 luafar3

 Timestamp is 6146ab37 (Sun Sep 19 04:15:03 2021)

 Preferred load address is 10000000

 Start         Length     Name                   Class
 0001:00000000 0004ace0H .text$mn                CODE
 0001:0004ace0 00000040H .text$x                 CODE
 0001:0004ad20 00000082H .text$yd                CODE
 0002:00000000 00000390H .idata$5                DATA
 0002:00000390 00000004H .00cfg                  DATA
 0002:00000394 00000004H .CRT$XCA                DATA
 0002:00000398 00000004H .CRT$XCZ                DATA
 0002:0000039c 00000004H .CRT$XIA                DATA
 0002:000003a0 0000000cH .CRT$XIC                DATA
 0002:000003ac 00000004H .CRT$XIZ                DATA
 0002:000003b0 00000004H .CRT$XPA                DATA
 0002:000003b4 0000000cH .CRT$XPX                DATA
 0002:000003c0 00000004H .CRT$XPXA               DATA
 0002:000003c4 00000004H .CRT$XPZ                DATA
 0002:000003c8 00000004H .CRT$XTA                DATA
 0002:000003cc 00000004H .CRT$XTZ                DATA
 0002:000003d0 00000000H .gfids$y                DATA
 0002:000003d0 0001228cH .rdata                  DATA
 0002:0001265c 000000e4H .rdata$r                DATA
 0002:00012740 0000001cH .rdata$sxdata           DATA
 0002:0001275c 000002fcH .rdata$zzzdbg           DATA
 0002:00012a58 00000004H .rtc$IAA                DATA
 0002:00012a5c 00000004H .rtc$IZZ                DATA
 0002:00012a60 00000004H .rtc$TAA                DATA
 0002:00012a64 00000004H .rtc$TZZ                DATA
 0002:00012a68 00000988H .xdata$x                DATA
 0002:000133f0 0000049cH .edata                  DATA
 0002:0001388c 00000078H .idata$2                DATA
 0002:00013904 00000014H .idata$3                DATA
 0002:00013918 00000390H .idata$4                DATA
 0002:00013ca8 00000fa8H .idata$6                DATA
 0003:00000000 0000b9f0H .data                   DATA
 0003:0000b9f0 00000060H .data$r                 DATA
 0003:0000ba50 00000b18H .bss                    DATA
 0004:00000000 00000060H .rsrc$01                DATA
 0004:00000060 00000320H .rsrc$02                DATA

  Address         Publics by Value              Rva+Base       Lib:Object

 0000:00000000       ___hybrid_code_map_count   00000000     <absolute>
 0000:00000000       ___guard_fids_count        00000000     <absolute>
 0000:00000000       ___guard_iat_count         00000000     <absolute>
 0000:00000000       ___guard_fids_table        00000000     <absolute>
 0000:00000000       ___dynamic_value_reloc_table 00000000     <absolute>
 0000:00000000       ___guard_longjmp_count     00000000     <absolute>
 0000:00000000       __except_list              00000000     <absolute>
 0000:00000000       ___guard_iat_table         00000000     <absolute>
 0000:00000000       ___guard_longjmp_table     00000000     <absolute>
 0000:00000000       ___hybrid_auxiliary_iat    00000000     <absolute>
 0000:00000000       ___enclave_config          00000000     <absolute>
 0000:00000000       ___volatile_metadata       00000000     <absolute>
 0000:00000000       ___AbsoluteZero            00000000     <absolute>
 0000:00000000       ___hybrid_code_map         00000000     <absolute>
 0000:00000007       ___safe_se_handler_count   00000007     <absolute>
 0000:00000100       ___guard_flags             00000100     <absolute>
 0000:00000000       ___ImageBase               10000000     <linker-defined>
 0001:00000000       ___local_stdio_printf_options 10001000 f i bit64.obj
 0001:00000010       _sprintf                   10001010 f i bit64.obj
 0001:00000050       _bit64_pushuserdata        10001050 f   bit64.obj
 0001:00000090       _bit64_push                10001090 f   bit64.obj
 0001:00000130       _bit64_getvalue            10001130 f   bit64.obj
 0001:000001b0       _check64                   100011b0 f   bit64.obj
 0001:00000dd0       _luaopen_bit64             10001dd0 f   bit64.obj
 0001:00000e30       _traceback                 10001e30 f   exported.obj
 0001:00000ed0       _GetExportFunction         10001ed0 f   exported.obj
 0001:00000f60       _pcall_msg                 10001f60 f   exported.obj
 0001:000010e0       _PushPluginObject          100020e0 f   exported.obj
 0001:00001140       _PushPluginPair            10002140 f   exported.obj
 0001:000011a0       _ReplacePluginInfoCollector 100021a0 f   exported.obj
 0001:000011d0       __AddStringToCollector     100021d0 f   exported.obj
 0001:000012c0       _AddStringToCollectorField 100022c0 f   exported.obj
 0001:000012f0       _AddBufToCollector         100022f0 f   exported.obj
 0001:00001340       _CreateStringsArray        10002340 f   exported.obj
 0001:00001450       _FarPanelItemFreeCallback@8 10002450 f   exported.obj
 0001:00001480       _FillPluginPanelItem       10002480 f   exported.obj
 0001:00001b20       _FillFindData              10002b20 f   exported.obj
 0001:00001ee0       _LF_GetFindData            10002ee0 f   exported.obj
 0001:00001fd0       _LF_FreeFindData           10002fd0 f   exported.obj
 0001:00002030       _UpdateFileSelection       10003030 f   exported.obj
 0001:000021d0       _LF_GetFiles               100031d0 f   exported.obj
 0001:000023c0       _RunDefaultScript          100033c0 f   exported.obj
 0001:00002680       _LF_RunDefaultScript       10003680 f   exported.obj
 0001:00002850       _LF_Analyse                10003850 f   exported.obj
 0001:000028f0       _LF_CloseAnalyse           100038f0 f   exported.obj
 0001:00002910       _LF_GetOpenPanelInfo       10003910 f   exported.obj
 0001:00003200       _PushFarMacroValue         10004200 f   exported.obj
 0001:000033b0       _PackMacroValues           100043b0 f   exported.obj
 0001:000036f0       _LF_Open                   100046f0 f   exported.obj
 0001:00003c10       _LF_ClosePanel             10004c10 f   exported.obj
 0001:00003c70       _LF_Compare                10004c70 f   exported.obj
 0001:00003d00       _LF_Configure              10004d00 f   exported.obj
 0001:00003d60       _LF_DeleteFiles            10004d60 f   exported.obj
 0001:00003e30       _LF_MakeDirectory          10004e30 f   exported.obj
 0001:00003f00       _LF_ProcessPanelEvent      10004f00 f   exported.obj
 0001:00004040       _LF_ProcessHostFile        10005040 f   exported.obj
 0001:00004140       _LF_ProcessPanelInput      10005140 f   exported.obj
 0001:000041b0       _LF_PutFiles               100051b0 f   exported.obj
 0001:00004360       _LF_SetDirectory           10005360 f   exported.obj
 0001:000044a0       _LF_SetFindList            100054a0 f   exported.obj
 0001:00004550       _LF_ExitFAR                10005550 f   exported.obj
 0001:000045d0       _getPluginMenuItems        100055d0 f   exported.obj
 0001:00004670       _LF_GetPluginInfo          10005670 f   exported.obj
 0001:000047d0       _LF_ProcessEditorInput     100057d0 f   exported.obj
 0001:00004830       _LF_ProcessEditorEvent     10005830 f   exported.obj
 0001:00004b00       _LF_ProcessViewerEvent     10005b00 f   exported.obj
 0001:00004bb0       _LF_ProcessDialogEvent     10005bb0 f   exported.obj
 0001:00004ec0       _LF_ProcessSynchroEvent    10005ec0 f   exported.obj
 0001:00005080       _LF_GetContentFields       10006080 f   exported.obj
 0001:000051c0       _LF_GetContentData         100061c0 f   exported.obj
 0001:000054b0       _LF_FreeContentData        100064b0 f   exported.obj
 0001:000054e0       _LF_GetGlobalInfo          100064e0 f   exported.obj
 0001:00005880       _LF_ProcessConsoleInput    10006880 f   exported.obj
 0001:00005a40       _LF_LoadFile               10006a40 f   lflua.obj
 0001:00005d80       _luaB_loadfileW            10006d80 f   lflua.obj
 0001:00005e70       _luaB_dofileW              10006e70 f   lflua.obj
 0001:00005f60       _LF_Gsub                   10006f60 f   lflua.obj
 0001:000060c0       _method_gc                 100070c0 f   lregex.obj
 0001:00006120       _method_tostring           10007120 f   lregex.obj
 0001:00006170       _check_regex_pattern       10007170 f   lregex.obj
 0001:00006210       _push_far_regex            10007210 f   lregex.obj
 0001:00006290       __regex_gmatch_closure     10007290 f   lregex.obj
 0001:000063a0       _regex_gmatch_closure      100073a0 f   lregex.obj
 0001:000063b0       _regex_gmatch_closureW     100073b0 f   lregex.obj
 0001:000063d0       __Gmatch                   100073d0 f   lregex.obj
 0001:00006550       _func_Gmatch               10007550 f   lregex.obj
 0001:00006560       _func_GmatchW              10007560 f   lregex.obj
 0001:00006580       _rx_find_match             10007580 f   lregex.obj
 0001:000069b0       _method_bracketscount      100079b0 f   lregex.obj
 0001:00006a10       _rx_gsub                   10007a10 f   lregex.obj
 0001:00007510       _func_New                  10008510 f   lregex.obj
 0001:00007550       _method_find               10008550 f   lregex.obj
 0001:00007570       _func_find                 10008570 f   lregex.obj
 0001:00007590       _method_findW              10008590 f   lregex.obj
 0001:000075b0       _func_findW                100085b0 f   lregex.obj
 0001:000075d0       _method_match              100085d0 f   lregex.obj
 0001:000075f0       _func_match                100085f0 f   lregex.obj
 0001:00007610       _method_matchW             10008610 f   lregex.obj
 0001:00007630       _func_matchW               10008630 f   lregex.obj
 0001:00007650       _method_exec               10008650 f   lregex.obj
 0001:00007670       _func_exec                 10008670 f   lregex.obj
 0001:00007690       _method_execW              10008690 f   lregex.obj
 0001:000076b0       _func_execW                100086b0 f   lregex.obj
 0001:000076d0       _method_gsub               100086d0 f   lregex.obj
 0001:000076f0       _func_gsub                 100086f0 f   lregex.obj
 0001:00007710       _method_gsubW              10008710 f   lregex.obj
 0001:00007730       _func_gsubW                10008730 f   lregex.obj
 0001:00007750       _luaopen_regex             10008750 f   lregex.obj
 0001:00007a20       _Open_Luamacro             10008a20 f   luamacro.obj
 0001:00007f60       _far_MacroCallFar          10008f60 f   luamacro.obj
 0001:00008180       _far_FarMacroCallToLua     10009180 f   luamacro.obj
 0001:00008240       _uc_len                    10009240 f   lusercontrol.obj
 0001:000085e0       _luaopen_usercontrol       100095e0 f   lusercontrol.obj
 0001:00008620       _CreateRegKey              10009620 f   reg.obj
 0001:00008660       _fprintf                   10009660 f i service.obj
 0001:00008690       _DllMain@12                10009690 f   service.obj
 0001:000089e0       _GetFlagCombination        100099e0 f   service.obj
 0001:00008c70       _OptFlags                  10009c70 f   service.obj
 0001:00008d80       _PutFlagsToTable           10009d80 f   service.obj
 0001:00008e40       _ConvertLuaValue           10009e40 f   service.obj
 0001:00009320       _StoreTempString           1000a320 f   service.obj
 0001:00009580       _PushPanelItem             1000a580 f   service.obj
 0001:00009b80       _PushPanelItems            1000ab80 f   service.obj
 0001:0000c2b0       _GetFarColor               1000d2b0 f   service.obj
 0001:0000c470       _PushFarColor              1000d470 f   service.obj
 0001:0000cc60       _PushInputRecord           1000dc60 f   service.obj
 0001:0000d090       _FillInputRecord           1000e090 f   service.obj
 0001:0000e3e0       _LF_Message                1000f3e0 f   service.obj
 0001:0000e920       _LF_Error                  1000f920 f   service.obj
 0001:00010cf0       _CreateList                10011cf0 f   service.obj
 0001:00011bf0       _NewDialogData             10012bf0 f   service.obj
 0001:00011c70       _DialogHandleEqual         10012c70 f   service.obj
 0001:00013040       _PushDNParams              10014040 f   service.obj
 0001:000132c0       _ProcessDNResult           100142c0 f   service.obj
 0001:00013570       _LF_DlgProc                10014570 f   service.obj
 0001:00018170       _MacroAddCallback@12       10019170 f   service.obj
 0001:00018940       _pushFileTime              10019940 f   service.obj
 0001:00018d90       _NewVirtualKeyTable        10019d90 f   service.obj
 0001:0001a320       _TimerCallback@8           1001b320 f   service.obj
 0001:0001cb30       _LF_RunLuafarInit          1001db30 f   service.obj
 0001:0001cc10       @_guard_check_icall_nop@4  1001dc10 f   LIBCMT:guard_support.obj
 0001:0001cc10       _LF_ProcessEnvVars         1001dc10 f   service.obj
 0001:0001cc20       _LF_InitLuaState1          1001dc20 f   service.obj
 0001:0001ce40       _LF_InitLuaState2          1001de40 f   service.obj
 0001:0001cee0       _LF_MacroCallback          1001dee0 f   service.obj
 0001:0001cf00       _LF_DoFile                 1001df00 f   service.obj
 0001:0001d020       _LF_GetLuafarAPI           1001e020 f   service.obj
 0001:0001d060       _luaopen_luafar3           1001e060 f   service.obj
 0001:0001d1f0       __snwprintf                1001e1f0 f i slnunico.obj
 0001:0001db50       _luaopen_unicode           1001eb50 f   slnunico.obj
 0001:000216c0       _luaopen_utf8              100226c0 f   lutf8lib.obj
 0001:000218c0       ___local_stdio_scanf_options 100228c0 f i uliolib51.obj
 0001:000218d0       _fscanf                    100228d0 f i uliolib51.obj
 0001:000231e0       _luaopen_uio               100241e0 f   uliolib51.obj
 0001:000243c0       _luaopen_upackage          100253c0 f   uloadlib51.obj
 0001:00024580       _pusherror                 10025580 f   ustring.obj
 0001:00024610       _SysErrorReturn            10025610 f   ustring.obj
 0001:00024690       _PutIntToArray             10025690 f   ustring.obj
 0001:000246d0       _PutIntToTable             100256d0 f   ustring.obj
 0001:00024710       _PutNumToTable             10025710 f   ustring.obj
 0001:00024740       _PutBoolToTable            10025740 f   ustring.obj
 0001:00024770       _PutStrToTable             10025770 f   ustring.obj
 0001:000247a0       _PutStrToArray             100257a0 f   ustring.obj
 0001:000247d0       _PutWStrToTable            100257d0 f   ustring.obj
 0001:00024800       _PutWStrToArray            10025800 f   ustring.obj
 0001:00024830       _PutLStrToTable            10025830 f   ustring.obj
 0001:00024860       _GetOptNumFromTable        10025860 f   ustring.obj
 0001:000248c0       _GetOptIntFromTable        100258c0 f   ustring.obj
 0001:00024910       _GetOptIntFromArray        10025910 f   ustring.obj
 0001:00024960       _GetBoolFromTable          10025960 f   ustring.obj
 0001:000249a0       _GetOptBoolFromTable       100259a0 f   ustring.obj
 0001:00024a00       _check_utf8_string         10025a00 f   ustring.obj
 0001:00024ad0       _utf8_to_utf16             10025ad0 f   ustring.obj
 0001:00024ba0       _opt_utf8_string           10025ba0 f   ustring.obj
 0001:00024bd0       _push_utf8_string          10025bd0 f   ustring.obj
 0001:00024c80       _ustring_WideCharToMultiByte 10025c80 f   ustring.obj
 0001:00024db0       _ustring_MultiByteToWideChar 10025db0 f   ustring.obj
 0001:00024f70       _ustring_OemToUtf8         10025f70 f   ustring.obj
 0001:00025030       _ustring_Utf8ToOem         10026030 f   ustring.obj
 0001:00025170       _ustring_Utf16ToUtf8       10026170 f   ustring.obj
 0001:000251a0       _ustring_Utf8ToUtf16       100261a0 f   ustring.obj
 0001:00025250       _ustring_GetACP            10026250 f   ustring.obj
 0001:00025270       _ustring_GetOEMCP          10026270 f   ustring.obj
 0001:00025290       _ustring_GetConsoleCP      10026290 f   ustring.obj
 0001:000252b0       _ustring_SetConsoleCP      100262b0 f   ustring.obj
 0001:000252f0       _ustring_GetConsoleOutputCP 100262f0 f   ustring.obj
 0001:00025310       _ustring_SetConsoleOutputCP 10026310 f   ustring.obj
 0001:00025350       _EnumCodePagesProc@4       10026350 f   ustring.obj
 0001:00025420       _ustring_EnumSystemCodePages 10026420 f   ustring.obj
 0001:00025480       _ustring_GetCPInfo         10026480 f   ustring.obj
 0001:000256d0       _ustring_GetLogicalDriveStrings 100266d0 f   ustring.obj
 0001:00025890       _ustring_GetDriveType      10026890 f   ustring.obj
 0001:000259b0       _ustring_Uuid              100269b0 f   ustring.obj
 0001:00025ab0       _ustring_SearchPath        10026ab0 f   ustring.obj
 0001:00025eb0       _ustring_GlobalMemoryStatus 10026eb0 f   ustring.obj
 0001:000261b0       _ustring_Sleep             100271b0 f   ustring.obj
 0001:000261f0       _PushAttrString            100271f0 f   ustring.obj
 0001:000262c0       _DecodeAttributes          100272c0 f   ustring.obj
 0001:000263f0       _SetAttrWords              100273f0 f   ustring.obj
 0001:000265d0       _ustring_SetFileAttr       100275d0 f   ustring.obj
 0001:000266b0       _ustring_GetFileAttr       100276b0 f   ustring.obj
 0001:00026780       _ustring_SHGetFolderPath   10027780 f   ustring.obj
 0001:000268a0       _push_utf16_string         100278a0 f   ustring.obj
 0001:000268e0       _ustring_sub               100278e0 f   ustring.obj
 0001:00026970       _ustring_len               10027970 f   ustring.obj
 0001:000269a0       _check_utf16_string        100279a0 f   ustring.obj
 0001:000269d0       _opt_utf16_string          100279d0 f   ustring.obj
 0001:00026c00       _ustring_GetCurrentDir     10027c00 f   ustring.obj
 0001:00026de0       _ustring_SetCurrentDir     10027de0 f   ustring.obj
 0001:00026eb0       _ustring_GetKeyState       10027eb0 f   ustring.obj
 0001:00026f00       _luaopen_ustring           10027f00 f   ustring.obj
 0001:00026f60       _GetIntFromArray           10027f60 f   util.obj
 0001:00026fe0       _GetFileSizeFromTable      10027fe0 f   util.obj
 0001:00027070       _GetFileTimeFromTable      10028070 f   util.obj
 0001:00027160       _PutFileTimeToTable        10028160 f   util.obj
 0001:0002a420       _win_WriteConsole          1002b420 f   win.obj
 0001:0002a5d0       _win_IsWinVersion          1002b5d0 f   win.obj
 0001:0002b1f0       _luaopen_win               1002c1f0 f   win.obj
 0001:0002b270       _EncodePointerWrapper@4    1002c270 f   vc_crt_fix_impl.obj
 0001:0002b330       _DecodePointerWrapper@4    1002c330 f   vc_crt_fix_impl.obj
 0001:0002b380       _GetModuleHandleExWWrapper@12 1002c380 f   vc_crt_fix_impl.obj
 0001:0002b6c0       _InitializeSListHeadWrapper@4 1002c6c0 f   vc_crt_fix_impl.obj
 0001:0002b710       _InterlockedFlushSListWrapper@4 1002c710 f   vc_crt_fix_impl.obj
 0001:0002b760       _InterlockedPopEntrySListWrapper@4 1002c760 f   vc_crt_fix_impl.obj
 0001:0002b7b0       _InterlockedPushEntrySListWrapper@8 1002c7b0 f   vc_crt_fix_impl.obj
 0001:0002b800       _InterlockedPushListSListExWrapper@16 1002c800 f   vc_crt_fix_impl.obj
 0001:0002b850       _RtlFirstEntrySListWrapper@4 1002c850 f   vc_crt_fix_impl.obj
 0001:0002b8a0       _QueryDepthSListWrapper@4  1002c8a0 f   vc_crt_fix_impl.obj
 0001:0002b8f0       _GetNumaHighestNodeNumberWrapper@4 1002c8f0 f   vc_crt_fix_impl.obj
 0001:0002b960       _GetLogicalProcessorInformationWrapper@8 1002c960 f   vc_crt_fix_impl.obj
 0001:0002b9c0       _SetThreadStackGuaranteeWrapper@4 1002c9c0 f   vc_crt_fix_impl.obj
 0001:0002ba20       _InitializeCriticalSectionExWrapper@12 1002ca20 f   vc_crt_fix_impl.obj
 0001:0002baa0       _CompareStringExWrapper@36 1002caa0 f   vc_crt_fix_impl.obj
 0001:0002bb20       _LCMapStringExWrapper@36   1002cb20 f   vc_crt_fix_impl.obj
 0001:0002bba0       _luaopen_table             1002cba0 f   lua51:lua51.dll
 0001:0002bba6       _luaopen_base              1002cba6 f   lua51:lua51.dll
 0001:0002bbac       _luaopen_os                1002cbac f   lua51:lua51.dll
 0001:0002bbb2       _luaopen_string            1002cbb2 f   lua51:lua51.dll
 0001:0002bbb8       _luaopen_math              1002cbb8 f   lua51:lua51.dll
 0001:0002bbbe       _luaopen_debug             1002cbbe f   lua51:lua51.dll
 0001:0002bbc4       @__security_check_cookie@4 1002cbc4 f   LIBCMT:secchk.obj
 0001:0002bbd5       ___raise_securityfailure   1002cbd5 f   LIBCMT:gs_report.obj
 0001:0002bbfd       ___report_gsfailure        1002cbfd f   LIBCMT:gs_report.obj
 0001:0002bd3a       ___scrt_acquire_startup_lock 1002cd3a f   LIBCMT:utility.obj
 0001:0002bd6c       ___scrt_dllmain_after_initialize_c 1002cd6c f   LIBCMT:utility.obj
 0001:0002bd97       ___scrt_dllmain_before_initialize_c 1002cd97 f   LIBCMT:utility.obj
 0001:0002bda5       ___scrt_dllmain_crt_thread_attach 1002cda5 f   LIBCMT:utility.obj
 0001:0002bdc4       ___scrt_dllmain_crt_thread_detach 1002cdc4 f   LIBCMT:utility.obj
 0001:0002bdd1       ___scrt_dllmain_exception_filter 1002cdd1 f   LIBCMT:utility.obj
 0001:0002be05       ___scrt_dllmain_uninitialize_c 1002ce05 f   LIBCMT:utility.obj
 0001:0002be28       ___scrt_dllmain_uninitialize_critical 1002ce28 f   LIBCMT:utility.obj
 0001:0002be35       ___scrt_initialize_crt     1002ce35 f   LIBCMT:utility.obj
 0001:0002be6e       ___scrt_initialize_onexit_tables 1002ce6e f   LIBCMT:utility.obj
 0001:0002bef5       ___scrt_is_nonwritable_in_current_image 1002cef5 f   LIBCMT:utility.obj
 0001:0002bf89       ___scrt_release_startup_lock 1002cf89 f   LIBCMT:utility.obj
 0001:0002bfa6       ___scrt_uninitialize_crt   1002cfa6 f   LIBCMT:utility.obj
 0001:0002bfce       __onexit                   1002cfce f   LIBCMT:utility.obj
 0001:0002bffb       _atexit                    1002cffb f   LIBCMT:utility.obj
 0001:0002c34b       __DllMainCRTStartup@12     1002d34b f   LIBCMT:dll_dllmain.obj
 0001:0002c36e       ___isa_available_init      1002d36e f   LIBCMT:cpu_disp.obj
 0001:0002c53e       __get_startup_argv_mode    1002d53e f   LIBCMT:argv_mode.obj
 0001:0002c542       ___scrt_is_ucrt_dll_in_use 1002d542 f   LIBCMT:ucrt_detection.obj
 0001:0002c54e       ___scrt_fastfail           1002d54e f   LIBCMT:utility_desktop.obj
 0001:0002c668       __crt_debugger_hook        1002d668 f   LIBCMT:utility_desktop.obj
 0001:0002c670       __SEH_prolog4              1002d670 f   LIBCMT:sehprolg4.obj
 0001:0002c6b6       __SEH_epilog4              1002d6b6 f   LIBCMT:sehprolg4.obj
 0001:0002c718       ___security_init_cookie    1002d718 f   LIBCMT:gs_support.obj
 0001:0002c763       ?__scrt_initialize_type_info@@YAXXZ 1002d763 f   LIBCMT:tncleanup.obj
 0001:0002c76f       ?__scrt_uninitialize_type_info@@YAXXZ 1002d76f f   LIBCMT:tncleanup.obj
 0001:0002c77b       ___scrt_initialize_default_local_stdio_options 1002d77b f   LIBCMT:default_local_stdio_options.obj
 0001:0002c798       ___scrt_get_dyn_tls_init_callback 1002d798 f   LIBCMT:dyn_tls_init.obj
 0001:0002c79e       __RTC_Initialize           1002d79e f   LIBCMT:initsect.obj
 0001:0002c7ca       __RTC_Terminate            1002d7ca f   LIBCMT:initsect.obj
 0001:0002c7f6       _wcsrchr                   1002d7f6 f   libvcruntime:wcsrchr.obj
 0001:0002c898       _wcsstr                    1002d898 f   libvcruntime:wcsstr.obj
 0001:0002cb14       _wcschr                    1002db14 f   libvcruntime:wcschr.obj
 0001:0002cbe0       _strchr                    1002dbe0 f   libvcruntime:strchr.obj
 0001:0002cc4e       ___from_strstr_to_strchr   1002dc4e     libvcruntime:strchr.obj
 0001:0002cd10       _strrchr                   1002dd10 f   libvcruntime:strrchr.obj
 0001:0002ce47       ?GetRangeOfTrysToCheck@__FrameHandler3@@SA?AU?$pair@Viterator@TryBlockMap@__FrameHandler3@@V123@@std@@AAVTryBlockMap@1@HPAXPBU_s_FuncInfo@@H@Z 1002de47 f   libvcruntime:trnsctrl.obj
 0001:0002ceb7       ?_CallCatchBlock2@@YAPAXPAUEHRegistrationNode@@PBU_s_FuncInfo@@PAXHK@Z 1002deb7 f   libvcruntime:trnsctrl.obj
 0001:0002cf15       ?_CallSETranslator@@YAHPAUEHExceptionRecord@@PAUEHRegistrationNode@@PAX2PBU_s_FuncInfo@@H1@Z 1002df15 f   libvcruntime:trnsctrl.obj
 0001:0002cffb       ?_JumpToContinuation@@YGXPAXPAUEHRegistrationNode@@@Z 1002dffb f   libvcruntime:trnsctrl.obj
 0001:0002d02b       ?_UnwindNestedFrames@@YGXPAUEHRegistrationNode@@PAUEHExceptionRecord@@@Z 1002e02b f   libvcruntime:trnsctrl.obj
 0001:0002d07e       __CatchGuardHandler        1002e07e f   libvcruntime:trnsctrl.obj
 0001:0002d0af       __CreateFrameInfo          1002e0af f   libvcruntime:trnsctrl.obj
 0001:0002d0d3       __FindAndUnlinkFrame       1002e0d3 f   libvcruntime:trnsctrl.obj
 0001:0002d11b       __TranslatorGuardHandler   1002e11b f   libvcruntime:trnsctrl.obj
 0001:0002d1b8       ___CxxFrameHandler3        1002e1b8 f   libvcruntime:trnsctrl.obj
 0001:0002d1ee       ___DestructExceptionObject 1002e1ee f   libvcruntime:ehhelpers.obj
 0001:0002d28f       ?_CallMemberFunction0@@YGXQAX0@Z 1002e28f f i libvcruntime:ehhelpers.obj
 0001:0002d2f4       __IsExceptionObjectToBeDestroyed 1002e2f4 f   libvcruntime:ehhelpers.obj
 0001:0002d31a       ___AdjustPointer           1002e31a f   libvcruntime:ehhelpers.obj
 0001:0002d33f       ___FrameUnwindFilter       1002e33f f   libvcruntime:ehhelpers.obj
 0001:0002d395       ___std_terminate           1002e395 f   libvcruntime:ehhelpers.obj
 0001:0002d39a       ___vcrt_initialize         1002e39a f   libvcruntime:initialization.obj
 0001:0002d3b9       ___vcrt_thread_attach      1002e3b9 f   libvcruntime:initialization.obj
 0001:0002d3c4       ___vcrt_thread_detach      1002e3c4 f   libvcruntime:initialization.obj
 0001:0002d3cf       ___vcrt_uninitialize       1002e3cf f   libvcruntime:initialization.obj
 0001:0002d3e6       ___vcrt_uninitialize_critical 1002e3e6 f   libvcruntime:initialization.obj
 0001:0002d430       __except_handler4          1002e430 f   libvcruntime:chandler4.obj
 0001:0002d590       _memset                    1002e590 f   libvcruntime:memset.obj
 0001:0002d6ea       ___std_type_info_compare   1002e6ea f   libvcruntime:std_type_info.obj
 0001:0002d726       ___std_type_info_destroy_list 1002e726 f   libvcruntime:std_type_info.obj
 0001:0002d749       ___vcrt_freefls@4          1002e749 f   libvcruntime:per_thread_data.obj
 0001:0002d765       ___vcrt_freeptd            1002e765 f   libvcruntime:per_thread_data.obj
 0001:0002d79b       ___vcrt_getptd             1002e79b f   libvcruntime:per_thread_data.obj
 0001:0002d7a9       ___vcrt_getptd_noexit      1002e7a9 f   libvcruntime:per_thread_data.obj
 0001:0002d83b       ___vcrt_initialize_ptd     1002e83b f   libvcruntime:per_thread_data.obj
 0001:0002d86e       ___vcrt_uninitialize_ptd   1002e86e f   libvcruntime:per_thread_data.obj
 0001:0002dfcc       ??$TypeMatchHelper@V__FrameHandler3@@@@YAHPBU_s_HandlerType@@PBU_s_CatchableType@@PBU_s_ThrowInfo@@@Z 1002efcc f i libvcruntime:frame.obj
 0001:0002e05a       ??$__InternalCxxFrameHandler@V__FrameHandler3@@@@YA?AW4_EXCEPTION_DISPOSITION@@PAUEHExceptionRecord@@PAUEHRegistrationNode@@PAU_CONTEXT@@PAXPBU_s_FuncInfo@@H1E@Z 1002f05a f i libvcruntime:frame.obj
 0001:0002e15c       ??0bad_exception@std@@QAE@ABV01@@Z 1002f15c f i libvcruntime:frame.obj
 0001:0002e177       ??0bad_exception@std@@QAE@XZ 1002f177 f i libvcruntime:frame.obj
 0001:0002e18f       ??0exception@std@@QAE@ABV01@@Z 1002f18f f i libvcruntime:frame.obj
 0001:0002e1bb       ??1bad_exception@std@@UAE@XZ 1002f1bb f i libvcruntime:frame.obj
 0001:0002e1cc       ??8type_info@@QBE_NABV0@@Z 1002f1cc f i libvcruntime:frame.obj
 0001:0002e1eb       ??_Gbad_exception@std@@UAEPAXI@Z 1002f1eb f i libvcruntime:frame.obj
 0001:0002e1eb       ??_Gexception@std@@UAEPAXI@Z 1002f1eb f i libvcruntime:frame.obj
 0001:0002e1eb       ??_Ebad_exception@std@@UAEPAXI@Z 1002f1eb f i libvcruntime:frame.obj
 0001:0002e1eb       ??_Eexception@std@@UAEPAXI@Z 1002f1eb f i libvcruntime:frame.obj
 0001:0002e460       ?FrameUnwindToEmptyState@__FrameHandler3@@SAXPAUEHRegistrationNode@@PAXPBU_s_FuncInfo@@@Z 1002f460 f   libvcruntime:frame.obj
 0001:0002e478       ?FrameUnwindToState@__FrameHandler3@@SAXPAUEHRegistrationNode@@PAXPBU_s_FuncInfo@@H@Z 1002f478 f   libvcruntime:frame.obj
 0001:0002e5fa       ?_CallMemberFunction1@@YGXQAX00@Z 1002f5fa f i libvcruntime:frame.obj
 0001:0002e60a       ?_CallMemberFunction2@@YGXQAX00H@Z 1002f60a f i libvcruntime:frame.obj
 0001:0002e61d       ?getESTypes@__FrameHandler3@@SAPBU_s_ESTypeList@@PBU_s_FuncInfo@@@Z 1002f61d f i libvcruntime:frame.obj
 0001:0002e628       ?what@exception@std@@UBEPBDXZ 1002f628 f i libvcruntime:frame.obj
 0001:0002e640       __CallSettingFrame@12      1002f640 f   libvcruntime:lowhelpr.obj
 0001:0002e667       __NLG_Return               1002f667     libvcruntime:lowhelpr.obj
 0001:0002e68c       ___except_validate_context_record 1002f68c f   libvcruntime:jbcxrval.obj
 0001:0002e6bc       ___except_validate_jump_buffer 1002f6bc f   libvcruntime:jbcxrval.obj
 0001:0002e6e9       ___vcrt_initialize_locks   1002f6e9 f   libvcruntime:locks.obj
 0001:0002e725       ___vcrt_uninitialize_locks 1002f725 f   libvcruntime:locks.obj
 0001:0002e760       __local_unwind4            1002f760 f   libvcruntime:exsup4.obj
 0001:0002e838       __seh_longjmp_unwind4@4    1002f838 f   libvcruntime:exsup4.obj
 0001:0002e860       @_EH4_CallFilterFunc@8     1002f860 f   libvcruntime:exsup4.obj
 0001:0002e878       @_EH4_TransferToHandler@8  1002f878 f   libvcruntime:exsup4.obj
 0001:0002e894       @_EH4_GlobalUnwind2@8      1002f894 f   libvcruntime:exsup4.obj
 0001:0002e8b0       @_EH4_LocalUnwind@16       1002f8b0 f   libvcruntime:exsup4.obj
 0001:0002e9bc       ___vcrt_FlsAlloc           1002f9bc f   libvcruntime:winapi_downlevel.obj
 0001:0002e9f7       ___vcrt_FlsFree            1002f9f7 f   libvcruntime:winapi_downlevel.obj
 0001:0002ea32       ___vcrt_FlsGetValue        1002fa32 f   libvcruntime:winapi_downlevel.obj
 0001:0002ea6d       ___vcrt_FlsSetValue        1002fa6d f   libvcruntime:winapi_downlevel.obj
 0001:0002eaab       ___vcrt_InitializeCriticalSectionEx 1002faab f   libvcruntime:winapi_downlevel.obj
 0001:0002eaf2       _unexpected                1002faf2 f   libvcruntime:unexpected.obj
 0001:0002eb0f       ?GetCurrentState@__FrameHandler3@@SAHPAUEHRegistrationNode@@PAXPBU_s_FuncInfo@@@Z 1002fb0f f   libvcruntime:ehstate.obj
 0001:0002eb2c       ?SetState@__FrameHandler3@@SAXPAUEHRegistrationNode@@PBU_s_FuncInfo@@H@Z 1002fb2c f   libvcruntime:ehstate.obj
 0001:0002eb3a       ___std_exception_copy      1002fb3a f   libvcruntime:std_exception.obj
 0001:0002eb9d       ___std_exception_destroy   1002fb9d f   libvcruntime:std_exception.obj
 0001:0002ebbc       __CxxThrowException@8      1002fbbc f   libvcruntime:throw.obj
 0001:0002ec30       _memmove                   1002fc30 f   libvcruntime:memmove.obj
 0001:0002f1b0       __global_unwind2           100301b0 f   libvcruntime:exsup.obj
 0001:0002f216       __local_unwind2            10030216 f   libvcruntime:exsup.obj
 0001:0002f29a       __abnormal_termination     1003029a f   libvcruntime:exsup.obj
 0001:0002f2c0       __NLG_Notify1              100302c0 f   libvcruntime:exsup.obj
 0001:0002f2cc       __NLG_Notify               100302cc f   libvcruntime:exsup.obj
 0001:0002f2e3       __NLG_Dispatch2            100302e3     libvcruntime:exsup.obj
 0001:0002f2e3       __NLG_Dispatch             100302e3     libvcruntime:exsup.obj
 0001:0002f2eb       __NLG_Call                 100302eb f   libvcruntime:exsup.obj
 0001:0002f2ed       __NLG_Return2              100302ed     libvcruntime:exsup.obj
 0001:0002f2f0       _memcpy                    100302f0 f   libvcruntime:memcpy.obj
 0001:0002fbc4       ??$count@D@formatting_buffer@__crt_stdio_output@@QBEIXZ 10030bc4 f i libucrt:output.obj
 0001:0002fbdc       ??$count@_W@formatting_buffer@__crt_stdio_output@@QBEIXZ 10030bdc f i libucrt:output.obj
 0001:0002fbf5       ??$ensure_buffer_is_big_enough@D@formatting_buffer@__crt_stdio_output@@QAE_NI@Z 10030bf5 f i libucrt:output.obj
 0001:0002fc72       ??$ensure_buffer_is_big_enough@_W@formatting_buffer@__crt_stdio_output@@QAE_NI@Z 10030c72 f i libucrt:output.obj
 0001:0002fcf0       ??$is_wide_character_specifier@D@__crt_stdio_output@@YA_N_KDW4length_modifier@0@@Z 10030cf0 f i libucrt:output.obj
 0001:0002fd21       ??$is_wide_character_specifier@_W@__crt_stdio_output@@YA_N_K_WW4length_modifier@0@@Z 10030d21 f i libucrt:output.obj
 0001:0002fd6f       ??$scratch_data@D@formatting_buffer@__crt_stdio_output@@QAEPADXZ 10030d6f f i libucrt:output.obj
 0001:0002fd8d       ??$type_case_integer_parse_into_buffer@I@?$output_processor@DV?$string_output_adapter@D@__crt_stdio_output@@V?$standard_base@DV?$string_output_adapter@D@__crt_stdio_output@@@2@@__crt_stdio_output@@AAEXII_N@Z 10030d8d f i libucrt:output.obj
 0001:0002fd8d       ??$type_case_integer_parse_into_buffer@I@?$output_processor@DV?$stream_output_adapter@D@__crt_stdio_output@@V?$standard_base@DV?$stream_output_adapter@D@__crt_stdio_output@@@2@@__crt_stdio_output@@AAEXII_N@Z 10030d8d f i libucrt:output.obj
 0001:0002fe00       ??$type_case_integer_parse_into_buffer@I@?$output_processor@_WV?$string_output_adapter@_W@__crt_stdio_output@@V?$standard_base@_WV?$string_output_adapter@_W@__crt_stdio_output@@@2@@__crt_stdio_output@@AAEXII_N@Z 10030e00 f i libucrt:output.obj
 0001:0002fe87       ??$type_case_integer_parse_into_buffer@_K@?$output_processor@DV?$string_output_adapter@D@__crt_stdio_output@@V?$standard_base@DV?$string_output_adapter@D@__crt_stdio_output@@@2@@__crt_stdio_output@@AAEX_KI_N@Z 10030e87 f i libucrt:output.obj
 0001:0002fe87       ??$type_case_integer_parse_into_buffer@_K@?$output_processor@DV?$stream_output_adapter@D@__crt_stdio_output@@V?$standard_base@DV?$stream_output_adapter@D@__crt_stdio_output@@@2@@__crt_stdio_output@@AAEX_KI_N@Z 10030e87 f i libucrt:output.obj
 0001:0002ff15       ??$type_case_integer_parse_into_buffer@_K@?$output_processor@_WV?$string_output_adapter@_W@__crt_stdio_output@@V?$standard_base@_WV?$string_output_adapter@_W@__crt_stdio_output@@@2@@__crt_stdio_output@@AAEX_KI_N@Z 10030f15 f i libucrt:output.obj
 0001:0002ffb7       ??$write_multiple_characters@V?$stream_output_adapter@D@__crt_stdio_output@@D@__crt_stdio_output@@YAXABV?$stream_output_adapter@D@0@DHQAH@Z 10030fb7 f i libucrt:output.obj
 0001:0002fff2       ??$write_multiple_characters@V?$string_output_adapter@D@__crt_stdio_output@@D@__crt_stdio_output@@YAXABV?$string_output_adapter@D@0@DHQAH@Z 10030ff2 f i libucrt:output.obj
 0001:0003001e       ??$write_multiple_characters@V?$string_output_adapter@_W@__crt_stdio_output@@D@__crt_stdio_output@@YAXABV?$string_output_adapter@_W@0@DHQAH@Z 1003101e f i libucrt:output.obj
 0001:0003004f       ??0?$common_data@D@__crt_stdio_output@@IAE@XZ 1003104f f i libucrt:output.obj
 0001:00030094       ??0?$common_data@_W@__crt_stdio_output@@IAE@XZ 10031094 f i libucrt:output.obj
 0001:000300de       ??0?$output_adapter_data@DV?$string_output_adapter@D@__crt_stdio_output@@@__crt_stdio_output@@IAE@ABV?$string_output_adapter@D@1@_KQBDQAU__crt_locale_pointers@@QAD@Z 100310de f i libucrt:output.obj
 0001:000300de       ??0?$output_adapter_data@DV?$stream_output_adapter@D@__crt_stdio_output@@@__crt_stdio_output@@IAE@ABV?$stream_output_adapter@D@1@_KQBDQAU__crt_locale_pointers@@QAD@Z 100310de f i libucrt:output.obj
 0001:0003011a       ??0?$output_adapter_data@_WV?$string_output_adapter@_W@__crt_stdio_output@@@__crt_stdio_output@@IAE@ABV?$string_output_adapter@_W@1@_KQB_WQAU__crt_locale_pointers@@QAD@Z 1003111a f i libucrt:output.obj
 0001:00030156       ??0_LocaleUpdate@@QAE@QAU__crt_locale_pointers@@@Z 10031156 f i libucrt:output.obj
 0001:000301d9       ??1formatting_buffer@__crt_stdio_output@@QAE@XZ 100311d9 f i libucrt:output.obj
 0001:000301f3       ??4?$__crt_unique_heap_ptr@DU__crt_internal_free_policy@@@@QAEAAV0@$$QAV0@@Z 100311f3 f i libucrt:output.obj
 0001:000302d6       ?crop_zeroes@__crt_stdio_output@@YAXPADQAU__crt_locale_pointers@@@Z 100312d6 f i libucrt:output.obj
 0001:00030336       ?find_next_state@?$output_processor@DV?$string_output_adapter@D@__crt_stdio_output@@V?$standard_base@DV?$string_output_adapter@D@__crt_stdio_output@@@2@@__crt_stdio_output@@ABE?AW4state@2@DW432@@Z 10031336 f i libucrt:output.obj
 0001:00030336       ?find_next_state@?$output_processor@DV?$stream_output_adapter@D@__crt_stdio_output@@V?$standard_base@DV?$stream_output_adapter@D@__crt_stdio_output@@@2@@__crt_stdio_output@@ABE?AW4state@2@DW432@@Z 10031336 f i libucrt:output.obj
 0001:00030373       ?find_next_state@?$output_processor@_WV?$string_output_adapter@_W@__crt_stdio_output@@V?$standard_base@_WV?$string_output_adapter@_W@__crt_stdio_output@@@2@@__crt_stdio_output@@ABE?AW4state@2@_WW432@@Z 10031373 f i libucrt:output.obj
 0001:000303b2       ?force_decimal_point@__crt_stdio_output@@YAXPADQAU__crt_locale_pointers@@@Z 100313b2 f i libucrt:output.obj
 0001:0003040e       ?parse_int_from_format_string@?$output_processor@DV?$stream_output_adapter@D@__crt_stdio_output@@V?$standard_base@DV?$stream_output_adapter@D@__crt_stdio_output@@@2@@__crt_stdio_output@@AAE_NQAH@Z 1003140e f i libucrt:output.obj
 0001:0003040e       ?parse_int_from_format_string@?$output_processor@DV?$string_output_adapter@D@__crt_stdio_output@@V?$standard_base@DV?$string_output_adapter@D@__crt_stdio_output@@@2@@__crt_stdio_output@@AAE_NQAH@Z 1003140e f i libucrt:output.obj
 0001:00030482       ?parse_int_from_format_string@?$output_processor@_WV?$string_output_adapter@_W@__crt_stdio_output@@V?$standard_base@_WV?$string_output_adapter@_W@__crt_stdio_output@@@2@@__crt_stdio_output@@AAE_NQAH@Z 10031482 f i libucrt:output.obj
 0001:000304f8       ?process@?$output_processor@DV?$stream_output_adapter@D@__crt_stdio_output@@V?$standard_base@DV?$stream_output_adapter@D@__crt_stdio_output@@@2@@__crt_stdio_output@@QAEHXZ 100314f8 f i libucrt:output.obj
 0001:0003060c       ?process@?$output_processor@DV?$string_output_adapter@D@__crt_stdio_output@@V?$standard_base@DV?$string_output_adapter@D@__crt_stdio_output@@@2@@__crt_stdio_output@@QAEHXZ 1003160c f i libucrt:output.obj
 0001:00030720       ?process@?$output_processor@_WV?$string_output_adapter@_W@__crt_stdio_output@@V?$standard_base@_WV?$string_output_adapter@_W@__crt_stdio_output@@@2@@__crt_stdio_output@@QAEHXZ 10031720 f i libucrt:output.obj
 0001:0003083c       ?state_case_flag@?$output_processor@DV?$stream_output_adapter@D@__crt_stdio_output@@V?$standard_base@DV?$stream_output_adapter@D@__crt_stdio_output@@@2@@__crt_stdio_output@@AAE_NXZ 1003183c f i libucrt:output.obj
 0001:0003083c       ?state_case_flag@?$output_processor@DV?$string_output_adapter@D@__crt_stdio_output@@V?$standard_base@DV?$string_output_adapter@D@__crt_stdio_output@@@2@@__crt_stdio_output@@AAE_NXZ 1003183c f i libucrt:output.obj
 0001:00030879       ?state_case_flag@?$output_processor@_WV?$string_output_adapter@_W@__crt_stdio_output@@V?$standard_base@_WV?$string_output_adapter@_W@__crt_stdio_output@@@2@@__crt_stdio_output@@AAE_NXZ 10031879 f i libucrt:output.obj
 0001:000308b6       ?state_case_normal@?$output_processor@DV?$stream_output_adapter@D@__crt_stdio_output@@V?$standard_base@DV?$stream_output_adapter@D@__crt_stdio_output@@@2@@__crt_stdio_output@@AAE_NXZ 100318b6 f i libucrt:output.obj
 0001:000308d5       ?state_case_normal@?$output_processor@DV?$string_output_adapter@D@__crt_stdio_output@@V?$standard_base@DV?$string_output_adapter@D@__crt_stdio_output@@@2@@__crt_stdio_output@@AAE_NXZ 100318d5 f i libucrt:output.obj
 0001:000308f4       ?state_case_normal@?$output_processor@_WV?$string_output_adapter@_W@__crt_stdio_output@@V?$standard_base@_WV?$string_output_adapter@_W@__crt_stdio_output@@@2@@__crt_stdio_output@@AAE_NXZ 100318f4 f i libucrt:output.obj
 0001:00030913       ?state_case_normal_common@?$output_processor@DV?$stream_output_adapter@D@__crt_stdio_output@@V?$standard_base@DV?$stream_output_adapter@D@__crt_stdio_output@@@2@@__crt_stdio_output@@AAE_NXZ 10031913 f i libucrt:output.obj
 0001:0003094d       ?state_case_normal_common@?$output_processor@DV?$string_output_adapter@D@__crt_stdio_output@@V?$standard_base@DV?$string_output_adapter@D@__crt_stdio_output@@@2@@__crt_stdio_output@@AAE_NXZ 1003194d f i libucrt:output.obj
 0001:00030977       ?state_case_normal_common@?$output_processor@_WV?$string_output_adapter@_W@__crt_stdio_output@@V?$standard_base@_WV?$string_output_adapter@_W@__crt_stdio_output@@@2@@__crt_stdio_output@@AAE_NXZ 10031977 f i libucrt:output.obj
 0001:00030992       ?state_case_normal_tchar@?$output_processor@DV?$stream_output_adapter@D@__crt_stdio_output@@V?$standard_base@DV?$stream_output_adapter@D@__crt_stdio_output@@@2@@__crt_stdio_output@@AAE_ND@Z 10031992 f i libucrt:output.obj
 0001:000309ff       ?state_case_normal_tchar@?$output_processor@DV?$string_output_adapter@D@__crt_stdio_output@@V?$standard_base@DV?$string_output_adapter@D@__crt_stdio_output@@@2@@__crt_stdio_output@@AAE_ND@Z 100319ff f i libucrt:output.obj
 0001:00030a63       ?state_case_precision@?$output_processor@DV?$string_output_adapter@D@__crt_stdio_output@@V?$standard_base@DV?$string_output_adapter@D@__crt_stdio_output@@@2@@__crt_stdio_output@@AAE_NXZ 10031a63 f i libucrt:output.obj
 0001:00030a63       ?state_case_precision@?$output_processor@DV?$stream_output_adapter@D@__crt_stdio_output@@V?$standard_base@DV?$stream_output_adapter@D@__crt_stdio_output@@@2@@__crt_stdio_output@@AAE_NXZ 10031a63 f i libucrt:output.obj
 0001:00030a89       ?state_case_precision@?$output_processor@_WV?$string_output_adapter@_W@__crt_stdio_output@@V?$standard_base@_WV?$string_output_adapter@_W@__crt_stdio_output@@@2@@__crt_stdio_output@@AAE_NXZ 10031a89 f i libucrt:output.obj
 0001:00030ab0       ?state_case_size@?$output_processor@DV?$stream_output_adapter@D@__crt_stdio_output@@V?$standard_base@DV?$stream_output_adapter@D@__crt_stdio_output@@@2@@__crt_stdio_output@@AAE_NXZ 10031ab0 f i libucrt:output.obj
 0001:00030bfe       ?state_case_size@?$output_processor@DV?$string_output_adapter@D@__crt_stdio_output@@V?$standard_base@DV?$string_output_adapter@D@__crt_stdio_output@@@2@@__crt_stdio_output@@AAE_NXZ 10031bfe f i libucrt:output.obj
 0001:00030d4c       ?state_case_size@?$output_processor@_WV?$string_output_adapter@_W@__crt_stdio_output@@V?$standard_base@_WV?$string_output_adapter@_W@__crt_stdio_output@@@2@@__crt_stdio_output@@AAE_NXZ 10031d4c f i libucrt:output.obj
 0001:00030ec4       ?state_case_type@?$output_processor@DV?$stream_output_adapter@D@__crt_stdio_output@@V?$standard_base@DV?$stream_output_adapter@D@__crt_stdio_output@@@2@@__crt_stdio_output@@AAE_NXZ 10031ec4 f i libucrt:output.obj
 0001:000310f6       ?state_case_type@?$output_processor@DV?$string_output_adapter@D@__crt_stdio_output@@V?$standard_base@DV?$string_output_adapter@D@__crt_stdio_output@@@2@@__crt_stdio_output@@AAE_NXZ 100320f6 f i libucrt:output.obj
 0001:00031328       ?state_case_type@?$output_processor@_WV?$string_output_adapter@_W@__crt_stdio_output@@V?$standard_base@_WV?$string_output_adapter@_W@__crt_stdio_output@@@2@@__crt_stdio_output@@AAE_NXZ 10032328 f i libucrt:output.obj
 0001:0003158d       ?state_case_width@?$output_processor@DV?$string_output_adapter@D@__crt_stdio_output@@V?$standard_base@DV?$string_output_adapter@D@__crt_stdio_output@@@2@@__crt_stdio_output@@AAE_NXZ 1003258d f i libucrt:output.obj
 0001:0003158d       ?state_case_width@?$output_processor@DV?$stream_output_adapter@D@__crt_stdio_output@@V?$standard_base@DV?$stream_output_adapter@D@__crt_stdio_output@@@2@@__crt_stdio_output@@AAE_NXZ 1003258d f i libucrt:output.obj
 0001:000315b8       ?state_case_width@?$output_processor@_WV?$string_output_adapter@_W@__crt_stdio_output@@V?$standard_base@_WV?$string_output_adapter@_W@__crt_stdio_output@@@2@@__crt_stdio_output@@AAE_NXZ 100325b8 f i libucrt:output.obj
 0001:000315e4       ?to_integer_size@__crt_stdio_output@@YAIW4length_modifier@1@@Z 100325e4 f i libucrt:output.obj
 0001:00031638       ?type_case_Z@?$output_processor@DV?$stream_output_adapter@D@__crt_stdio_output@@V?$standard_base@DV?$stream_output_adapter@D@__crt_stdio_output@@@2@@__crt_stdio_output@@AAE_NXZ 10032638 f i libucrt:output.obj
 0001:00031638       ?type_case_Z@?$output_processor@DV?$string_output_adapter@D@__crt_stdio_output@@V?$standard_base@DV?$string_output_adapter@D@__crt_stdio_output@@@2@@__crt_stdio_output@@AAE_NXZ 10032638 f i libucrt:output.obj
 0001:00031692       ?type_case_Z@?$output_processor@_WV?$string_output_adapter@_W@__crt_stdio_output@@V?$standard_base@_WV?$string_output_adapter@_W@__crt_stdio_output@@@2@@__crt_stdio_output@@AAE_NXZ 10032692 f i libucrt:output.obj
 0001:000316ec       ?type_case_a@?$output_processor@DV?$string_output_adapter@D@__crt_stdio_output@@V?$standard_base@DV?$string_output_adapter@D@__crt_stdio_output@@@2@@__crt_stdio_output@@AAE_NXZ 100326ec f i libucrt:output.obj
 0001:000316ec       ?type_case_a@?$output_processor@DV?$stream_output_adapter@D@__crt_stdio_output@@V?$standard_base@DV?$stream_output_adapter@D@__crt_stdio_output@@@2@@__crt_stdio_output@@AAE_NXZ 100326ec f i libucrt:output.obj
 0001:0003183b       ?type_case_a@?$output_processor@_WV?$string_output_adapter@_W@__crt_stdio_output@@V?$standard_base@_WV?$string_output_adapter@_W@__crt_stdio_output@@@2@@__crt_stdio_output@@AAE_NXZ 1003283b f i libucrt:output.obj
 0001:000319a0       ?type_case_c_tchar@?$output_processor@DV?$string_output_adapter@D@__crt_stdio_output@@V?$standard_base@DV?$string_output_adapter@D@__crt_stdio_output@@@2@@__crt_stdio_output@@AAE_ND@Z 100329a0 f i libucrt:output.obj
 0001:000319a0       ?type_case_c_tchar@?$output_processor@DV?$stream_output_adapter@D@__crt_stdio_output@@V?$standard_base@DV?$stream_output_adapter@D@__crt_stdio_output@@@2@@__crt_stdio_output@@AAE_ND@Z 100329a0 f i libucrt:output.obj
 0001:00031a30       ?type_case_c_tchar@?$output_processor@_WV?$string_output_adapter@_W@__crt_stdio_output@@V?$standard_base@_WV?$string_output_adapter@_W@__crt_stdio_output@@@2@@__crt_stdio_output@@AAE_N_W@Z 10032a30 f i libucrt:output.obj
 0001:00031ac6       ?type_case_integer@?$output_processor@DV?$stream_output_adapter@D@__crt_stdio_output@@V?$standard_base@DV?$stream_output_adapter@D@__crt_stdio_output@@@2@@__crt_stdio_output@@AAE_NI_N@Z 10032ac6 f i libucrt:output.obj
 0001:00031ac6       ?type_case_integer@?$output_processor@DV?$string_output_adapter@D@__crt_stdio_output@@V?$standard_base@DV?$string_output_adapter@D@__crt_stdio_output@@@2@@__crt_stdio_output@@AAE_NI_N@Z 10032ac6 f i libucrt:output.obj
 0001:00031c17       ?type_case_integer@?$output_processor@_WV?$string_output_adapter@_W@__crt_stdio_output@@V?$standard_base@_WV?$string_output_adapter@_W@__crt_stdio_output@@@2@@__crt_stdio_output@@AAE_NI_N@Z 10032c17 f i libucrt:output.obj
 0001:00031d6c       ?type_case_n@?$output_processor@DV?$stream_output_adapter@D@__crt_stdio_output@@V?$standard_base@DV?$stream_output_adapter@D@__crt_stdio_output@@@2@@__crt_stdio_output@@AAE_NXZ 10032d6c f i libucrt:output.obj
 0001:00031d6c       ?type_case_n@?$output_processor@DV?$string_output_adapter@D@__crt_stdio_output@@V?$standard_base@DV?$string_output_adapter@D@__crt_stdio_output@@@2@@__crt_stdio_output@@AAE_NXZ 10032d6c f i libucrt:output.obj
 0001:00031d6c       ?type_case_n@?$output_processor@_WV?$string_output_adapter@_W@__crt_stdio_output@@V?$standard_base@_WV?$string_output_adapter@_W@__crt_stdio_output@@@2@@__crt_stdio_output@@AAE_NXZ 10032d6c f i libucrt:output.obj
 0001:00031de0       ?type_case_o@?$output_processor@DV?$stream_output_adapter@D@__crt_stdio_output@@V?$standard_base@DV?$stream_output_adapter@D@__crt_stdio_output@@@2@@__crt_stdio_output@@AAE_NXZ 10032de0 f i libucrt:output.obj
 0001:00031de0       ?type_case_o@?$output_processor@DV?$string_output_adapter@D@__crt_stdio_output@@V?$standard_base@DV?$string_output_adapter@D@__crt_stdio_output@@@2@@__crt_stdio_output@@AAE_NXZ 10032de0 f i libucrt:output.obj
 0001:00031dff       ?type_case_o@?$output_processor@_WV?$string_output_adapter@_W@__crt_stdio_output@@V?$standard_base@_WV?$string_output_adapter@_W@__crt_stdio_output@@@2@@__crt_stdio_output@@AAE_NXZ 10032dff f i libucrt:output.obj
 0001:00031e1e       ?type_case_p@?$output_processor@DV?$stream_output_adapter@D@__crt_stdio_output@@V?$standard_base@DV?$stream_output_adapter@D@__crt_stdio_output@@@2@@__crt_stdio_output@@AAE_NXZ 10032e1e f i libucrt:output.obj
 0001:00031e1e       ?type_case_p@?$output_processor@DV?$string_output_adapter@D@__crt_stdio_output@@V?$standard_base@DV?$string_output_adapter@D@__crt_stdio_output@@@2@@__crt_stdio_output@@AAE_NXZ 10032e1e f i libucrt:output.obj
 0001:00031e36       ?type_case_p@?$output_processor@_WV?$string_output_adapter@_W@__crt_stdio_output@@V?$standard_base@_WV?$string_output_adapter@_W@__crt_stdio_output@@@2@@__crt_stdio_output@@AAE_NXZ 10032e36 f i libucrt:output.obj
 0001:00031e4e       ?type_case_s@?$output_processor@DV?$string_output_adapter@D@__crt_stdio_output@@V?$standard_base@DV?$string_output_adapter@D@__crt_stdio_output@@@2@@__crt_stdio_output@@AAE_NXZ 10032e4e f i libucrt:output.obj
 0001:00031e4e       ?type_case_s@?$output_processor@DV?$stream_output_adapter@D@__crt_stdio_output@@V?$standard_base@DV?$stream_output_adapter@D@__crt_stdio_output@@@2@@__crt_stdio_output@@AAE_NXZ 10032e4e f i libucrt:output.obj
 0001:00031ebf       ?type_case_s@?$output_processor@_WV?$string_output_adapter@_W@__crt_stdio_output@@V?$standard_base@_WV?$string_output_adapter@_W@__crt_stdio_output@@@2@@__crt_stdio_output@@AAE_NXZ 10032ebf f i libucrt:output.obj
 0001:00031f32       ?type_case_s_compute_narrow_string_length@?$output_processor@_WV?$string_output_adapter@_W@__crt_stdio_output@@V?$standard_base@_WV?$string_output_adapter@_W@__crt_stdio_output@@@2@@__crt_stdio_output@@ABEHH_W@Z 10032f32 f i libucrt:output.obj
 0001:00031f79       ?validate@?$stream_input_adapter@D@__crt_stdio_input@@QBE_NXZ 10032f79 f i libucrt:input.obj
 0001:00031f79       ?validate@?$stream_output_adapter@D@__crt_stdio_output@@QBE_NXZ 10032f79 f i libucrt:output.obj
 0001:00031f9a       ?validate@?$string_output_adapter@_W@__crt_stdio_output@@QBE_NXZ 10032f9a f i libucrt:output.obj
 0001:00031f9a       ?validate@?$c_string_character_source@_W@__crt_strtox@@QBE_NXZ 10032f9a f i libucrt:atox.obj
 0001:00031f9a       ?validate@?$string_output_adapter@D@__crt_stdio_output@@QBE_NXZ 10032f9a f i libucrt:output.obj
 0001:00031f9a       ?validate@?$c_string_character_source@D@__crt_strtox@@QBE_NXZ 10032f9a f i libucrt:atox.obj
 0001:00031fb5       ?validate_stream_is_ansi_if_required@?$__acrt_stdio_char_traits@D@@SA_NQAU_iobuf@@@Z 10032fb5 f i libucrt:output.obj
 0001:0003203c       ?write_character@?$string_output_adapter@D@__crt_stdio_output@@QBE_NDQAH@Z 1003303c f i libucrt:output.obj
 0001:0003207e       ?write_character@?$string_output_adapter@_W@__crt_stdio_output@@QBE_N_WQAH@Z 1003307e f i libucrt:output.obj
 0001:000320c3       ?write_character_without_count_update@?$stream_output_adapter@D@__crt_stdio_output@@QBE_ND@Z 100330c3 f i libucrt:output.obj
 0001:000320f9       ?write_stored_string_tchar@?$output_processor@DV?$stream_output_adapter@D@__crt_stdio_output@@V?$standard_base@DV?$stream_output_adapter@D@__crt_stdio_output@@@2@@__crt_stdio_output@@AAE_ND@Z 100330f9 f i libucrt:output.obj
 0001:000321a0       ?write_stored_string_tchar@?$output_processor@DV?$string_output_adapter@D@__crt_stdio_output@@V?$standard_base@DV?$string_output_adapter@D@__crt_stdio_output@@@2@@__crt_stdio_output@@AAE_ND@Z 100331a0 f i libucrt:output.obj
 0001:00032247       ?write_stored_string_tchar@?$output_processor@_WV?$string_output_adapter@_W@__crt_stdio_output@@V?$standard_base@_WV?$string_output_adapter@_W@__crt_stdio_output@@@2@@__crt_stdio_output@@AAE_N_W@Z 10033247 f i libucrt:output.obj
 0001:000322da       ?write_string@?$stream_output_adapter@D@__crt_stdio_output@@QBEXQBDHQAHAAV__crt_deferred_errno_cache@@@Z 100332da f i libucrt:output.obj
 0001:00032306       ?write_string@?$string_output_adapter@D@__crt_stdio_output@@QBEXQBDHQAHAAV__crt_deferred_errno_cache@@@Z 10033306 f i libucrt:output.obj
 0001:0003236d       ?write_string@?$string_output_adapter@_W@__crt_stdio_output@@QBEXQB_WHQAHAAV__crt_deferred_errno_cache@@@Z 1003336d f i libucrt:output.obj
 0001:000323de       ?write_string_impl@?$output_adapter_common@DV?$stream_output_adapter@D@__crt_stdio_output@@@__crt_stdio_output@@IBEXQBDHQAHAAV__crt_deferred_errno_cache@@@Z 100333de f i libucrt:output.obj
 0001:0003247c       ___acrt_locale_get_ctype_array_value 1003347c f i libucrt:output.obj
 0001:0003249e       ___stdio_common_vfprintf   1003349e f   libucrt:output.obj
 0001:00032521       ___stdio_common_vsprintf   10033521 f   libucrt:output.obj
 0001:00032545       ___stdio_common_vswprintf  10033545 f   libucrt:output.obj
 0001:00032569       __fclose_nolock            10033569 f   libucrt:fclose.obj
 0001:000325e0       _fclose                    100335e0 f   libucrt:fclose.obj
 0001:00032664       _wcsdup                    10033664 f   libucrt:wcsdup.obj
 0001:00032664       __wcsdup                   10033664 f   libucrt:wcsdup.obj
 0001:0003276a       __clearfp                  1003376a f   libucrt:ieee87.obj
 0001:00032848       __control87                10033848 f   libucrt:ieee87.obj
 0001:00032c9d       __wfopen                   10033c9d f   libucrt:fopen.obj
 0001:00032cb4       _free                      10033cb4 f   libucrt:free.obj
 0001:00032ccf       _malloc                    10033ccf f   libucrt:malloc.obj
 0001:00032cda       _feof                      10033cda f   libucrt:feoferr.obj
 0001:00032d06       _ferror                    10033d06 f   libucrt:feoferr.obj
 0001:00032d32       ___acrt_initialize_stdio   10033d32 f   libucrt:_file.obj
 0001:00032dfa       ___acrt_iob_func           10033dfa f   libucrt:_file.obj
 0001:00032e0a       ___acrt_uninitialize_stdio 10033e0a f   libucrt:_file.obj
 0001:00032e56       __lock_file                10033e56 f   libucrt:_file.obj
 0001:00032e6a       __unlock_file              10033e6a f   libucrt:_file.obj
 0001:00032e7e       __fgetc_nolock             10033e7e f   libucrt:fgetc.obj
 0001:00032eba       __getc_nolock              10033eba f   libucrt:fgetc.obj
 0001:00032ec5       _fgetc                     10033ec5 f   libucrt:fgetc.obj
 0001:00032fcd       _getc                      10033fcd f   libucrt:fgetc.obj
 0001:000330e1       __wfreopen                 100340e1 f   libucrt:freopen.obj
 0001:00033107       _rewind                    10034107 f   libucrt:rewind.obj
 0001:000331d4       ___acrt_errno_from_os_error 100341d4 f   libucrt:errno.obj
 0001:00033217       ___acrt_errno_map_os_error 10034217 f   libucrt:errno.obj
 0001:0003323a       ___doserrno                1003423a f   libucrt:errno.obj
 0001:0003324d       __errno                    1003424d f   libucrt:errno.obj
 0001:00033260       __ungetc_nolock            10034260 f   libucrt:ungetc.obj
 0001:0003335a       _ungetc                    1003435a f   libucrt:ungetc.obj
 0001:000333cd       __fread_nolock_s           100343cd f   libucrt:fread.obj
 0001:000335b3       _fread                     100345b3 f   libucrt:fread.obj
 0001:000335d0       _fread_s                   100345d0 f   libucrt:fread.obj
 0001:00033763       __get_sys_err_msg          10034763 f i libucrt:strerror.obj
 0001:00033787       _strerror                  10034787 f   libucrt:strerror.obj
 0001:00033792       ___ascii_wcsicmp           10034792 f   libucrt:wcsicmp.obj
 0001:000337cf       __towlower_internal        100347cf f i libucrt:wcsicmp.obj
 0001:0003380e       __wcsicmp                  1003480e f   libucrt:wcsicmp.obj
 0001:00033857       __wcsicmp_l                10034857 f   libucrt:wcsicmp.obj
 0001:0003390f       _iswctype                  1003490f f   libucrt:iswctype.obj
 0001:00033978       _wcsncpy                   10034978 f   libucrt:wcsncpy.obj
 0001:000339c0       _strncmp                   100349c0 f   libucrt:strncmp.obj
 0001:00033a38       __ischartype_l             10034a38 f i libucrt:_ctype.obj
 0001:00033a8c       __isdigit_l                10034a8c f i libucrt:_ctype.obj
 0001:00033ac2       __isspace_l                10034ac2 f i libucrt:_ctype.obj
 0001:00033af8       _isdigit                   10034af8 f i libucrt:_ctype.obj
 0001:00033b29       _isspace                   10034b29 f i libucrt:_ctype.obj
 0001:00033b60       _strncpy                   10034b60 f   libucrt:strncpy.obj
 0001:00033c90       _strpbrk                   10034c90 f   libucrt:strpbrk.obj
 0001:00034226       ?__crt_stdio_path_requires_backslash@@YA_NQB_W@Z 10035226 f i libucrt:popen.obj
 0001:000342d2       __pclose                   100352d2 f   libucrt:popen.obj
 0001:000343a9       __wpopen                   100353a9 f   libucrt:popen.obj
 0001:000345f1       ___acrt_stdio_flush_nolock 100355f1 f   libucrt:fflush.obj
 0001:00034656       __fflush_nolock            10035656 f   libucrt:fflush.obj
 0001:0003469e       __flushall                 1003569e f   libucrt:fflush.obj
 0001:000346a7       _fflush                    100356a7 f   libucrt:fflush.obj
 0001:000346fc       _clearerr                  100356fc f   libucrt:clearerr.obj
 0001:00034701       _clearerr_s                10035701 f   libucrt:clearerr.obj
 0001:0003486e       _fgets                     1003586e f   libucrt:fgets.obj
 0001:00034bae       ___acrt_stdio_free_tmpfile_name_buffers_nolock 10035bae f   libucrt:tmpfile.obj
 0001:00034c09       _tmpfile                   10035c09 f   libucrt:tmpfile.obj
 0001:00034cc3       __fwrite_nolock            10035cc3 f   libucrt:fwrite.obj
 0001:00034e44       _fwrite                    10035e44 f   libucrt:fwrite.obj
 0001:00034fcf       _setvbuf                   10035fcf f   libucrt:setvbuf.obj
 0001:000350ac       ??$assemble_floating_point_snan@N@__crt_strtox@@YAX_NAAN@Z 100360ac f i libucrt:input.obj
 0001:000350cd       ??$assemble_floating_point_value_t@M@__crt_strtox@@YA?AW4SLD_STATUS@@_NH_KAAM@Z 100360cd f i libucrt:input.obj
 0001:000350fd       ??$assemble_floating_point_value_t@N@__crt_strtox@@YA?AW4SLD_STATUS@@_NH_KAAN@Z 100360fd f i libucrt:input.obj
 0001:0003513f       ??$convert_decimal_string_to_floating_type@M@__crt_strtox@@YA?AW4SLD_STATUS@@ABUfloating_point_string@0@AAM@Z 1003613f f i libucrt:input.obj
 0001:00035160       ??$convert_decimal_string_to_floating_type@N@__crt_strtox@@YA?AW4SLD_STATUS@@ABUfloating_point_string@0@AAN@Z 10036160 f i libucrt:input.obj
 0001:00035181       ??$convert_hexadecimal_string_to_floating_type@M@__crt_strtox@@YA?AW4SLD_STATUS@@ABUfloating_point_string@0@AAM@Z 10036181 f i libucrt:input.obj
 0001:000351a2       ??$convert_hexadecimal_string_to_floating_type@N@__crt_strtox@@YA?AW4SLD_STATUS@@ABUfloating_point_string@0@AAN@Z 100361a2 f i libucrt:input.obj
 0001:000351c3       ??$is_overflow_condition@_K@__crt_strtox@@YA_NI_K@Z 100361c3 f i libucrt:input.obj
 0001:00035204       ??$make_input_adapter_character_source@V?$stream_input_adapter@D@__crt_stdio_input@@@__crt_strtox@@YA?AV?$input_adapter_character_source@V?$stream_input_adapter@D@__crt_stdio_input@@@0@QAV?$stream_input_adapter@D@__crt_stdio_input@@_KQA_N@Z 10036204 f i libucrt:input.obj
 0001:00035222       ??$parse_floating_point@V?$input_adapter_character_source@V?$stream_input_adapter@D@__crt_stdio_input@@@__crt_strtox@@M@__crt_strtox@@YA?AW4SLD_STATUS@@QAU__crt_locale_pointers@@V?$input_adapter_character_source@V?$stream_input_adapter@D@__crt_stdio_input@@@0@QAM@Z 10036222 f i libucrt:input.obj
 0001:0003529b       ??$parse_floating_point@V?$input_adapter_character_source@V?$stream_input_adapter@D@__crt_stdio_input@@@__crt_strtox@@N@__crt_strtox@@YA?AW4SLD_STATUS@@QAU__crt_locale_pointers@@V?$input_adapter_character_source@V?$stream_input_adapter@D@__crt_stdio_input@@@0@QAN@Z 1003629b f i libucrt:input.obj
 0001:00035314       ??$parse_floating_point_from_source@V?$input_adapter_character_source@V?$stream_input_adapter@D@__crt_stdio_input@@@__crt_strtox@@@__crt_strtox@@YA?AW4floating_point_parse_result@0@QAU__crt_locale_pointers@@AAV?$input_adapter_character_source@V?$stream_input_adapter@D@__crt_stdio_input@@@0@AAUfloating_point_string@0@@Z 10036314 f i libucrt:input.obj
 0001:00035771       ??$parse_floating_point_possible_infinity@DV?$input_adapter_character_source@V?$stream_input_adapter@D@__crt_stdio_input@@@__crt_strtox@@_K@__crt_strtox@@YA?AW4floating_point_parse_result@0@AADAAV?$input_adapter_character_source@V?$stream_input_adapter@D@__crt_stdio_input@@@0@_K@Z 10036771 f i libucrt:input.obj
 0001:00035830       ??$parse_floating_point_possible_nan@DV?$input_adapter_character_source@V?$stream_input_adapter@D@__crt_stdio_input@@@__crt_strtox@@_K@__crt_strtox@@YA?AW4floating_point_parse_result@0@AADAAV?$input_adapter_character_source@V?$stream_input_adapter@D@__crt_stdio_input@@@0@_K@Z 10036830 f i libucrt:input.obj
 0001:0003594b       ??$parse_floating_point_possible_nan_is_ind@DV?$input_adapter_character_source@V?$stream_input_adapter@D@__crt_stdio_input@@@__crt_strtox@@@__crt_strtox@@YA_NAADAAV?$input_adapter_character_source@V?$stream_input_adapter@D@__crt_stdio_input@@@0@@Z 1003694b f i libucrt:input.obj
 0001:00035985       ??$parse_floating_point_possible_nan_is_snan@DV?$input_adapter_character_source@V?$stream_input_adapter@D@__crt_stdio_input@@@__crt_strtox@@@__crt_strtox@@YA_NAADAAV?$input_adapter_character_source@V?$stream_input_adapter@D@__crt_stdio_input@@@0@@Z 10036985 f i libucrt:input.obj
 0001:000359bf       ??$parse_floating_point_write_result@M@__crt_strtox@@YA?AW4SLD_STATUS@@W4floating_point_parse_result@0@ABUfloating_point_string@0@QAM@Z 100369bf f i libucrt:input.obj
 0001:00035b2b       ??$parse_floating_point_write_result@N@__crt_strtox@@YA?AW4SLD_STATUS@@W4floating_point_parse_result@0@ABUfloating_point_string@0@QAN@Z 10036b2b f i libucrt:input.obj
 0001:00035c4f       ??$parse_integer@_KV?$input_adapter_character_source@V?$stream_input_adapter@D@__crt_stdio_input@@@__crt_strtox@@@__crt_strtox@@YA_KQAU__crt_locale_pointers@@V?$input_adapter_character_source@V?$stream_input_adapter@D@__crt_stdio_input@@@0@H_N@Z 10036c4f f i libucrt:input.obj
 0001:00035f0d       ??$process_floating_point_specifier_t@M@?$input_processor@DV?$stream_input_adapter@D@__crt_stdio_input@@@__crt_stdio_input@@AAE_NXZ 10036f0d f i libucrt:input.obj
 0001:00035f73       ??$process_floating_point_specifier_t@N@?$input_processor@DV?$stream_input_adapter@D@__crt_stdio_input@@@__crt_stdio_input@@AAE_NXZ 10036f73 f i libucrt:input.obj
 0001:00035fd9       ??$process_string_specifier_tchar@D@?$input_processor@DV?$stream_input_adapter@D@__crt_stdio_input@@@__crt_stdio_input@@AAE_NW4conversion_mode@1@D@Z 10036fd9 f i libucrt:input.obj
 0001:0003614a       ??$process_string_specifier_tchar@_W@?$input_processor@DV?$stream_input_adapter@D@__crt_stdio_input@@@__crt_stdio_input@@AAE_NW4conversion_mode@1@_W@Z 1003714a f i libucrt:input.obj
 0001:000362c5       ??$skip_whitespace@Vstream_input_adapter@__crt_stdio_input@@D@__crt_stdio_input@@YAHAAV?$stream_input_adapter@D@0@QAU__crt_locale_pointers@@@Z 100372c5 f i libucrt:input.obj
 0001:000362fc       ??$write_floating_point@M@?$input_processor@DV?$stream_input_adapter@D@__crt_stdio_input@@@__crt_stdio_input@@AAE_NABM@Z 100372fc f i libucrt:input.obj
 0001:00036330       ??$write_floating_point@N@?$input_processor@DV?$stream_input_adapter@D@__crt_stdio_input@@@__crt_stdio_input@@AAE_NABN@Z 10037330 f i libucrt:input.obj
 0001:0003636a       ??0?$format_string_parser@D@__crt_stdio_input@@QAE@_KQBE@Z 1003736a f i libucrt:input.obj
 0001:000363b4       ??0?$input_adapter_character_source@V?$stream_input_adapter@D@__crt_stdio_input@@@__crt_strtox@@QAE@QAV?$stream_input_adapter@D@__crt_stdio_input@@_KQA_N@Z 100373b4 f i libucrt:input.obj
 0001:000363e5       ??0?$input_processor@DV?$stream_input_adapter@D@__crt_stdio_input@@@__crt_stdio_input@@QAE@ABV?$stream_input_adapter@D@1@_KQBDQAU__crt_locale_pointers@@QAD@Z 100373e5 f i libucrt:input.obj
 0001:000364d8       ?advance@?$format_string_parser@D@__crt_stdio_input@@QAE_NXZ 100374d8 f i libucrt:input.obj
 0001:000365f0       ?as_double@floating_point_value@__crt_strtox@@QBEAANXZ 100375f0 f i libucrt:input.obj
 0001:00036615       ?as_float@floating_point_value@__crt_strtox@@QBEAAMXZ 10037615 f i libucrt:input.obj
 0001:0003663a       ?assemble_floating_point_infinity@__crt_strtox@@YAX_NABVfloating_point_value@1@@Z 1003763a f i libucrt:input.obj
 0001:0003667a       ?assemble_floating_point_value@__crt_strtox@@YA?AW4SLD_STATUS@@_KH_N1ABVfloating_point_value@1@@Z 1003767a f i libucrt:input.obj
 0001:000369c3       ?assemble_floating_point_value_from_big_integer@__crt_strtox@@YA?AW4SLD_STATUS@@ABUbig_integer@1@I_N1ABVfloating_point_value@1@@Z 100379c3 f i libucrt:input.obj
 0001:00036b57       ?assemble_floating_point_zero@__crt_strtox@@YAX_NABVfloating_point_value@1@@Z 10037b57 f i libucrt:input.obj
 0001:00036b8c       ?convert_decimal_string_to_floating_type_common@__crt_strtox@@YA?AW4SLD_STATUS@@ABUfloating_point_string@1@ABVfloating_point_value@1@@Z 10037b8c f i libucrt:input.obj
 0001:000388cb       ?convert_hexadecimal_string_to_floating_type_common@__crt_strtox@@YA?AW4SLD_STATUS@@ABUfloating_point_string@1@ABVfloating_point_value@1@@Z 100398cb f i libucrt:input.obj
 0001:00038971       ?denormal_mantissa_mask@floating_point_value@__crt_strtox@@QBE_KXZ 10039971 f i libucrt:input.obj
 0001:00038990       ?divide@__crt_strtox@@YA_KAAUbig_integer@1@ABU21@@Z 10039990 f i libucrt:input.obj
 0001:00038e28       ?get@?$input_adapter_character_source@V?$stream_input_adapter@D@__crt_stdio_input@@@__crt_strtox@@QAEDXZ 10039e28 f i libucrt:input.obj
 0001:00038e67       ?invert@?$scanset_buffer@E@__crt_stdio_input@@QAEXXZ 10039e67 f i libucrt:input.obj
 0001:00038e85       ?is_character_allowed_in_string@?$input_processor@DV?$stream_input_adapter@D@__crt_stdio_input@@@__crt_stdio_input@@ABE_NW4conversion_mode@2@H@Z 10039e85 f i libucrt:input.obj
 0001:00038ed5       ?length@?$format_string_parser@D@__crt_stdio_input@@QBEIXZ 10039ed5 f i libucrt:input.obj
 0001:00038f16       ?normal_mantissa_mask@floating_point_value@__crt_strtox@@QBE_KXZ 10039f16 f i libucrt:input.obj
 0001:00038f2d       ?process@?$input_processor@DV?$stream_input_adapter@D@__crt_stdio_input@@@__crt_stdio_input@@QAEHXZ 10039f2d f i libucrt:input.obj
 0001:00038fb8       ?process_character_count_specifier@?$input_processor@DV?$stream_input_adapter@D@__crt_stdio_input@@@__crt_stdio_input@@AAE_NXZ 10039fb8 f i libucrt:input.obj
 0001:00038fcc       ?process_conversion_specifier@?$input_processor@DV?$stream_input_adapter@D@__crt_stdio_input@@@__crt_stdio_input@@AAE_NXZ 10039fcc f i libucrt:input.obj
 0001:00039040       ?process_floating_point_specifier@?$input_processor@DV?$stream_input_adapter@D@__crt_stdio_input@@@__crt_stdio_input@@AAE_NXZ 1003a040 f i libucrt:input.obj
 0001:00039070       ?process_integer_specifier@?$input_processor@DV?$stream_input_adapter@D@__crt_stdio_input@@@__crt_stdio_input@@AAE_NI_N@Z 1003a070 f i libucrt:input.obj
 0001:000390d2       ?process_literal_character@?$input_processor@DV?$stream_input_adapter@D@__crt_stdio_input@@@__crt_stdio_input@@AAE_NXZ 1003a0d2 f i libucrt:input.obj
 0001:00039108       ?process_literal_character_tchar@?$input_processor@DV?$stream_input_adapter@D@__crt_stdio_input@@@__crt_stdio_input@@AAE_ND@Z 1003a108 f i libucrt:input.obj
 0001:0003915f       ?process_state@?$input_processor@DV?$stream_input_adapter@D@__crt_stdio_input@@@__crt_stdio_input@@AAE_NXZ 1003a15f f i libucrt:input.obj
 0001:000391a1       ?process_string_specifier@?$input_processor@DV?$stream_input_adapter@D@__crt_stdio_input@@@__crt_stdio_input@@AAE_NW4conversion_mode@2@@Z 1003a1a1 f i libucrt:input.obj
 0001:000391e9       ?process_whitespace@?$input_processor@DV?$stream_input_adapter@D@__crt_stdio_input@@@__crt_stdio_input@@AAE_NXZ 1003a1e9 f i libucrt:input.obj
 0001:00039206       ?restore_state@?$input_adapter_character_source@V?$stream_input_adapter@D@__crt_stdio_input@@@__crt_strtox@@QAE_N_K@Z 1003a206 f i libucrt:input.obj
 0001:0003922b       ?scan_conversion_specifier@?$format_string_parser@D@__crt_stdio_input@@AAE_NXZ 1003a22b f i libucrt:input.obj
 0001:0003939b       ?scan_optional_field_width@?$format_string_parser@D@__crt_stdio_input@@AAE_NXZ 1003a39b f i libucrt:input.obj
 0001:00039438       ?scan_optional_length_modifier@?$format_string_parser@D@__crt_stdio_input@@AAEXXZ 1003a438 f i libucrt:input.obj
 0001:00039547       ?scan_optional_literal_character_trail_bytes_tchar@?$format_string_parser@D@__crt_stdio_input@@AAE_ND@Z 1003a547 f i libucrt:input.obj
 0001:00039599       ?scan_optional_wide_modifier@?$format_string_parser@D@__crt_stdio_input@@AAEXXZ 1003a599 f i libucrt:input.obj
 0001:000395b7       ?scan_scanset_range@?$format_string_parser@D@__crt_stdio_input@@AAE_NXZ 1003a5b7 f i libucrt:input.obj
 0001:000396ef       ?set_wide_for_c_s_or_scanset@?$format_string_parser@D@__crt_stdio_input@@AAEXXZ 1003a6ef f i libucrt:input.obj
 0001:0003970f       ?to_floating_point_length@__crt_stdio_input@@YAIW4length_modifier@1@@Z 1003a70f f i libucrt:input.obj
 0001:00039732       ?to_integer_length@__crt_stdio_input@@YAIW4length_modifier@1@@Z 1003a732 f i libucrt:input.obj
 0001:00039785       ?unget@?$input_adapter_character_source@V?$stream_input_adapter@D@__crt_stdio_input@@@__crt_strtox@@QAEXD@Z 1003a785 f i libucrt:input.obj
 0001:000397cc       ?unget@?$stream_input_adapter@D@__crt_stdio_input@@QAEXH@Z 1003a7cc f i libucrt:input.obj
 0001:000397ea       ?validate@?$format_string_parser@D@__crt_stdio_input@@QBE_NXZ 1003a7ea f i libucrt:input.obj
 0001:00039806       ?validate@?$input_adapter_character_source@V?$stream_input_adapter@D@__crt_stdio_input@@@__crt_strtox@@QBE_NXZ 1003a806 f i libucrt:input.obj
 0001:00039827       ?write_character@?$input_processor@DV?$stream_input_adapter@D@__crt_stdio_input@@@__crt_stdio_input@@AAE_NQA_WIAAPA_WAAID@Z 1003a827 f i libucrt:input.obj
 0001:0003989d       ?write_integer@?$input_processor@DV?$stream_input_adapter@D@__crt_stdio_input@@@__crt_stdio_input@@AAE_N_K@Z 1003a89d f i libucrt:input.obj
 0001:0003990b       ___stdio_common_vfscanf    1003a90b f   libucrt:input.obj
 0001:00039f68       __ftelli64                 1003af68 f   libucrt:ftell.obj
 0001:00039f73       __ftelli64_nolock          1003af73 f   libucrt:ftell.obj
 0001:00039f7e       ?LongLongSub@@YAJ_J0PA_J@Z 1003af7e f i libucrt:fseek.obj
 0001:0003a23a       __fseeki64                 1003b23a f   libucrt:fseek.obj
 0001:0003a469       __wdupenv_s                1003b469 f   libucrt:getenv.obj
 0001:0003a487       __wgetenv                  1003b487 f   libucrt:getenv.obj
 0001:0003a590       __wsystem                  1003b590 f   libucrt:system.obj
 0001:0003a59b       _wcscmp                    1003b59b f   libucrt:wcscmp.obj
 0001:0003a5db       __seh_filter_dll           1003b5db f   libucrt:exception_filter.obj
 0001:0003a5fb       __seh_filter_exe           1003b5fb f   libucrt:exception_filter.obj
 0001:0003a9c9       ___acrt_initialize_thread_local_exit_callback 1003b9c9 f   libucrt:exit.obj
 0001:0003a9d8       __cexit                    1003b9d8 f   libucrt:exit.obj
 0001:0003a9e7       __exit                     1003b9e7 f   libucrt:exit.obj
 0001:0003a9fd       __is_c_termination_complete 1003b9fd f   libucrt:exit.obj
 0001:0003acb1       ___acrt_allocate_buffer_for_argv 1003bcb1 f   libucrt:argv_parsing.obj
 0001:0003ad00       __configure_narrow_argv    1003bd00 f   libucrt:argv_parsing.obj
 0001:0003b061       ??$uninitialize@A6AXAAPAPAD@Z@?$dual_state_global@PAPAD@__crt_state_management@@QAEXA6AXAAPAPAD@Z@Z 1003c061 f i libucrt:environment_initialization.obj
 0001:0003b061       ??$uninitialize@A6AXAAPAPA_W@Z@?$dual_state_global@PAPA_W@__crt_state_management@@QAEXA6AXAAPAPA_W@Z@Z 1003c061 f i libucrt:environment_initialization.obj
 0001:0003b0c0       ___dcrt_get_or_create_wide_environment_nolock 1003c0c0 f   libucrt:environment_initialization.obj
 0001:0003b0c5       ___dcrt_uninitialize_environments_nolock 1003c0c5 f   libucrt:environment_initialization.obj
 0001:0003b0fc       __initialize_narrow_environment 1003c0fc f   libucrt:environment_initialization.obj
 0001:0003b1b7       ??$__crt_fast_encode_pointer@PAP6AXXZ@@YAPAP6AXXZQAP6AXXZ@Z 1003c1b7 f i libucrt:onexit.obj
 0001:0003b1b7       ??$__crt_fast_encode_pointer@PAX@@YAPAXQAX@Z 1003c1b7 f i libucrt:initialization.obj
 0001:0003b1b7       ??$__crt_fast_encode_pointer@P6AHXZ@@YAP6AHXZQ6AHXZ@Z 1003c1b7 f i libucrt:onexit.obj
 0001:0003b3d9       __crt_atexit               1003c3d9 f   libucrt:onexit.obj
 0001:0003b3ef       __execute_onexit_table     1003c3ef f   libucrt:onexit.obj
 0001:0003b41c       __initialize_onexit_table  1003c41c f   libucrt:onexit.obj
 0001:0003b445       __register_onexit_function 1003c445 f   libucrt:onexit.obj
 0001:0003b478       ___acrt_uninitialize_command_line 1003c478 f   libucrt:argv_data.obj
 0001:0003b576       ___acrt_initialize         1003c576 f   libucrt:initialization.obj
 0001:0003b588       ___acrt_thread_attach      1003c588 f   libucrt:initialization.obj
 0001:0003b593       ___acrt_thread_detach      1003c593 f   libucrt:initialization.obj
 0001:0003b59b       ___acrt_uninitialize       1003c59b f   libucrt:initialization.obj
 0001:0003b5cb       ___acrt_uninitialize_critical 1003c5cb f   libucrt:initialization.obj
 0001:0003b5dd       __initterm                 1003c5dd f   libucrt:initterm.obj
 0001:0003b622       __initterm_e               1003c622 f   libucrt:initterm.obj
 0001:0003b650       _terminate                 1003c650 f   libucrt:terminate.obj
 0001:0003b7f8       __freea_crt                1003c7f8 f i libucrt:strupr.obj
 0001:0003b818       __strupr                   1003c818 f   libucrt:strupr.obj
 0001:0003b818       _strupr                    1003c818 f   libucrt:strupr.obj
 0001:0003b874       __strupr_s_l               1003c874 f   libucrt:strupr.obj
 0001:0003b8ab       ___ascii_stricmp           1003c8ab f   libucrt:stricmp.obj
 0001:0003b8e4       __stricmp                  1003c8e4 f   libucrt:stricmp.obj
 0001:0003b8e4       _stricmp                   1003c8e4 f   libucrt:stricmp.obj
 0001:0003b92d       __stricmp_l                1003c92d f   libucrt:stricmp.obj
 0001:0003b9bb       _abort                     1003c9bb f   libucrt:abort.obj
 0001:0003b9ff       _strcpy_s                  1003c9ff f   libucrt:strcpy_s.obj
 0001:0003ba59       _calloc                    1003ca59 f   libucrt:calloc.obj
 0001:0003ba64       ??$is_overflow_condition@K@__crt_strtox@@YA_NIK@Z 1003ca64 f i libucrt:atox.obj
 0001:0003ba95       ??$parse_integer@KV?$c_string_character_source@D@__crt_strtox@@@__crt_strtox@@YAKQAU__crt_locale_pointers@@V?$c_string_character_source@D@0@H_N@Z 1003ca95 f i libucrt:atox.obj
 0001:0003bcba       ??$parse_integer@KV?$c_string_character_source@_W@__crt_strtox@@@__crt_strtox@@YAKQAU__crt_locale_pointers@@V?$c_string_character_source@_W@0@H_N@Z 1003ccba f i libucrt:atox.obj
 0001:0003c2c2       ??$parse_integer@_KV?$c_string_character_source@D@__crt_strtox@@@__crt_strtox@@YA_KQAU__crt_locale_pointers@@V?$c_string_character_source@D@0@H_N@Z 1003d2c2 f i libucrt:atox.obj
 0001:0003c568       ?unget@?$c_string_character_source@D@__crt_strtox@@QAEXD@Z 1003d568 f i libucrt:atox.obj
 0001:0003c591       ?unget@?$c_string_character_source@_W@__crt_strtox@@QAEX_W@Z 1003d591 f i libucrt:atox.obj
 0001:0003c5bf       _wcsncmp                   1003d5bf f   libucrt:wcsncmp.obj
 0001:0003c5f9       ___acrt_call_reportfault   1003d5f9 f   libucrt:invalid_parameter.obj
 0001:0003c732       ___acrt_initialize_invalid_parameter_handler 1003d732 f   libucrt:invalid_parameter.obj
 0001:0003c741       __invalid_parameter        1003d741 f   libucrt:invalid_parameter.obj
 0001:0003c7a5       __invalid_parameter_noinfo 1003d7a5 f   libucrt:invalid_parameter.obj
 0001:0003c7b5       __invoke_watson            1003d7b5 f   libucrt:invalid_parameter.obj
 0001:0003c7e9       __free_base                1003d7e9 f   libucrt:free_base.obj
 0001:0003c823       __malloc_base              1003d823 f   libucrt:malloc_base.obj
 0001:0003c871       ??$make_c_string_character_source@DPAPAD@__crt_strtox@@YA?AV?$c_string_character_source@D@0@QBDQAPAD@Z 1003d871 f i libucrt:strtox.obj
 0001:0003c871       ??$make_c_string_character_source@_WPAPA_W@__crt_strtox@@YA?AV?$c_string_character_source@_W@0@QB_WQAPA_W@Z 1003d871 f i libucrt:strtox.obj
 0001:0003c88c       _strtol                    1003d88c f   libucrt:strtox.obj
 0001:0003c8b6       _strtoull                  1003d8b6 f   libucrt:strtox.obj
 0001:0003c8e0       _wcstol                    1003d8e0 f   libucrt:strtox.obj
 0001:0003c90a       __mbtowc_l                 1003d90a f   libucrt:mbtowc.obj
 0001:0003ca4c       _mbtowc                    1003da4c f   libucrt:mbtowc.obj
 0001:0003ca66       __wctomb_s_l               1003da66 f   libucrt:wctomb.obj
 0001:0003cbc1       _wctomb_s                  1003dbc1 f   libucrt:wctomb.obj
 0001:0003cbde       _strnlen                   1003dbde f   libucrt:strnlen.obj
 0001:0003cd00       _wcsnlen                   1003dd00 f   libucrt:strnlen.obj
 0001:0003d1ee       ___acrt_freeptd            1003e1ee f   libucrt:per_thread_data.obj
 0001:0003d21a       ___acrt_getptd             1003e21a f   libucrt:per_thread_data.obj
 0001:0003d2d7       ___acrt_getptd_head        1003e2d7 f   libucrt:per_thread_data.obj
 0001:0003d371       ___acrt_getptd_noexit      1003e371 f   libucrt:per_thread_data.obj
 0001:0003d426       ___acrt_initialize_ptd     1003e426 f   libucrt:per_thread_data.obj
 0001:0003d452       ___acrt_uninitialize_ptd   1003e452 f   libucrt:per_thread_data.obj
 0001:0003d46c       ___acrt_update_locale_info 1003e46c f   libucrt:locale_update.obj
 0001:0003d499       ___acrt_update_multibyte_info 1003e499 f   libucrt:locale_update.obj
 0001:0003d4c6       ?__acrt_fp_classify@@YA?AW4__acrt_fp_class@@ABN@Z 1003e4c6 f i libucrt:cvt.obj
 0001:0003dd11       ___acrt_fp_format          1003ed11 f   libucrt:cvt.obj
 0001:0003de4c       __fileno                   1003ee4c f   libucrt:fileno.obj
 0001:0003de73       __fputc_nolock             1003ee73 f   libucrt:fputc.obj
 0001:0003de9c       __get_printf_count_output  1003ee9c f   libucrt:printf_count_output.obj
 0001:0003deb1       ___acrt_stdio_begin_temporary_buffering_nolock 1003eeb1 f   libucrt:_sftbuf.obj
 0001:0003df64       ___acrt_stdio_end_temporary_buffering_nolock 1003ef64 f   libucrt:_sftbuf.obj
 0001:0003e00c       ___acrt_set_locale_changed 1003f00c f   libucrt:wsetlocale.obj
 0001:0003e017       ___acrt_uninitialize_locale 1003f017 f   libucrt:wsetlocale.obj
 0001:0003e1a8       ___acrt_initialize_lowio   1003f1a8 f   libucrt:ioinit.obj
 0001:0003e208       ___acrt_uninitialize_lowio 1003f208 f   libucrt:ioinit.obj
 0001:0003e2c0       __close                    1003f2c0 f   libucrt:close.obj
 0001:0003e34d       __close_nolock             1003f34d f   libucrt:close.obj
 0001:0003e3e9       ?__acrt_stdio_allocate_stream@@YA?AV__crt_stdio_stream@@XZ 1003f3e9 f   libucrt:stream.obj
 0001:0003e452       ?__acrt_stdio_free_stream@@YAXV__crt_stdio_stream@@@Z 1003f452 f   libucrt:stream.obj
 0001:0003e54f       ___acrt_stdio_free_buffer_nolock 1003f54f f   libucrt:_freebuf.obj
 0001:0003e58f       _wcscpy_s                  1003f58f f   libucrt:wcscpy_s.obj
 0001:0003e6c1       ___acrt_get_sigabrt_handler 1003f6c1 f   libucrt:signal.obj
 0001:0003e6e8       ___acrt_initialize_signal_handlers 1003f6e8 f   libucrt:signal.obj
 0001:0003e706       ___fpecode                 1003f706 f   libucrt:signal.obj
 0001:0003e70f       _raise                     1003f70f f   libucrt:signal.obj
 0001:0003e90a       ___set_fpsr_sse2           1003f90a f   libucrt:fpctrl.obj
 0001:0003e98a       __clrfp                    1003f98a f   libucrt:fpctrl.obj
 0001:0003e99b       __ctrlfp                   1003f99b f   libucrt:fpctrl.obj
 0001:0003e9c5       __set_statfp               1003f9c5 f   libucrt:fpctrl.obj
 0001:0003ea1e       __statfp                   1003fa1e f   libucrt:fpctrl.obj
 0001:0003ea2e       ??$__acrt_stdio_parse_mode@_W@@YA?AU__acrt_stdio_stream_mode@@QB_W@Z 1003fa2e f i libucrt:openfile.obj
 0001:0003ed1c       ?__acrt_stdio_parse_mode_D@@YA_NAAU__acrt_stdio_stream_mode@@@Z 1003fd1c f i libucrt:openfile.obj
 0001:0003ed37       ?__acrt_stdio_parse_mode_T@@YA_NAAU__acrt_stdio_stream_mode@@@Z 1003fd37 f i libucrt:openfile.obj
 0001:0003ed56       ?__acrt_stdio_parse_mode_b@@YA_NAAU__acrt_stdio_stream_mode@@@Z 1003fd56 f i libucrt:openfile.obj
 0001:0003ed76       ?__acrt_stdio_parse_mode_c@@YA_NAAU__acrt_stdio_stream_mode@@AA_N@Z 1003fd76 f i libucrt:openfile.obj
 0001:0003ed98       ?__acrt_stdio_parse_mode_n@@YA_NAAU__acrt_stdio_stream_mode@@AA_N@Z 1003fd98 f i libucrt:openfile.obj
 0001:0003edba       ?__acrt_stdio_parse_mode_plus@@YA_NAAU__acrt_stdio_stream_mode@@AA_N@Z 1003fdba f i libucrt:openfile.obj
 0001:0003edf0       ?__acrt_stdio_parse_mode_t@@YA_NAAU__acrt_stdio_stream_mode@@@Z 1003fdf0 f i libucrt:openfile.obj
 0001:0003ee10       ?__acrt_stdio_parse_mode_x@@YA_NAAU__acrt_stdio_stream_mode@@@Z 1003fe10 f i libucrt:openfile.obj
 0001:0003ee30       __wopenfile                1003fe30 f   libucrt:openfile.obj
 0001:0003ee3b       __calloc_base              1003fe3b f   libucrt:calloc_base.obj
 0001:0003f04a       ___acrt_AppPolicyGetProcessTerminationMethodInternal@4 1004004a f   libucrt:winapi_thunks.obj
 0001:0003f08a       ___acrt_AreFileApisANSI@0  1004008a f   libucrt:winapi_thunks.obj
 0001:0003f0a9       ___acrt_CompareStringEx@36 100400a9 f   libucrt:winapi_thunks.obj
 0001:0003f106       ___acrt_FlsAlloc@4         10040106 f   libucrt:winapi_thunks.obj
 0001:0003f145       ___acrt_FlsFree@4          10040145 f   libucrt:winapi_thunks.obj
 0001:0003f184       ___acrt_FlsGetValue@4      10040184 f   libucrt:winapi_thunks.obj
 0001:0003f1c3       ___acrt_FlsSetValue@8      100401c3 f   libucrt:winapi_thunks.obj
 0001:0003f205       ___acrt_InitializeCriticalSectionEx@12 10040205 f   libucrt:winapi_thunks.obj
 0001:0003f250       ___acrt_LCMapStringEx@36   10040250 f   libucrt:winapi_thunks.obj
 0001:0003f2ad       ___acrt_LocaleNameToLCID@8 100402ad f   libucrt:winapi_thunks.obj
 0001:0003f2de       ___acrt_initialize_winapi_thunks 100402de f   libucrt:winapi_thunks.obj
 0001:0003f309       ___acrt_uninitialize_winapi_thunks 10040309 f   libucrt:winapi_thunks.obj
 0001:0003f33f       __fcloseall                1004033f f   libucrt:closeall.obj
 0001:0003f574       ___acrt_stdio_refill_and_read_narrow_nolock 10040574 f   libucrt:_filbuf.obj
 0001:0003f8d2       __lseek                    100408d2 f   libucrt:lseek.obj
 0001:0003f8dd       __lseeki64                 100408dd f   libucrt:lseek.obj
 0001:0003f8f8       __lseeki64_nolock          100408f8 f   libucrt:lseek.obj
 0001:0003f913       ___acrt_stdio_allocate_buffer_nolock 10040913 f   libucrt:_getbuf.obj
 0001:0003fe70       __read                     10040e70 f   libucrt:read.obj
 0001:0003ff84       __read_nolock              10040f84 f   libucrt:read.obj
 0001:00040334       ___sys_errlist             10041334 f   libucrt:syserr.obj
 0001:0004033a       ___sys_nerr                1004133a f   libucrt:syserr.obj
 0001:000403f3       _strncpy_s                 100413f3 f   libucrt:strncpy_s.obj
 0001:000403fe       __towlower_l               100413fe f   libucrt:towlower.obj
 0001:000404a0       ___pctype_func             100414a0 f   libucrt:ctype.obj
 0001:000404c4       ___acrt_GetStringTypeW     100414c4 f   libucrt:getstringtypew.obj
 0001:000404dd       __isctype_l                100414dd f   libucrt:isctype.obj
 0001:000405a8       __recalloc_base            100415a8 f   libucrt:recalloc.obj
 0001:00040615       _wcscat_s                  10041615 f   libucrt:wcscat_s.obj
 0001:0004068a       __cwait                    1004168a f   libucrt:wait.obj
 0001:0004084b       ___acrt_wgetpath           1004184b f   libucrt:getpath.obj
 0001:00040908       ??$__acrt_mbs_to_wcs_cp@U__crt_win32_buffer_internal_dynamic_resizing@@@@YAHQBDAAV?$__crt_win32_buffer@_WU__crt_win32_buffer_internal_dynamic_resizing@@@@I@Z 10041908 f i libucrt:createprocessa.obj
 0001:00040925       ?__acrt_get_utf8_acp_compatibility_codepage@@YAIXZ 10041925 f i libucrt:createprocessa.obj
 0001:00040964       ?_deallocate@?$__crt_win32_buffer@_WU__crt_win32_buffer_internal_dynamic_resizing@@@@AAEXXZ 10041964 f i libucrt:createprocessa.obj
 0001:00040964       ?_deallocate@?$__crt_win32_buffer@DU__crt_win32_buffer_internal_dynamic_resizing@@@@AAEXXZ 10041964 f i libucrt:argv_wildcards.obj
 0001:0004097e       ?allocate@?$__crt_win32_buffer@_WU__crt_win32_buffer_internal_dynamic_resizing@@@@QAEHI@Z 1004197e f i libucrt:createprocessa.obj
 0001:000409bd       ?allocate@__crt_win32_buffer_internal_dynamic_resizing@@SAHQAPAXIABV__crt_win32_buffer_empty_debug_info@@@Z 100419bd f i libucrt:createprocessa.obj
 0001:000409dc       ___acrt_initialize_locks   100419dc f   libucrt:locks.obj
 0001:00040a1d       ___acrt_lock               10041a1d f   libucrt:locks.obj
 0001:00040a34       ___acrt_uninitialize_locks 10041a34 f   libucrt:locks.obj
 0001:00040a65       ___acrt_unlock             10041a65 f   libucrt:locks.obj
 0001:00040a7c       __waccess_s                10041a7c f   libucrt:waccess.obj
 0001:00040b3a       __pipe                     10041b3a f   libucrt:pipe.obj
 0001:00040eb6       __wfdopen                  10041eb6 f   libucrt:fdopen.obj
 0001:00040f63       __commit                   10041f63 f   libucrt:commit.obj
 0001:00041759       __write                    10042759 f   libucrt:write.obj
 0001:0004184b       __write_nolock             1004284b f   libucrt:write.obj
 0001:00041b67       __ui64toa_s                10042b67 f   libucrt:xtoa.obj
 0001:00041b87       __strdup                   10042b87 f   libucrt:strdup.obj
 0001:00041bdb       ___acrt_GetTempPathA       10042bdb f   libucrt:gettemppath.obj
 0001:000422ea       __sopen_nolock             100432ea f   libucrt:open.obj
 0001:00042358       __sopen_s                  10043358 f   libucrt:open.obj
 0001:00042378       __wsopen_nolock            10043378 f   libucrt:open.obj
 0001:000426a2       __wsopen_s                 100436a2 f   libucrt:open.obj
 0001:000426c2       ___acrt_uninitialize_tmpfile 100436c2 f   libucrt:rmtmp.obj
 0001:000426cc       __rmtmp                    100436cc f   libucrt:rmtmp.obj
 0001:000429d4       ___acrt_stdio_flush_and_write_narrow_nolock 100439d4 f   libucrt:_flsbuf.obj
 0001:000429df       _fegetround                100439df f   libucrt:fegetround.obj
 0001:000429ec       __wcsnicoll                100439ec f   libucrt:wcsnicol.obj
 0001:00042a59       __wcsnicoll_l              10043a59 f   libucrt:wcsnicol.obj
 0001:00043107       __wspawnve                 10044107 f   libucrt:spawnv.obj
 0001:0004340f       __wspawnvpe                1004440f f   libucrt:spawnvp.obj
 0001:0004341a       ___acrt_get_process_end_policy 1004441a f   libucrt:win_policies.obj
 0001:00043a29       ?allocate@?$__crt_win32_buffer@DU__crt_win32_buffer_internal_dynamic_resizing@@@@QAEHI@Z 10044a29 f i libucrt:argv_wildcards.obj
 0001:00043aec       ___acrt_expand_narrow_argv_wildcards 10044aec f   libucrt:argv_wildcards.obj
 0001:00043bbe       ?allocate@?$__crt_win32_buffer@DU__crt_win32_buffer_no_resizing@@@@QAEHI@Z 10044bbe f i libucrt:getmodulefilenamea.obj
 0001:00043be5       ?set_to_nullptr@?$__crt_win32_buffer@DU__crt_win32_buffer_no_resizing@@@@QAEXXZ 10044be5 f i libucrt:getmodulefilenamea.obj
 0001:00043bf9       ___acrt_GetModuleFileNameA 10044bf9 f   libucrt:getmodulefilenamea.obj
 0001:000441b8       ___acrt_initialize_multibyte 100451b8 f   libucrt:mbctype.obj
 0001:00044200       ___acrt_update_thread_multibyte_data 10045200 f   libucrt:mbctype.obj
 0001:00044213       __setmbcp_nolock           10045213 f   libucrt:mbctype.obj
 0001:0004445d       __ismbblead                1004545d f   libucrt:ismbbyte.obj
 0001:00044475       ___acrt_initialize_command_line 10045475 f   libucrt:argv_data.obj
 0001:0004448e       ___acrt_MultiByteToWideChar 1004548e f   libucrt:multibytetowidechar.obj
 0001:0004450a       ___acrt_WideCharToMultiByte 1004550a f   libucrt:widechartomultibyte.obj
 0001:000445ee       ___dcrt_get_narrow_environment_from_os 100455ee f   libucrt:get_environment_from_os.obj
 0001:00044672       ___dcrt_get_wide_environment_from_os 10045672 f   libucrt:get_environment_from_os.obj
 0001:00044a45       ___dcrt_set_variable_in_wide_environment_nolock 10045a45 f   libucrt:setenv.obj
 0001:00044a50       ___acrt_initialize_heap    10045a50 f   libucrt:heap_handle.obj
 0001:00044a61       ___acrt_uninitialize_heap  10045a61 f   libucrt:heap_handle.obj
 0001:00044a6b       ___acrt_execute_initializers 10045a6b f   libucrt:shared_initialization.obj
 0001:00044ad3       ___acrt_execute_uninitializers 10045ad3 f   libucrt:shared_initialization.obj
 0001:00044b04       ___acrt_initialize_new_handler 10045b04 f   libucrt:new_handler.obj
 0001:00044b13       __callnewh                 10045b13 f   libucrt:new_handler.obj
 0001:00044b40       __query_new_handler        10045b40 f   libucrt:new_handler.obj
 0001:00044b9c       ___acrt_has_user_matherr   10045b9c f   libucrt:matherr.obj
 0001:00044bb4       ___acrt_initialize_user_matherr 10045bb4 f   libucrt:matherr.obj
 0001:00044bc3       ___acrt_invoke_user_matherr 10045bc3 f   libucrt:matherr.obj
 0001:00044ddf       ___acrt_LCMapStringA       10045ddf f   libucrt:lcmapstringa.obj
 0001:00044e28       __query_new_mode           10045e28 f   libucrt:new_mode.obj
 0001:00044e2f       __isleadbyte_l             10045e2f f i libucrt:_wctype.obj
 0001:00044e95       ?__mbrtowc_utf8@__crt_mbstring@@YAIPA_WPBDIPAU_Mbstatet@@@Z 10045e95 f   libucrt:mbrtowc.obj
 0001:00044ed5       ?__mbsrtowcs_utf8@__crt_mbstring@@YAIPA_WPAPBDIPAU_Mbstatet@@@Z 10045ed5 f   libucrt:mbrtowc.obj
 0001:00044fd0       ?__c32rtomb_utf8@__crt_mbstring@@YAIPAD_UPAU_Mbstatet@@@Z 10045fd0 f   libucrt:c32rtomb.obj
 0001:0004507b       ?return_illegal_sequence@__crt_mbstring@@YAIPAU_Mbstatet@@@Z 1004607b f i libucrt:c32rtomb.obj
 0001:0004509a       ___acrt_add_locale_ref     1004609a f   libucrt:locale_refcounting.obj
 0001:00045117       ___acrt_free_locale        10046117 f   libucrt:locale_refcounting.obj
 0001:0004525f       ___acrt_locale_add_lc_time_reference 1004625f f   libucrt:locale_refcounting.obj
 0001:00045288       ___acrt_locale_free_lc_time_if_unreferenced 10046288 f   libucrt:locale_refcounting.obj
 0001:000452b9       ___acrt_locale_release_lc_time_reference 100462b9 f   libucrt:locale_refcounting.obj
 0001:000452e2       ___acrt_release_locale_ref 100462e2 f   libucrt:locale_refcounting.obj
 0001:00045363       ___acrt_update_thread_locale_data 10046363 f   libucrt:locale_refcounting.obj
 0001:000453e4       __updatetlocinfoEx_nolock  100463e4 f   libucrt:locale_refcounting.obj
 0001:00045434       ___acrt_fp_strflt_to_string 10046434 f   libucrt:_fptostr.obj
 0001:000454f4       ___acrt_fltout             100464f4 f   libucrt:cfout.obj
 0001:0004683e       __isatty                   1004783e f   libucrt:isatty.obj
 0001:00046894       ___acrt_locale_free_monetary 10047894 f   libucrt:initmon.obj
 0001:00046992       ___acrt_locale_free_numeric 10047992 f   libucrt:initnum.obj
 0001:00046a33       ___acrt_locale_free_time   10047a33 f   libucrt:inittime.obj
 0001:00046b17       ___acrt_GetStringTypeA     10047b17 f   libucrt:getstringtypea.obj
 0001:00046c1a       ___acrt_lowio_create_handle_array 10047c1a f   libucrt:osfinfo.obj
 0001:00046c95       ___acrt_lowio_destroy_handle_array 10047c95 f   libucrt:osfinfo.obj
 0001:00046cca       ___acrt_lowio_ensure_fh_exists 10047cca f   libucrt:osfinfo.obj
 0001:00046d68       ___acrt_lowio_lock_fh      10047d68 f   libucrt:osfinfo.obj
 0001:00046d8b       ___acrt_lowio_set_os_handle 10047d8b f   libucrt:osfinfo.obj
 0001:00046e1d       ___acrt_lowio_unlock_fh    10047e1d f   libucrt:osfinfo.obj
 0001:00046e40       __alloc_osfhnd             10047e40 f   libucrt:osfinfo.obj
 0001:00046f53       __free_osfhnd              10047f53 f   libucrt:osfinfo.obj
 0001:00046fe4       __get_osfhandle            10047fe4 f   libucrt:osfinfo.obj
 0001:0004704e       ___ascii_wcsnicmp          1004804e f   libucrt:wcsnicmp.obj
 0001:0004709d       __wcsnicmp                 1004809d f   libucrt:wcsnicmp.obj
 0001:000470e9       __wcsnicmp_l               100480e9 f   libucrt:wcsnicmp.obj
 0001:0004720c       ___acrt_DownlevelLocaleNameToLCID 1004820c f   libucrt:lcidtoname_downlevel.obj
 0001:00047238       ___acrt_LCMapStringW       10048238 f   libucrt:lcmapstringw.obj
 0001:00047276       __msize_base               10048276 f   libucrt:msize.obj
 0001:000472a9       __realloc_base             100482a9 f   libucrt:realloc_base.obj
 0001:00047312       __get_fmode                10048312 f   libucrt:setmode.obj
 0001:0004733f       __setmode_nolock           1004833f f   libucrt:setmode.obj
 0001:0004740e       __putwch_nolock            1004840e f   libucrt:putwch.obj
 0001:00047440       ??0__crt_seek_guard@@QAE@H_J@Z 10048440 f i libucrt:chsize.obj
 0001:0004748d       __chsize_nolock            1004848d f   libucrt:chsize.obj
 0001:0004790a       ___acrt_fenv_get_common_round_control 1004890a f   libucrt:_fenvutils.obj
 0001:0004792c       ___acrt_fenv_get_control   1004892c f   libucrt:_fenvutils.obj
 0001:000479ac       ___acrt_fenv_get_status    100489ac f   libucrt:_fenvutils.obj
 0001:00047a64       ___acrt_fenv_set_control   10048a64 f   libucrt:_fenvutils.obj
 0001:00047acc       ___acrt_fenv_set_status    10048acc f   libucrt:_fenvutils.obj
 0001:00047bc3       ___acrt_CompareStringW     10048bc3 f   libucrt:comparestringw.obj
 0001:0004804e       ___acrt_pack_wide_command_line_and_environment 1004904e f   libucrt:cenvarg.obj
 0001:00048110       _qsort                     10049110 f   libucrt:qsort.obj
 0001:00048554       __mbsdec                   10049554 f   libucrt:mbsdec.obj
 0001:0004856b       __mbsdec_l                 1004956b f   libucrt:mbsdec.obj
 0001:00048607       ___strncnt                 10049607 f   libucrt:strncnt.obj
 0001:00048623       ?__mbrtoc32_utf8@__crt_mbstring@@YAIPA_UPBDIPAU_Mbstatet@@@Z 10049623 f   libucrt:mbrtoc32.obj
 0001:000487ca       _fegetenv                  100497ca f   libucrt:fegetenv.obj
 0001:000487e7       _fesetenv                  100497e7 f   libucrt:fesetenv.obj
 0001:00048832       _feholdexcept              10049832 f   libucrt:feholdexcept.obj
 0001:00048880       __CIlog10                  10049880 f   libucrt:log10_impl.obj
 0001:000488bb       __CIlog10_default          100498bb f   libucrt:log10_impl.obj
 0001:000488cf       __log10_default            100498cf     libucrt:log10_impl.obj
 0001:00048990       _ceil                      10049990 f   libucrt:ceil_pentium4.obj
 0001:000489d0       __ceil_pentium4            100499d0 f   libucrt:ceil_pentium4.obj
 0001:00048aad       __query_app_type           10049aad f   libucrt:report_runtime_error.obj
 0001:00048ac0       ___ascii_strnicmp          10049ac0 f   libucrt:_strnicm.obj
 0001:00048b40       ___dcrt_lowio_ensure_console_output_initialized 10049b40 f   libucrt:initcon.obj
 0001:00048b5f       ___dcrt_terminate_console_output 10049b5f f   libucrt:initcon.obj
 0001:00048b76       ___dcrt_write_console      10049b76 f   libucrt:initcon.obj
 0001:00048bcb       ___acrt_initialize_sse2    10049bcb f   libucrt:mathfcns.obj
 0001:00048be0       __CIlog10_pentium4         10049be0 f   libucrt:log10_pentium4.obj
 0001:00048bf8       __log10_pentium4           10049bf8     libucrt:log10_pentium4.obj
 0001:00048e90       __fFEXP                    10049e90 f   libucrt:87tran.obj
 0001:00048ee7       __rtinfpopse               10049ee7     libucrt:87tran.obj
 0001:00048ee9       __rtinfnpopse              10049ee9     libucrt:87tran.obj
 0001:00048ef9       __fFLN                     10049ef9     libucrt:87tran.obj
 0001:00048fae       __rtinfpop                 10049fae     libucrt:87tran.obj
 0001:00048fb0       __rtinfnpop                10049fb0     libucrt:87tran.obj
 0001:00048fc0       __rtforexpinf              10049fc0 f   libucrt:87tran.obj
 0001:00048fcd       __ffexpm1                  10049fcd     libucrt:87tran.obj
 0001:00049080       __trandisp1                1004a080 f   libucrt:87disp.obj
 0001:000490f5       __trandisp2                1004a0f5 f   libucrt:87disp.obj
 0001:0004918f       __rttospopde               1004a18f     libucrt:87disp.obj
 0001:00049194       __rttospop                 1004a194     libucrt:87disp.obj
 0001:000491a0       __rtnospop                 1004a1a0 f   libucrt:87disp.obj
 0001:000491b0       __rttosnpop                1004a1b0 f   libucrt:87disp.obj
 0001:000491b1       __rtnospopde               1004a1b1     libucrt:87disp.obj
 0001:000491b8       __rtzeropop                1004a1b8     libucrt:87disp.obj
 0001:000491ba       __rtzeronpop               1004a1ba     libucrt:87disp.obj
 0001:000491c0       __rtzerospop               1004a1c0 f   libucrt:87disp.obj
 0001:000491cd       __rtonepop                 1004a1cd     libucrt:87disp.obj
 0001:000491d0       __rtonenpop                1004a1d0 f   libucrt:87disp.obj
 0001:000491e0       __tosnan1                  1004a1e0 f   libucrt:87disp.obj
 0001:00049210       __nosnan2                  1004a210 f   libucrt:87disp.obj
 0001:00049220       __tosnan2                  1004a220 f   libucrt:87disp.obj
 0001:00049250       __nan2                     1004a250 f   libucrt:87disp.obj
 0001:00049290       __rtindfpop                1004a290 f   libucrt:87disp.obj
 0001:00049292       __rtindfnpop               1004a292     libucrt:87disp.obj
 0001:000492a3       __rttosnpopde              1004a2a3     libucrt:87disp.obj
 0001:000492b0       __rtatan2inf               1004a2b0 f   libucrt:87disp.obj
 0001:000492cd       __rtchsifneg               1004a2cd     libucrt:87disp.obj
 0001:000492e0       __twoToTOS                 1004a2e0 f   libucrt:common.obj
 0001:000492f5       __load_CW                  1004a2f5 f   libucrt:common.obj
 0001:0004930c       __convertTOStoQNaN         1004a30c f   libucrt:common.obj
 0001:00049325       __fload_withFB             1004a325 f   libucrt:common.obj
 0001:00049368       __checkTOS_withFB          1004a368 f   libucrt:common.obj
 0001:0004937e       __fast_exit                1004a37e f   libucrt:common.obj
 0001:0004938b       __math_exit                1004a38b f   libucrt:common.obj
 0001:000493b5       __check_overflow_exit      1004a3b5 f   libucrt:common.obj
 0001:000493c9       __check_range_exit         1004a3c9 f   libucrt:common.obj
 0001:00049470       __startTwoArgErrorHandling 1004a470 f   libucrt:genexcep.obj
 0001:00049487       __startOneArgErrorHandling 1004a487 f   libucrt:genexcep.obj
 0001:000494c3       ___libm_error_support      1004a4c3 f   libucrt:libm_error.obj
 0001:000496b7       __ceil_default             1004a6b7 f   libucrt:ceil.obj
 0001:0004976c       __d_inttype                1004a76c f   libucrt:powhlp.obj
 0001:000497d4       __powhlp                   1004a7d4 f   libucrt:powhlp.obj
 0001:000498ff       __87except                 1004a8ff f   libucrt:87except.obj
 0001:00049a09       __frnd                     1004aa09 f   libucrt:frnd.obj
 0001:00049a1d       __errcode                  1004aa1d f   libucrt:fpexcept.obj
 0001:00049a51       __except1                  1004aa51 f   libucrt:fpexcept.obj
 0001:00049b1f       __handle_exc               1004ab1f f   libucrt:fpexcept.obj
 0001:00049d0a       __raise_exc                1004ad0a f   libucrt:fpexcept.obj
 0001:00049d2d       __raise_exc_ex             1004ad2d f   libucrt:fpexcept.obj
 0001:0004a023       __set_errno_from_matherr   1004b023 f   libucrt:fpexcept.obj
 0001:0004a052       __umatherr                 1004b052 f   libucrt:fpexcept.obj
 0001:0004a0f2       __decomp                   1004b0f2 f   libucrt:util.obj
 0001:0004a1c4       __set_exp                  1004b1c4 f   libucrt:util.obj
 0001:0004a1f1       __sptype                   1004b1f1 f   libucrt:util.obj
 0001:0004a24f       __fpclass                  1004b24f f   libucrt:ieeemisc.obj
 0001:0004a2f3       _IsProcessorFeaturePresent@4 1004b2f3 f   kernel32:KERNEL32.dll
 0001:0004a2f9       ??_Gtype_info@@UAEPAXI@Z   1004b2f9 f i LIBCMT:std_type_info_static.obj
 0001:0004a2f9       ??_Etype_info@@UAEPAXI@Z   1004b2f9 f i LIBCMT:std_type_info_static.obj
 0001:0004a320       __FindPESection            1004b320 f   LIBCMT:pesect.obj
 0001:0004a370       __IsNonwritableInCurrentImage 1004b370 f   LIBCMT:pesect.obj
 0001:0004a430       __ValidateImageBase        1004b430 f   LIBCMT:pesect.obj
 0001:0004a463       ??3@YAXPAXI@Z              1004b463 f   LIBCMT:delete_scalar_size.obj
 0001:0004a471       __EH_prolog3_catch         1004b471 f   LIBCMT:ehprolg3.obj
 0001:0004a4b0       __aulldvrm                 1004b4b0 f   LIBCMT:ulldvrm.obj
 0001:0004a550       __SEH_prolog4_GS           1004b550 f   LIBCMT:sehprolg4gs.obj
 0001:0004a599       __SEH_epilog4_GS           1004b599 f   LIBCMT:sehprolg4gs.obj
 0001:0004a5b0       __allmul                   1004b5b0 f   LIBCMT:llmul.obj
 0001:0004a5f0       __allshl                   1004b5f0 f   LIBCMT:llshl.obj
 0001:0004a610       __aullshr                  1004b610 f   LIBCMT:ullshr.obj
 0001:0004a630       __alldiv                   1004b630 f   LIBCMT:lldiv.obj
 0001:0004a6e0       __alloca_probe             1004b6e0 f   LIBCMT:chkstk.obj
 0001:0004a6e0       __chkstk                   1004b6e0 f   LIBCMT:chkstk.obj
 0001:0004a710       __alloca_probe_16          1004b710 f   LIBCMT:alloca16.obj
 0001:0004a726       __alloca_probe_8           1004b726     LIBCMT:alloca16.obj
 0001:0004a740       __alldvrm                  1004b740 f   LIBCMT:lldvrm.obj
 0001:0004a820       __ftol2_sse                1004b820     LIBCMT:ftol2.obj
 0001:0004a820       __ftol2_sse_excpt          1004b820     LIBCMT:ftol2.obj
 0001:0004a820       __ftoi2                    1004b820 f   LIBCMT:ftol2.obj
 0001:0004a8a0       __ftoui2                   1004b8a0 f   LIBCMT:ftol2.obj
 0001:0004a950       __ftol2                    1004b950 f   LIBCMT:ftol2.obj
 0001:0004aa00       __ftoul2                   1004ba00 f   LIBCMT:ftol2.obj
 0001:0004aab9       ??3@YAXPAX@Z               1004bab9 f   LIBCMT:delete_scalar.obj
 0001:0004aabe       __filter_x86_sse2_floating_point_exception_default 1004babe f   LIBCMT:x86_exception_filter.obj
 0001:0004aabe       __filter_x86_sse2_floating_point_exception 1004babe f   LIBCMT:x86_exception_filter.obj
 0001:0004ab40       __allrem                   1004bb40 f   LIBCMT:llrem.obj
 0001:0004ac00       __allshr                   1004bc00 f   LIBCMT:llshr.obj
 0001:0004ac30       _memchr                    1004bc30 f   libvcruntime:memchr.obj
 0002:00000000       __imp__RegDeleteKeyW@8     1004c000     advapi32:ADVAPI32.dll
 0002:00000004       __imp__RegEnumKeyExW@32    1004c004     advapi32:ADVAPI32.dll
 0002:00000008       __imp__RegDeleteValueW@8   1004c008     advapi32:ADVAPI32.dll
 0002:0000000c       __imp__RegEnumValueW@32    1004c00c     advapi32:ADVAPI32.dll
 0002:00000010       __imp__RegCloseKey@4       1004c010     advapi32:ADVAPI32.dll
 0002:00000014       __imp__RegCreateKeyExW@36  1004c014     advapi32:ADVAPI32.dll
 0002:00000018       __imp__RegSetValueExW@24   1004c018     advapi32:ADVAPI32.dll
 0002:0000001c       __imp__RegOpenKeyExW@20    1004c01c     advapi32:ADVAPI32.dll
 0002:00000020       __imp__RegQueryValueExW@24 1004c020     advapi32:ADVAPI32.dll
 0002:00000024       \177ADVAPI32_NULL_THUNK_DATA 1004c024     advapi32:ADVAPI32.dll
 0002:00000028       __imp__DeleteTimerQueueTimer@12 1004c028     kernel32:KERNEL32.dll
 0002:0000002c       __imp__CreateTimerQueue@0  1004c02c     kernel32:KERNEL32.dll
 0002:00000030       __imp__GetModuleFileNameW@12 1004c030     kernel32:KERNEL32.dll
 0002:00000034       __imp__LoadLibraryW@4      1004c034     kernel32:KERNEL32.dll
 0002:00000038       __imp__FreeLibrary@4       1004c038     kernel32:KERNEL32.dll
 0002:0000003c       __imp__GetCPInfoExW@12     1004c03c     kernel32:KERNEL32.dll
 0002:00000040       __imp__GetOEMCP@0          1004c040     kernel32:KERNEL32.dll
 0002:00000044       __imp__SearchPathW@24      1004c044     kernel32:KERNEL32.dll
 0002:00000048       __imp__GetConsoleOutputCP@0 1004c048     kernel32:KERNEL32.dll
 0002:0000004c       __imp__GetConsoleCP@0      1004c04c     kernel32:KERNEL32.dll
 0002:00000050       __imp__EnumSystemCodePagesW@8 1004c050     kernel32:KERNEL32.dll
 0002:00000054       __imp__GetACP@0            1004c054     kernel32:KERNEL32.dll
 0002:00000058       __imp__SetFileAttributesW@8 1004c058     kernel32:KERNEL32.dll
 0002:0000005c       __imp__GetLogicalDriveStringsW@8 1004c05c     kernel32:KERNEL32.dll
 0002:00000060       __imp__MultiByteToWideChar@24 1004c060     kernel32:KERNEL32.dll
 0002:00000064       __imp__Sleep@4             1004c064     kernel32:KERNEL32.dll
 0002:00000068       __imp__FormatMessageW@28   1004c068     kernel32:KERNEL32.dll
 0002:0000006c       __imp__GetLastError@0      1004c06c     kernel32:KERNEL32.dll
 0002:00000070       __imp__OutputDebugStringW@4 1004c070     kernel32:KERNEL32.dll
 0002:00000074       __imp__GetCurrentDirectoryW@8 1004c074     kernel32:KERNEL32.dll
 0002:00000078       __imp__SetCurrentDirectoryW@4 1004c078     kernel32:KERNEL32.dll
 0002:0000007c       __imp__SetConsoleCP@4      1004c07c     kernel32:KERNEL32.dll
 0002:00000080       __imp__GlobalMemoryStatusEx@4 1004c080     kernel32:KERNEL32.dll
 0002:00000084       __imp__WideCharToMultiByte@32 1004c084     kernel32:KERNEL32.dll
 0002:00000088       __imp__SetConsoleOutputCP@4 1004c088     kernel32:KERNEL32.dll
 0002:0000008c       __imp__GetDriveTypeW@4     1004c08c     kernel32:KERNEL32.dll
 0002:00000090       __imp__CreateDirectoryW@8  1004c090     kernel32:KERNEL32.dll
 0002:00000094       __imp__FindFirstFileW@8    1004c094     kernel32:KERNEL32.dll
 0002:00000098       __imp__GetModuleHandleW@4  1004c098     kernel32:KERNEL32.dll
 0002:0000009c       __imp__RemoveDirectoryW@4  1004c09c     kernel32:KERNEL32.dll
 0002:000000a0       __imp__SetFileTime@16      1004c0a0     kernel32:KERNEL32.dll
 0002:000000a4       __imp__SetEnvironmentVariableW@8 1004c0a4     kernel32:KERNEL32.dll
 0002:000000a8       __imp__FindClose@4         1004c0a8     kernel32:KERNEL32.dll
 0002:000000ac       __imp__CreateFileW@28      1004c0ac     kernel32:KERNEL32.dll
 0002:000000b0       __imp__ReadConsoleInputW@16 1004c0b0     kernel32:KERNEL32.dll
 0002:000000b4       __imp__FileTimeToSystemTime@8 1004c0b4     kernel32:KERNEL32.dll
 0002:000000b8       __imp__DeleteFileW@4       1004c0b8     kernel32:KERNEL32.dll
 0002:000000bc       __imp__CloseHandle@4       1004c0bc     kernel32:KERNEL32.dll
 0002:000000c0       __imp__FileTimeToLocalFileTime@8 1004c0c0     kernel32:KERNEL32.dll
 0002:000000c4       __imp__PeekConsoleInputW@16 1004c0c4     kernel32:KERNEL32.dll
 0002:000000c8       __imp__WriteConsoleW@20    1004c0c8     kernel32:KERNEL32.dll
 0002:000000cc       __imp__MoveFileExW@12      1004c0cc     kernel32:KERNEL32.dll
 0002:000000d0       __imp__VerSetConditionMask@16 1004c0d0     kernel32:KERNEL32.dll
 0002:000000d4       __imp__SystemTimeToFileTime@8 1004c0d4     kernel32:KERNEL32.dll
 0002:000000d8       __imp__CopyFileW@12        1004c0d8     kernel32:KERNEL32.dll
 0002:000000dc       __imp__VerifyVersionInfoW@16 1004c0dc     kernel32:KERNEL32.dll
 0002:000000e0       __imp__GetSystemTimeAsFileTime@4 1004c0e0     kernel32:KERNEL32.dll
 0002:000000e4       __imp__GetFileTime@16      1004c0e4     kernel32:KERNEL32.dll
 0002:000000e8       __imp__SetLastError@4      1004c0e8     kernel32:KERNEL32.dll
 0002:000000ec       __imp__EnterCriticalSection@4 1004c0ec     kernel32:KERNEL32.dll
 0002:000000f0       __imp__LeaveCriticalSection@4 1004c0f0     kernel32:KERNEL32.dll
 0002:000000f4       __imp__InitializeCriticalSection@4 1004c0f4     kernel32:KERNEL32.dll
 0002:000000f8       __imp__GetCurrentThread@0  1004c0f8     kernel32:KERNEL32.dll
 0002:000000fc       __imp__DeleteCriticalSection@4 1004c0fc     kernel32:KERNEL32.dll
 0002:00000100       __imp__LCMapStringW@24     1004c100     kernel32:KERNEL32.dll
 0002:00000104       __imp__GetThreadTimes@20   1004c104     kernel32:KERNEL32.dll
 0002:00000108       __imp__VirtualQuery@12     1004c108     kernel32:KERNEL32.dll
 0002:0000010c       __imp__HeapReAlloc@16      1004c10c     kernel32:KERNEL32.dll
 0002:00000110       __imp__GetProcAddress@8    1004c110     kernel32:KERNEL32.dll
 0002:00000114       __imp__ChangeTimerQueueTimer@16 1004c114     kernel32:KERNEL32.dll
 0002:00000118       __imp__GetModuleHandleA@4  1004c118     kernel32:KERNEL32.dll
 0002:0000011c       __imp__GetFileAttributesW@4 1004c11c     kernel32:KERNEL32.dll
 0002:00000120       __imp__GetEnvironmentVariableW@12 1004c120     kernel32:KERNEL32.dll
 0002:00000124       __imp__GetStdHandle@4      1004c124     kernel32:KERNEL32.dll
 0002:00000128       __imp__GetConsoleScreenBufferInfo@8 1004c128     kernel32:KERNEL32.dll
 0002:0000012c       __imp__CreateTimerQueueTimer@28 1004c12c     kernel32:KERNEL32.dll
 0002:00000130       __imp__CompareStringW@24   1004c130     kernel32:KERNEL32.dll
 0002:00000134       __imp__DeleteTimerQueueEx@8 1004c134     kernel32:KERNEL32.dll
 0002:00000138       __imp__HeapSize@12         1004c138     kernel32:KERNEL32.dll
 0002:0000013c       __imp__SetStdHandle@8      1004c13c     kernel32:KERNEL32.dll
 0002:00000140       __imp__GetProcessHeap@0    1004c140     kernel32:KERNEL32.dll
 0002:00000144       __imp__FreeEnvironmentStringsW@4 1004c144     kernel32:KERNEL32.dll
 0002:00000148       __imp__GetEnvironmentStringsW@0 1004c148     kernel32:KERNEL32.dll
 0002:0000014c       __imp__GetCommandLineW@0   1004c14c     kernel32:KERNEL32.dll
 0002:00000150       __imp__GetCommandLineA@0   1004c150     kernel32:KERNEL32.dll
 0002:00000154       __imp__GetCPInfo@8         1004c154     kernel32:KERNEL32.dll
 0002:00000158       __imp__IsValidCodePage@4   1004c158     kernel32:KERNEL32.dll
 0002:0000015c       __imp__FindNextFileW@8     1004c15c     kernel32:KERNEL32.dll
 0002:00000160       __imp__FindFirstFileExW@24 1004c160     kernel32:KERNEL32.dll
 0002:00000164       __imp__GetFileSizeEx@8     1004c164     kernel32:KERNEL32.dll
 0002:00000168       __imp__WriteFile@20        1004c168     kernel32:KERNEL32.dll
 0002:0000016c       __imp__FlushFileBuffers@4  1004c16c     kernel32:KERNEL32.dll
 0002:00000170       __imp__CreatePipe@16       1004c170     kernel32:KERNEL32.dll
 0002:00000174       __imp__GetFileAttributesExW@12 1004c174     kernel32:KERNEL32.dll
 0002:00000178       __imp__GetExitCodeProcess@8 1004c178     kernel32:KERNEL32.dll
 0002:0000017c       __imp__WaitForSingleObject@8 1004c17c     kernel32:KERNEL32.dll
 0002:00000180       __imp__GetStringTypeW@16   1004c180     kernel32:KERNEL32.dll
 0002:00000184       __imp__ReadConsoleW@20     1004c184     kernel32:KERNEL32.dll
 0002:00000188       __imp__GetConsoleMode@8    1004c188     kernel32:KERNEL32.dll
 0002:0000018c       __imp__SetFilePointerEx@20 1004c18c     kernel32:KERNEL32.dll
 0002:00000190       __imp__GetFileType@4       1004c190     kernel32:KERNEL32.dll
 0002:00000194       __imp__HeapAlloc@12        1004c194     kernel32:KERNEL32.dll
 0002:00000198       __imp__HeapFree@12         1004c198     kernel32:KERNEL32.dll
 0002:0000019c       __imp__ExitProcess@4       1004c19c     kernel32:KERNEL32.dll
 0002:000001a0       __imp__ReadFile@20         1004c1a0     kernel32:KERNEL32.dll
 0002:000001a4       __imp__GetTempPathW@8      1004c1a4     kernel32:KERNEL32.dll
 0002:000001a8       __imp__CreateProcessW@40   1004c1a8     kernel32:KERNEL32.dll
 0002:000001ac       __imp__DuplicateHandle@28  1004c1ac     kernel32:KERNEL32.dll
 0002:000001b0       __imp__RaiseException@16   1004c1b0     kernel32:KERNEL32.dll
 0002:000001b4       __imp__LoadLibraryExW@12   1004c1b4     kernel32:KERNEL32.dll
 0002:000001b8       __imp__SetEndOfFile@4      1004c1b8     kernel32:KERNEL32.dll
 0002:000001bc       __imp__TlsFree@4           1004c1bc     kernel32:KERNEL32.dll
 0002:000001c0       __imp__TlsSetValue@8       1004c1c0     kernel32:KERNEL32.dll
 0002:000001c4       __imp__TlsGetValue@4       1004c1c4     kernel32:KERNEL32.dll
 0002:000001c8       __imp__TlsAlloc@0          1004c1c8     kernel32:KERNEL32.dll
 0002:000001cc       __imp__InitializeCriticalSectionAndSpinCount@8 1004c1cc     kernel32:KERNEL32.dll
 0002:000001d0       __imp__RtlUnwind@16        1004c1d0     kernel32:KERNEL32.dll
 0002:000001d4       __imp__GetCurrentThreadId@0 1004c1d4     kernel32:KERNEL32.dll
 0002:000001d8       __imp__GetCurrentProcessId@0 1004c1d8     kernel32:KERNEL32.dll
 0002:000001dc       __imp__QueryPerformanceCounter@4 1004c1dc     kernel32:KERNEL32.dll
 0002:000001e0       __imp__GetStartupInfoW@4   1004c1e0     kernel32:KERNEL32.dll
 0002:000001e4       __imp__IsDebuggerPresent@0 1004c1e4     kernel32:KERNEL32.dll
 0002:000001e8       __imp__IsProcessorFeaturePresent@4 1004c1e8     kernel32:KERNEL32.dll
 0002:000001ec       __imp__TerminateProcess@8  1004c1ec     kernel32:KERNEL32.dll
 0002:000001f0       __imp__GetCurrentProcess@0 1004c1f0     kernel32:KERNEL32.dll
 0002:000001f4       __imp__SetUnhandledExceptionFilter@4 1004c1f4     kernel32:KERNEL32.dll
 0002:000001f8       __imp__UnhandledExceptionFilter@4 1004c1f8     kernel32:KERNEL32.dll
 0002:000001fc       \177KERNEL32_NULL_THUNK_DATA 1004c1fc     kernel32:KERNEL32.dll
 0002:00000200       __imp__UuidCreate@4        1004c200     rpcrt4:RPCRT4.dll
 0002:00000204       __imp__UuidToStringA@8     1004c204     rpcrt4:RPCRT4.dll
 0002:00000208       __imp__RpcStringFreeA@4    1004c208     rpcrt4:RPCRT4.dll
 0002:0000020c       __imp__UuidFromStringA@8   1004c20c     rpcrt4:RPCRT4.dll
 0002:00000210       \177RPCRT4_NULL_THUNK_DATA 1004c210     rpcrt4:RPCRT4.dll
 0002:00000214       __imp__SHGetFolderPathW@20 1004c214     shell32:SHELL32.dll
 0002:00000218       __imp__ShellExecuteW@24    1004c218     shell32:SHELL32.dll
 0002:0000021c       \177SHELL32_NULL_THUNK_DATA 1004c21c     shell32:SHELL32.dll
 0002:00000220       __imp__GetKeyState@4       1004c220     user32:USER32.dll
 0002:00000224       \177USER32_NULL_THUNK_DATA 1004c224     user32:USER32.dll
 0002:00000228       __imp__luaL_optinteger     1004c228     lua51:lua51.dll
 0002:0000022c       __imp__lua_checkstack      1004c22c     lua51:lua51.dll
 0002:00000230       __imp__luaL_optlstring     1004c230     lua51:lua51.dll
 0002:00000234       __imp__lua_getinfo         1004c234     lua51:lua51.dll
 0002:00000238       __imp__lua_getstack        1004c238     lua51:lua51.dll
 0002:0000023c       __imp__luaL_checktype      1004c23c     lua51:lua51.dll
 0002:00000240       __imp__luaopen_table       1004c240     lua51:lua51.dll
 0002:00000244       __imp__luaL_findtable      1004c244     lua51:lua51.dll
 0002:00000248       __imp__lua_getallocf       1004c248     lua51:lua51.dll
 0002:0000024c       __imp__luaL_checkany       1004c24c     lua51:lua51.dll
 0002:00000250       __imp__lua_settable        1004c250     lua51:lua51.dll
 0002:00000254       __imp__lua_getfenv         1004c254     lua51:lua51.dll
 0002:00000258       __imp__luaopen_base        1004c258     lua51:lua51.dll
 0002:0000025c       __imp__lua_next            1004c25c     lua51:lua51.dll
 0002:00000260       __imp__luaopen_os          1004c260     lua51:lua51.dll
 0002:00000264       __imp__luaL_optnumber      1004c264     lua51:lua51.dll
 0002:00000268       __imp__luaopen_string      1004c268     lua51:lua51.dll
 0002:0000026c       __imp__luaopen_math        1004c26c     lua51:lua51.dll
 0002:00000270       __imp__luaL_checknumber    1004c270     lua51:lua51.dll
 0002:00000274       __imp__luaL_typerror       1004c274     lua51:lua51.dll
 0002:00000278       __imp__lua_setfenv         1004c278     lua51:lua51.dll
 0002:0000027c       __imp__luaopen_debug       1004c27c     lua51:lua51.dll
 0002:00000280       __imp__lua_setallocf       1004c280     lua51:lua51.dll
 0002:00000284       __imp__lua_dump            1004c284     lua51:lua51.dll
 0002:00000288       __imp__luaL_prepbuffer     1004c288     lua51:lua51.dll
 0002:0000028c       __imp__luaL_checkstack     1004c28c     lua51:lua51.dll
 0002:00000290       __imp__lua_typename        1004c290     lua51:lua51.dll
 0002:00000294       __imp__lua_tocfunction     1004c294     lua51:lua51.dll
 0002:00000298       __imp__luaL_checkoption    1004c298     lua51:lua51.dll
 0002:0000029c       __imp__lua_iscfunction     1004c29c     lua51:lua51.dll
 0002:000002a0       __imp__luaL_gsub           1004c2a0     lua51:lua51.dll
 0002:000002a4       __imp__lua_isuserdata      1004c2a4     lua51:lua51.dll
 0002:000002a8       __imp__luaL_checkudata     1004c2a8     lua51:lua51.dll
 0002:000002ac       __imp__luaL_loadstring     1004c2ac     lua51:lua51.dll
 0002:000002b0       __imp__lua_insert          1004c2b0     lua51:lua51.dll
 0002:000002b4       __imp__lua_rawseti         1004c2b4     lua51:lua51.dll
 0002:000002b8       __imp__lua_toboolean       1004c2b8     lua51:lua51.dll
 0002:000002bc       __imp__lua_pcall           1004c2bc     lua51:lua51.dll
 0002:000002c0       __imp__luaL_addvalue       1004c2c0     lua51:lua51.dll
 0002:000002c4       __imp__lua_rawset          1004c2c4     lua51:lua51.dll
 0002:000002c8       __imp__lua_rawget          1004c2c8     lua51:lua51.dll
 0002:000002cc       __imp__luaL_unref          1004c2cc     lua51:lua51.dll
 0002:000002d0       __imp__lua_remove          1004c2d0     lua51:lua51.dll
 0002:000002d4       __imp__lua_rawgeti         1004c2d4     lua51:lua51.dll
 0002:000002d8       __imp__lua_objlen          1004c2d8     lua51:lua51.dll
 0002:000002dc       __imp__lua_topointer       1004c2dc     lua51:lua51.dll
 0002:000002e0       __imp__lua_isstring        1004c2e0     lua51:lua51.dll
 0002:000002e4       __imp__lua_tointeger       1004c2e4     lua51:lua51.dll
 0002:000002e8       __imp__lua_createtable     1004c2e8     lua51:lua51.dll
 0002:000002ec       __imp__lua_gettable        1004c2ec     lua51:lua51.dll
 0002:000002f0       __imp__lua_pushlightuserdata 1004c2f0     lua51:lua51.dll
 0002:000002f4       __imp__lua_pushlstring     1004c2f4     lua51:lua51.dll
 0002:000002f8       __imp__lua_isnumber        1004c2f8     lua51:lua51.dll
 0002:000002fc       __imp__lua_pushinteger     1004c2fc     lua51:lua51.dll
 0002:00000300       __imp__lua_pushnil         1004c300     lua51:lua51.dll
 0002:00000304       __imp__lua_replace         1004c304     lua51:lua51.dll
 0002:00000308       __imp__luaL_argerror       1004c308     lua51:lua51.dll
 0002:0000030c       __imp__lua_pushvalue       1004c30c     lua51:lua51.dll
 0002:00000310       __imp__luaL_newmetatable   1004c310     lua51:lua51.dll
 0002:00000314       __imp__lua_settop          1004c314     lua51:lua51.dll
 0002:00000318       __imp__lua_setmetatable    1004c318     lua51:lua51.dll
 0002:0000031c       __imp__luaL_register       1004c31c     lua51:lua51.dll
 0002:00000320       __imp__lua_getfield        1004c320     lua51:lua51.dll
 0002:00000324       __imp__lua_gettop          1004c324     lua51:lua51.dll
 0002:00000328       __imp__lua_pushnumber      1004c328     lua51:lua51.dll
 0002:0000032c       __imp__lua_pushstring      1004c32c     lua51:lua51.dll
 0002:00000330       __imp__lua_touserdata      1004c330     lua51:lua51.dll
 0002:00000334       __imp__lua_call            1004c334     lua51:lua51.dll
 0002:00000338       __imp__lua_tolstring       1004c338     lua51:lua51.dll
 0002:0000033c       __imp__lua_pushboolean     1004c33c     lua51:lua51.dll
 0002:00000340       __imp__lua_tonumber        1004c340     lua51:lua51.dll
 0002:00000344       __imp__lua_newuserdata     1004c344     lua51:lua51.dll
 0002:00000348       __imp__luaL_checkinteger   1004c348     lua51:lua51.dll
 0002:0000034c       __imp__lua_setfield        1004c34c     lua51:lua51.dll
 0002:00000350       __imp__lua_type            1004c350     lua51:lua51.dll
 0002:00000354       __imp__lua_rawequal        1004c354     lua51:lua51.dll
 0002:00000358       __imp__lua_getmetatable    1004c358     lua51:lua51.dll
 0002:0000035c       __imp__lua_pushcclosure    1004c35c     lua51:lua51.dll
 0002:00000360       __imp__luaL_error          1004c360     lua51:lua51.dll
 0002:00000364       __imp__luaL_checklstring   1004c364     lua51:lua51.dll
 0002:00000368       __imp__luaL_buffinit       1004c368     lua51:lua51.dll
 0002:0000036c       __imp__luaL_addlstring     1004c36c     lua51:lua51.dll
 0002:00000370       __imp__lua_load            1004c370     lua51:lua51.dll
 0002:00000374       __imp__lua_error           1004c374     lua51:lua51.dll
 0002:00000378       __imp__lua_pushfstring     1004c378     lua51:lua51.dll
 0002:0000037c       __imp__lua_concat          1004c37c     lua51:lua51.dll
 0002:00000380       __imp__lua_gc              1004c380     lua51:lua51.dll
 0002:00000384       __imp__luaL_pushresult     1004c384     lua51:lua51.dll
 0002:00000388       __imp__luaL_ref            1004c388     lua51:lua51.dll
 0002:0000038c       \177lua51_NULL_THUNK_DATA  1004c38c     lua51:lua51.dll
 0002:00000390       ___guard_check_icall_fptr  1004c390     LIBCMT:guard_support.obj
 0002:00000394       ___xc_a                    1004c394     LIBCMT:initializers.obj
 0002:00000398       ___xc_z                    1004c398     LIBCMT:initializers.obj
 0002:0000039c       ___xi_a                    1004c39c     LIBCMT:initializers.obj
 0002:000003a0       ___acrt_stdio_initializer  1004c3a0     libucrt:stdio_initializer.obj
 0002:000003a4       ___acrt_multibyte_initializer 1004c3a4     libucrt:multibyte_initializer.obj
 0002:000003a8       ___acrt_tran_sse2_initializer 1004c3a8     libucrt:sse2_initializer.obj
 0002:000003ac       ___xi_z                    1004c3ac     LIBCMT:initializers.obj
 0002:000003b0       ___xp_a                    1004c3b0     LIBCMT:initializers.obj
 0002:000003b4       ___acrt_locale_terminator  1004c3b4     libucrt:locale_initializer.obj
 0002:000003b8       ___acrt_tmpfile_terminator 1004c3b8     libucrt:tmpfile_initializer.obj
 0002:000003bc       ___dcrt_console_output_terminator 1004c3bc     libucrt:console_output_initializer.obj
 0002:000003c0       ___acrt_stdio_terminator   1004c3c0     libucrt:stdio_initializer.obj
 0002:000003c4       ___xp_z                    1004c3c4     LIBCMT:initializers.obj
 0002:000003c8       ___xt_a                    1004c3c8     LIBCMT:initializers.obj
 0002:000003cc       ___xt_z                    1004c3cc     LIBCMT:initializers.obj
 0002:000003d0       __imp__EncodePointer@4     1004c3d0     vc_crt_fix.obj
 0002:000003d4       __imp__DecodePointer@4     1004c3d4     vc_crt_fix.obj
 0002:000003d8       __imp__GetModuleHandleExW@12 1004c3d8     vc_crt_fix.obj
 0002:000003dc       __imp__InitializeSListHead@4 1004c3dc     vc_crt_fix.obj
 0002:000003e0       __imp__InterlockedFlushSList@4 1004c3e0     vc_crt_fix.obj
 0002:000003e4       __imp__InterlockedPopEntrySList@4 1004c3e4     vc_crt_fix.obj
 0002:000003e8       __imp__InterlockedPushEntrySList@8 1004c3e8     vc_crt_fix.obj
 0002:000003ec       __imp__InterlockedPushListSListEx@16 1004c3ec     vc_crt_fix.obj
 0002:000003f0       __imp__RtlFirstEntrySList@4 1004c3f0     vc_crt_fix.obj
 0002:000003f4       __imp__QueryDepthSList@4   1004c3f4     vc_crt_fix.obj
 0002:000003f8       __imp__GetNumaHighestNodeNumber@4 1004c3f8     vc_crt_fix.obj
 0002:000003fc       __imp__GetLogicalProcessorInformation@8 1004c3fc     vc_crt_fix.obj
 0002:00000400       __imp__SetThreadStackGuarantee@4 1004c400     vc_crt_fix.obj
 0002:00000404       __imp__InitializeCriticalSectionEx@12 1004c404     vc_crt_fix.obj
 0002:00000408       __imp__CompareStringEx@36  1004c408     vc_crt_fix.obj
 0002:0000040c       __imp__LCMapStringEx@36    1004c40c     vc_crt_fix.obj
 0002:00000418       __pRawDllMain              1004c418     LIBCMT:dll_dllmain.obj
 0002:00000418       __pDefaultRawDllMain       1004c418     LIBCMT:dll_dllmain.obj
 0002:0000041c       __pDestructExceptionObject 1004c41c     libvcruntime:ehhelpers.obj
 0002:00000424       ??_7exception@std@@6B@     1004c424     libvcruntime:frame.obj
 0002:0000042c       ??_C@_0BC@EOODALEL@Unknown?5exception@ 1004c42c     libvcruntime:frame.obj
 0002:00000444       ??_7bad_exception@std@@6B@ 1004c444     libvcruntime:frame.obj
 0002:0000044c       ??_C@_0O@DPKOEFFH@bad?5exception@ 1004c44c     libvcruntime:frame.obj
 0002:000007e0       ??_C@_08EHJDFFNH@__based?$CI@ 1004c7e0     libvcruntime:undname.obj
 0002:000007ec       ??_C@_07KOLFKCDI@__cdecl@  1004c7ec     libvcruntime:undname.obj
 0002:000007f4       ??_C@_08GHMPAG@__pascal@   1004c7f4     libvcruntime:undname.obj
 0002:00000800       ??_C@_09IFJBGAPI@__stdcall@ 1004c800     libvcruntime:undname.obj
 0002:0000080c       ??_C@_0L@NPHFGOKO@__thiscall@ 1004c80c     libvcruntime:undname.obj
 0002:00000818       ??_C@_0L@JMKHOMEK@__fastcall@ 1004c818     libvcruntime:undname.obj
 0002:00000824       ??_C@_0N@BCKKPABJ@__vectorcall@ 1004c824     libvcruntime:undname.obj
 0002:00000834       ??_C@_09HIJEGCPM@__clrcall@ 1004c834     libvcruntime:undname.obj
 0002:00000840       ??_C@_06GHPCKEAG@__eabi@   1004c840     libvcruntime:undname.obj
 0002:00000848       ??_C@_09IOPIDJLG@__swift_1@ 1004c848     libvcruntime:undname.obj
 0002:00000854       ??_C@_09KFNFGKHF@__swift_2@ 1004c854     libvcruntime:undname.obj
 0002:00000860       ??_C@_07JOMMBBKO@__ptr64@  1004c860     libvcruntime:undname.obj
 0002:00000868       ??_C@_0L@PILCLIHE@__restrict@ 1004c868     libvcruntime:undname.obj
 0002:00000874       ??_C@_0M@GFIIJFMG@__unaligned@ 1004c874     libvcruntime:undname.obj
 0002:00000880       ??_C@_09DHDLOLLB@restrict?$CI@ 1004c880     libvcruntime:undname.obj
 0002:0000088c       ??_C@_04NIHEBCM@?5new@     1004c88c     libvcruntime:undname.obj
 0002:00000894       ??_C@_07FPCDHGMM@?5delete@ 1004c894     libvcruntime:undname.obj
 0002:0000089c       ??_C@_01NEMOKFLO@?$DN@     1004c89c     libvcruntime:undname.obj
 0002:000008a0       ??_C@_02GPIOPFAK@?$DO?$DO@ 1004c8a0     libvcruntime:undname.obj
 0002:000008a4       ??_C@_02FODMEDOG@?$DM?$DM@ 1004c8a4     libvcruntime:undname.obj
 0002:000008a8       ??_C@_01DCLJPIOD@?$CB@     1004c8a8     libvcruntime:undname.obj
 0002:000008ac       ??_C@_02EGOFBIJA@?$DN?$DN@ 1004c8ac     libvcruntime:undname.obj
 0002:000008b0       ??_C@_02FDNJECIE@?$CB?$DN@ 1004c8b0     libvcruntime:undname.obj
 0002:000008b4       ??_C@_02GPECMEKF@?$FL?$FN@ 1004c8b4     libvcruntime:undname.obj
 0002:000008b8       ??_C@_08LHJFAFGD@operator@ 1004c8b8     libvcruntime:undname.obj
 0002:000008c4       ??_C@_02HBOOOICD@?9?$DO@   1004c8c4     libvcruntime:undname.obj
 0002:000008c8       ??_C@_01NBENCBCI@?$CK@     1004c8c8     libvcruntime:undname.obj
 0002:000008cc       ??_C@_02ECNGHCIF@?$CL?$CL@ 1004c8cc     libvcruntime:undname.obj
 0002:000008d0       ??_C@_02BAABKJLB@?9?9@     1004c8d0     libvcruntime:undname.obj
 0002:000008d4       ??_C@_01JOAMLHOP@?9@       1004c8d4     libvcruntime:undname.obj
 0002:000008d8       ??_C@_01MIFGBAGJ@?$CL@     1004c8d8     libvcruntime:undname.obj
 0002:000008dc       ??_C@_01HNPIGOCE@?$CG@     1004c8dc     libvcruntime:undname.obj
 0002:000008e0       ??_C@_03MNHNFDLC@?9?$DO?$CK@ 1004c8e0     libvcruntime:undname.obj
 0002:000008e4       ??_C@_01FGNFDNOH@?$CF@     1004c8e4     libvcruntime:undname.obj
 0002:000008e8       ??_C@_01MNNFJEPP@?$DM@     1004c8e8     libvcruntime:undname.obj
 0002:000008ec       ??_C@_02EHCHHCKH@?$DM?$DN@ 1004c8ec     libvcruntime:undname.obj
 0002:000008f0       ??_C@_01PPODPGHN@?$DO@     1004c8f0     libvcruntime:undname.obj
 0002:000008f4       ??_C@_02EEKDKGMJ@?$DO?$DN@ 1004c8f4     libvcruntime:undname.obj
 0002:000008f8       ??_C@_01IHBHIGKO@?0@       1004c8f8     libvcruntime:undname.obj
 0002:000008fc       ??_C@_02HCKGKOFO@?$CI?$CJ@ 1004c8fc     libvcruntime:undname.obj
 0002:00000900       ??_C@_01PJKLJHI@?$HO@      1004c900     libvcruntime:undname.obj
 0002:00000904       ??_C@_01JKBOJNNK@?$FO@     1004c904     libvcruntime:undname.obj
 0002:00000908       ??_C@_01DNKMNLPK@?$HM@     1004c908     libvcruntime:undname.obj
 0002:0000090c       ??_C@_02PPKAJPJL@?$CG?$CG@ 1004c90c     libvcruntime:undname.obj
 0002:00000910       ??_C@_02NONPIBCD@?$HM?$HM@ 1004c910     libvcruntime:undname.obj
 0002:00000914       ??_C@_02FPIMKNGF@?$CK?$DN@ 1004c914     libvcruntime:undname.obj
 0002:00000918       ??_C@_02FOEOMHFC@?$CL?$DN@ 1004c918     libvcruntime:undname.obj
 0002:0000091c       ??_C@_02FKMDLLOA@?9?$DN@   1004c91c     libvcruntime:undname.obj
 0002:00000920       ??_C@_02FJEHGPIO@?1?$DN@   1004c920     libvcruntime:undname.obj
 0002:00000924       ??_C@_02FENAOKFI@?$CF?$DN@ 1004c924     libvcruntime:undname.obj
 0002:00000928       ??_C@_03IKFCCPFF@?$DO?$DO?$DN@ 1004c928     libvcruntime:undname.obj
 0002:0000092c       ??_C@_03CDNPDDLA@?$DM?$DM?$DN@ 1004c92c     libvcruntime:undname.obj
 0002:00000930       ??_C@_02FGJGFEAB@?$CG?$DN@ 1004c930     libvcruntime:undname.obj
 0002:00000934       ??_C@_02DHLNPPGH@?$HM?$DN@ 1004c934     libvcruntime:undname.obj
 0002:00000938       ??_C@_02MHEGNOJ@?$FO?$DN@  1004c938     libvcruntime:undname.obj
 0002:0000093c       ??_C@_09IFPLHPGF@?$GAvftable?8@ 1004c93c     libvcruntime:undname.obj
 0002:00000948       ??_C@_09BLBHBJP@?$GAvbtable?8@ 1004c948     libvcruntime:undname.obj
 0002:00000954       ??_C@_07FEEIOKP@?$GAvcall?8@ 1004c954     libvcruntime:undname.obj
 0002:0000095c       ??_C@_08LLFFHHDJ@?$GAtypeof?8@ 1004c95c     libvcruntime:undname.obj
 0002:00000968       ??_C@_0BF@KDPPACIK@?$GAlocal?5static?5guard?8@ 1004c968     libvcruntime:undname.obj
 0002:00000980       ??_C@_08OBABFOLI@?$GAstring?8@ 1004c980     libvcruntime:undname.obj
 0002:0000098c       ??_C@_0BD@JDLKDPAB@?$GAvbase?5destructor?8@ 1004c98c     libvcruntime:undname.obj
 0002:000009a0       ??_C@_0BN@DEGPLNFK@?$GAvector?5deleting?5destructor?8@ 1004c9a0     libvcruntime:undname.obj
 0002:000009c0       ??_C@_0BO@OBMKPJIG@?$GAdefault?5constructor?5closure?8@ 1004c9c0     libvcruntime:undname.obj
 0002:000009e0       ??_C@_0BN@IMDCHIKM@?$GAscalar?5deleting?5destructor?8@ 1004c9e0     libvcruntime:undname.obj
 0002:00000a00       ??_C@_0BO@PFGOCPJJ@?$GAvector?5constructor?5iterator?8@ 1004ca00     libvcruntime:undname.obj
 0002:00000a20       ??_C@_0BN@LFPFMEDL@?$GAvector?5destructor?5iterator?8@ 1004ca20     libvcruntime:undname.obj
 0002:00000a40       ??_C@_0CE@IKBNEHA@?$GAvector?5vbase?5constructor?5itera@ 1004ca40     libvcruntime:undname.obj
 0002:00000a64       ??_C@_0BL@NILFHHPC@?$GAvirtual?5displacement?5map?8@ 1004ca64     libvcruntime:undname.obj
 0002:00000a80       ??_C@_0CB@JONCMFFK@?$GAeh?5vector?5constructor?5iterator@ 1004ca80     libvcruntime:undname.obj
 0002:00000aa4       ??_C@_0CA@GCEOPDGL@?$GAeh?5vector?5destructor?5iterator?8@ 1004caa4     libvcruntime:undname.obj
 0002:00000ac4       ??_C@_0CH@OOJPLCPH@?$GAeh?5vector?5vbase?5constructor?5it@ 1004cac4     libvcruntime:undname.obj
 0002:00000aec       ??_C@_0BL@LLKPOHJI@?$GAcopy?5constructor?5closure?8@ 1004caec     libvcruntime:undname.obj
 0002:00000b08       ??_C@_0BA@KBCDOMBN@?$GAudt?5returning?8@ 1004cb08     libvcruntime:undname.obj
 0002:00000b18       ??_C@_03KLGMFNMG@?$GAEH@   1004cb18     libvcruntime:undname.obj
 0002:00000b1c       ??_C@_05KHLCHHI@?$GARTTI@  1004cb1c     libvcruntime:undname.obj
 0002:00000b24       ??_C@_0BA@KKLDJDLB@?$GAlocal?5vftable?8@ 1004cb24     libvcruntime:undname.obj
 0002:00000b34       ??_C@_0CE@IIHCMGGL@?$GAlocal?5vftable?5constructor?5clos@ 1004cb34     libvcruntime:undname.obj
 0002:00000b58       ??_C@_06FHBGPFGH@?5new?$FL?$FN@ 1004cb58     libvcruntime:undname.obj
 0002:00000b60       ??_C@_09LBNFPBCA@?5delete?$FL?$FN@ 1004cb60     libvcruntime:undname.obj
 0002:00000b6c       ??_C@_0P@HJKNJFNN@?$GAomni?5callsig?8@ 1004cb6c     libvcruntime:undname.obj
 0002:00000b7c       ??_C@_0BL@CNOONJFP@?$GAplacement?5delete?5closure?8@ 1004cb7c     libvcruntime:undname.obj
 0002:00000b98       ??_C@_0BN@CKNJLHMB@?$GAplacement?5delete?$FL?$FN?5closure?8@ 1004cb98     libvcruntime:undname.obj
 0002:00000bb8       ??_C@_0CG@CFDHKGGD@?$GAmanaged?5vector?5constructor?5ite@ 1004cbb8     libvcruntime:undname.obj
 0002:00000be0       ??_C@_0CF@IMGKMJNO@?$GAmanaged?5vector?5destructor?5iter@ 1004cbe0     libvcruntime:undname.obj
 0002:00000c08       ??_C@_0CG@HLDDJMAG@?$GAeh?5vector?5copy?5constructor?5ite@ 1004cc08     libvcruntime:undname.obj
 0002:00000c30       ??_C@_0CM@FCBBDIGB@?$GAeh?5vector?5vbase?5copy?5construct@ 1004cc30     libvcruntime:undname.obj
 0002:00000c5c       ??_C@_0BL@CLIPGLGB@?$GAdynamic?5initializer?5for?5?8@ 1004cc5c     libvcruntime:undname.obj
 0002:00000c78       ??_C@_0CB@PDBIFEP@?$GAdynamic?5atexit?5destructor?5for?5@ 1004cc78     libvcruntime:undname.obj
 0002:00000c9c       ??_C@_0CD@CGAJBKEJ@?$GAvector?5copy?5constructor?5iterat@ 1004cc9c     libvcruntime:undname.obj
 0002:00000cc0       ??_C@_0CJ@GJELGAMM@?$GAvector?5vbase?5copy?5constructor?5@ 1004ccc0     libvcruntime:undname.obj
 0002:00000cec       ??_C@_0CL@FGIJHLCE@?$GAmanaged?5vector?5copy?5constructo@ 1004ccec     libvcruntime:undname.obj
 0002:00000d18       ??_C@_0BM@PMGGMLDN@?$GAlocal?5static?5thread?5guard?8@ 1004cd18     libvcruntime:undname.obj
 0002:00000d34       ??_C@_0N@BDNMDMOL@operator?5?$CC?$CC?5@ 1004cd34     libvcruntime:undname.obj
 0002:00000d44       ??_C@_0BC@GGEBGALA@operator?5co_await@ 1004cd44     libvcruntime:undname.obj
 0002:00000d58       ??_C@_0M@GAAIMMOH@operator?$DM?$DN?$DO@ 1004cd58     libvcruntime:undname.obj
 0002:00000d64       ??_C@_0BC@DAFEJGAK@?5Type?5Descriptor?8@ 1004cd64     libvcruntime:undname.obj
 0002:00000d78       ??_C@_0BM@LDKODKLH@?5Base?5Class?5Descriptor?5at?5?$CI@ 1004cd78     libvcruntime:undname.obj
 0002:00000d94       ??_C@_0BD@LGICGFMM@?5Base?5Class?5Array?8@ 1004cd94     libvcruntime:undname.obj
 0002:00000da8       ??_C@_0BN@MECKDCOJ@?5Class?5Hierarchy?5Descriptor?8@ 1004cda8     libvcruntime:undname.obj
 0002:00000dc8       ??_C@_0BK@CFCOFLF@?5Complete?5Object?5Locator?8@ 1004cdc8     libvcruntime:undname.obj
 0002:00000de4       ??_C@_0BG@JNJLAMPM@?$GAanonymous?5namespace?8@ 1004cde4     libvcruntime:undname.obj
 0002:00000e08       ??_C@_1DM@KHCHBNEB@?$AAa?$AAp?$AAi?$AA?9?$AAm?$AAs?$AA?9?$AAw?$AAi?$AAn?$AA?9?$AAc?$AAo?$AAr?$AAe@ 1004ce08     libvcruntime:winapi_downlevel.obj
 0002:00000e44       ??_C@_1DK@LPPGFMPP@?$AAa?$AAp?$AAi?$AA?9?$AAm?$AAs?$AA?9?$AAw?$AAi?$AAn?$AA?9?$AAc?$AAo?$AAr?$AAe@ 1004ce44     libvcruntime:winapi_downlevel.obj
 0002:00000e80       ??_C@_1BC@GDMECMAK@?$AAk?$AAe?$AAr?$AAn?$AAe?$AAl?$AA3?$AA2@ 1004ce80     libvcruntime:winapi_downlevel.obj
 0002:00000e94       ??_C@_1BA@PFFKHIOG@?$AAa?$AAp?$AAi?$AA?9?$AAm?$AAs?$AA?9@ 1004ce94     libvcruntime:winapi_downlevel.obj
 0002:00000eac       ??_C@_08KNHFBNJ@FlsAlloc@  1004ceac     libvcruntime:winapi_downlevel.obj
 0002:00000ec0       ??_C@_07PEJMOBNF@FlsFree@  1004cec0     libvcruntime:winapi_downlevel.obj
 0002:00000ed0       ??_C@_0M@GDNOONDI@FlsGetValue@ 1004ced0     libvcruntime:winapi_downlevel.obj
 0002:00000ee4       ??_C@_0M@JCPCPOEF@FlsSetValue@ 1004cee4     libvcruntime:winapi_downlevel.obj
 0002:00000ef8       _standard_lookup_table     1004cef8     libucrt:output.obj
 0002:00000f54       ??_C@_1O@CEDCILHN@?$AA?$CI?$AAn?$AAu?$AAl?$AAl?$AA?$CJ@ 1004cf54     libucrt:output.obj
 0002:00000f64       ??_C@_06OJHGLDPL@?$CInull?$CJ@ 1004cf64     libucrt:output.obj
 0002:000010d8       ??_C@_0EA@FCLIIPNN@Visual?5C?$CL?$CL?5CRT?3?5Not?5enough?5memo@ 1004d0d8     libucrt:strerror.obj
 0002:00001158       ?large_power_data@?1??multiply_by_power_of_ten@__crt_strtox@@YA_NAAUbig_integer@2@I@Z@4QBIB 1004d158     libucrt:input.obj
 0002:00001af8       ?small_powers_of_ten@?1??multiply_by_power_of_ten@__crt_strtox@@YA_NAAUbig_integer@2@I@Z@4QBIB 1004daf8     libucrt:input.obj
 0002:00001b20       ??_C@_1GE@DPGDJKLM@?$AAm?$AAi?$AAn?$AAk?$AAe?$AAr?$AAn?$AAe?$AAl?$AA?2?$AAc?$AAr?$AAt?$AAs?$AA?2@ 1004db20     libucrt:input.obj
 0002:00001b88       ??_C@_1FM@FELNCOBF@?$AA_?$AA_?$AAc?$AAr?$AAt?$AA_?$AAs?$AAt?$AAr?$AAt?$AAo?$AAx?$AA?3?$AA?3?$AAf@ 1004db88     libucrt:input.obj
 0002:00001be4       ??_C@_1BG@GEMHBGAF@?$AA_?$AAi?$AAs?$AA_?$AAd?$AAo?$AAu?$AAb?$AAl?$AAe@ 1004dbe4     libucrt:input.obj
 0002:00001c00       ??_C@_1FK@JOJELFFO@?$AA_?$AA_?$AAc?$AAr?$AAt?$AA_?$AAs?$AAt?$AAr?$AAt?$AAo?$AAx?$AA?3?$AA?3?$AAf@ 1004dc00     libucrt:input.obj
 0002:00001c5c       ??_C@_1BI@BANMPGJI@?$AA?$CB?$AA_?$AAi?$AAs?$AA_?$AAd?$AAo?$AAu?$AAb?$AAl?$AAe@ 1004dc5c     libucrt:input.obj
 0002:00001c78       ?constraints@?1??is_length_valid@__crt_stdio_input@@YA_NW4conversion_mode@2@W4length_modifier@2@@Z@4QAY0M@$$CBEA 1004dc78     libucrt:input.obj
 0002:00001cf0       ?inf_uppercase@?1???$parse_floating_point_possible_infinity@DV?$input_adapter_character_source@V?$stream_input_adapter@D@__crt_stdio_input@@@__crt_strtox@@_K@__crt_strtox@@YA?AW4floating_point_parse_result@1@AADAAV?$input_adapter_character_source@V?$stream_input_adapter@D@__crt_stdio_input@@@1@_K@Z@4QBDB 1004dcf0     libucrt:input.obj
 0002:00001cf4       ?inf_lowercase@?1???$parse_floating_point_possible_infinity@DV?$input_adapter_character_source@V?$stream_input_adapter@D@__crt_stdio_input@@@__crt_strtox@@_K@__crt_strtox@@YA?AW4floating_point_parse_result@1@AADAAV?$input_adapter_character_source@V?$stream_input_adapter@D@__crt_stdio_input@@@1@_K@Z@4QBDB 1004dcf4     libucrt:input.obj
 0002:00001cf8       ?inity_uppercase@?1???$parse_floating_point_possible_infinity@DV?$input_adapter_character_source@V?$stream_input_adapter@D@__crt_stdio_input@@@__crt_strtox@@_K@__crt_strtox@@YA?AW4floating_point_parse_result@1@AADAAV?$input_adapter_character_source@V?$stream_input_adapter@D@__crt_stdio_input@@@1@_K@Z@4QBDB 1004dcf8     libucrt:input.obj
 0002:00001d00       ?inity_lowercase@?1???$parse_floating_point_possible_infinity@DV?$input_adapter_character_source@V?$stream_input_adapter@D@__crt_stdio_input@@@__crt_strtox@@_K@__crt_strtox@@YA?AW4floating_point_parse_result@1@AADAAV?$input_adapter_character_source@V?$stream_input_adapter@D@__crt_stdio_input@@@1@_K@Z@4QBDB 1004dd00     libucrt:input.obj
 0002:00001d08       ?uppercase@?1???$parse_floating_point_possible_nan@DV?$input_adapter_character_source@V?$stream_input_adapter@D@__crt_stdio_input@@@__crt_strtox@@_K@__crt_strtox@@YA?AW4floating_point_parse_result@1@AADAAV?$input_adapter_character_source@V?$stream_input_adapter@D@__crt_stdio_input@@@1@_K@Z@4QBDB 1004dd08     libucrt:input.obj
 0002:00001d0c       ?lowercase@?1???$parse_floating_point_possible_nan@DV?$input_adapter_character_source@V?$stream_input_adapter@D@__crt_stdio_input@@@__crt_strtox@@_K@__crt_strtox@@YA?AW4floating_point_parse_result@1@AADAAV?$input_adapter_character_source@V?$stream_input_adapter@D@__crt_stdio_input@@@1@_K@Z@4QBDB 1004dd0c     libucrt:input.obj
 0002:00001d10       ?uppercase@?1???$parse_floating_point_possible_nan_is_snan@DV?$input_adapter_character_source@V?$stream_input_adapter@D@__crt_stdio_input@@@__crt_strtox@@@__crt_strtox@@YA_NAADAAV?$input_adapter_character_source@V?$stream_input_adapter@D@__crt_stdio_input@@@1@@Z@4QBDB 1004dd10     libucrt:input.obj
 0002:00001d18       ?lowercase@?1???$parse_floating_point_possible_nan_is_snan@DV?$input_adapter_character_source@V?$stream_input_adapter@D@__crt_stdio_input@@@__crt_strtox@@@__crt_strtox@@YA_NAADAAV?$input_adapter_character_source@V?$stream_input_adapter@D@__crt_stdio_input@@@1@@Z@4QBDB 1004dd18     libucrt:input.obj
 0002:00001d20       ?uppercase@?1???$parse_floating_point_possible_nan_is_ind@DV?$input_adapter_character_source@V?$stream_input_adapter@D@__crt_stdio_input@@@__crt_strtox@@@__crt_strtox@@YA_NAADAAV?$input_adapter_character_source@V?$stream_input_adapter@D@__crt_stdio_input@@@1@@Z@4QBDB 1004dd20     libucrt:input.obj
 0002:00001d24       ?lowercase@?1???$parse_floating_point_possible_nan_is_ind@DV?$input_adapter_character_source@V?$stream_input_adapter@D@__crt_stdio_input@@@__crt_strtox@@@__crt_strtox@@YA_NAADAAV?$input_adapter_character_source@V?$stream_input_adapter@D@__crt_stdio_input@@@1@@Z@4QBDB 1004dd24     libucrt:input.obj
 0002:00001d50       ___acrt_exception_action_table 1004dd50     libucrt:exception_filter.obj
 0002:00001de0       ___acrt_signal_action_table_count 1004dde0     libucrt:exception_filter.obj
 0002:00001de4       ___acrt_signal_action_first_fpe_index 1004dde4     libucrt:exception_filter.obj
 0002:00001de8       ___acrt_signal_action_fpe_count 1004dde8     libucrt:exception_filter.obj
 0002:00001dec       ??_C@_1BI@BGOHAHKC@?$AAm?$AAs?$AAc?$AAo?$AAr?$AAe?$AAe?$AA?4?$AAd?$AAl?$AAl@ 1004ddec     libucrt:exit.obj
 0002:00001e04       ??_C@_0P@MIGLKIOC@CorExitProcess@ 1004de04     libucrt:exit.obj
 0002:00001ed8       ??_C@_03OEIAHPBN@INF@      1004ded8     libucrt:cvt.obj
 0002:00001edc       ??_C@_03OJHLLCGB@inf@      1004dedc     libucrt:cvt.obj
 0002:00001ee0       ??_C@_03LKNCIKJB@NAN@      1004dee0     libucrt:cvt.obj
 0002:00001ee4       ??_C@_03LHCJEHON@nan@      1004dee4     libucrt:cvt.obj
 0002:00001ee8       ??_C@_09OFJJIMPC@NAN?$CISNAN?$CJ@ 1004dee8     libucrt:cvt.obj
 0002:00001ef4       ??_C@_09IPFBKMDL@nan?$CIsnan?$CJ@ 1004def4     libucrt:cvt.obj
 0002:00001f00       ??_C@_08IKHNHAJ@NAN?$CIIND?$CJ@ 1004df00     libucrt:cvt.obj
 0002:00001f0c       ??_C@_08OFCDMILK@nan?$CIind?$CJ@ 1004df0c     libucrt:cvt.obj
 0002:00001f18       ??_C@_05KLBDPFGC@e?$CL000@ 1004df18     libucrt:cvt.obj
 0002:00001f20       ___lc_time_c               1004df20     libucrt:nlsdata.obj
 0002:00002084       ??_C@_03KOEHGMDN@Sun@      1004e084     libucrt:nlsdata.obj
 0002:00002088       ??_C@_03PDAGKDH@Mon@       1004e088     libucrt:nlsdata.obj
 0002:0000208c       ??_C@_03NAGEINEP@Tue@      1004e08c     libucrt:nlsdata.obj
 0002:00002090       ??_C@_03MHOMLAJA@Wed@      1004e090     libucrt:nlsdata.obj
 0002:00002094       ??_C@_03IOFIKPDN@Thu@      1004e094     libucrt:nlsdata.obj
 0002:00002098       ??_C@_03IDIOELNC@Fri@      1004e098     libucrt:nlsdata.obj
 0002:0000209c       ??_C@_03FEFJNEK@Sat@       1004e09c     libucrt:nlsdata.obj
 0002:000020a0       ??_C@_06OOPIFAJ@Sunday@    1004e0a0     libucrt:nlsdata.obj
 0002:000020a8       ??_C@_06JLEDEDGH@Monday@   1004e0a8     libucrt:nlsdata.obj
 0002:000020b0       ??_C@_07BAAGCFCM@Tuesday@  1004e0b0     libucrt:nlsdata.obj
 0002:000020b8       ??_C@_09DLIGFAKA@Wednesday@ 1004e0b8     libucrt:nlsdata.obj
 0002:000020c4       ??_C@_08HACCIKIA@Thursday@ 1004e0c4     libucrt:nlsdata.obj
 0002:000020d0       ??_C@_06JECMNKMI@Friday@   1004e0d0     libucrt:nlsdata.obj
 0002:000020d8       ??_C@_08INBOOONO@Saturday@ 1004e0d8     libucrt:nlsdata.obj
 0002:000020e4       ??_C@_03JIHJHPIE@Jan@      1004e0e4     libucrt:nlsdata.obj
 0002:000020e8       ??_C@_03HJBDCHOM@Feb@      1004e0e8     libucrt:nlsdata.obj
 0002:000020ec       ??_C@_03ODNJBKGA@Mar@      1004e0ec     libucrt:nlsdata.obj
 0002:000020f0       ??_C@_03LEOLGMJP@Apr@      1004e0f0     libucrt:nlsdata.obj
 0002:000020f4       ??_C@_03CNMDKL@May@        1004e0f4     libucrt:nlsdata.obj
 0002:000020f8       ??_C@_03IDFGHECI@Jun@      1004e0f8     libucrt:nlsdata.obj
 0002:000020fc       ??_C@_03LBGABGKK@Jul@      1004e0fc     libucrt:nlsdata.obj
 0002:00002100       ??_C@_03IFJFEIGA@Aug@      1004e100     libucrt:nlsdata.obj
 0002:00002104       ??_C@_03GGCAPAJC@Sep@      1004e104     libucrt:nlsdata.obj
 0002:00002108       ??_C@_03BMAOKBAD@Oct@      1004e108     libucrt:nlsdata.obj
 0002:0000210c       ??_C@_03JPJOFNIA@Nov@      1004e10c     libucrt:nlsdata.obj
 0002:00002110       ??_C@_03MKABNOCG@Dec@      1004e110     libucrt:nlsdata.obj
 0002:00002114       ??_C@_07CGJPFGJA@January@  1004e114     libucrt:nlsdata.obj
 0002:0000211c       ??_C@_08GNJGEPFN@February@ 1004e11c     libucrt:nlsdata.obj
 0002:00002128       ??_C@_05HPCKOFNC@March@    1004e128     libucrt:nlsdata.obj
 0002:00002130       ??_C@_05DMJDNLEJ@April@    1004e130     libucrt:nlsdata.obj
 0002:00002138       ??_C@_04CNLMGBGM@June@     1004e138     libucrt:nlsdata.obj
 0002:00002140       ??_C@_04MIEPOIFP@July@     1004e140     libucrt:nlsdata.obj
 0002:00002148       ??_C@_06LBBHFDDG@August@   1004e148     libucrt:nlsdata.obj
 0002:00002150       ??_C@_09BHHEALKD@September@ 1004e150     libucrt:nlsdata.obj
 0002:0000215c       ??_C@_07JJNFCEND@October@  1004e15c     libucrt:nlsdata.obj
 0002:00002164       ??_C@_08HCHEGEOA@November@ 1004e164     libucrt:nlsdata.obj
 0002:00002170       ??_C@_08EDHMEBNP@December@ 1004e170     libucrt:nlsdata.obj
 0002:0000217c       ??_C@_02DEDBPAFC@AM@       1004e17c     libucrt:nlsdata.obj
 0002:00002180       ??_C@_02CJNFDJBF@PM@       1004e180     libucrt:nlsdata.obj
 0002:00002184       ??_C@_08BPBNCDIB@MM?1dd?1yy@ 1004e184     libucrt:nlsdata.obj
 0002:00002190       ??_C@_0BE@CKGJFCPC@dddd?0?5MMMM?5dd?0?5yyyy@ 1004e190     libucrt:nlsdata.obj
 0002:000021a4       ??_C@_08JCCMCCIL@HH?3mm?3ss@ 1004e1a4     libucrt:nlsdata.obj
 0002:000021b0       ??_C@_17MBGCMIPB@?$AAS?$AAu?$AAn@ 1004e1b0     libucrt:nlsdata.obj
 0002:000021b8       ??_C@_17KBOMKBF@?$AAM?$AAo?$AAn@ 1004e1b8     libucrt:nlsdata.obj
 0002:000021c0       ??_C@_17BMKGEGOJ@?$AAT?$AAu?$AAe@ 1004e1c0     libucrt:nlsdata.obj
 0002:000021c8       ??_C@_17CJEDCEPE@?$AAW?$AAe?$AAd@ 1004e1c8     libucrt:nlsdata.obj
 0002:000021d0       ??_C@_17PDPHAADD@?$AAT?$AAh?$AAu@ 1004e1d0     libucrt:nlsdata.obj
 0002:000021d8       ??_C@_17HFOLPPLP@?$AAF?$AAr?$AAi@ 1004e1d8     libucrt:nlsdata.obj
 0002:000021e0       ??_C@_17GGIBDPIH@?$AAS?$AAa?$AAt@ 1004e1e0     libucrt:nlsdata.obj
 0002:000021e8       ??_C@_1O@IHNHDHPB@?$AAS?$AAu?$AAn?$AAd?$AAa?$AAy@ 1004e1e8     libucrt:nlsdata.obj
 0002:000021f8       ??_C@_1O@MMNBFLIA@?$AAM?$AAo?$AAn?$AAd?$AAa?$AAy@ 1004e1f8     libucrt:nlsdata.obj
 0002:00002208       ??_C@_1BA@ENFBFFEK@?$AAT?$AAu?$AAe?$AAs?$AAd?$AAa?$AAy@ 1004e208     libucrt:nlsdata.obj
 0002:00002218       ??_C@_1BE@EBOGMDOH@?$AAW?$AAe?$AAd?$AAn?$AAe?$AAs?$AAd?$AAa?$AAy@ 1004e218     libucrt:nlsdata.obj
 0002:0000222c       ??_C@_1BC@HHMNLIHE@?$AAT?$AAh?$AAu?$AAr?$AAs?$AAd?$AAa?$AAy@ 1004e22c     libucrt:nlsdata.obj
 0002:00002240       ??_C@_1O@PDICJHAG@?$AAF?$AAr?$AAi?$AAd?$AAa?$AAy@ 1004e240     libucrt:nlsdata.obj
 0002:00002250       ??_C@_1BC@ENMNNPAJ@?$AAS?$AAa?$AAt?$AAu?$AAr?$AAd?$AAa?$AAy@ 1004e250     libucrt:nlsdata.obj
 0002:00002264       ??_C@_17DKNBKCHM@?$AAJ?$AAa?$AAn@ 1004e264     libucrt:nlsdata.obj
 0002:0000226c       ??_C@_17LMDJEKJN@?$AAF?$AAe?$AAb@ 1004e26c     libucrt:nlsdata.obj
 0002:00002274       ??_C@_17CKNLEDEC@?$AAM?$AAa?$AAr@ 1004e274     libucrt:nlsdata.obj
 0002:0000227c       ??_C@_17LFPOIHDD@?$AAA?$AAp?$AAr@ 1004e27c     libucrt:nlsdata.obj
 0002:00002284       ??_C@_17PNNKMEED@?$AAM?$AAa?$AAy@ 1004e284     libucrt:nlsdata.obj
 0002:0000228c       ??_C@_17KCJGOCPB@?$AAJ?$AAu?$AAn@ 1004e28c     libucrt:nlsdata.obj
 0002:00002294       ??_C@_17IJPCKHK@?$AAJ?$AAu?$AAl@ 1004e294     libucrt:nlsdata.obj
 0002:0000229c       ??_C@_17ICPELBCN@?$AAA?$AAu?$AAg@ 1004e29c     libucrt:nlsdata.obj
 0002:000022a4       ??_C@_17HCHCOKMG@?$AAS?$AAe?$AAp@ 1004e2a4     libucrt:nlsdata.obj
 0002:000022ac       ??_C@_17FNLKOI@?$AAO?$AAc?$AAt@ 1004e2ac     libucrt:nlsdata.obj
 0002:000022b4       ??_C@_17BBDMLCIG@?$AAN?$AAo?$AAv@ 1004e2b4     libucrt:nlsdata.obj
 0002:000022bc       ??_C@_17EGKACKIF@?$AAD?$AAe?$AAc@ 1004e2bc     libucrt:nlsdata.obj
 0002:000022c4       ??_C@_1BA@EFMEIEBA@?$AAJ?$AAa?$AAn?$AAu?$AAa?$AAr?$AAy@ 1004e2c4     libucrt:nlsdata.obj
 0002:000022d4       ??_C@_1BC@JGDDFFAM@?$AAF?$AAe?$AAb?$AAr?$AAu?$AAa?$AAr?$AAy@ 1004e2d4     libucrt:nlsdata.obj
 0002:000022e8       ??_C@_1M@IKEENEDF@?$AAM?$AAa?$AAr?$AAc?$AAh@ 1004e2e8     libucrt:nlsdata.obj
 0002:000022f4       ??_C@_1M@GJNLMHFD@?$AAA?$AAp?$AAr?$AAi?$AAl@ 1004e2f4     libucrt:nlsdata.obj
 0002:00002300       ??_C@_19EPFLPGAP@?$AAJ?$AAu?$AAn?$AAe@ 1004e300     libucrt:nlsdata.obj
 0002:0000230c       ??_C@_19BIFMLPCD@?$AAJ?$AAu?$AAl?$AAy@ 1004e30c     libucrt:nlsdata.obj
 0002:00002318       ??_C@_1O@PAHLKOAC@?$AAA?$AAu?$AAg?$AAu?$AAs?$AAt@ 1004e318     libucrt:nlsdata.obj
 0002:00002328       ??_C@_1BE@DKAAMBJL@?$AAS?$AAe?$AAp?$AAt?$AAe?$AAm?$AAb?$AAe?$AAr@ 1004e328     libucrt:nlsdata.obj
 0002:0000233c       ??_C@_1BA@EPANDLNG@?$AAO?$AAc?$AAt?$AAo?$AAb?$AAe?$AAr@ 1004e33c     libucrt:nlsdata.obj
 0002:0000234c       ??_C@_1BC@BGLIFPF@?$AAN?$AAo?$AAv?$AAe?$AAm?$AAb?$AAe?$AAr@ 1004e34c     libucrt:nlsdata.obj
 0002:00002360       ??_C@_1BC@FEMKIFH@?$AAD?$AAe?$AAc?$AAe?$AAm?$AAb?$AAe?$AAr@ 1004e360     libucrt:nlsdata.obj
 0002:00002374       ??_C@_15ODEHAHHF@?$AAA?$AAM@ 1004e374     libucrt:nlsdata.obj
 0002:0000237c       ??_C@_15CLMNNGEL@?$AAP?$AAM@ 1004e37c     libucrt:nlsdata.obj
 0002:00002384       ??_C@_1BC@IEBCMHCM@?$AAM?$AAM?$AA?1?$AAd?$AAd?$AA?1?$AAy?$AAy@ 1004e384     libucrt:nlsdata.obj
 0002:00002398       ??_C@_1CI@KNAKOEBC@?$AAd?$AAd?$AAd?$AAd?$AA?0?$AA?5?$AAM?$AAM?$AAM?$AAM?$AA?5?$AAd?$AAd?$AA?0?$AA?5@ 1004e398     libucrt:nlsdata.obj
 0002:000023c0       ??_C@_1BC@GDGBMEMK@?$AAH?$AAH?$AA?3?$AAm?$AAm?$AA?3?$AAs?$AAs@ 1004e3c0     libucrt:nlsdata.obj
 0002:000023d4       ??_C@_1M@BMHNFIME@?$AAe?$AAn?$AA?9?$AAU?$AAS@ 1004e3d4     libucrt:nlsdata.obj
 0002:000023f8       ?ccs@?1???$__acrt_stdio_parse_mode@_W@@YA?AU__acrt_stdio_stream_mode@@QB_W@Z@4QB_WB 1004e3f8     libucrt:openfile.obj
 0002:00002400       ?utf8_encoding@?1???$__acrt_stdio_parse_mode@_W@@YA?AU__acrt_stdio_stream_mode@@QB_W@Z@4QB_WB 1004e400     libucrt:openfile.obj
 0002:0000240c       ?utf16_encoding@?1???$__acrt_stdio_parse_mode@_W@@YA?AU__acrt_stdio_stream_mode@@QB_W@Z@4QB_WB 1004e40c     libucrt:openfile.obj
 0002:0000241c       ?unicode_encoding@?1???$__acrt_stdio_parse_mode@_W@@YA?AU__acrt_stdio_stream_mode@@QB_W@Z@4QB_WB 1004e41c     libucrt:openfile.obj
 0002:00002480       ??_C@_1EA@JGEFHKEI@?$AAa?$AAp?$AAi?$AA?9?$AAm?$AAs?$AA?9?$AAw?$AAi?$AAn?$AA?9?$AAc?$AAo?$AAr?$AAe@ 1004e480     libucrt:winapi_thunks.obj
 0002:000024c0       ??_C@_1DI@IJCEHOCB@?$AAa?$AAp?$AAi?$AA?9?$AAm?$AAs?$AA?9?$AAw?$AAi?$AAn?$AA?9?$AAc?$AAo?$AAr?$AAe@ 1004e4c0     libucrt:winapi_thunks.obj
 0002:000024f8       ??_C@_1EI@MPIAOHOC@?$AAa?$AAp?$AAi?$AA?9?$AAm?$AAs?$AA?9?$AAw?$AAi?$AAn?$AA?9?$AAc?$AAo?$AAr?$AAe@ 1004e4f8     libucrt:winapi_thunks.obj
 0002:00002540       ??_C@_1FK@FPHCKFIE@?$AAa?$AAp?$AAi?$AA?9?$AAm?$AAs?$AA?9?$AAw?$AAi?$AAn?$AA?9?$AAc?$AAo?$AAr?$AAe@ 1004e540     libucrt:winapi_thunks.obj
 0002:000025a0       ??_C@_1EM@DILCGIIO@?$AAa?$AAp?$AAi?$AA?9?$AAm?$AAs?$AA?9?$AAw?$AAi?$AAn?$AA?9?$AAc?$AAo?$AAr?$AAe@ 1004e5a0     libucrt:winapi_thunks.obj
 0002:000025ec       ??_C@_1DM@LNCGDDPN@?$AAa?$AAp?$AAi?$AA?9?$AAm?$AAs?$AA?9?$AAw?$AAi?$AAn?$AA?9?$AAc?$AAo?$AAr?$AAe@ 1004e5ec     libucrt:winapi_thunks.obj
 0002:00002628       ??_C@_1DO@FPAPJEMD@?$AAa?$AAp?$AAi?$AA?9?$AAm?$AAs?$AA?9?$AAw?$AAi?$AAn?$AA?9?$AAc?$AAo?$AAr?$AAe@ 1004e628     libucrt:winapi_thunks.obj
 0002:00002668       ??_C@_1DK@NDHNAHIO@?$AAa?$AAp?$AAi?$AA?9?$AAm?$AAs?$AA?9?$AAw?$AAi?$AAn?$AA?9?$AAc?$AAo?$AAr?$AAe@ 1004e668     libucrt:winapi_thunks.obj
 0002:000026a4       ??_C@_1DM@KGHDGBCM@?$AAa?$AAp?$AAi?$AA?9?$AAm?$AAs?$AA?9?$AAw?$AAi?$AAn?$AA?9?$AAc?$AAo?$AAr?$AAe@ 1004e6a4     libucrt:winapi_thunks.obj
 0002:000026e0       ??_C@_1EO@IJIOEFOH@?$AAa?$AAp?$AAi?$AA?9?$AAm?$AAs?$AA?9?$AAw?$AAi?$AAn?$AA?9?$AAr?$AAt?$AAc?$AAo@ 1004e6e0     libucrt:winapi_thunks.obj
 0002:00002730       ??_C@_1FG@HHGEKANL@?$AAa?$AAp?$AAi?$AA?9?$AAm?$AAs?$AA?9?$AAw?$AAi?$AAn?$AA?9?$AAs?$AAe?$AAc?$AAu@ 1004e730     libucrt:winapi_thunks.obj
 0002:00002788       ??_C@_1EG@DBIOJECG@?$AAe?$AAx?$AAt?$AA?9?$AAm?$AAs?$AA?9?$AAw?$AAi?$AAn?$AA?9?$AAn?$AAt?$AAu?$AAs@ 1004e788     libucrt:winapi_thunks.obj
 0002:000027d0       ??_C@_1EO@FIHMJCLF@?$AAe?$AAx?$AAt?$AA?9?$AAm?$AAs?$AA?9?$AAw?$AAi?$AAn?$AA?9?$AAn?$AAt?$AAu?$AAs@ 1004e7d0     libucrt:winapi_thunks.obj
 0002:00002820       ??_C@_1BC@DNHGCMLG@?$AAa?$AAd?$AAv?$AAa?$AAp?$AAi?$AA3?$AA2@ 1004e820     libucrt:winapi_thunks.obj
 0002:00002834       ??_C@_1M@OAIMIKLP@?$AAn?$AAt?$AAd?$AAl?$AAl@ 1004e834     libucrt:winapi_thunks.obj
 0002:00002840       ??_C@_1EG@DPGNFKGC@?$AAa?$AAp?$AAi?$AA?9?$AAm?$AAs?$AA?9?$AAw?$AAi?$AAn?$AA?9?$AAa?$AAp?$AAp?$AAm@ 1004e840     libucrt:winapi_thunks.obj
 0002:00002888       ??_C@_1O@BCCLBEOE@?$AAu?$AAs?$AAe?$AAr?$AA3?$AA2@ 1004e888     libucrt:winapi_thunks.obj
 0002:00002898       ??_C@_1BA@IAIFMGEF@?$AAe?$AAx?$AAt?$AA?9?$AAm?$AAs?$AA?9@ 1004e898     libucrt:winapi_thunks.obj
 0002:000028ac       ??_C@_0BA@FHFNEAED@AreFileApisANSI@ 1004e8ac     libucrt:winapi_thunks.obj
 0002:000028f4       ??_C@_0O@KKBNKAPF@LCMapStringEx@ 1004e8f4     libucrt:winapi_thunks.obj
 0002:0000290c       ??_C@_0BB@HBDEELFH@LocaleNameToLCID@ 1004e90c     libucrt:winapi_thunks.obj
 0002:00002924       ??_C@_0CF@OJOFEIGO@AppPolicyGetProcessTerminationM@ 1004e924     libucrt:winapi_thunks.obj
 0002:00002950       __sys_errlist              1004e950     libucrt:syserr.obj
 0002:00002a00       ??_C@_08INEPGKHH@No?5error@ 1004ea00     libucrt:syserr.obj
 0002:00002a0c       ??_C@_0BI@BJFCGOHL@Operation?5not?5permitted@ 1004ea0c     libucrt:syserr.obj
 0002:00002a24       ??_C@_0BK@FMDHKPNF@No?5such?5file?5or?5directory@ 1004ea24     libucrt:syserr.obj
 0002:00002a40       ??_C@_0BA@FKIAIBGA@No?5such?5process@ 1004ea40     libucrt:syserr.obj
 0002:00002a50       ??_C@_0BK@FJBOAFDK@Interrupted?5function?5call@ 1004ea50     libucrt:syserr.obj
 0002:00002a6c       ??_C@_0BD@KKNFOBBD@Input?1output?5error@ 1004ea6c     libucrt:syserr.obj
 0002:00002a80       ??_C@_0BK@DPKMCKJ@No?5such?5device?5or?5address@ 1004ea80     libucrt:syserr.obj
 0002:00002a9c       ??_C@_0BC@MFFGCDFL@Arg?5list?5too?5long@ 1004ea9c     libucrt:syserr.obj
 0002:00002ab0       ??_C@_0BC@HKPNECK@Exec?5format?5error@ 1004eab0     libucrt:syserr.obj
 0002:00002ac4       ??_C@_0BE@NFGDDCEF@Bad?5file?5descriptor@ 1004eac4     libucrt:syserr.obj
 0002:00002ad8       ??_C@_0BD@LOHELEP@No?5child?5processes@ 1004ead8     libucrt:syserr.obj
 0002:00002aec       ??_C@_0CB@EPFKGNAK@Resource?5temporarily?5unavailabl@ 1004eaec     libucrt:syserr.obj
 0002:00002b10       ??_C@_0BB@IMDKMPFB@Not?5enough?5space@ 1004eb10     libucrt:syserr.obj
 0002:00002b24       ??_C@_0BC@HFNFNKAI@Permission?5denied@ 1004eb24     libucrt:syserr.obj
 0002:00002b38       ??_C@_0M@LOEHLCJD@Bad?5address@ 1004eb38     libucrt:syserr.obj
 0002:00002b44       ??_C@_0O@NIPGCINC@Unknown?5error@ 1004eb44     libucrt:syserr.obj
 0002:00002b54       ??_C@_0BA@BIBLIOEK@Resource?5device@ 1004eb54     libucrt:syserr.obj
 0002:00002b64       ??_C@_0M@NAAJNNGH@File?5exists@ 1004eb64     libucrt:syserr.obj
 0002:00002b70       ??_C@_0O@OAMDNOCP@Improper?5link@ 1004eb70     libucrt:syserr.obj
 0002:00002b80       ??_C@_0P@NLEIANHE@No?5such?5device@ 1004eb80     libucrt:syserr.obj
 0002:00002b90       ??_C@_0BA@CJBACOOL@Not?5a?5directory@ 1004eb90     libucrt:syserr.obj
 0002:00002ba0       ??_C@_0P@NDHGCGKE@Is?5a?5directory@ 1004eba0     libucrt:syserr.obj
 0002:00002bb0       ??_C@_0BB@HMGGCEBG@Invalid?5argument@ 1004ebb0     libucrt:syserr.obj
 0002:00002bc4       ??_C@_0BO@IIFBODJE@Too?5many?5open?5files?5in?5system@ 1004ebc4     libucrt:syserr.obj
 0002:00002be4       ??_C@_0BE@INBJMKGG@Too?5many?5open?5files@ 1004ebe4     libucrt:syserr.obj
 0002:00002bf8       ??_C@_0CE@ONOKNLPF@Inappropriate?5I?1O?5control?5opera@ 1004ebf8     libucrt:syserr.obj
 0002:00002c1c       ??_C@_0P@LFMMIPAE@File?5too?5large@ 1004ec1c     libucrt:syserr.obj
 0002:00002c2c       ??_C@_0BI@FEALHKLD@No?5space?5left?5on?5device@ 1004ec2c     libucrt:syserr.obj
 0002:00002c44       ??_C@_0N@FEHLOILP@Invalid?5seek@ 1004ec44     libucrt:syserr.obj
 0002:00002c54       ??_C@_0BG@DDBFNKBH@Read?9only?5file?5system@ 1004ec54     libucrt:syserr.obj
 0002:00002c6c       ??_C@_0P@PKCJJLLM@Too?5many?5links@ 1004ec6c     libucrt:syserr.obj
 0002:00002c7c       ??_C@_0M@LHEPIIOM@Broken?5pipe@ 1004ec7c     libucrt:syserr.obj
 0002:00002c88       ??_C@_0N@MMJPGLJK@Domain?5error@ 1004ec88     libucrt:syserr.obj
 0002:00002c98       ??_C@_0BB@FCBJFCAJ@Result?5too?5large@ 1004ec98     libucrt:syserr.obj
 0002:00002cac       ??_C@_0BK@JAEBMJJM@Resource?5deadlock?5avoided@ 1004ecac     libucrt:syserr.obj
 0002:00002cc8       ??_C@_0BC@BEDIHIDK@Filename?5too?5long@ 1004ecc8     libucrt:syserr.obj
 0002:00002cdc       ??_C@_0BD@CLHBCGPB@No?5locks?5available@ 1004ecdc     libucrt:syserr.obj
 0002:00002cf0       ??_C@_0BJ@IHEHINLI@Function?5not?5implemented@ 1004ecf0     libucrt:syserr.obj
 0002:00002d0c       ??_C@_0BE@ICMCHPHH@Directory?5not?5empty@ 1004ed0c     libucrt:syserr.obj
 0002:00002d20       ??_C@_0BG@KLEAJEFJ@Illegal?5byte?5sequence@ 1004ed20     libucrt:syserr.obj
 0002:00002d38       __sys_nerr                 1004ed38     libucrt:syserr.obj
 0002:00002d40       ___newctype                1004ed40     libucrt:ctype.obj
 0002:00003040       ___newclmap                1004f040     libucrt:ctype.obj
 0002:000031c0       ___newcumap                1004f1c0     libucrt:ctype.obj
 0002:00003340       __wctype                   1004f340     libucrt:ctype.obj
 0002:00003584       ??_C@_1M@HPNHIDJI@?$AAj?$AAa?$AA?9?$AAJ?$AAP@ 1004f584     libucrt:mbctype.obj
 0002:00003590       ??_C@_1M@BIBDDEMK@?$AAz?$AAh?$AA?9?$AAC?$AAN@ 1004f590     libucrt:mbctype.obj
 0002:0000359c       ??_C@_1M@JLOOOEGK@?$AAk?$AAo?$AA?9?$AAK?$AAR@ 1004f59c     libucrt:mbctype.obj
 0002:000035a8       ??_C@_1M@CLNBBOPM@?$AAz?$AAh?$AA?9?$AAT?$AAW@ 1004f5a8     libucrt:mbctype.obj
 0002:00003650       ??_C@_05DNEBIAHO@1?$CDINF@ 1004f650     libucrt:cfout.obj
 0002:00003658       ??_C@_06IMKFLFPG@1?$CDQNAN@ 1004f658     libucrt:cfout.obj
 0002:00003660       ??_C@_06PGGFOGJG@1?$CDSNAN@ 1004f660     libucrt:cfout.obj
 0002:00003668       ??_C@_05PHHOCPM@1?$CDIND@  1004f668     libucrt:cfout.obj
 0002:00003670       ??_C@_15PJPFLCCM@?$AAu?$AAk@ 1004f670     libucrt:get_qualified_locale.obj
 0002:00003d98       ??_C@_15EMKDOKLE@?$AAa?$AAr@ 1004fd98     libucrt:lcidtoname_downlevel.obj
 0002:00003da0       ??_C@_15KNPADPLH@?$AAb?$AAg@ 1004fda0     libucrt:lcidtoname_downlevel.obj
 0002:00003da8       ??_C@_15EDMHLDMO@?$AAc?$AAa@ 1004fda8     libucrt:lcidtoname_downlevel.obj
 0002:00003db0       ??_C@_1O@BPEAJADD@?$AAz?$AAh?$AA?9?$AAC?$AAH?$AAS@ 1004fdb0     libucrt:lcidtoname_downlevel.obj
 0002:00003dc0       ??_C@_15LJNHCMNK@?$AAc?$AAs@ 1004fdc0     libucrt:lcidtoname_downlevel.obj
 0002:00003dc8       ??_C@_15FOMCIDHG@?$AAd?$AAa@ 1004fdc8     libucrt:lcidtoname_downlevel.obj
 0002:00003dd0       ??_C@_15NBKABECB@?$AAd?$AAe@ 1004fdd0     libucrt:lcidtoname_downlevel.obj
 0002:00003dd8       ??_C@_15GHPEIIAO@?$AAe?$AAl@ 1004fdd8     libucrt:lcidtoname_downlevel.obj
 0002:00003de0       ??_C@_15MNPNEAIF@?$AAe?$AAn@ 1004fde0     libucrt:lcidtoname_downlevel.obj
 0002:00003de8       ??_C@_15GPIOMPMH@?$AAe?$AAs@ 1004fde8     libucrt:lcidtoname_downlevel.obj
 0002:00003df0       ??_C@_15NGLOAKJC@?$AAf?$AAi@ 1004fdf0     libucrt:lcidtoname_downlevel.obj
 0002:00003df8       ??_C@_15FBKGNKAM@?$AAf?$AAr@ 1004fdf8     libucrt:lcidtoname_downlevel.obj
 0002:00003e00       ??_C@_15KGGCNEFK@?$AAh?$AAe@ 1004fe00     libucrt:lcidtoname_downlevel.obj
 0002:00003e08       ??_C@_15PGHLIDMF@?$AAh?$AAu@ 1004fe08     libucrt:lcidtoname_downlevel.obj
 0002:00003e10       ??_C@_15BIEMAPLM@?$AAi?$AAs@ 1004fe10     libucrt:lcidtoname_downlevel.obj
 0002:00003e18       ??_C@_15IFJLDHAF@?$AAi?$AAt@ 1004fe18     libucrt:lcidtoname_downlevel.obj
 0002:00003e20       ??_C@_15GEMIOCAG@?$AAj?$AAa@ 1004fe20     libucrt:lcidtoname_downlevel.obj
 0002:00003e28       ??_C@_15EPELEGJA@?$AAk?$AAo@ 1004fe28     libucrt:lcidtoname_downlevel.obj
 0002:00003e30       ??_C@_15NDDHIMN@?$AAn?$AAl@ 1004fe30     libucrt:lcidtoname_downlevel.obj
 0002:00003e38       ??_C@_15BPIGNHCD@?$AAn?$AAo@ 1004fe38     libucrt:lcidtoname_downlevel.obj
 0002:00003e40       ??_C@_15DEOPBLCG@?$AAp?$AAl@ 1004fe40     libucrt:lcidtoname_downlevel.obj
 0002:00003e48       ??_C@_15KBECGEFG@?$AAp?$AAt@ 1004fe48     libucrt:lcidtoname_downlevel.obj
 0002:00003e50       ??_C@_15GLJCBFMD@?$AAr?$AAo@ 1004fe50     libucrt:lcidtoname_downlevel.obj
 0002:00003e58       ??_C@_15FEDGKCDI@?$AAr?$AAu@ 1004fe58     libucrt:lcidtoname_downlevel.obj
 0002:00003e60       ??_C@_15GLKMLLHM@?$AAh?$AAr@ 1004fe60     libucrt:lcidtoname_downlevel.obj
 0002:00003e68       ??_C@_15CPKMFBDB@?$AAs?$AAk@ 1004fe68     libucrt:lcidtoname_downlevel.obj
 0002:00003e70       ??_C@_15BAAIOGMK@?$AAs?$AAq@ 1004fe70     libucrt:lcidtoname_downlevel.obj
 0002:00003e78       ??_C@_15INNPNOHD@?$AAs?$AAv@ 1004fe78     libucrt:lcidtoname_downlevel.obj
 0002:00003e80       ??_C@_15CABMMOGH@?$AAt?$AAh@ 1004fe80     libucrt:lcidtoname_downlevel.obj
 0002:00003e88       ??_C@_15BPLIHJJM@?$AAt?$AAr@ 1004fe88     libucrt:lcidtoname_downlevel.obj
 0002:00003e90       ??_C@_15NEOEKKDJ@?$AAu?$AAr@ 1004fe90     libucrt:lcidtoname_downlevel.obj
 0002:00003e98       ??_C@_15NFICGAJK@?$AAi?$AAd@ 1004fe98     libucrt:lcidtoname_downlevel.obj
 0002:00003ea0       ??_C@_15HPJPHDM@?$AAb?$AAe@ 1004fea0     libucrt:lcidtoname_downlevel.obj
 0002:00003ea8       ??_C@_15LCHLGJII@?$AAs?$AAl@ 1004fea8     libucrt:lcidtoname_downlevel.obj
 0002:00003eb0       ??_C@_15PCFJPHHO@?$AAe?$AAt@ 1004feb0     libucrt:lcidtoname_downlevel.obj
 0002:00003eb8       ??_C@_15HPFPGODN@?$AAl?$AAv@ 1004feb8     libucrt:lcidtoname_downlevel.obj
 0002:00003ec0       ??_C@_15NFFGKGLG@?$AAl?$AAt@ 1004fec0     libucrt:lcidtoname_downlevel.obj
 0002:00003ec8       ??_C@_15BDAKCCHN@?$AAf?$AAa@ 1004fec8     libucrt:lcidtoname_downlevel.obj
 0002:00003ed0       ??_C@_15NFGIAIAJ@?$AAv?$AAi@ 1004fed0     libucrt:lcidtoname_downlevel.obj
 0002:00003ed8       ??_C@_15LMKNDMHN@?$AAh?$AAy@ 1004fed8     libucrt:lcidtoname_downlevel.obj
 0002:00003ee0       ??_C@_15IJBHMCFL@?$AAa?$AAz@ 1004fee0     libucrt:lcidtoname_downlevel.obj
 0002:00003ee8       ??_C@_15EKOFJABL@?$AAe?$AAu@ 1004fee8     libucrt:lcidtoname_downlevel.obj
 0002:00003ef0       ??_C@_15BGHADCNK@?$AAm?$AAk@ 1004fef0     libucrt:lcidtoname_downlevel.obj
 0002:00003ef8       ??_C@_15JDNICKHM@?$AAa?$AAf@ 1004fef8     libucrt:lcidtoname_downlevel.obj
 0002:00003f00       ??_C@_15KPJEDBKD@?$AAk?$AAa@ 1004ff00     libucrt:lcidtoname_downlevel.obj
 0002:00003f08       ??_C@_15PDNFFFEO@?$AAf?$AAo@ 1004ff08     libucrt:lcidtoname_downlevel.obj
 0002:00003f10       ??_C@_15OMLEGLOC@?$AAh?$AAi@ 1004ff10     libucrt:lcidtoname_downlevel.obj
 0002:00003f18       ??_C@_15IDNNENKK@?$AAm?$AAs@ 1004ff18     libucrt:lcidtoname_downlevel.obj
 0002:00003f20       ??_C@_15MACJNBMH@?$AAk?$AAk@ 1004ff20     libucrt:lcidtoname_downlevel.obj
 0002:00003f28       ??_C@_15DKDJEOND@?$AAk?$AAy@ 1004ff28     libucrt:lcidtoname_downlevel.obj
 0002:00003f30       ??_C@_15DFGDLJBG@?$AAs?$AAw@ 1004ff30     libucrt:lcidtoname_downlevel.obj
 0002:00003f38       ??_C@_15BBFAICNG@?$AAu?$AAz@ 1004ff38     libucrt:lcidtoname_downlevel.obj
 0002:00003f40       ??_C@_15DKNDCGEA@?$AAt?$AAt@ 1004ff40     libucrt:lcidtoname_downlevel.obj
 0002:00003f48       ??_C@_15MGIFMDPL@?$AAp?$AAa@ 1004ff48     libucrt:lcidtoname_downlevel.obj
 0002:00003f50       ??_C@_15HCNDBBA@?$AAg?$AAu@ 1004ff50     libucrt:lcidtoname_downlevel.obj
 0002:00003f58       ??_C@_15FNBEIBON@?$AAt?$AAa@ 1004ff58     libucrt:lcidtoname_downlevel.obj
 0002:00003f60       ??_C@_15NCHGBGLK@?$AAt?$AAe@ 1004ff60     libucrt:lcidtoname_downlevel.obj
 0002:00003f68       ??_C@_15PHPHCBPF@?$AAk?$AAn@ 1004ff68     libucrt:lcidtoname_downlevel.obj
 0002:00003f70       ??_C@_15DLGBCKMP@?$AAm?$AAr@ 1004ff70     libucrt:lcidtoname_downlevel.obj
 0002:00003f78       ??_C@_15EABBLBFF@?$AAs?$AAa@ 1004ff78     libucrt:lcidtoname_downlevel.obj
 0002:00003f80       ??_C@_15CBKOMCOI@?$AAm?$AAn@ 1004ff80     libucrt:lcidtoname_downlevel.obj
 0002:00003f88       ??_C@_15CKDMCJAF@?$AAg?$AAl@ 1004ff88     libucrt:lcidtoname_downlevel.obj
 0002:00003f90       ??_C@_17CNJFBPG@?$AAk?$AAo?$AAk@ 1004ff90     libucrt:lcidtoname_downlevel.obj
 0002:00003f98       ??_C@_17FFBJICPL@?$AAs?$AAy?$AAr@ 1004ff98     libucrt:lcidtoname_downlevel.obj
 0002:00003fa0       ??_C@_17KPNDCPAF@?$AAd?$AAi?$AAv@ 1004ffa0     libucrt:lcidtoname_downlevel.obj
 0002:00003fa8       ??_C@_1M@OKAHONE@?$AAa?$AAr?$AA?9?$AAS?$AAA@ 1004ffa8     libucrt:lcidtoname_downlevel.obj
 0002:00003fb4       ??_C@_1M@FFFIGIGK@?$AAb?$AAg?$AA?9?$AAB?$AAG@ 1004ffb4     libucrt:lcidtoname_downlevel.obj
 0002:00003fc0       ??_C@_1M@BJNKEDC@?$AAc?$AAa?$AA?9?$AAE?$AAS@ 1004ffc0     libucrt:lcidtoname_downlevel.obj
 0002:00003fcc       ??_C@_1M@IJJHFJHA@?$AAc?$AAs?$AA?9?$AAC?$AAZ@ 1004ffcc     libucrt:lcidtoname_downlevel.obj
 0002:00003fd8       ??_C@_1M@CLPEOBGI@?$AAd?$AAa?$AA?9?$AAD?$AAK@ 1004ffd8     libucrt:lcidtoname_downlevel.obj
 0002:00003fe4       ??_C@_1M@MCMADGCB@?$AAd?$AAe?$AA?9?$AAD?$AAE@ 1004ffe4     libucrt:lcidtoname_downlevel.obj
 0002:00003ff0       ??_C@_1M@OOCKEMAM@?$AAe?$AAl?$AA?9?$AAG?$AAR@ 1004fff0     libucrt:lcidtoname_downlevel.obj
 0002:00003ffc       ??_C@_1M@DDNJFGID@?$AAf?$AAi?$AA?9?$AAF?$AAI@ 1004fffc     libucrt:lcidtoname_downlevel.obj
 0002:00004008       ??_C@_1M@GLIPPMAC@?$AAf?$AAr?$AA?9?$AAF?$AAR@ 10050008     libucrt:lcidtoname_downlevel.obj
 0002:00004014       ??_C@_1M@GFMCHPE@?$AAh?$AAe?$AA?9?$AAI?$AAL@ 10050014     libucrt:lcidtoname_downlevel.obj
 0002:00004020       ??_C@_1M@MHLPGNKM@?$AAh?$AAu?$AA?9?$AAH?$AAU@ 10050020     libucrt:lcidtoname_downlevel.obj
 0002:0000402c       ??_C@_1M@LPDDNNPN@?$AAi?$AAs?$AA?9?$AAI?$AAS@ 1005002c     libucrt:lcidtoname_downlevel.obj
 0002:00004038       ??_C@_1M@MADIPODN@?$AAi?$AAt?$AA?9?$AAI?$AAT@ 10050038     libucrt:lcidtoname_downlevel.obj
 0002:00004044       ??_C@_1M@IHBJJGG@?$AAn?$AAl?$AA?9?$AAN?$AAL@ 10050044     libucrt:lcidtoname_downlevel.obj
 0002:00004050       ??_C@_1M@EANAGDL@?$AAn?$AAb?$AA?9?$AAN?$AAO@ 10050050     libucrt:lcidtoname_downlevel.obj
 0002:0000405c       ??_C@_1M@NEIEMEGP@?$AAp?$AAl?$AA?9?$AAP?$AAL@ 1005005c     libucrt:lcidtoname_downlevel.obj
 0002:00004068       ??_C@_1M@BOCFIGEP@?$AAp?$AAt?$AA?9?$AAB?$AAR@ 10050068     libucrt:lcidtoname_downlevel.obj
 0002:00004074       ??_C@_1M@IMPFOPBG@?$AAr?$AAo?$AA?9?$AAR?$AAO@ 10050074     libucrt:lcidtoname_downlevel.obj
 0002:00004080       ??_C@_1M@IDNNEJMM@?$AAr?$AAu?$AA?9?$AAR?$AAU@ 10050080     libucrt:lcidtoname_downlevel.obj
 0002:0000408c       ??_C@_1M@LILEEOGM@?$AAh?$AAr?$AA?9?$AAH?$AAR@ 1005008c     libucrt:lcidtoname_downlevel.obj
 0002:00004098       ??_C@_1M@FKIFEHPB@?$AAs?$AAk?$AA?9?$AAS?$AAK@ 10050098     libucrt:lcidtoname_downlevel.obj
 0002:000040a4       ??_C@_1M@LJMAMNPJ@?$AAs?$AAq?$AA?9?$AAA?$AAL@ 100500a4     libucrt:lcidtoname_downlevel.obj
 0002:000040b0       ??_C@_1M@GIAKDKJK@?$AAs?$AAv?$AA?9?$AAS?$AAE@ 100500b0     libucrt:lcidtoname_downlevel.obj
 0002:000040bc       ??_C@_1M@MKJKIKCL@?$AAt?$AAh?$AA?9?$AAT?$AAH@ 100500bc     libucrt:lcidtoname_downlevel.obj
 0002:000040c8       ??_C@_1M@MFLCCMPB@?$AAt?$AAr?$AA?9?$AAT?$AAR@ 100500c8     libucrt:lcidtoname_downlevel.obj
 0002:000040d4       ??_C@_1M@OIJHDKJN@?$AAu?$AAr?$AA?9?$AAP?$AAK@ 100500d4     libucrt:lcidtoname_downlevel.obj
 0002:000040e0       ??_C@_1M@LHIPCIEK@?$AAi?$AAd?$AA?9?$AAI?$AAD@ 100500e0     libucrt:lcidtoname_downlevel.obj
 0002:000040ec       ??_C@_1M@MFMOBGI@?$AAu?$AAk?$AA?9?$AAU?$AAA@ 100500ec     libucrt:lcidtoname_downlevel.obj
 0002:000040f8       ??_C@_1M@OBGLJIPL@?$AAb?$AAe?$AA?9?$AAB?$AAY@ 100500f8     libucrt:lcidtoname_downlevel.obj
 0002:00004104       ??_C@_1M@BCFAJEAD@?$AAs?$AAl?$AA?9?$AAS?$AAI@ 10050104     libucrt:lcidtoname_downlevel.obj
 0002:00004110       ??_C@_1M@FKFFEDDN@?$AAe?$AAt?$AA?9?$AAE?$AAE@ 10050110     libucrt:lcidtoname_downlevel.obj
 0002:0000411c       ??_C@_1M@KGKKAACI@?$AAl?$AAv?$AA?9?$AAL?$AAV@ 1005011c     libucrt:lcidtoname_downlevel.obj
 0002:00004128       ??_C@_1M@IFGBIJO@?$AAl?$AAt?$AA?9?$AAL?$AAT@ 10050128     libucrt:lcidtoname_downlevel.obj
 0002:00004134       ??_C@_1M@FGEAHEDM@?$AAf?$AAa?$AA?9?$AAI?$AAR@ 10050134     libucrt:lcidtoname_downlevel.obj
 0002:00004140       ??_C@_1M@KBMAIBFN@?$AAv?$AAi?$AA?9?$AAV?$AAN@ 10050140     libucrt:lcidtoname_downlevel.obj
 0002:0000414c       ??_C@_1M@GPCBKDJK@?$AAh?$AAy?$AA?9?$AAA?$AAM@ 1005014c     libucrt:lcidtoname_downlevel.obj
 0002:00004158       ??_C@_1BG@BECMDDJB@?$AAa?$AAz?$AA?9?$AAA?$AAZ?$AA?9?$AAL?$AAa?$AAt?$AAn@ 10050158     libucrt:lcidtoname_downlevel.obj
 0002:00004170       ??_C@_1M@MAOFCAEA@?$AAe?$AAu?$AA?9?$AAE?$AAS@ 10050170     libucrt:lcidtoname_downlevel.obj
 0002:0000417c       ??_C@_1M@IGHABKPI@?$AAm?$AAk?$AA?9?$AAM?$AAK@ 1005017c     libucrt:lcidtoname_downlevel.obj
 0002:00004188       ??_C@_1M@IAIGNEJG@?$AAt?$AAn?$AA?9?$AAZ?$AAA@ 10050188     libucrt:lcidtoname_downlevel.obj
 0002:00004194       ??_C@_1M@IIJCOJFA@?$AAx?$AAh?$AA?9?$AAZ?$AAA@ 10050194     libucrt:lcidtoname_downlevel.obj
 0002:000041a0       ??_C@_1M@LGPJHNJH@?$AAz?$AAu?$AA?9?$AAZ?$AAA@ 100501a0     libucrt:lcidtoname_downlevel.obj
 0002:000041ac       ??_C@_1M@HOKAOIO@?$AAa?$AAf?$AA?9?$AAZ?$AAA@ 100501ac     libucrt:lcidtoname_downlevel.obj
 0002:000041b8       ??_C@_1M@DPCLHLIE@?$AAk?$AAa?$AA?9?$AAG?$AAE@ 100501b8     libucrt:lcidtoname_downlevel.obj
 0002:000041c4       ??_C@_1M@BLKMHJBI@?$AAf?$AAo?$AA?9?$AAF?$AAO@ 100501c4     libucrt:lcidtoname_downlevel.obj
 0002:000041d0       ??_C@_1M@LGGJAPPB@?$AAh?$AAi?$AA?9?$AAI?$AAN@ 100501d0     libucrt:lcidtoname_downlevel.obj
 0002:000041dc       ??_C@_1M@FIKPIHFE@?$AAm?$AAt?$AA?9?$AAM?$AAT@ 100501dc     libucrt:lcidtoname_downlevel.obj
 0002:000041e8       ??_C@_1M@HEGGPBFA@?$AAs?$AAe?$AA?9?$AAN?$AAO@ 100501e8     libucrt:lcidtoname_downlevel.obj
 0002:000041f4       ??_C@_1M@EIBJEEPA@?$AAm?$AAs?$AA?9?$AAM?$AAY@ 100501f4     libucrt:lcidtoname_downlevel.obj
 0002:00004200       ??_C@_1M@FHLBGMPP@?$AAk?$AAk?$AA?9?$AAK?$AAZ@ 10050200     libucrt:lcidtoname_downlevel.obj
 0002:0000420c       ??_C@_1M@NGJJLCGI@?$AAk?$AAy?$AA?9?$AAK?$AAG@ 1005020c     libucrt:lcidtoname_downlevel.obj
 0002:00004218       ??_C@_1M@GIENNBFC@?$AAs?$AAw?$AA?9?$AAK?$AAE@ 10050218     libucrt:lcidtoname_downlevel.obj
 0002:00004224       ??_C@_1BG@NDGMJIMJ@?$AAu?$AAz?$AA?9?$AAU?$AAZ?$AA?9?$AAL?$AAa?$AAt?$AAn@ 10050224     libucrt:lcidtoname_downlevel.obj
 0002:0000423c       ??_C@_1M@IDCCIHBC@?$AAt?$AAt?$AA?9?$AAR?$AAU@ 1005023c     libucrt:lcidtoname_downlevel.obj
 0002:00004248       ??_C@_1M@LOICPMOJ@?$AAb?$AAn?$AA?9?$AAI?$AAN@ 10050248     libucrt:lcidtoname_downlevel.obj
 0002:00004254       ??_C@_1M@KPKKNEAH@?$AAp?$AAa?$AA?9?$AAI?$AAN@ 10050254     libucrt:lcidtoname_downlevel.obj
 0002:00004260       ??_C@_1M@PJGPPBOG@?$AAg?$AAu?$AA?9?$AAI?$AAN@ 10050260     libucrt:lcidtoname_downlevel.obj
 0002:0000426c       ??_C@_1M@KMKMOPHI@?$AAt?$AAa?$AA?9?$AAI?$AAN@ 1005026c     libucrt:lcidtoname_downlevel.obj
 0002:00004278       ??_C@_1M@KFEHEPAC@?$AAt?$AAe?$AA?9?$AAI?$AAN@ 10050278     libucrt:lcidtoname_downlevel.obj
 0002:00004284       ??_C@_1M@CDCLMGHI@?$AAk?$AAn?$AA?9?$AAI?$AAN@ 10050284     libucrt:lcidtoname_downlevel.obj
 0002:00004290       ??_C@_1M@MIODLDKF@?$AAm?$AAl?$AA?9?$AAI?$AAN@ 10050290     libucrt:lcidtoname_downlevel.obj
 0002:0000429c       ??_C@_1M@PBIEACPO@?$AAm?$AAr?$AA?9?$AAI?$AAN@ 1005029c     libucrt:lcidtoname_downlevel.obj
 0002:000042a8       ??_C@_1M@NIDEAGPH@?$AAs?$AAa?$AA?9?$AAI?$AAN@ 100502a8     libucrt:lcidtoname_downlevel.obj
 0002:000042b4       ??_C@_1M@FHIHCBIO@?$AAm?$AAn?$AA?9?$AAM?$AAN@ 100502b4     libucrt:lcidtoname_downlevel.obj
 0002:000042c0       ??_C@_1M@JAIJPENP@?$AAc?$AAy?$AA?9?$AAG?$AAB@ 100502c0     libucrt:lcidtoname_downlevel.obj
 0002:000042cc       ??_C@_1M@PHGFBEPN@?$AAg?$AAl?$AA?9?$AAE?$AAS@ 100502cc     libucrt:lcidtoname_downlevel.obj
 0002:000042d8       ??_C@_1O@KPIPDNCP@?$AAk?$AAo?$AAk?$AA?9?$AAI?$AAN@ 100502d8     libucrt:lcidtoname_downlevel.obj
 0002:000042e8       ??_C@_1O@KNHJLDJA@?$AAs?$AAy?$AAr?$AA?9?$AAS?$AAY@ 100502e8     libucrt:lcidtoname_downlevel.obj
 0002:000042f8       ??_C@_1O@MKEKBLAH@?$AAd?$AAi?$AAv?$AA?9?$AAM?$AAV@ 100502f8     libucrt:lcidtoname_downlevel.obj
 0002:00004308       ??_C@_1O@OHDCKDDF@?$AAq?$AAu?$AAz?$AA?9?$AAB?$AAO@ 10050308     libucrt:lcidtoname_downlevel.obj
 0002:00004318       ??_C@_1M@LEPJNLFD@?$AAn?$AAs?$AA?9?$AAZ?$AAA@ 10050318     libucrt:lcidtoname_downlevel.obj
 0002:00004324       ??_C@_1M@OMLEIIJB@?$AAm?$AAi?$AA?9?$AAN?$AAZ@ 10050324     libucrt:lcidtoname_downlevel.obj
 0002:00004330       ??_C@_1M@PMPEAILG@?$AAa?$AAr?$AA?9?$AAI?$AAQ@ 10050330     libucrt:lcidtoname_downlevel.obj
 0002:0000433c       ??_C@_1M@CNKPNOEE@?$AAd?$AAe?$AA?9?$AAC?$AAH@ 1005033c     libucrt:lcidtoname_downlevel.obj
 0002:00004348       ??_C@_1M@LKMGMLKO@?$AAe?$AAn?$AA?9?$AAG?$AAB@ 10050348     libucrt:lcidtoname_downlevel.obj
 0002:00004354       ??_C@_1M@PGKJFFGL@?$AAe?$AAs?$AA?9?$AAM?$AAX@ 10050354     libucrt:lcidtoname_downlevel.obj
 0002:00004360       ??_C@_1M@DNNANBDC@?$AAf?$AAr?$AA?9?$AAB?$AAE@ 10050360     libucrt:lcidtoname_downlevel.obj
 0002:0000436c       ??_C@_1M@HLGMDFHM@?$AAi?$AAt?$AA?9?$AAC?$AAH@ 1005036c     libucrt:lcidtoname_downlevel.obj
 0002:00004378       ??_C@_1M@CLLBGJH@?$AAn?$AAl?$AA?9?$AAB?$AAE@ 10050378     libucrt:lcidtoname_downlevel.obj
 0002:00004384       ??_C@_1M@BODBOGLF@?$AAn?$AAn?$AA?9?$AAN?$AAO@ 10050384     libucrt:lcidtoname_downlevel.obj
 0002:00004390       ??_C@_1M@HFFAHKAD@?$AAp?$AAt?$AA?9?$AAP?$AAT@ 10050390     libucrt:lcidtoname_downlevel.obj
 0002:0000439c       ??_C@_1BG@LNOAKHIE@?$AAs?$AAr?$AA?9?$AAS?$AAP?$AA?9?$AAL?$AAa?$AAt?$AAn@ 1005039c     libucrt:lcidtoname_downlevel.obj
 0002:000043b4       ??_C@_1M@HBMHBGAK@?$AAs?$AAv?$AA?9?$AAF?$AAI@ 100503b4     libucrt:lcidtoname_downlevel.obj
 0002:000043c0       ??_C@_1BG@DGCJGJBE@?$AAa?$AAz?$AA?9?$AAA?$AAZ?$AA?9?$AAC?$AAy?$AAr?$AAl@ 100503c0     libucrt:lcidtoname_downlevel.obj
 0002:000043d8       ??_C@_1M@KEJDAAHB@?$AAs?$AAe?$AA?9?$AAS?$AAE@ 100503d8     libucrt:lcidtoname_downlevel.obj
 0002:000043e4       ??_C@_1M@HEIBJJAD@?$AAm?$AAs?$AA?9?$AAB?$AAN@ 100503e4     libucrt:lcidtoname_downlevel.obj
 0002:000043f0       ??_C@_1BG@PBGJMCEM@?$AAu?$AAz?$AA?9?$AAU?$AAZ?$AA?9?$AAC?$AAy?$AAr?$AAl@ 100503f0     libucrt:lcidtoname_downlevel.obj
 0002:00004408       ??_C@_1O@LAOBCMDF@?$AAq?$AAu?$AAz?$AA?9?$AAE?$AAC@ 10050408     libucrt:lcidtoname_downlevel.obj
 0002:00004418       ??_C@_1M@POEEMAIO@?$AAa?$AAr?$AA?9?$AAE?$AAG@ 10050418     libucrt:lcidtoname_downlevel.obj
 0002:00004424       ??_C@_1M@EFAKDEDL@?$AAz?$AAh?$AA?9?$AAH?$AAK@ 10050424     libucrt:lcidtoname_downlevel.obj
 0002:00004430       ??_C@_1M@HKKIJHGI@?$AAd?$AAe?$AA?9?$AAA?$AAT@ 10050430     libucrt:lcidtoname_downlevel.obj
 0002:0000443c       ??_C@_1M@KBFBEHJF@?$AAe?$AAn?$AA?9?$AAA?$AAU@ 1005043c     libucrt:lcidtoname_downlevel.obj
 0002:00004448       ??_C@_1M@MNPLFAAH@?$AAe?$AAs?$AA?9?$AAE?$AAS@ 10050448     libucrt:lcidtoname_downlevel.obj
 0002:00004454       ??_C@_1M@HJOOJFMA@?$AAf?$AAr?$AA?9?$AAC?$AAA@ 10050454     libucrt:lcidtoname_downlevel.obj
 0002:00004460       ??_C@_1BG@JPOFPNAB@?$AAs?$AAr?$AA?9?$AAS?$AAP?$AA?9?$AAC?$AAy?$AAr?$AAl@ 10050460     libucrt:lcidtoname_downlevel.obj
 0002:00004478       ??_C@_1M@LNFOCMOB@?$AAs?$AAe?$AA?9?$AAF?$AAI@ 10050478     libucrt:lcidtoname_downlevel.obj
 0002:00004484       ??_C@_1O@MGJBOAMB@?$AAq?$AAu?$AAz?$AA?9?$AAP?$AAE@ 10050484     libucrt:lcidtoname_downlevel.obj
 0002:00004494       ??_C@_1M@GJINLBOK@?$AAa?$AAr?$AA?9?$AAL?$AAY@ 10050494     libucrt:lcidtoname_downlevel.obj
 0002:000044a0       ??_C@_1M@GGMNHJNL@?$AAz?$AAh?$AA?9?$AAS?$AAG@ 100504a0     libucrt:lcidtoname_downlevel.obj
 0002:000044ac       ??_C@_1M@HOIKODND@?$AAd?$AAe?$AA?9?$AAL?$AAU@ 100504ac     libucrt:lcidtoname_downlevel.obj
 0002:000044b8       ??_C@_1M@DDOCCGFG@?$AAe?$AAn?$AA?9?$AAC?$AAA@ 100504b8     libucrt:lcidtoname_downlevel.obj
 0002:000044c4       ??_C@_1M@BNOEMJLF@?$AAe?$AAs?$AA?9?$AAG?$AAT@ 100504c4     libucrt:lcidtoname_downlevel.obj
 0002:000044d0       ??_C@_1M@EOGNKEK@?$AAf?$AAr?$AA?9?$AAC?$AAH@ 100504d0     libucrt:lcidtoname_downlevel.obj
 0002:000044dc       ??_C@_1M@FLIDJFHL@?$AAh?$AAr?$AA?9?$AAB?$AAA@ 100504dc     libucrt:lcidtoname_downlevel.obj
 0002:000044e8       ??_C@_1O@FMCELNAJ@?$AAs?$AAm?$AAj?$AA?9?$AAN?$AAO@ 100504e8     libucrt:lcidtoname_downlevel.obj
 0002:000044f8       ??_C@_1M@JHGLJMGJ@?$AAa?$AAr?$AA?9?$AAD?$AAZ@ 100504f8     libucrt:lcidtoname_downlevel.obj
 0002:00004504       ??_C@_1M@JKKFDCNP@?$AAz?$AAh?$AA?9?$AAM?$AAO@ 10050504     libucrt:lcidtoname_downlevel.obj
 0002:00004510       ??_C@_1M@GEEFALPE@?$AAd?$AAe?$AA?9?$AAL?$AAI@ 10050510     libucrt:lcidtoname_downlevel.obj
 0002:0000451c       ??_C@_1M@IGEOFBG@?$AAe?$AAn?$AA?9?$AAN?$AAZ@ 1005051c     libucrt:lcidtoname_downlevel.obj
 0002:00004528       ??_C@_1M@KDBONEHP@?$AAe?$AAs?$AA?9?$AAC?$AAR@ 10050528     libucrt:lcidtoname_downlevel.obj
 0002:00004534       ??_C@_1M@FHMDOHNN@?$AAf?$AAr?$AA?9?$AAL?$AAU@ 10050534     libucrt:lcidtoname_downlevel.obj
 0002:00004540       ??_C@_1BG@NFKKMAFG@?$AAb?$AAs?$AA?9?$AAB?$AAA?$AA?9?$AAL?$AAa?$AAt?$AAn@ 10050540     libucrt:lcidtoname_downlevel.obj
 0002:00004558       ??_C@_1O@IMNBEMCI@?$AAs?$AAm?$AAj?$AA?9?$AAS?$AAE@ 10050558     libucrt:lcidtoname_downlevel.obj
 0002:00004568       ??_C@_1M@DHHMBNDP@?$AAa?$AAr?$AA?9?$AAM?$AAA@ 10050568     libucrt:lcidtoname_downlevel.obj
 0002:00004574       ??_C@_1M@BNBLJCGH@?$AAe?$AAn?$AA?9?$AAI?$AAE@ 10050574     libucrt:lcidtoname_downlevel.obj
 0002:00004580       ??_C@_1M@GEPAFMDL@?$AAe?$AAs?$AA?9?$AAP?$AAA@ 10050580     libucrt:lcidtoname_downlevel.obj
 0002:0000458c       ??_C@_1M@OJONDMDL@?$AAf?$AAr?$AA?9?$AAM?$AAC@ 1005058c     libucrt:lcidtoname_downlevel.obj
 0002:00004598       ??_C@_1BG@OBCNFJB@?$AAs?$AAr?$AA?9?$AAB?$AAA?$AA?9?$AAL?$AAa?$AAt?$AAn@ 10050598     libucrt:lcidtoname_downlevel.obj
 0002:000045b0       ??_C@_1O@KEMEEGPO@?$AAs?$AAm?$AAa?$AA?9?$AAN?$AAO@ 100505b0     libucrt:lcidtoname_downlevel.obj
 0002:000045c0       ??_C@_1M@ELMGFODK@?$AAa?$AAr?$AA?9?$AAT?$AAN@ 100505c0     libucrt:lcidtoname_downlevel.obj
 0002:000045cc       ??_C@_1M@BHDLHFAF@?$AAe?$AAn?$AA?9?$AAZ?$AAA@ 100505cc     libucrt:lcidtoname_downlevel.obj
 0002:000045d8       ??_C@_1M@BMGIGLIF@?$AAe?$AAs?$AA?9?$AAD?$AAO@ 100505d8     libucrt:lcidtoname_downlevel.obj
 0002:000045e4       ??_C@_1BG@CMBHIPBE@?$AAs?$AAr?$AA?9?$AAB?$AAA?$AA?9?$AAC?$AAy?$AAr?$AAl@ 100505e4     libucrt:lcidtoname_downlevel.obj
 0002:000045fc       ??_C@_1O@HEDBLHNP@?$AAs?$AAm?$AAa?$AA?9?$AAS?$AAE@ 100505fc     libucrt:lcidtoname_downlevel.obj
 0002:0000460c       ??_C@_1M@DAGCADIM@?$AAa?$AAr?$AA?9?$AAO?$AAM@ 1005060c     libucrt:lcidtoname_downlevel.obj
 0002:00004618       ??_C@_1M@FODLMICG@?$AAe?$AAn?$AA?9?$AAJ?$AAM@ 10050618     libucrt:lcidtoname_downlevel.obj
 0002:00004624       ??_C@_1M@DNMLCIHB@?$AAe?$AAs?$AA?9?$AAV?$AAE@ 10050624     libucrt:lcidtoname_downlevel.obj
 0002:00004630       ??_C@_1O@EOKHMKJK@?$AAs?$AAm?$AAs?$AA?9?$AAF?$AAI@ 10050630     libucrt:lcidtoname_downlevel.obj
 0002:00004640       ??_C@_1M@CAFJMKOF@?$AAa?$AAr?$AA?9?$AAY?$AAE@ 10050640     libucrt:lcidtoname_downlevel.obj
 0002:0000464c       ??_C@_1M@CBFHIJLI@?$AAe?$AAn?$AA?9?$AAC?$AAB@ 1005064c     libucrt:lcidtoname_downlevel.obj
 0002:00004658       ??_C@_1M@BGNFLDN@?$AAe?$AAs?$AA?9?$AAC?$AAO@ 10050658     libucrt:lcidtoname_downlevel.obj
 0002:00004664       ??_C@_1O@JMPHMAMC@?$AAs?$AAm?$AAn?$AA?9?$AAF?$AAI@ 10050664     libucrt:lcidtoname_downlevel.obj
 0002:00004674       ??_C@_1M@JLANABKE@?$AAa?$AAr?$AA?9?$AAS?$AAY@ 10050674     libucrt:lcidtoname_downlevel.obj
 0002:00004680       ??_C@_1M@HPKGCFGN@?$AAe?$AAn?$AA?9?$AAB?$AAZ@ 10050680     libucrt:lcidtoname_downlevel.obj
 0002:0000468c       ??_C@_1M@OLJCMLGM@?$AAe?$AAs?$AA?9?$AAP?$AAE@ 1005068c     libucrt:lcidtoname_downlevel.obj
 0002:00004698       ??_C@_1M@MKKGFKLE@?$AAa?$AAr?$AA?9?$AAJ?$AAO@ 10050698     libucrt:lcidtoname_downlevel.obj
 0002:000046a4       ??_C@_1M@EKPGLDNI@?$AAe?$AAn?$AA?9?$AAT?$AAT@ 100506a4     libucrt:lcidtoname_downlevel.obj
 0002:000046b0       ??_C@_1M@OONGHFHE@?$AAe?$AAs?$AA?9?$AAA?$AAR@ 100506b0     libucrt:lcidtoname_downlevel.obj
 0002:000046bc       ??_C@_1M@OOJFGBHE@?$AAa?$AAr?$AA?9?$AAL?$AAB@ 100506bc     libucrt:lcidtoname_downlevel.obj
 0002:000046c8       ??_C@_1M@GCEJHNEG@?$AAe?$AAn?$AA?9?$AAZ?$AAW@ 100506c8     libucrt:lcidtoname_downlevel.obj
 0002:000046d4       ??_C@_1M@JNOCAHJI@?$AAe?$AAs?$AA?9?$AAE?$AAC@ 100506d4     libucrt:lcidtoname_downlevel.obj
 0002:000046e0       ??_C@_1M@JEFHPGGB@?$AAa?$AAr?$AA?9?$AAK?$AAW@ 100506e0     libucrt:lcidtoname_downlevel.obj
 0002:000046ec       ??_C@_1M@MLKIBJOJ@?$AAe?$AAn?$AA?9?$AAP?$AAH@ 100506ec     libucrt:lcidtoname_downlevel.obj
 0002:000046f8       ??_C@_1M@BDNIPEND@?$AAe?$AAs?$AA?9?$AAC?$AAL@ 100506f8     libucrt:lcidtoname_downlevel.obj
 0002:00004704       ??_C@_1M@MPNMEKBD@?$AAa?$AAr?$AA?9?$AAA?$AAE@ 10050704     libucrt:lcidtoname_downlevel.obj
 0002:00004710       ??_C@_1M@KBJALCPI@?$AAe?$AAs?$AA?9?$AAU?$AAY@ 10050710     libucrt:lcidtoname_downlevel.obj
 0002:0000471c       ??_C@_1M@LLCCOAGA@?$AAa?$AAr?$AA?9?$AAB?$AAH@ 1005071c     libucrt:lcidtoname_downlevel.obj
 0002:00004728       ??_C@_1M@PBFNCDEL@?$AAe?$AAs?$AA?9?$AAP?$AAY@ 10050728     libucrt:lcidtoname_downlevel.obj
 0002:00004734       ??_C@_1M@EDGINPNP@?$AAa?$AAr?$AA?9?$AAQ?$AAA@ 10050734     libucrt:lcidtoname_downlevel.obj
 0002:00004740       ??_C@_1M@MKDBIIJI@?$AAe?$AAs?$AA?9?$AAB?$AAO@ 10050740     libucrt:lcidtoname_downlevel.obj
 0002:0000474c       ??_C@_1M@CPKKEBLD@?$AAe?$AAs?$AA?9?$AAS?$AAV@ 1005074c     libucrt:lcidtoname_downlevel.obj
 0002:00004758       ??_C@_1M@NDBGMMJL@?$AAe?$AAs?$AA?9?$AAH?$AAN@ 10050758     libucrt:lcidtoname_downlevel.obj
 0002:00004764       ??_C@_1M@JIJIBHDP@?$AAe?$AAs?$AA?9?$AAN?$AAI@ 10050764     libucrt:lcidtoname_downlevel.obj
 0002:00004770       ??_C@_1M@CGFMKEEK@?$AAe?$AAs?$AA?9?$AAP?$AAR@ 10050770     libucrt:lcidtoname_downlevel.obj
 0002:0000477c       ??_C@_1O@ICJHKIIK@?$AAz?$AAh?$AA?9?$AAC?$AAH?$AAT@ 1005077c     libucrt:lcidtoname_downlevel.obj
 0002:0000478c       ??_C@_15CLNEJCE@?$AAs?$AAr@ 1005078c     libucrt:lcidtoname_downlevel.obj
 0002:00004eb8       ??_C@_1M@KAHEKEIG@?$AAa?$AAf?$AA?9?$AAz?$AAa@ 10050eb8     libucrt:lcidtoname_downlevel.obj
 0002:00004ec4       ??_C@_1M@GIECOABL@?$AAa?$AAr?$AA?9?$AAa?$AAe@ 10050ec4     libucrt:lcidtoname_downlevel.obj
 0002:00004ed0       ??_C@_1M@BMLMEKGI@?$AAa?$AAr?$AA?9?$AAb?$AAh@ 10050ed0     libucrt:lcidtoname_downlevel.obj
 0002:00004edc       ??_C@_1M@DAPFDGGB@?$AAa?$AAr?$AA?9?$AAd?$AAz@ 10050edc     libucrt:lcidtoname_downlevel.obj
 0002:00004ee8       ??_C@_1M@FJNKGKIG@?$AAa?$AAr?$AA?9?$AAe?$AAg@ 10050ee8     libucrt:lcidtoname_downlevel.obj
 0002:00004ef4       ??_C@_1M@FLGKKCLO@?$AAa?$AAr?$AA?9?$AAi?$AAq@ 10050ef4     libucrt:lcidtoname_downlevel.obj
 0002:00004f00       ??_C@_1M@GNDIPALM@?$AAa?$AAr?$AA?9?$AAj?$AAo@ 10050f00     libucrt:lcidtoname_downlevel.obj
 0002:00004f0c       ??_C@_1M@DDMJFMGJ@?$AAa?$AAr?$AA?9?$AAk?$AAw@ 10050f0c     libucrt:lcidtoname_downlevel.obj
 0002:00004f18       ??_C@_1M@EJALMLHM@?$AAa?$AAr?$AA?9?$AAl?$AAb@ 10050f18     libucrt:lcidtoname_downlevel.obj
 0002:00004f24       ??_C@_1M@MOBDBLOC@?$AAa?$AAr?$AA?9?$AAl?$AAy@ 10050f24     libucrt:lcidtoname_downlevel.obj
 0002:00004f30       ??_C@_1M@JAOCLHDH@?$AAa?$AAr?$AA?9?$AAm?$AAa@ 10050f30     libucrt:lcidtoname_downlevel.obj
 0002:00004f3c       ??_C@_1M@JHPMKJIE@?$AAa?$AAr?$AA?9?$AAo?$AAm@ 10050f3c     libucrt:lcidtoname_downlevel.obj
 0002:00004f48       ??_C@_1M@OEPGHFNH@?$AAa?$AAr?$AA?9?$AAq?$AAa@ 10050f48     libucrt:lcidtoname_downlevel.obj
 0002:00004f54       ??_C@_1M@KJDONENM@?$AAa?$AAr?$AA?9?$AAs?$AAa@ 10050f54     libucrt:lcidtoname_downlevel.obj
 0002:00004f60       ??_C@_1M@DMJDKLKM@?$AAa?$AAr?$AA?9?$AAs?$AAy@ 10050f60     libucrt:lcidtoname_downlevel.obj
 0002:00004f6c       ??_C@_1M@OMFIPEDC@?$AAa?$AAr?$AA?9?$AAt?$AAn@ 10050f6c     libucrt:lcidtoname_downlevel.obj
 0002:00004f78       ??_C@_1M@IHMHGAON@?$AAa?$AAr?$AA?9?$AAy?$AAe@ 10050f78     libucrt:lcidtoname_downlevel.obj
 0002:00004f84       ??_C@_1BG@KDCPGJGB@?$AAa?$AAz?$AA?9?$AAa?$AAz?$AA?9?$AAc?$AAy?$AAr?$AAl@ 10050f84     libucrt:lcidtoname_downlevel.obj
 0002:00004f9c       ??_C@_1BG@IBCKDDOE@?$AAa?$AAz?$AA?9?$AAa?$AAz?$AA?9?$AAl?$AAa?$AAt?$AAn@ 10050f9c     libucrt:lcidtoname_downlevel.obj
 0002:00004fb4       ??_C@_1M@EGPFDCPD@?$AAb?$AAe?$AA?9?$AAb?$AAy@ 10050fb4     libucrt:lcidtoname_downlevel.obj
 0002:00004fc0       ??_C@_1M@PCMGMCGC@?$AAb?$AAg?$AA?9?$AAb?$AAg@ 10050fc0     libucrt:lcidtoname_downlevel.obj
 0002:00004fcc       ??_C@_1M@BJBMFGOB@?$AAb?$AAn?$AA?9?$AAi?$AAn@ 10050fcc     libucrt:lcidtoname_downlevel.obj
 0002:00004fd8       ??_C@_1BG@EAKMMACD@?$AAb?$AAs?$AA?9?$AAb?$AAa?$AA?9?$AAl?$AAa?$AAt?$AAn@ 10050fd8     libucrt:lcidtoname_downlevel.obj
 0002:00004ff0       ??_C@_1M@KGADAODK@?$AAc?$AAa?$AA?9?$AAe?$AAs@ 10050ff0     libucrt:lcidtoname_downlevel.obj
 0002:00004ffc       ??_C@_1M@COAJPDHI@?$AAc?$AAs?$AA?9?$AAc?$AAz@ 10050ffc     libucrt:lcidtoname_downlevel.obj
 0002:00005008       ??_C@_1M@DHBHFONH@?$AAc?$AAy?$AA?9?$AAg?$AAb@ 10051008     libucrt:lcidtoname_downlevel.obj
 0002:00005014       ??_C@_1M@IMGKELGA@?$AAd?$AAa?$AA?9?$AAd?$AAk@ 10051014     libucrt:lcidtoname_downlevel.obj
 0002:00005020       ??_C@_1M@NNDGDNGA@?$AAd?$AAe?$AA?9?$AAa?$AAt@ 10051020     libucrt:lcidtoname_downlevel.obj
 0002:0000502c       ??_C@_1M@IKDBHEEM@?$AAd?$AAe?$AA?9?$AAc?$AAh@ 1005102c     libucrt:lcidtoname_downlevel.obj
 0002:00005038       ??_C@_1M@GFFOJMCJ@?$AAd?$AAe?$AA?9?$AAd?$AAe@ 10051038     libucrt:lcidtoname_downlevel.obj
 0002:00005044       ??_C@_1M@MDNLKBPM@?$AAd?$AAe?$AA?9?$AAl?$AAi@ 10051044     libucrt:lcidtoname_downlevel.obj
 0002:00005050       ??_C@_1M@NJBEEJNL@?$AAd?$AAe?$AA?9?$AAl?$AAu@ 10051050     libucrt:lcidtoname_downlevel.obj
 0002:0000505c       ??_C@_1O@GNNELBAP@?$AAd?$AAi?$AAv?$AA?9?$AAm?$AAv@ 1005105c     libucrt:lcidtoname_downlevel.obj
 0002:0000506c       ??_C@_1M@EJLEOGAE@?$AAe?$AAl?$AA?9?$AAg?$AAr@ 1005106c     libucrt:lcidtoname_downlevel.obj
 0002:00005078       ??_C@_1M@GMPONJN@?$AAe?$AAn?$AA?9?$AAa?$AAu@ 10051078     libucrt:lcidtoname_downlevel.obj
 0002:00005084       ??_C@_1M@NIDIIPGF@?$AAe?$AAn?$AA?9?$AAb?$AAz@ 10051084     libucrt:lcidtoname_downlevel.obj
 0002:00005090       ??_C@_1M@JEHMIMFO@?$AAe?$AAn?$AA?9?$AAc?$AAa@ 10051090     libucrt:lcidtoname_downlevel.obj
 0002:0000509c       ??_C@_1M@IGMJCDLA@?$AAe?$AAn?$AA?9?$AAc?$AAb@ 1005109c     libucrt:lcidtoname_downlevel.obj
 0002:000050a8       ??_C@_1M@BNFIGBKG@?$AAe?$AAn?$AA?9?$AAg?$AAb@ 100510a8     libucrt:lcidtoname_downlevel.obj
 0002:000050b4       ??_C@_1M@LKIFDIGP@?$AAe?$AAn?$AA?9?$AAi?$AAe@ 100510b4     libucrt:lcidtoname_downlevel.obj
 0002:000050c0       ??_C@_1M@PJKFGCCO@?$AAe?$AAn?$AA?9?$AAj?$AAm@ 100510c0     libucrt:lcidtoname_downlevel.obj
 0002:000050cc       ??_C@_1M@KPPKEPBO@?$AAe?$AAn?$AA?9?$AAn?$AAz@ 100510cc     libucrt:lcidtoname_downlevel.obj
 0002:000050d8       ??_C@_1M@GMDGLDOB@?$AAe?$AAn?$AA?9?$AAp?$AAh@ 100510d8     libucrt:lcidtoname_downlevel.obj
 0002:000050e4       ??_C@_1M@ONGIBJNA@?$AAe?$AAn?$AA?9?$AAt?$AAt@ 100510e4     libucrt:lcidtoname_downlevel.obj
 0002:000050f0       ??_C@_1M@LLODPCMM@?$AAe?$AAn?$AA?9?$AAu?$AAs@ 100510f0     libucrt:lcidtoname_downlevel.obj
 0002:000050fc       ??_C@_1M@LAKFNPAN@?$AAe?$AAn?$AA?9?$AAz?$AAa@ 100510fc     libucrt:lcidtoname_downlevel.obj
 0002:00005108       ??_C@_1M@MFNHNHEO@?$AAe?$AAn?$AA?9?$AAz?$AAw@ 10051108     libucrt:lcidtoname_downlevel.obj
 0002:00005114       ??_C@_1M@EJEINPHM@?$AAe?$AAs?$AA?9?$AAa?$AAr@ 10051114     libucrt:lcidtoname_downlevel.obj
 0002:00005120       ??_C@_1M@GNKPCCJA@?$AAe?$AAs?$AA?9?$AAb?$AAo@ 10051120     libucrt:lcidtoname_downlevel.obj
 0002:0000512c       ??_C@_1M@LEEGFONL@?$AAe?$AAs?$AA?9?$AAc?$AAl@ 1005112c     libucrt:lcidtoname_downlevel.obj
 0002:00005138       ??_C@_1M@KGPDPBDF@?$AAe?$AAs?$AA?9?$AAc?$AAo@ 10051138     libucrt:lcidtoname_downlevel.obj
 0002:00005144       ??_C@_1M@EIAHOHH@?$AAe?$AAs?$AA?9?$AAc?$AAr@ 10051144     libucrt:lcidtoname_downlevel.obj
 0002:00005150       ??_C@_1M@LLPGMBIN@?$AAe?$AAs?$AA?9?$AAd?$AAo@ 10051150     libucrt:lcidtoname_downlevel.obj
 0002:0000515c       ??_C@_1M@DKHMKNJA@?$AAe?$AAs?$AA?9?$AAe?$AAc@ 1005115c     libucrt:lcidtoname_downlevel.obj
 0002:00005168       ??_C@_1M@GKGFPKAP@?$AAe?$AAs?$AA?9?$AAe?$AAs@ 10051168     libucrt:lcidtoname_downlevel.obj
 0002:00005174       ??_C@_1M@LKHKGDLN@?$AAe?$AAs?$AA?9?$AAg?$AAt@ 10051174     libucrt:lcidtoname_downlevel.obj
 0002:00005180       ??_C@_1M@HEIIGGJD@?$AAe?$AAs?$AA?9?$AAh?$AAn@ 10051180     libucrt:lcidtoname_downlevel.obj
 0002:0000518c       ??_C@_1M@FBDHPPGD@?$AAe?$AAs?$AA?9?$AAm?$AAx@ 1005118c     libucrt:lcidtoname_downlevel.obj
 0002:00005198       ??_C@_1M@DPAGLNDH@?$AAe?$AAs?$AA?9?$AAn?$AAi@ 10051198     libucrt:lcidtoname_downlevel.obj
 0002:000051a4       ??_C@_1M@MDGOPGDD@?$AAe?$AAs?$AA?9?$AAp?$AAa@ 100511a4     libucrt:lcidtoname_downlevel.obj
 0002:000051b0       ??_C@_1M@EMAMGBGE@?$AAe?$AAs?$AA?9?$AAp?$AAe@ 100511b0     libucrt:lcidtoname_downlevel.obj
 0002:000051bc       ??_C@_1M@IBMCAOEC@?$AAe?$AAs?$AA?9?$AAp?$AAr@ 100511bc     libucrt:lcidtoname_downlevel.obj
 0002:000051c8       ??_C@_1M@FGMDIJED@?$AAe?$AAs?$AA?9?$AAp?$AAy@ 100511c8     libucrt:lcidtoname_downlevel.obj
 0002:000051d4       ??_C@_1M@IIDEOLLL@?$AAe?$AAs?$AA?9?$AAs?$AAv@ 100511d4     libucrt:lcidtoname_downlevel.obj
 0002:000051e0       ??_C@_1M@GAOBIPA@?$AAe?$AAs?$AA?9?$AAu?$AAy@ 100511e0     libucrt:lcidtoname_downlevel.obj
 0002:000051ec       ??_C@_1M@JKFFICHJ@?$AAe?$AAs?$AA?9?$AAv?$AAe@ 100511ec     libucrt:lcidtoname_downlevel.obj
 0002:000051f8       ??_C@_1M@PNMLOJDF@?$AAe?$AAt?$AA?9?$AAe?$AAe@ 100511f8     libucrt:lcidtoname_downlevel.obj
 0002:00005204       ??_C@_1M@GHHLIKEI@?$AAe?$AAu?$AA?9?$AAe?$AAs@ 10051204     libucrt:lcidtoname_downlevel.obj
 0002:00005210       ??_C@_1M@PBNONODE@?$AAf?$AAa?$AA?9?$AAi?$AAr@ 10051210     libucrt:lcidtoname_downlevel.obj
 0002:0000521c       ??_C@_1M@JEEHPMIL@?$AAf?$AAi?$AA?9?$AAf?$AAi@ 1005121c     libucrt:lcidtoname_downlevel.obj
 0002:00005228       ??_C@_1M@LMDCNDBA@?$AAf?$AAo?$AA?9?$AAf?$AAo@ 10051228     libucrt:lcidtoname_downlevel.obj
 0002:00005234       ??_C@_1M@JKEOHLDK@?$AAf?$AAr?$AA?9?$AAb?$AAe@ 10051234     libucrt:lcidtoname_downlevel.obj
 0002:00005240       ??_C@_1M@NOHADPMI@?$AAf?$AAr?$AA?9?$AAc?$AAa@ 10051240     libucrt:lcidtoname_downlevel.obj
 0002:0000524c       ??_C@_1M@KDHIHAEC@?$AAf?$AAr?$AA?9?$AAc?$AAh@ 1005124c     libucrt:lcidtoname_downlevel.obj
 0002:00005258       ??_C@_1M@MMBBFGAK@?$AAf?$AAr?$AA?9?$AAf?$AAr@ 10051258     libucrt:lcidtoname_downlevel.obj
 0002:00005264       ??_C@_1M@PAFNENNF@?$AAf?$AAr?$AA?9?$AAl?$AAu@ 10051264     libucrt:lcidtoname_downlevel.obj
 0002:00005270       ??_C@_1M@EOHDJGDD@?$AAf?$AAr?$AA?9?$AAm?$AAc@ 10051270     libucrt:lcidtoname_downlevel.obj
 0002:0000527c       ??_C@_1M@FAPLLOPF@?$AAg?$AAl?$AA?9?$AAe?$AAs@ 1005127c     libucrt:lcidtoname_downlevel.obj
 0002:00005288       ??_C@_1M@FOPBFLOO@?$AAg?$AAu?$AA?9?$AAi?$AAn@ 10051288     libucrt:lcidtoname_downlevel.obj
 0002:00005294       ??_C@_1M@KBMCINPM@?$AAh?$AAe?$AA?9?$AAi?$AAl@ 10051294     libucrt:lcidtoname_downlevel.obj
 0002:000052a0       ??_C@_1M@BBPHKFPJ@?$AAh?$AAi?$AA?9?$AAi?$AAn@ 100512a0     libucrt:lcidtoname_downlevel.obj
 0002:000052ac       ??_C@_1M@PMBNDPHD@?$AAh?$AAr?$AA?9?$AAb?$AAa@ 100512ac     libucrt:lcidtoname_downlevel.obj
 0002:000052b8       ??_C@_1M@BPCKOEGE@?$AAh?$AAr?$AA?9?$AAh?$AAr@ 100512b8     libucrt:lcidtoname_downlevel.obj
 0002:000052c4       ??_C@_1M@GACBMHKE@?$AAh?$AAu?$AA?9?$AAh?$AAu@ 100512c4     libucrt:lcidtoname_downlevel.obj
 0002:000052d0       ??_C@_1M@MILPAJJC@?$AAh?$AAy?$AA?9?$AAa?$AAm@ 100512d0     libucrt:lcidtoname_downlevel.obj
 0002:000052dc       ??_C@_1M@BABBICEC@?$AAi?$AAd?$AA?9?$AAi?$AAd@ 100512dc     libucrt:lcidtoname_downlevel.obj
 0002:000052e8       ??_C@_1M@BIKNHHPF@?$AAi?$AAs?$AA?9?$AAi?$AAs@ 100512e8     libucrt:lcidtoname_downlevel.obj
 0002:000052f4       ??_C@_1M@NMPCJPHE@?$AAi?$AAt?$AA?9?$AAc?$AAh@ 100512f4     libucrt:lcidtoname_downlevel.obj
 0002:00005300       ??_C@_1M@GHKGFEDF@?$AAi?$AAt?$AA?9?$AAi?$AAt@ 10051300     libucrt:lcidtoname_downlevel.obj
 0002:0000530c       ??_C@_1M@NIEJCJJA@?$AAj?$AAa?$AA?9?$AAj?$AAp@ 1005130c     libucrt:lcidtoname_downlevel.obj
 0002:00005318       ??_C@_1M@JILFNBIM@?$AAk?$AAa?$AA?9?$AAg?$AAe@ 10051318     libucrt:lcidtoname_downlevel.obj
 0002:00005324       ??_C@_1M@PACPMGPH@?$AAk?$AAk?$AA?9?$AAk?$AAz@ 10051324     libucrt:lcidtoname_downlevel.obj
 0002:00005330       ??_C@_1M@IELFGMHA@?$AAk?$AAn?$AA?9?$AAi?$AAn@ 10051330     libucrt:lcidtoname_downlevel.obj
 0002:0000533c       ??_C@_1O@IBBJHCH@?$AAk?$AAo?$AAk?$AA?9?$AAi?$AAn@ 1005133c     libucrt:lcidtoname_downlevel.obj
 0002:0000534c       ??_C@_1M@DMHAEOGC@?$AAk?$AAo?$AA?9?$AAk?$AAr@ 1005134c     libucrt:lcidtoname_downlevel.obj
 0002:00005358       ??_C@_1M@HBAHBIGA@?$AAk?$AAy?$AA?9?$AAk?$AAg@ 10051358     libucrt:lcidtoname_downlevel.obj
 0002:00005364       ??_C@_1M@KPMILCJG@?$AAl?$AAt?$AA?9?$AAl?$AAt@ 10051364     libucrt:lcidtoname_downlevel.obj
 0002:00005370       ??_C@_1M@BDEKKCA@?$AAl?$AAv?$AA?9?$AAl?$AAv@ 10051370     libucrt:lcidtoname_downlevel.obj
 0002:0000537c       ??_C@_1M@ELCKCCJJ@?$AAm?$AAi?$AA?9?$AAn?$AAz@ 1005137c     libucrt:lcidtoname_downlevel.obj
 0002:00005388       ??_C@_1M@CBOOLAPA@?$AAm?$AAk?$AA?9?$AAm?$AAk@ 10051388     libucrt:lcidtoname_downlevel.obj
 0002:00005394       ??_C@_1M@GPHNBJKN@?$AAm?$AAl?$AA?9?$AAi?$AAn@ 10051394     libucrt:lcidtoname_downlevel.obj
 0002:000053a0       ??_C@_1M@PABJILIG@?$AAm?$AAn?$AA?9?$AAm?$AAn@ 100513a0     libucrt:lcidtoname_downlevel.obj
 0002:000053ac       ??_C@_1M@FGBKKIPG@?$AAm?$AAr?$AA?9?$AAi?$AAn@ 100513ac     libucrt:lcidtoname_downlevel.obj
 0002:000053b8       ??_C@_1M@NDBPDDAL@?$AAm?$AAs?$AA?9?$AAb?$AAn@ 100513b8     libucrt:lcidtoname_downlevel.obj
 0002:000053c4       ??_C@_1M@OPIHOOPI@?$AAm?$AAs?$AA?9?$AAm?$AAy@ 100513c4     libucrt:lcidtoname_downlevel.obj
 0002:000053d0       ??_C@_1M@PPDBCNFM@?$AAm?$AAt?$AA?9?$AAm?$AAt@ 100513d0     libucrt:lcidtoname_downlevel.obj
 0002:000053dc       ??_C@_1M@KDJDKMDD@?$AAn?$AAb?$AA?9?$AAn?$AAo@ 100513dc     libucrt:lcidtoname_downlevel.obj
 0002:000053e8       ??_C@_1M@KFCFLMJP@?$AAn?$AAl?$AA?9?$AAb?$AAe@ 100513e8     libucrt:lcidtoname_downlevel.obj
 0002:000053f4       ??_C@_1M@KPOPDDGO@?$AAn?$AAl?$AA?9?$AAn?$AAl@ 100513f4     libucrt:lcidtoname_downlevel.obj
 0002:00005400       ??_C@_1M@LJKPEMLN@?$AAn?$AAn?$AA?9?$AAn?$AAo@ 10051400     libucrt:lcidtoname_downlevel.obj
 0002:0000540c       ??_C@_1M@BDGHHBFL@?$AAn?$AAs?$AA?9?$AAz?$AAa@ 1005140c     libucrt:lcidtoname_downlevel.obj
 0002:00005418       ??_C@_1M@IDEHOAP@?$AAp?$AAa?$AA?9?$AAi?$AAn@ 10051418     libucrt:lcidtoname_downlevel.obj
 0002:00005424       ??_C@_1M@HDBKGOGH@?$AAp?$AAl?$AA?9?$AAp?$AAl@ 10051424     libucrt:lcidtoname_downlevel.obj
 0002:00005430       ??_C@_1M@LJLLCMEH@?$AAp?$AAt?$AA?9?$AAb?$AAr@ 10051430     libucrt:lcidtoname_downlevel.obj
 0002:0000543c       ??_C@_1M@NCMONAAL@?$AAp?$AAt?$AA?9?$AAp?$AAt@ 1005143c     libucrt:lcidtoname_downlevel.obj
 0002:00005448       ??_C@_1O@EAKMAJDN@?$AAq?$AAu?$AAz?$AA?9?$AAb?$AAo@ 10051448     libucrt:lcidtoname_downlevel.obj
 0002:00005458       ??_C@_1O@BHHPIGDN@?$AAq?$AAu?$AAz?$AA?9?$AAe?$AAc@ 10051458     libucrt:lcidtoname_downlevel.obj
 0002:00005468       ??_C@_1O@GBAPEKMJ@?$AAq?$AAu?$AAz?$AA?9?$AAp?$AAe@ 10051468     libucrt:lcidtoname_downlevel.obj
 0002:00005478       ??_C@_1M@CLGLEFBO@?$AAr?$AAo?$AA?9?$AAr?$AAo@ 10051478     libucrt:lcidtoname_downlevel.obj
 0002:00005484       ??_C@_1M@CEEDODME@?$AAr?$AAu?$AA?9?$AAr?$AAu@ 10051484     libucrt:lcidtoname_downlevel.obj
 0002:00005490       ??_C@_1M@HPKKKMPP@?$AAs?$AAa?$AA?9?$AAi?$AAn@ 10051490     libucrt:lcidtoname_downlevel.obj
 0002:0000549c       ??_C@_1M@BKMAIGOJ@?$AAs?$AAe?$AA?9?$AAf?$AAi@ 1005149c     libucrt:lcidtoname_downlevel.obj
 0002:000054a8       ??_C@_1M@NDPIFLFI@?$AAs?$AAe?$AA?9?$AAn?$AAo@ 100514a8     libucrt:lcidtoname_downlevel.obj
 0002:000054b4       ??_C@_1M@DANKKHJ@?$AAs?$AAe?$AA?9?$AAs?$AAe@ 100514b4     libucrt:lcidtoname_downlevel.obj
 0002:000054c0       ??_C@_1M@PNBLONPJ@?$AAs?$AAk?$AA?9?$AAs?$AAk@ 100514c0     libucrt:lcidtoname_downlevel.obj
 0002:000054cc       ??_C@_1M@LFMODOAL@?$AAs?$AAl?$AA?9?$AAs?$AAi@ 100514cc     libucrt:lcidtoname_downlevel.obj
 0002:000054d8       ??_C@_1O@DFKOMPG@?$AAs?$AAm?$AAa?$AA?9?$AAn?$AAo@ 100514d8     libucrt:lcidtoname_downlevel.obj
 0002:000054e8       ??_C@_1O@NDKPBNNH@?$AAs?$AAm?$AAa?$AA?9?$AAs?$AAe@ 100514e8     libucrt:lcidtoname_downlevel.obj
 0002:000054f8       ??_C@_1O@PLLKBHAB@?$AAs?$AAm?$AAj?$AA?9?$AAn?$AAo@ 100514f8     libucrt:lcidtoname_downlevel.obj
 0002:00005508       ??_C@_1O@CLEPOGCA@?$AAs?$AAm?$AAj?$AA?9?$AAs?$AAe@ 10051508     libucrt:lcidtoname_downlevel.obj
 0002:00005518       ??_C@_1O@DLGJGKMK@?$AAs?$AAm?$AAn?$AA?9?$AAf?$AAi@ 10051518     libucrt:lcidtoname_downlevel.obj
 0002:00005528       ??_C@_1O@OJDJGAJC@?$AAs?$AAm?$AAs?$AA?9?$AAf?$AAi@ 10051528     libucrt:lcidtoname_downlevel.obj
 0002:00005538       ??_C@_1M@BOFOGHPB@?$AAs?$AAq?$AA?9?$AAa?$AAl@ 10051538     libucrt:lcidtoname_downlevel.obj
 0002:00005544       ??_C@_1BG@LJBBIPGB@?$AAs?$AAr?$AA?9?$AAb?$AAa?$AA?9?$AAc?$AAy?$AAr?$AAl@ 10051544     libucrt:lcidtoname_downlevel.obj
 0002:0000555c       ??_C@_1BG@JLBENFOE@?$AAs?$AAr?$AA?9?$AAb?$AAa?$AA?9?$AAl?$AAa?$AAt?$AAn@ 1005155c     libucrt:lcidtoname_downlevel.obj
 0002:00005574       ??_C@_1BG@KODPNHE@?$AAs?$AAr?$AA?9?$AAs?$AAp?$AA?9?$AAc?$AAy?$AAr?$AAl@ 10051574     libucrt:lcidtoname_downlevel.obj
 0002:0000558c       ??_C@_1BG@CIOGKHPB@?$AAs?$AAr?$AA?9?$AAs?$AAp?$AA?9?$AAl?$AAa?$AAt?$AAn@ 1005158c     libucrt:lcidtoname_downlevel.obj
 0002:000055a4       ??_C@_1M@NGFJLMAC@?$AAs?$AAv?$AA?9?$AAf?$AAi@ 100515a4     libucrt:lcidtoname_downlevel.obj
 0002:000055b0       ??_C@_1M@MPJEJAJC@?$AAs?$AAv?$AA?9?$AAs?$AAe@ 100515b0     libucrt:lcidtoname_downlevel.obj
 0002:000055bc       ??_C@_1M@MPNDHLFK@?$AAs?$AAw?$AA?9?$AAk?$AAe@ 100515bc     libucrt:lcidtoname_downlevel.obj
 0002:000055c8       ??_C@_1O@KOHBJJI@?$AAs?$AAy?$AAr?$AA?9?$AAs?$AAy@ 100515c8     libucrt:lcidtoname_downlevel.obj
 0002:000055d8       ??_C@_1M@LDCEFHA@?$AAt?$AAa?$AA?9?$AAi?$AAn@ 100515d8     libucrt:lcidtoname_downlevel.obj
 0002:000055e4       ??_C@_1M@CNJOFAK@?$AAt?$AAe?$AA?9?$AAi?$AAn@ 100515e4     libucrt:lcidtoname_downlevel.obj
 0002:000055f0       ??_C@_1M@GNAECACD@?$AAt?$AAh?$AA?9?$AAt?$AAh@ 100515f0     libucrt:lcidtoname_downlevel.obj
 0002:000055fc       ??_C@_1M@CHBIHOJO@?$AAt?$AAn?$AA?9?$AAz?$AAa@ 100515fc     libucrt:lcidtoname_downlevel.obj
 0002:00005608       ??_C@_1M@GCCMIGPJ@?$AAt?$AAr?$AA?9?$AAt?$AAr@ 10051608     libucrt:lcidtoname_downlevel.obj
 0002:00005614       ??_C@_1M@CELMCNBK@?$AAt?$AAt?$AA?9?$AAr?$AAu@ 10051614     libucrt:lcidtoname_downlevel.obj
 0002:00005620       ??_C@_1M@KLMCELGA@?$AAu?$AAk?$AA?9?$AAu?$AAa@ 10051620     libucrt:lcidtoname_downlevel.obj
 0002:0000562c       ??_C@_1M@EPAJJAJF@?$AAu?$AAr?$AA?9?$AAp?$AAk@ 1005162c     libucrt:lcidtoname_downlevel.obj
 0002:00005638       ??_C@_1BG@GEGPMCDJ@?$AAu?$AAz?$AA?9?$AAu?$AAz?$AA?9?$AAc?$AAy?$AAr?$AAl@ 10051638     libucrt:lcidtoname_downlevel.obj
 0002:00005650       ??_C@_1BG@EGGKJILM@?$AAu?$AAz?$AA?9?$AAu?$AAz?$AA?9?$AAl?$AAa?$AAt?$AAn@ 10051650     libucrt:lcidtoname_downlevel.obj
 0002:00005668       ??_C@_1M@GFOCLFF@?$AAv?$AAi?$AA?9?$AAv?$AAn@ 10051668     libucrt:lcidtoname_downlevel.obj
 0002:00005674       ??_C@_1M@CPAMEDFI@?$AAx?$AAh?$AA?9?$AAz?$AAa@ 10051674     libucrt:lcidtoname_downlevel.obj
 0002:00005680       ??_C@_1O@EBKIFIGN@?$AAz?$AAh?$AA?9?$AAc?$AAh?$AAs@ 10051680     libucrt:lcidtoname_downlevel.obj
 0002:00005690       ??_C@_1O@NMHPGANE@?$AAz?$AAh?$AA?9?$AAc?$AAh?$AAt@ 10051690     libucrt:lcidtoname_downlevel.obj
 0002:000056a0       ??_C@_1M@LPINJOMC@?$AAz?$AAh?$AA?9?$AAc?$AAn@ 100516a0     libucrt:lcidtoname_downlevel.obj
 0002:000056ac       ??_C@_1M@OCJEJODD@?$AAz?$AAh?$AA?9?$AAh?$AAk@ 100516ac     libucrt:lcidtoname_downlevel.obj
 0002:000056b8       ??_C@_1M@DNDLJINH@?$AAz?$AAh?$AA?9?$AAm?$AAo@ 100516b8     libucrt:lcidtoname_downlevel.obj
 0002:000056c4       ??_C@_1M@MBFDNDND@?$AAz?$AAh?$AA?9?$AAs?$AAg@ 100516c4     libucrt:lcidtoname_downlevel.obj
 0002:000056d0       ??_C@_1M@IMEPLEPE@?$AAz?$AAh?$AA?9?$AAt?$AAw@ 100516d0     libucrt:lcidtoname_downlevel.obj
 0002:000056dc       ??_C@_1M@BBGHNHJP@?$AAz?$AAu?$AA?9?$AAz?$AAa@ 100516dc     libucrt:lcidtoname_downlevel.obj
 0002:00005748       ??_C@_1BA@BALFACEM@?$AAC?$AAO?$AAN?$AAO?$AAU?$AAT?$AA$@ 10051748     libucrt:initcon.obj
 0002:00005860       __infinity                 10051860     libucrt:87tran.obj
 0002:0000586a       __minfinity                1005186a     libucrt:87tran.obj
 0002:00005874       __logemax                  10051874     libucrt:87tran.obj
 0002:0000589a       __OP_EXPjmptab             1005189a     libucrt:87tran.obj
 0002:000058c0       __indefinite               100518c0     libucrt:87disp.obj
 0002:000058ca       __piby2                    100518ca     libucrt:87disp.obj
 0002:000058d4       __piby4                    100518d4     libucrt:87disp.obj
 0002:00005908       __DEFAULT_CW_in_mem        10051908     libucrt:common.obj
 0002:0000590a       __pi_by_2_to_61            1005190a     libucrt:common.obj
 0002:00005944       ??_C@_03MGHMBJCF@log@      10051944     libucrt:libm_error.obj
 0002:00005948       ??_C@_05HGHHAHAP@log10@    10051948     libucrt:libm_error.obj
 0002:00005950       ??_C@_03KHJOGHMM@exp@      10051950     libucrt:libm_error.obj
 0002:00005954       ??_C@_03JGHBODFD@pow@      10051954     libucrt:libm_error.obj
 0002:00005958       ??_C@_04FIHNOPOL@asin@     10051958     libucrt:libm_error.obj
 0002:00005960       ??_C@_04PDIFKINK@acos@     10051960     libucrt:libm_error.obj
 0002:00005968       ??_C@_04EIAKFFMI@sqrt@     10051968     libucrt:libm_error.obj
 0002:00005970       ___acrt_log10_table_t      10051970     libucrt:log10_tables.obj
 0002:00005d80       ___acrt_log10_table_cb     10051d80     libucrt:log10_tables.obj
 0002:00006190       __real@3fe0000000000000    10052190     libucrt:powhlp.obj
 0002:00006280       ??_C@_04COOMCNPB@sinh@     10052280     libucrt:fpexcept.obj
 0002:00006288       ??_C@_04HPJJNFIM@cosh@     10052288     libucrt:fpexcept.obj
 0002:00006290       ??_C@_04FJHINJAO@tanh@     10052290     libucrt:fpexcept.obj
 0002:00006298       ??_C@_04MLLJIGOK@atan@     10052298     libucrt:fpexcept.obj
 0002:000062a0       ??_C@_05KNGEOGJB@atan2@    100522a0     libucrt:fpexcept.obj
 0002:000062a8       ??_C@_03BLEJJJBH@sin@      100522a8     libucrt:fpexcept.obj
 0002:000062ac       ??_C@_03LALBNOCG@cos@      100522ac     libucrt:fpexcept.obj
 0002:000062b0       ??_C@_03IIINPABG@tan@      100522b0     libucrt:fpexcept.obj
 0002:000062b4       ??_C@_04GFPJNGEK@ceil@     100522b4     libucrt:fpexcept.obj
 0002:000062bc       ??_C@_05PBJFFIGL@floor@    100522bc     libucrt:fpexcept.obj
 0002:000062c4       ??_C@_04ODHECPBC@fabs@     100522c4     libucrt:fpexcept.obj
 0002:000062cc       ??_C@_04EHEDPDJG@modf@     100522cc     libucrt:fpexcept.obj
 0002:000062d4       ??_C@_05CEJMAHNP@ldexp@    100522d4     libucrt:fpexcept.obj
 0002:000062dc       ??_C@_05KBKMEMPO@_cabs@    100522dc     libucrt:fpexcept.obj
 0002:000062e4       ??_C@_06MEIMCGCF@_hypot@   100522e4     libucrt:fpexcept.obj
 0002:000062ec       ??_C@_04KEPJIHGP@fmod@     100522ec     libucrt:fpexcept.obj
 0002:000062f4       ??_C@_05GKKHEGJL@frexp@    100522f4     libucrt:fpexcept.obj
 0002:000062fc       ??_C@_03MJLDFKDL@_y0@      100522fc     libucrt:fpexcept.obj
 0002:00006300       ??_C@_03NAKIGLHK@_y1@      10052300     libucrt:fpexcept.obj
 0002:00006304       ??_C@_03ONILCKOB@_yn@      10052304     libucrt:fpexcept.obj
 0002:00006308       ??_C@_05JGDBENOH@_logb@    10052308     libucrt:fpexcept.obj
 0002:00006310       ??_C@_0L@KDOEJCKC@_nextafter@ 10052310     libucrt:fpexcept.obj
 0002:00006320       __d_inf                    10052320     libucrt:util.obj
 0002:00006328       __d_max                    10052328     libucrt:util.obj
 0002:00006330       __d_mzero                  10052330     libucrt:util.obj
 0002:0000633c       ??_7type_info@@6B@         1005233c     LIBCMT:std_type_info_static.obj
 0002:0000634c       ??_C@_09GPALILFO@bad?5int64@ 1005234c     bit64.obj
 0002:00006358       ??_C@_05LLAMLEHD@?$CFI64d@ 10052358     bit64.obj
 0002:00006360       ??_C@_04JAOJMBA@bnot@      10052360     bit64.obj
 0002:00006368       ??_C@_04BKGNPECA@band@     10052368     bit64.obj
 0002:00006370       ??_C@_03BBBGIIAC@bor@      10052370     bit64.obj
 0002:00006374       ??_C@_04CKCGDDNF@bxor@     10052374     bit64.obj
 0002:0000637c       ??_C@_06ELFGPGBK@lshift@   1005237c     bit64.obj
 0002:00006384       ??_C@_06HMLHBBIJ@rshift@   10052384     bit64.obj
 0002:0000638c       ??_C@_07JILILBLL@arshift@  1005238c     bit64.obj
 0002:00006394       ??_C@_03CLCAEGCJ@new@      10052394     bit64.obj
 0002:00006398       ??_C@_03BDGOHNNK@add@      10052398     bit64.obj
 0002:0000639c       ??_C@_03KCMAIMAP@sub@      1005239c     bit64.obj
 0002:000063a0       ??_C@_03IMIFIBCN@mul@      100523a0     bit64.obj
 0002:000063a4       ??_C@_03FEJMGOGI@div@      100523a4     bit64.obj
 0002:000063a8       ??_C@_03FFONCNID@mod@      100523a8     bit64.obj
 0002:000063ac       ??_C@_02HIIGGHJB@eq@       100523ac     bit64.obj
 0002:000063b0       ??_C@_02KCAKIFL@lt@        100523b0     bit64.obj
 0002:000063b4       ??_C@_02FJPJILEL@le@       100523b4     bit64.obj
 0002:000063b8       ??_C@_04GPMDFGEJ@type@     100523b8     bit64.obj
 0002:000063c0       ??_C@_05MEHDOBFN@__add@    100523c0     bit64.obj
 0002:000063c8       ??_C@_05HFNNBAII@__sub@    100523c8     bit64.obj
 0002:000063d0       ??_C@_05FLJIBNKK@__mul@    100523d0     bit64.obj
 0002:000063d8       ??_C@_05IDIBPCOP@__div@    100523d8     bit64.obj
 0002:000063e0       ??_C@_05ICPALBAE@__mod@    100523e0     bit64.obj
 0002:000063e8       ??_C@_05MHFNBPAK@__unm@    100523e8     bit64.obj
 0002:000063f0       ??_C@_04GIMIAOHA@__eq@     100523f0     bit64.obj
 0002:000063f8       ??_C@_04BKGOMBLK@__lt@     100523f8     bit64.obj
 0002:00006400       ??_C@_04EJLHOCKK@__le@     10052400     bit64.obj
 0002:00006408       ??_C@_0L@HDFPAPPH@__tostring@ 10052408     bit64.obj
 0002:00006414       ??_C@_08JOIMPOJO@tonumber@ 10052414     bit64.obj
 0002:00006420       ??_C@_07NHABFFHN@__index@  10052420     bit64.obj
 0002:00006428       ??_C@_05OALCLICP@bit64@    10052428     bit64.obj
 0002:00006430       _metatable_name            10052430     bit64.obj
 0002:00006530       ??_C@_05GFCDIDHO@debug@    10052530     exported.obj
 0002:00006538       ??_C@_09GPFEECNC@traceback@ 10052538     exported.obj
 0002:00006544       ??_C@_06NKNNMLDJ@export@   10052544     exported.obj
 0002:0000654c       ??_C@_07PCNKBAGB@OnError@  1005254c     exported.obj
 0002:00006554       ??_C@_0N@NJMIGDDL@CreationTime@ 10052554     exported.obj
 0002:00006564       ??_C@_0P@MFHPCDDH@LastAccessTime@ 10052564     exported.obj
 0002:00006574       ??_C@_0O@FCFNCAHK@LastWriteTime@ 10052574     exported.obj
 0002:00006584       ??_C@_0L@FCILKIIG@ChangeTime@ 10052584     exported.obj
 0002:00006590       ??_C@_08BHIEONMC@FileSize@ 10052590     exported.obj
 0002:0000659c       ??_C@_0P@JBACEJLL@AllocationSize@ 1005259c     exported.obj
 0002:000065ac       ??_C@_05BOOEKJH@Flags@     100525ac     exported.obj
 0002:000065b4       ??_C@_0O@DLGJHFNH@NumberOfLinks@ 100525b4     exported.obj
 0002:000065c4       ??_C@_05MHNOECFO@CRC32@    100525c4     exported.obj
 0002:000065cc       ??_C@_08FDCJCDOL@FileName@ 100525cc     exported.obj
 0002:000065d8       ??_C@_0BC@COCBGKAE@AlternateFileName@ 100525d8     exported.obj
 0002:000065ec       ??_C@_0M@OHKMKKDH@Description@ 100525ec     exported.obj
 0002:000065f8       ??_C@_05HDCNEILF@Owner@    100525f8     exported.obj
 0002:00006600       ??_C@_0BB@OKGMKOG@CustomColumnData@ 10052600     exported.obj
 0002:00006614       ??_C@_01LOCGONAA@?$AA@     10052614     service.obj
 0002:00006614       ??_C@_11LOCGONAA@@         10052614     exported.obj
 0002:00006618       ??_C@_08JNHPECBG@UserData@ 10052618     exported.obj
 0002:00006624       ??_C@_0M@BDCAMGGD@ExtUserData@ 10052624     exported.obj
 0002:00006630       ??_C@_0N@LHFGLEGJ@FreeUserData@ 10052630     exported.obj
 0002:00006640       ??_C@_0M@DFMHDHBL@GetFindData@ 10052640     exported.obj
 0002:0000664c       ??_C@_08FFPEEIHA@GetFiles@ 1005264c     exported.obj
 0002:00006658       ??_C@_0BC@IECOKJFL@GetFiles?4DestPath@ 10052658     exported.obj
 0002:0000666c       ??_C@_05LFOKGKBN@?$DMboot@ 1005266c     exported.obj
 0002:00006674       ??_C@_15CBMDENPJ@?$AA?4?$AA?9@ 10052674     exported.obj
 0002:0000667c       ??_C@_07KNEGBPNO@package@  1005267c     exported.obj
 0002:00006684       ??_C@_07GCEAJMEA@preload@  10052684     exported.obj
 0002:0000668c       ??_C@_19BCNABNAK@?$AA?4?$AAl?$AAu?$AAa@ 1005268c     exported.obj
 0002:00006698       ??_C@_13BPINEIPE@?$AAr@    10052698     exported.obj
 0002:0000669c       ??_C@_1DC@PABHCCON@?$AAD?$AAe?$AAf?$AAa?$AAu?$AAl?$AAt?$AA?5?$AAs?$AAc?$AAr?$AAi?$AAp?$AAt?$AA?5@ 1005269c     exported.obj
 0002:000066d0       ??_C@_03JEOKDCFP@far@      100526d0     exported.obj
 0002:000066d4       ??_C@_0BE@HCPAIELH@ReloadDefaultScript@ 100526d4     exported.obj
 0002:000066e8       ??_C@_0L@OCPPMCCK@StructSize@ 100526e8     exported.obj
 0002:000066f4       ??_C@_06LBMCOACO@Buffer@   100526f4     exported.obj
 0002:000066fc       ??_C@_06EPIAKPGD@OpMode@   100526fc     exported.obj
 0002:00006704       ??_C@_07GDADDFBD@Analyse@  10052704     exported.obj
 0002:0000670c       ??_C@_0BB@CKIGBGLB@GetOpenPanelInfo@ 1005270c     exported.obj
 0002:00006720       ??_C@_08KDMNIFGM@FreeSize@ 10052720     exported.obj
 0002:0000672c       ??_C@_08PAJOMFPO@HostFile@ 1005272c     exported.obj
 0002:00006738       ??_C@_06IBPEEEAJ@CurDir@   10052738     exported.obj
 0002:00006740       ??_C@_06PEPCFMNJ@Format@   10052740     exported.obj
 0002:00006748       ??_C@_0L@CMHIOLLB@PanelTitle@ 10052748     exported.obj
 0002:00006754       ??_C@_09PMEOAIAA@InfoLines@ 10052754     exported.obj
 0002:00006760       ??_C@_0BA@BLCGOCOG@InfoLinesNumber@ 10052760     exported.obj
 0002:00006770       ??_C@_04OJAHODMC@Text@     10052770     exported.obj
 0002:00006778       ??_C@_04DICKPMGH@Data@     10052778     exported.obj
 0002:00006780       ??_C@_0L@FPEHOFAI@DescrFiles@ 10052780     exported.obj
 0002:0000678c       ??_C@_0BA@BBOGKOKF@PanelModesArray@ 1005278c     exported.obj
 0002:0000679c       ??_C@_0BB@LFNABPEF@PanelModesNumber@ 1005279c     exported.obj
 0002:000067b0       ??_C@_0M@KDJPJFOF@ColumnTypes@ 100527b0     exported.obj
 0002:000067bc       ??_C@_0N@ILFJPGHI@ColumnWidths@ 100527bc     exported.obj
 0002:000067cc       ??_C@_0BC@KELOOKNK@StatusColumnTypes@ 100527cc     exported.obj
 0002:000067e0       ??_C@_0BD@DNDIPKDK@StatusColumnWidths@ 100527e0     exported.obj
 0002:000067f4       ??_C@_0N@EHCEJHEE@ColumnTitles@ 100527f4     exported.obj
 0002:00006804       ??_C@_0P@BEEDPJDK@StartPanelMode@ 10052804     exported.obj
 0002:00006814       ??_C@_0O@NIFKFGBJ@StartSortMode@ 10052814     exported.obj
 0002:00006824       ??_C@_0P@KMACBLNK@StartSortOrder@ 10052824     exported.obj
 0002:00006834       ??_C@_06ONGFDHIA@KeyBar@   10052834     exported.obj
 0002:0000683c       ??_C@_0P@PKDBPEJI@VirtualKeyCode@ 1005283c     exported.obj
 0002:0000684c       ??_C@_0BA@MFFHAKP@ControlKeyState@ 1005284c     exported.obj
 0002:0000685c       ??_C@_08DGDJEKCP@LongText@ 1005285c     exported.obj
 0002:00006868       ??_C@_0BE@OPMKBLIP@_ModuleShortcutData@ 10052868     exported.obj
 0002:0000687c       ??_C@_0N@IHDKLODA@ShortcutData@ 1005287c     exported.obj
 0002:0000688c       ??_C@_05HIFJDKLD@array@    1005288c     exported.obj
 0002:00006894       ??_C@_01EFFIKLCJ@n@        10052894     exported.obj
 0002:00006896       ??_C@_00CNPNBAHC@@         10052896     exported.obj
 0002:00006898       ??_C@_04DNCDCIAE@Open@     10052898     exported.obj
 0002:000068a0       ??_C@_04OPJIDECA@hDlg@     100528a0     exported.obj
 0002:000068a8       ??_C@_06BNNOMDLO@Handle@   100528a8     exported.obj
 0002:000068b0       ??_C@_05LNOAKADA@panel@    100528b0     exported.obj
 0002:000068b8       ??_C@_0L@JMPDJFBN@ClosePanel@ 100528b8     exported.obj
 0002:000068c4       ??_C@_07MBOMJGGF@Compare@  100528c4     exported.obj
 0002:000068cc       ??_C@_09NANCCILE@Configure@ 100528cc     exported.obj
 0002:000068d8       ??_C@_0M@MMKKMEFA@DeleteFiles@ 100528d8     exported.obj
 0002:000068e4       ??_C@_0O@GLLEDHJA@MakeDirectory@ 100528e4     exported.obj
 0002:000068f4       ??_C@_0BD@PJNONGDB@MakeDirectory?4Name@ 100528f4     exported.obj
 0002:00006908       ??_C@_0BC@COPMJGBI@ProcessPanelEvent@ 10052908     exported.obj
 0002:0000691c       ??_C@_0BA@DPJAKFGC@ProcessHostFile@ 1005291c     exported.obj
 0002:0000692c       ??_C@_0BC@HOBKGBBM@ProcessPanelInput@ 1005292c     exported.obj
 0002:00006940       ??_C@_08OBOOFGOD@PutFiles@ 10052940     exported.obj
 0002:0000694c       ??_C@_0N@KCFEBPAO@SetDirectory@ 1005294c     exported.obj
 0002:0000695c       ??_C@_0M@PNOHHCCH@SetFindList@ 1005295c     exported.obj
 0002:00006968       ??_C@_07EACELFAO@ExitFAR@  10052968     exported.obj
 0002:00006970       ??_C@_0O@OBCKADMD@GetPluginInfo@ 10052970     exported.obj
 0002:00006980       ??_C@_0O@GDMHGAFH@CommandPrefix@ 10052980     exported.obj
 0002:00006990       ??_C@_0O@PHBKMNMJ@DiskMenuGuids@ 10052990     exported.obj
 0002:000069a0       ??_C@_0BA@NLBDFPEO@DiskMenuStrings@ 100529a0     exported.obj
 0002:000069b0       ??_C@_0BA@FOMPNLJF@PluginMenuGuids@ 100529b0     exported.obj
 0002:000069c0       ??_C@_0BC@DJMJFBJC@PluginMenuStrings@ 100529c0     exported.obj
 0002:000069d4       ??_C@_0BC@ILBHAHCH@PluginConfigGuids@ 100529d4     exported.obj
 0002:000069e8       ??_C@_0BE@GAFPNGIP@PluginConfigStrings@ 100529e8     exported.obj
 0002:000069fc       ??_C@_0BD@DECJPBBK@ProcessEditorInput@ 100529fc     exported.obj
 0002:00006a10       ??_C@_0BD@GEMPAGBO@ProcessEditorEvent@ 10052a10     exported.obj
 0002:00006a24       ??_C@_04KOACHJEN@Type@     10052a24     exported.obj
 0002:00006a2c       ??_C@_0N@EKPHGDMI@StringNumber@ 10052a2c     exported.obj
 0002:00006a3c       ??_C@_07MOCFLHCN@FileEOL@  10052a3c     exported.obj
 0002:00006a44       ??_C@_08DOHJINHB@CodePage@ 10052a44     exported.obj
 0002:00006a50       ??_C@_0BD@GGKMLEJG@ProcessViewerEvent@ 10052a50     exported.obj
 0002:00006a64       ??_C@_0BD@FNHBEIC@ProcessDialogEvent@ 10052a64     exported.obj
 0002:00006a78       ??_C@_06CPBJDKAC@Param2@   10052a78     exported.obj
 0002:00006a80       ??_C@_06EDEGJMB@Param1@    10052a80     exported.obj
 0002:00006a88       ??_C@_03MLMOILGK@Msg@      10052a88     exported.obj
 0002:00006a8c       ??_C@_0BE@LHJGGGHN@ProcessSynchroEvent@ 10052a8c     exported.obj
 0002:00006aa0       ??_C@_0BB@PHIEFGHD@GetContentFields@ 10052aa0     exported.obj
 0002:00006ab4       ??_C@_0P@DPJDPMPI@GetContentData@ 10052ab4     exported.obj
 0002:00006ac4       ??_C@_0N@DDJEHLKE@?$DM_globalinfo@ 10052ac4     exported.obj
 0002:00006ad4       ??_C@_1CA@IBKDMBNJ@?$AA_?$AAg?$AAl?$AAo?$AAb?$AAa?$AAl?$AAi?$AAn?$AAf?$AAo?$AA?4?$AAl?$AAu?$AAa@ 10052ad4     exported.obj
 0002:00006af4       ??_C@_0O@GJMOPLGM@GetGlobalInfo@ 10052af4     exported.obj
 0002:00006b04       ??_C@_0O@CALOEOI@MinFarVersion@ 10052b04     exported.obj
 0002:00006b14       ??_C@_07NGFJPNPN@Version@  10052b14     exported.obj
 0002:00006b1c       ??_C@_04MJHIICBJ@Guid@     10052b1c     exported.obj
 0002:00006b24       ??_C@_05PABKJLOM@Title@    10052b24     exported.obj
 0002:00006b2c       ??_C@_06HHECMMLE@Author@   10052b2c     exported.obj
 0002:00006b34       ??_C@_0BE@DONMOPMJ@ProcessConsoleInput@ 10052b34     exported.obj
 0002:00006b48       _KEY_OBJECT                10052b48     exported.obj
 0002:00006b58       _COLLECTOR_GI              10052b58     exported.obj
 0002:00006b70       _COLLECTOR_OPI             10052b70     exported.obj
 0002:00006b88       _COLLECTOR_PI              10052b88     exported.obj
 0002:00006ba0       ??_C@_0BI@IDKIJMME@FARMANAGERVERSION_MAJOR@ 10052ba0     flags.obj
 0002:00006bb8       ??_C@_0BI@DMLKEAFC@FARMANAGERVERSION_MINOR@ 10052bb8     flags.obj
 0002:00006bd0       ??_C@_0BL@NMALNAFP@FARMANAGERVERSION_REVISION@ 10052bd0     flags.obj
 0002:00006bec       ??_C@_0BI@OLPFLLDD@FARMANAGERVERSION_BUILD@ 10052bec     flags.obj
 0002:00006c04       ??_C@_0BI@MOOFLFPC@FARMANAGERVERSION_STAGE@ 10052c04     flags.obj
 0002:00006c1c       ??_C@_0L@MIDBGFJO@CP_UNICODE@ 10052c1c     flags.obj
 0002:00006c28       ??_C@_0O@MNMCMEJH@CP_REVERSEBOM@ 10052c28     flags.obj
 0002:00006c38       ??_C@_0L@JDNPCEDH@CP_DEFAULT@ 10052c38     flags.obj
 0002:00006c44       ??_C@_0M@OMCMFJHA@CP_REDETECT@ 10052c44     flags.obj
 0002:00006c50       ??_C@_09MNAPNKKC@INDEXMASK@ 10052c50     flags.obj
 0002:00006c5c       ??_C@_09BLFIDJLF@COLORMASK@ 10052c5c     flags.obj
 0002:00006c68       ??_C@_09ENNBLPJC@ALPHAMASK@ 10052c68     flags.obj
 0002:00006c74       ??_C@_0L@EHFOPLFD@PANEL_NONE@ 10052c74     flags.obj
 0002:00006c80       ??_C@_0N@LPMKALBG@PANEL_ACTIVE@ 10052c80     flags.obj
 0002:00006c90       ??_C@_0O@HPKEABPN@PANEL_PASSIVE@ 10052c90     flags.obj
 0002:00006ca0       ??_C@_0L@GOEBPENN@PANEL_STOP@ 10052ca0     flags.obj
 0002:00006cac       ??_C@_0N@HLIFAAPJ@EEREDRAW_ALL@ 10052cac     flags.obj
 0002:00006cbc       ??_C@_0P@NHNDIKJ@CURRENT_EDITOR@ 10052cbc     flags.obj
 0002:00006ccc       ??_C@_0BN@PPNDCHHA@EDITOR_COLOR_NORMAL_PRIORITY@ 10052ccc     flags.obj
 0002:00006cec       ??_C@_07MGGAEAFF@DI_TEXT@  10052cec     flags.obj
 0002:00006cf4       ??_C@_08HODBDEHE@DI_VTEXT@ 10052cf4     flags.obj
 0002:00006d00       ??_C@_0N@IGKKGFMF@DI_SINGLEBOX@ 10052d00     flags.obj
 0002:00006d10       ??_C@_0N@EDCLIEAE@DI_DOUBLEBOX@ 10052d10     flags.obj
 0002:00006d20       ??_C@_07DOLIFAEF@DI_EDIT@  10052d20     flags.obj
 0002:00006d28       ??_C@_0L@EOMEIIFM@DI_PSWEDIT@ 10052d28     flags.obj
 0002:00006d34       ??_C@_0L@MGOIMBKF@DI_FIXEDIT@ 10052d34     flags.obj
 0002:00006d40       ??_C@_09GGAEMAPJ@DI_BUTTON@ 10052d40     flags.obj
 0002:00006d4c       ??_C@_0M@MHFHGPHJ@DI_CHECKBOX@ 10052d4c     flags.obj
 0002:00006d58       ??_C@_0P@GIPCGMBE@DI_RADIOBUTTON@ 10052d58     flags.obj
 0002:00006d68       ??_C@_0M@MAKBFNGC@DI_COMBOBOX@ 10052d68     flags.obj
 0002:00006d74       ??_C@_0L@ONDMPPPO@DI_LISTBOX@ 10052d74     flags.obj
 0002:00006d80       ??_C@_0P@GDJDPEIK@DI_USERCONTROL@ 10052d80     flags.obj
 0002:00006d90       ??_C@_08KAEGOLOB@DM_FIRST@ 10052d90     flags.obj
 0002:00006d9c       ??_C@_08MJMBFJHA@DM_CLOSE@ 10052d9c     flags.obj
 0002:00006da8       ??_C@_09KLJOCKAA@DM_ENABLE@ 10052da8     flags.obj
 0002:00006db4       ??_C@_0BA@KAMJGFDG@DM_ENABLEREDRAW@ 10052db4     flags.obj
 0002:00006dc4       ??_C@_0O@FKGMMKLP@DM_GETDLGDATA@ 10052dc4     flags.obj
 0002:00006dd4       ??_C@_0O@HEGKCPOI@DM_GETDLGITEM@ 10052dd4     flags.obj
 0002:00006de4       ??_C@_0O@BEHCGMCL@DM_GETDLGRECT@ 10052de4     flags.obj
 0002:00006df4       ??_C@_0L@ELBDNLFO@DM_GETTEXT@ 10052df4     flags.obj
 0002:00006e00       ??_C@_06IKGPEGEJ@DM_KEY@   10052e00     flags.obj
 0002:00006e08       ??_C@_0O@DIPLLJEH@DM_MOVEDIALOG@ 10052e08     flags.obj
 0002:00006e18       ??_C@_0O@EEEDHNPG@DM_SETDLGDATA@ 10052e18     flags.obj
 0002:00006e28       ??_C@_0O@GKEFJIKB@DM_SETDLGITEM@ 10052e28     flags.obj
 0002:00006e38       ??_C@_0M@GOFGHDFK@DM_SETFOCUS@ 10052e38     flags.obj
 0002:00006e44       ??_C@_09ILPFEDOM@DM_REDRAW@ 10052e44     flags.obj
 0002:00006e50       ??_C@_0L@LDOCOEIP@DM_SETTEXT@ 10052e50     flags.obj
 0002:00006e5c       ??_C@_0BE@LABEAIPD@DM_SETMAXTEXTLENGTH@ 10052e5c     flags.obj
 0002:00006e70       ??_C@_0O@BIFKIPIP@DM_SHOWDIALOG@ 10052e70     flags.obj
 0002:00006e80       ??_C@_0M@JPHKGACH@DM_GETFOCUS@ 10052e80     flags.obj
 0002:00006e8c       ??_C@_0BA@NLMONBKJ@DM_GETCURSORPOS@ 10052e8c     flags.obj
 0002:00006e9c       ??_C@_0BA@KPHABNOF@DM_SETCURSORPOS@ 10052e9c     flags.obj
 0002:00006eac       ??_C@_0O@LGEKFPKK@DM_SETTEXTPTR@ 10052eac     flags.obj
 0002:00006ebc       ??_C@_0M@NCOJHJKI@DM_SHOWITEM@ 10052ebc     flags.obj
 0002:00006ec8       ??_C@_0O@GKKCFHIM@DM_ADDHISTORY@ 10052ec8     flags.obj
 0002:00006ed8       ??_C@_0M@MCEMDFMD@DM_GETCHECK@ 10052ed8     flags.obj
 0002:00006ee4       ??_C@_0M@DDGACGLO@DM_SETCHECK@ 10052ee4     flags.obj
 0002:00006ef0       ??_C@_0N@MEGOPFGK@DM_SET3STATE@ 10052ef0     flags.obj
 0002:00006f00       ??_C@_0M@GEPBDDNC@DM_LISTSORT@ 10052f00     flags.obj
 0002:00006f0c       ??_C@_0P@NFJNHAKH@DM_LISTGETITEM@ 10052f0c     flags.obj
 0002:00006f1c       ??_C@_0BB@EEIMACNO@DM_LISTGETCURPOS@ 10052f1c     flags.obj
 0002:00006f30       ??_C@_0BB@GKMJCDEM@DM_LISTSETCURPOS@ 10052f30     flags.obj
 0002:00006f44       ??_C@_0O@NOPCAHGJ@DM_LISTDELETE@ 10052f44     flags.obj
 0002:00006f54       ??_C@_0L@BMEAECNG@DM_LISTADD@ 10052f54     flags.obj
 0002:00006f60       ??_C@_0O@HBHDMHP@DM_LISTADDSTR@ 10052f60     flags.obj
 0002:00006f70       ??_C@_0O@PDFCNPKN@DM_LISTUPDATE@ 10052f70     flags.obj
 0002:00006f80       ??_C@_0O@GAAGMJJL@DM_LISTINSERT@ 10052f80     flags.obj
 0002:00006f90       ??_C@_0BC@MIFCLOBD@DM_LISTFINDSTRING@ 10052f90     flags.obj
 0002:00006fa4       ??_C@_0M@EEAEBLKC@DM_LISTINFO@ 10052fa4     flags.obj
 0002:00006fb0       ??_C@_0P@PLJLJFPA@DM_LISTGETDATA@ 10052fb0     flags.obj
 0002:00006fc0       ??_C@_0P@DGKKKCB@DM_LISTSETDATA@ 10052fc0     flags.obj
 0002:00006fd0       ??_C@_0BB@CELMNLLN@DM_LISTSETTITLES@ 10052fd0     flags.obj
 0002:00006fe4       ??_C@_0BB@KPJPKCP@DM_LISTGETTITLES@ 10052fe4     flags.obj
 0002:00006ff8       ??_C@_0BA@ICDJCFLE@DM_RESIZEDIALOG@ 10052ff8     flags.obj
 0002:00007008       ??_C@_0BD@CNGGHGJF@DM_SETITEMPOSITION@ 10053008     flags.obj
 0002:0000701c       ??_C@_0BF@JMINBGBA@DM_GETDROPDOWNOPENED@ 1005301c     flags.obj
 0002:00007034       ??_C@_0BF@LJIGJNAO@DM_SETDROPDOWNOPENED@ 10053034     flags.obj
 0002:0000704c       ??_C@_0O@NPDKADMJ@DM_SETHISTORY@ 1005304c     flags.obj
 0002:0000705c       ??_C@_0BD@BPHAAEIM@DM_GETITEMPOSITION@ 1005305c     flags.obj
 0002:00007070       ??_C@_0BC@BENFKLNH@DM_SETINPUTNOTIFY@ 10053070     flags.obj
 0002:00007084       ??_C@_0BH@CFMLLNNM@DM_SETMOUSEEVENTNOTIFY@ 10053084     flags.obj
 0002:0000709c       ??_C@_0BF@IAGIACOD@DM_EDITUNCHANGEDFLAG@ 1005309c     flags.obj
 0002:000070b4       ??_C@_0P@OJKNHIPN@DM_GETITEMDATA@ 100530b4     flags.obj
 0002:000070c4       ??_C@_0P@OGLDKOHO@DM_SETITEMDATA@ 100530c4     flags.obj
 0002:000070d4       ??_C@_0L@KNFAKFKE@DM_LISTSET@ 100530d4     flags.obj
 0002:000070e0       ??_C@_0BB@EPMFHAFO@DM_GETCURSORSIZE@ 100530e0     flags.obj
 0002:000070f4       ??_C@_0BB@DANLMDCJ@DM_SETCURSORSIZE@ 100530f4     flags.obj
 0002:00007108       ??_C@_0BD@LAOOKGHD@DM_LISTGETDATASIZE@ 10053108     flags.obj
 0002:0000711c       ??_C@_0BA@BHGANJAP@DM_GETSELECTION@ 1005311c     flags.obj
 0002:0000712c       ??_C@_0BA@GDNOBFED@DM_SETSELECTION@ 1005312c     flags.obj
 0002:0000713c       ??_C@_0BD@FIHDGIGO@DM_GETEDITPOSITION@ 1005313c     flags.obj
 0002:00007150       ??_C@_0BD@GKGFBKHH@DM_SETEDITPOSITION@ 10053150     flags.obj
 0002:00007164       ??_C@_0BE@MCECGHBC@DM_SETCOMBOBOXEVENT@ 10053164     flags.obj
 0002:00007178       ??_C@_0BE@KGBLNJKA@DM_GETCOMBOBOXEVENT@ 10053178     flags.obj
 0002:0000718c       ??_C@_0BD@CJEPBACF@DM_GETCONSTTEXTPTR@ 1005318c     flags.obj
 0002:000071a0       ??_C@_0BD@HOOHICEG@DM_GETDLGITEMSHORT@ 100531a0     flags.obj
 0002:000071b4       ??_C@_0BD@EMPBPAFP@DM_SETDLGITEMSHORT@ 100531b4     flags.obj
 0002:000071c8       ??_C@_0BB@GAPFMPKE@DM_GETDIALOGINFO@ 100531c8     flags.obj
 0002:000071dc       ??_C@_0BC@KJOLMFGG@DM_GETDIALOGTITLE@ 100531dc     flags.obj
 0002:000071f0       ??_C@_08COMJOMAC@DN_FIRST@ 100531f0     flags.obj
 0002:000071fc       ??_C@_0M@NNNAPNMA@DN_BTNCLICK@ 100531fc     flags.obj
 0002:00007208       ??_C@_0BC@MJFJAANN@DN_CTLCOLORDIALOG@ 10053208     flags.obj
 0002:0000721c       ??_C@_0BD@HFGBIBBL@DN_CTLCOLORDLGITEM@ 1005321c     flags.obj
 0002:00007230       ??_C@_0BD@JMFJPHPD@DN_CTLCOLORDLGLIST@ 10053230     flags.obj
 0002:00007244       ??_C@_0O@NKBDPILK@DN_DRAWDIALOG@ 10053244     flags.obj
 0002:00007254       ??_C@_0P@KGKEDPBI@DN_DRAWDLGITEM@ 10053254     flags.obj
 0002:00007264       ??_C@_0O@JMKNGFLE@DN_EDITCHANGE@ 10053264     flags.obj
 0002:00007274       ??_C@_0M@JHFIBKOO@DN_GOTFOCUS@ 10053274     flags.obj
 0002:00007280       ??_C@_07NJJEMKPA@DN_HELP@  10053280     flags.obj
 0002:00007288       ??_C@_09EDGJFAK@DN_HOTKEY@ 10053288     flags.obj
 0002:00007294       ??_C@_0O@BJECHBCA@DN_INITDIALOG@ 10053294     flags.obj
 0002:000072a4       ??_C@_0N@CHLLLNBO@DN_KILLFOCUS@ 100532a4     flags.obj
 0002:000072b4       ??_C@_0O@CLPABIGO@DN_LISTCHANGE@ 100532b4     flags.obj
 0002:000072c4       ??_C@_0L@MLMFBHN@DN_DRAGGED@ 100532c4     flags.obj
 0002:000072d0       ??_C@_0BB@BOOOCAEG@DN_RESIZECONSOLE@ 100532d0     flags.obj
 0002:000072e4       ??_C@_0BC@FHPPFLKG@DN_DRAWDIALOGDONE@ 100532e4     flags.obj
 0002:000072f8       ??_C@_0O@EONPBNNP@DN_LISTHOTKEY@ 100532f8     flags.obj
 0002:00007308       ??_C@_08MDDLDGPO@DN_INPUT@ 10053308     flags.obj
 0002:00007314       ??_C@_0BA@FGOGLDBC@DN_CONTROLINPUT@ 10053314     flags.obj
 0002:00007324       ??_C@_08EHEOFOJD@DN_CLOSE@ 10053324     flags.obj
 0002:00007330       ??_C@_0M@POIFBPFN@DN_GETVALUE@ 10053330     flags.obj
 0002:0000733c       ??_C@_0BC@MHCBFAAO@DN_DROPDOWNOPENED@ 1005333c     flags.obj
 0002:00007350       ??_C@_0BD@NGEKAPIF@DN_DRAWDLGITEMDONE@ 10053350     flags.obj
 0002:00007364       ??_C@_07DIJJNCBA@DM_USER@  10053364     flags.obj
 0002:0000736c       ??_C@_0BB@HLBBGMAN@BSTATE_UNCHECKED@ 1005336c     flags.obj
 0002:00007380       ??_C@_0P@FALAMPGP@BSTATE_CHECKED@ 10053380     flags.obj
 0002:00007390       ??_C@_0O@KBIFGGHO@BSTATE_3STATE@ 10053390     flags.obj
 0002:000073a0       ??_C@_0O@ILJOJGLD@BSTATE_TOGGLE@ 100533a0     flags.obj
 0002:000073b0       ??_C@_08PPADCPCM@CBET_KEY@ 100533b0     flags.obj
 0002:000073bc       ??_C@_0L@KHCLMGFJ@CBET_MOUSE@ 100533bc     flags.obj
 0002:000073c8       ??_C@_0BA@KNHGEBNE@PTYPE_FILEPANEL@ 100533c8     flags.obj
 0002:000073d8       ??_C@_0BA@LPPHNHIG@PTYPE_TREEPANEL@ 100533d8     flags.obj
 0002:000073e8       ??_C@_0BB@JBINOKAI@PTYPE_QVIEWPANEL@ 100533e8     flags.obj
 0002:000073fc       ??_C@_0BA@NKMDEBG@PTYPE_INFOPANEL@ 100533fc     flags.obj
 0002:0000740c       ??_C@_0L@OPHJOKKE@SM_DEFAULT@ 1005340c     flags.obj
 0002:00007418       ??_C@_0M@JGBFGGEA@SM_UNSORTED@ 10053418     flags.obj
 0002:00007424       ??_C@_07KIFHAGIL@SM_NAME@  10053424     flags.obj
 0002:0000742c       ??_C@_0M@OAFEBGNH@SM_FULLNAME@ 1005342c     flags.obj
 0002:00007438       ??_C@_06GJJJNNFE@SM_EXT@   10053438     flags.obj
 0002:00007440       ??_C@_08FICJBKFN@SM_MTIME@ 10053440     flags.obj
 0002:0000744c       ??_C@_08GCCDHLCN@SM_CTIME@ 1005344c     flags.obj
 0002:00007458       ??_C@_08CPOLNKCG@SM_ATIME@ 10053458     flags.obj
 0002:00007464       ??_C@_07OMPKMIKC@SM_SIZE@  10053464     flags.obj
 0002:0000746c       ??_C@_08BCBPOLMA@SM_DESCR@ 1005346c     flags.obj
 0002:00007478       ??_C@_08MEAGCMBB@SM_OWNER@ 10053478     flags.obj
 0002:00007484       ??_C@_0BC@NKDBNAHD@SM_COMPRESSEDSIZE@ 10053484     flags.obj
 0002:00007498       ??_C@_0M@PKNLKFI@SM_NUMLINKS@ 10053498     flags.obj
 0002:000074a4       ??_C@_0O@CCKEKPHL@SM_NUMSTREAMS@ 100534a4     flags.obj
 0002:000074b4       ??_C@_0P@PKGMDPMD@SM_STREAMSSIZE@ 100534b4     flags.obj
 0002:000074c4       ??_C@_0M@KALDNPOO@SM_NAMEONLY@ 100534c4     flags.obj
 0002:000074d0       ??_C@_09KFKGJDHC@SM_CHTIME@ 100534d0     flags.obj
 0002:000074dc       ??_C@_08DOEDKINA@SM_COUNT@ 100534dc     flags.obj
 0002:000074e8       ??_C@_07EOOHOKCC@SM_USER@  100534e8     flags.obj
 0002:000074f0       ??_C@_0P@FEMAMJLE@EEC_OPEN_ERROR@ 100534f0     flags.obj
 0002:00007500       ??_C@_0N@GLMELIKF@EEC_MODIFIED@ 10053500     flags.obj
 0002:00007510       ??_C@_0BB@HALKEFOL@EEC_NOT_MODIFIED@ 10053510     flags.obj
 0002:00007524       ??_C@_0BI@CNPFKHKO@EEC_LOADING_INTERRUPTED@ 10053524     flags.obj
 0002:0000753c       ??_C@_0BK@PHBCABMB@ACTL_GETFARMANAGERVERSION@ 1005353c     flags.obj
 0002:00007558       ??_C@_0N@DPABJDML@ACTL_WAITKEY@ 10053558     flags.obj
 0002:00007568       ??_C@_0O@CEHHJAFD@ACTL_GETCOLOR@ 10053568     flags.obj
 0002:00007578       ??_C@_0BD@OKPAACIK@ACTL_GETARRAYCOLOR@ 10053578     flags.obj
 0002:0000758c       ??_C@_0BD@DIFEEKNN@ACTL_GETWINDOWINFO@ 1005358c     flags.obj
 0002:000075a0       ??_C@_0BE@PJBIPKOD@ACTL_GETWINDOWCOUNT@ 100535a0     flags.obj
 0002:000075b4       ??_C@_0BG@MNKPOEEN@ACTL_SETCURRENTWINDOW@ 100535b4     flags.obj
 0002:000075cc       ??_C@_0M@IHHFGPPA@ACTL_COMMIT@ 100535cc     flags.obj
 0002:000075d8       ??_C@_0BA@CLHFKJJP@ACTL_GETFARHWND@ 100535d8     flags.obj
 0002:000075e8       ??_C@_0BD@JFOOLBPN@ACTL_SETARRAYCOLOR@ 100535e8     flags.obj
 0002:000075fc       ??_C@_0P@JECKFIA@ACTL_REDRAWALL@ 100535fc     flags.obj
 0002:0000760c       ??_C@_0N@DHPLJLHO@ACTL_SYNCHRO@ 1005360c     flags.obj
 0002:0000761c       ??_C@_0BG@IJPADENB@ACTL_SETPROGRESSSTATE@ 1005361c     flags.obj
 0002:00007634       ??_C@_0BG@ICJFAPHK@ACTL_SETPROGRESSVALUE@ 10053634     flags.obj
 0002:0000764c       ??_C@_09HNDBKLDC@ACTL_QUIT@ 1005364c     flags.obj
 0002:00007658       ??_C@_0BA@LJCPDIKK@ACTL_GETFARRECT@ 10053658     flags.obj
 0002:00007668       ??_C@_0BC@FELBEIDG@ACTL_GETCURSORPOS@ 10053668     flags.obj
 0002:0000767c       ??_C@_0BC@CAAPIEHK@ACTL_SETCURSORPOS@ 1005367c     flags.obj
 0002:00007690       ??_C@_0BE@NPJGMDBM@ACTL_PROGRESSNOTIFY@ 10053690     flags.obj
 0002:000076a4       ??_C@_0BD@IPKOEBIA@ACTL_GETWINDOWTYPE@ 100536a4     flags.obj
 0002:000076b8       ??_C@_09CEDFMINA@MSSC_POST@ 100536b8     flags.obj
 0002:000076c4       ??_C@_0L@MOADGAEB@MSSC_CHECK@ 100536c4     flags.obj
 0002:000076d0       ??_C@_0BA@MMOAIEKP@MACROAREA_OTHER@ 100536d0     flags.obj
 0002:000076e0       ??_C@_0BA@DEBOOAEB@MACROAREA_SHELL@ 100536e0     flags.obj
 0002:000076f0       ??_C@_0BB@JIMPEHCD@MACROAREA_VIEWER@ 100536f0     flags.obj
 0002:00007704       ??_C@_0BB@KILFBFJH@MACROAREA_EDITOR@ 10053704     flags.obj
 0002:00007718       ??_C@_0BB@CADENPFI@MACROAREA_DIALOG@ 10053718     flags.obj
 0002:0000772c       ??_C@_0BB@MLMLHIGE@MACROAREA_SEARCH@ 1005372c     flags.obj
 0002:00007740       ??_C@_0BA@KKMKOLIK@MACROAREA_DISKS@ 10053740     flags.obj
 0002:00007750       ??_C@_0BD@IGOOIJP@MACROAREA_MAINMENU@ 10053750     flags.obj
 0002:00007764       ??_C@_0P@LFLMAHBF@MACROAREA_MENU@ 10053764     flags.obj
 0002:00007774       ??_C@_0P@DKPKIEO@MACROAREA_HELP@ 10053774     flags.obj
 0002:00007784       ??_C@_0BE@MDJPICHC@MACROAREA_INFOPANEL@ 10053784     flags.obj
 0002:00007798       ??_C@_0BF@NLJMHMPP@MACROAREA_QVIEWPANEL@ 10053798     flags.obj
 0002:000077b0       ??_C@_0BE@HBMEGBOC@MACROAREA_TREEPANEL@ 100537b0     flags.obj
 0002:000077c4       ??_C@_0BF@FCHKCGLL@MACROAREA_FINDFOLDER@ 100537c4     flags.obj
 0002:000077dc       ??_C@_0BD@JCFMJGDE@MACROAREA_USERMENU@ 100537dc     flags.obj
 0002:000077f0       ??_C@_0BO@OMLEPJPM@MACROAREA_SHELLAUTOCOMPLETION@ 100537f0     flags.obj
 0002:00007810       ??_C@_0BP@OIHAIGBK@MACROAREA_DIALOGAUTOCOMPLETION@ 10053810     flags.obj
 0002:00007830       ??_C@_0BC@EIJFKPMK@MACROAREA_GRABBER@ 10053830     flags.obj
 0002:00007844       ??_C@_0BC@GNLOCEJP@MACROAREA_DESKTOP@ 10053844     flags.obj
 0002:00007858       ??_C@_0BB@JPEEDDOG@MACROAREA_COMMON@ 10053858     flags.obj
 0002:0000786c       ??_C@_0BD@DIKEKAIJ@MACROSTATE_NOMACRO@ 1005386c     flags.obj
 0002:00007880       ??_C@_0BF@PCDEFEGP@MACROSTATE_EXECUTING@ 10053880     flags.obj
 0002:00007898       ??_C@_0BM@EJOFDENO@MACROSTATE_EXECUTING_COMMON@ 10053898     flags.obj
 0002:000078b4       ??_C@_0BF@BGODKPBB@MACROSTATE_RECORDING@ 100538b4     flags.obj
 0002:000078cc       ??_C@_0BM@OICPADFE@MACROSTATE_RECORDING_COMMON@ 100538cc     flags.obj
 0002:000078e8       ??_C@_0N@CGFFMLBC@MPEC_SUCCESS@ 100538e8     flags.obj
 0002:000078f8       ??_C@_0L@FJDDLDNN@MPEC_ERROR@ 100538f8     flags.obj
 0002:00007904       ??_C@_0N@IBOAADDD@FMVT_UNKNOWN@ 10053904     flags.obj
 0002:00007914       ??_C@_0N@BDMFKEKE@FMVT_INTEGER@ 10053914     flags.obj
 0002:00007924       ??_C@_0M@LFMLDDKI@FMVT_STRING@ 10053924     flags.obj
 0002:00007930       ??_C@_0M@CKDAIOEN@FMVT_DOUBLE@ 10053930     flags.obj
 0002:0000793c       ??_C@_0N@MHKOBOGF@FMVT_BOOLEAN@ 1005393c     flags.obj
 0002:0000794c       ??_C@_0M@GKPDICDA@FMVT_BINARY@ 1005394c     flags.obj
 0002:00007958       ??_C@_0N@FMHCFNDF@FMVT_POINTER@ 10053958     flags.obj
 0002:00007968       ??_C@_08DDPDBBNO@FMVT_NIL@ 10053968     flags.obj
 0002:00007974       ??_C@_0L@DJIKMOJA@FMVT_ARRAY@ 10053974     flags.obj
 0002:00007980       ??_C@_0L@PMDDFEBD@FMVT_PANEL@ 10053980     flags.obj
 0002:0000798c       ??_C@_0L@ELHBHIEH@FMVT_ERROR@ 1005398c     flags.obj
 0002:00007998       ??_C@_0O@OGHFLIKM@WTYPE_UNKNOWN@ 10053998     flags.obj
 0002:000079a8       ??_C@_0O@DCGKMPOM@WTYPE_DESKTOP@ 100539a8     flags.obj
 0002:000079b8       ??_C@_0N@FNCFCPIG@WTYPE_PANELS@ 100539b8     flags.obj
 0002:000079c8       ??_C@_0N@EJKMDMBK@WTYPE_VIEWER@ 100539c8     flags.obj
 0002:000079d8       ??_C@_0N@HJNGGOKO@WTYPE_EDITOR@ 100539d8     flags.obj
 0002:000079e8       ??_C@_0N@PBFHKEGB@WTYPE_DIALOG@ 100539e8     flags.obj
 0002:000079f8       ??_C@_0M@OMKLELFA@WTYPE_VMENU@ 100539f8     flags.obj
 0002:00007a04       ??_C@_0L@BCEMNGOG@WTYPE_HELP@ 10053a04     flags.obj
 0002:00007a10       ??_C@_0P@MMIDEOJJ@WTYPE_COMBOBOX@ 10053a10     flags.obj
 0002:00007a20       ??_C@_0O@BHEBEELJ@WTYPE_GRABBER@ 10053a20     flags.obj
 0002:00007a30       ??_C@_0M@NFHHCILL@WTYPE_HMENU@ 10053a30     flags.obj
 0002:00007a3c       ??_C@_0BA@IPEAOBGN@TBPS_NOPROGRESS@ 10053a3c     flags.obj
 0002:00007a4c       ??_C@_0BD@HMEHMDAL@TBPS_INDETERMINATE@ 10053a4c     flags.obj
 0002:00007a60       ??_C@_0M@KHLNKPHE@TBPS_NORMAL@ 10053a60     flags.obj
 0002:00007a6c       ??_C@_0L@DFDPCOFD@TBPS_ERROR@ 10053a6c     flags.obj
 0002:00007a78       ??_C@_0M@GHGAPHPP@TBPS_PAUSED@ 10053a78     flags.obj
 0002:00007a84       ??_C@_0O@MCNCFBLF@VSMT_VIEWMODE@ 10053a84     flags.obj
 0002:00007a94       ??_C@_09FLKONCNO@VSMT_WRAP@ 10053a94     flags.obj
 0002:00007aa0       ??_C@_0O@INKALKJK@VSMT_WORDWRAP@ 10053aa0     flags.obj
 0002:00007ab0       ??_C@_08FNEFFFEL@VMT_TEXT@ 10053ab0     flags.obj
 0002:00007abc       ??_C@_07FLIHDEDA@VMT_HEX@  10053abc     flags.obj
 0002:00007ac4       ??_C@_08BDDNDBMJ@VMT_DUMP@ 10053ac4     flags.obj
 0002:00007ad0       ??_C@_07OJCLGDHJ@VE_READ@  10053ad0     flags.obj
 0002:00007ad8       ??_C@_08JIBCCIDC@VE_CLOSE@ 10053ad8     flags.obj
 0002:00007ae4       ??_C@_0M@FEFKOOMJ@VE_GOTFOCUS@ 10053ae4     flags.obj
 0002:00007af0       ??_C@_0N@ICHCAKIB@VE_KILLFOCUS@ 10053af0     flags.obj
 0002:00007b00       ??_C@_07BLBPFFLB@EE_READ@  10053b00     flags.obj
 0002:00007b08       ??_C@_07KJGPGPOC@EE_SAVE@  10053b08     flags.obj
 0002:00007b10       ??_C@_09NPOPIKMK@EE_REDRAW@ 10053b10     flags.obj
 0002:00007b1c       ??_C@_08NFPFGIG@EE_CLOSE@  10053b1c     flags.obj
 0002:00007b28       ??_C@_0M@CPNMNBMF@EE_GOTFOCUS@ 10053b28     flags.obj
 0002:00007b34       ??_C@_0N@ILLPMAJF@EE_KILLFOCUS@ 10053b34     flags.obj
 0002:00007b44       ??_C@_09MIOGFFI@EE_CHANGE@ 10053b44     flags.obj
 0002:00007b50       ??_C@_0P@MBHAHBBG@DE_DLGPROCINIT@ 10053b50     flags.obj
 0002:00007b60       ??_C@_0BC@BMFEJAMO@DE_DEFDLGPROCINIT@ 10053b60     flags.obj
 0002:00007b74       ??_C@_0O@ICBCOJCG@DE_DLGPROCEND@ 10053b74     flags.obj
 0002:00007b84       ??_C@_0BB@MNODJNPE@SE_COMMONSYNCHRO@ 10053b84     flags.obj
 0002:00007b98       ??_C@_0N@HKGMPMJE@ESPT_TABSIZE@ 10053b98     flags.obj
 0002:00007ba8       ??_C@_0BA@GOKHPFCK@ESPT_EXPANDTABS@ 10053ba8     flags.obj
 0002:00007bb8       ??_C@_0BA@KOADDMLI@ESPT_AUTOINDENT@ 10053bb8     flags.obj
 0002:00007bc8       ??_C@_0BF@LPNONOMF@ESPT_CURSORBEYONDEOL@ 10053bc8     flags.obj
 0002:00007be0       ??_C@_0BC@OECOCGLJ@ESPT_CHARCODEBASE@ 10053be0     flags.obj
 0002:00007bf4       ??_C@_0O@PIAOJINE@ESPT_CODEPAGE@ 10053bf4     flags.obj
 0002:00007c04       ??_C@_0BG@HAPABMJH@ESPT_SAVEFILEPOSITION@ 10053c04     flags.obj
 0002:00007c1c       ??_C@_0O@KCPDJCKC@ESPT_LOCKMODE@ 10053c1c     flags.obj
 0002:00007c2c       ??_C@_0BA@EIGIAOHM@ESPT_SETWORDDIV@ 10053c2c     flags.obj
 0002:00007c3c       ??_C@_0BA@FGEHLJDF@ESPT_GETWORDDIV@ 10053c3c     flags.obj
 0002:00007c4c       ??_C@_0BE@MACJBCFP@ESPT_SHOWWHITESPACE@ 10053c4c     flags.obj
 0002:00007c60       ??_C@_0M@FICNFPPA@ESPT_SETBOM@ 10053c60     flags.obj
 0002:00007c6c       ??_C@_09FLEMPKKP@EUR_BEGIN@ 10053c6c     flags.obj
 0002:00007c78       ??_C@_07DDJDFJCN@EUR_END@  10053c78     flags.obj
 0002:00007c80       ??_C@_08FCONALGE@EUR_UNDO@ 10053c80     flags.obj
 0002:00007c8c       ??_C@_08DHMMFAHF@EUR_REDO@ 10053c8c     flags.obj
 0002:00007c98       ??_C@_0O@PKOIFEBO@EXPAND_NOTABS@ 10053c98     flags.obj
 0002:00007ca8       ??_C@_0P@MLHPCNDM@EXPAND_ALLTABS@ 10053ca8     flags.obj
 0002:00007cb8       ??_C@_0P@OONGIIBL@EXPAND_NEWTABS@ 10053cb8     flags.obj
 0002:00007cc8       ??_C@_0BD@DKHPEOHH@EOPT_EXPANDALLTABS@ 10053cc8     flags.obj
 0002:00007cdc       ??_C@_0BG@BOINMDEK@EOPT_PERSISTENTBLOCKS@ 10053cdc     flags.obj
 0002:00007cf4       ??_C@_0BG@PIIHHCAN@EOPT_DELREMOVESBLOCKS@ 10053cf4     flags.obj
 0002:00007d0c       ??_C@_0BA@KPJEAKBD@EOPT_AUTOINDENT@ 10053d0c     flags.obj
 0002:00007d1c       ??_C@_0BG@MBPADLG@EOPT_SAVEFILEPOSITION@ 10053d1c     flags.obj
 0002:00007d34       ??_C@_0BI@PFHCGCAI@EOPT_AUTODETECTCODEPAGE@ 10053d34     flags.obj
 0002:00007d4c       ??_C@_0BF@IMCOEIAL@EOPT_CURSORBEYONDEOL@ 10053d4c     flags.obj
 0002:00007d64       ??_C@_0BH@CJPAGGLC@EOPT_EXPANDONLYNEWTABS@ 10053d64     flags.obj
 0002:00007d7c       ??_C@_0BE@DDKCDJDC@EOPT_SHOWWHITESPACE@ 10053d7c     flags.obj
 0002:00007d90       ??_C@_08HMMLONBH@EOPT_BOM@ 10053d90     flags.obj
 0002:00007d9c       ??_C@_0BD@CLLAKGOA@EOPT_SHOWLINEBREAK@ 10053d9c     flags.obj
 0002:00007db0       ??_C@_0BC@JCJEPKEC@EOPT_SHOWTITLEBAR@ 10053db0     flags.obj
 0002:00007dc4       ??_C@_0BA@KPGMOBKI@EOPT_SHOWKEYBAR@ 10053dc4     flags.obj
 0002:00007dd4       ??_C@_0BD@EFCFEAD@EOPT_SHOWSCROLLBAR@ 10053dd4     flags.obj
 0002:00007de8       ??_C@_0L@BJCBJJNB@BTYPE_NONE@ 10053de8     flags.obj
 0002:00007df4       ??_C@_0N@OPHHGFPF@BTYPE_STREAM@ 10053df4     flags.obj
 0002:00007e04       ??_C@_0N@EMEGNPLI@BTYPE_COLUMN@ 10053e04     flags.obj
 0002:00007e14       ??_C@_0BB@BNPDAPGB@ECSTATE_MODIFIED@ 10053e14     flags.obj
 0002:00007e28       ??_C@_0O@GBBGHDFM@ECSTATE_SAVED@ 10053e28     flags.obj
 0002:00007e38       ??_C@_0P@BECIAJAM@ECSTATE_LOCKED@ 10053e38     flags.obj
 0002:00007e48       ??_C@_0P@DOBJCNIG@ECTYPE_CHANGED@ 10053e48     flags.obj
 0002:00007e58       ??_C@_0N@MDEFMEEA@ECTYPE_ADDED@ 10053e58     flags.obj
 0002:00007e68       ??_C@_0P@NMOJJPOB@ECTYPE_DELETED@ 10053e68     flags.obj
 0002:00007e78       ??_C@_08HHHKLJPB@PLT_PATH@ 10053e78     flags.obj
 0002:00007e84       ??_C@_08KBAMIIFB@PFM_GUID@ 10053e84     flags.obj
 0002:00007e90       ??_C@_0P@KKEMMPNI@PFM_MODULENAME@ 10053e90     flags.obj
 0002:00007ea0       ??_C@_09BOODOHKD@FFT_PANEL@ 10053ea0     flags.obj
 0002:00007eac       ??_C@_0N@GMEDAGNH@FFT_FINDFILE@ 10053eac     flags.obj
 0002:00007ebc       ??_C@_08KKCPIPGP@FFT_COPY@ 10053ebc     flags.obj
 0002:00007ec8       ??_C@_0L@EKPDMFDD@FFT_SELECT@ 10053ec8     flags.obj
 0002:00007ed4       ??_C@_0L@LGPEDLLD@FFT_CUSTOM@ 10053ed4     flags.obj
 0002:00007ee0       ??_C@_0M@OIOMMFOE@FST_UNKNOWN@ 10053ee0     flags.obj
 0002:00007eec       ??_C@_0L@GGGOEGKJ@FST_SUBKEY@ 10053eec     flags.obj
 0002:00007ef8       ??_C@_09LFEEAJIC@FST_QWORD@ 10053ef8     flags.obj
 0002:00007f04       ??_C@_0L@LPMPBKDL@FST_STRING@ 10053f04     flags.obj
 0002:00007f10       ??_C@_08EJJJCLIG@FST_DATA@ 10053f10     flags.obj
 0002:00007f1c       ??_C@_09OBBBBFPE@FSSF_ROOT@ 10053f1c     flags.obj
 0002:00007f28       ??_C@_0BB@HDKCPBIO@FSSF_HISTORY_CMD@ 10053f28     flags.obj
 0002:00007f3c       ??_C@_0BE@BLPOFODL@FSSF_HISTORY_FOLDER@ 10053f3c     flags.obj
 0002:00007f50       ??_C@_0BC@NJCJCCNH@FSSF_HISTORY_VIEW@ 10053f50     flags.obj
 0002:00007f64       ??_C@_0BC@CODELNPP@FSSF_HISTORY_EDIT@ 10053f64     flags.obj
 0002:00007f78       ??_C@_0BG@IFGEMJIF@FSSF_HISTORY_EXTERNAL@ 10053f78     flags.obj
 0002:00007f90       ??_C@_0BG@DGAKDKFK@FSSF_FOLDERSHORTCUT_0@ 10053f90     flags.obj
 0002:00007fa8       ??_C@_0BG@CPBBALBL@FSSF_FOLDERSHORTCUT_1@ 10053fa8     flags.obj
 0002:00007fc0       ??_C@_0BG@EDMFINI@FSSF_FOLDERSHORTCUT_2@ 10053fc0     flags.obj
 0002:00007fd8       ??_C@_0BG@BNCHGJJJ@FSSF_FOLDERSHORTCUT_3@ 10053fd8     flags.obj
 0002:00007ff0       ??_C@_0BG@FCGGPPFO@FSSF_FOLDERSHORTCUT_4@ 10053ff0     flags.obj
 0002:00008008       ??_C@_0BG@ELHNMOBP@FSSF_FOLDERSHORTCUT_5@ 10054008     flags.obj
 0002:00008020       ??_C@_0BG@GAFAJNNM@FSSF_FOLDERSHORTCUT_6@ 10054020     flags.obj
 0002:00008038       ??_C@_0BG@HJELKMJN@FSSF_FOLDERSHORTCUT_7@ 10054038     flags.obj
 0002:00008050       ??_C@_0BG@PONDLAFC@FSSF_FOLDERSHORTCUT_8@ 10054050     flags.obj
 0002:00008068       ??_C@_0BG@OHMIIBBD@FSSF_FOLDERSHORTCUT_9@ 10054068     flags.obj
 0002:00008080       ??_C@_0BD@PBIEGEHP@FSSF_CONFIRMATIONS@ 10054080     flags.obj
 0002:00008094       ??_C@_0M@PIGDMPJB@FSSF_SYSTEM@ 10054094     flags.obj
 0002:000080a0       ??_C@_0L@LBFNJGFB@FSSF_PANEL@ 100540a0     flags.obj
 0002:000080ac       ??_C@_0M@KJLIHDEL@FSSF_EDITOR@ 100540ac     flags.obj
 0002:000080b8       ??_C@_0M@KEMGKEOF@FSSF_SCREEN@ 100540b8     flags.obj
 0002:000080c4       ??_C@_0M@CBDJLJIE@FSSF_DIALOG@ 100540c4     flags.obj
 0002:000080d0       ??_C@_0P@OCDADNBF@FSSF_INTERFACE@ 100540d0     flags.obj
 0002:000080e0       ??_C@_0BB@GBBEBNKE@FSSF_PANELLAYOUT@ 100540e0     flags.obj
 0002:000080f4       ??_C@_0M@JCGHGLJF@PSL_ROAMING@ 100540f4     flags.obj
 0002:00008100       ??_C@_09EDBNDHCM@PSL_LOCAL@ 10054100     flags.obj
 0002:0000810c       ??_C@_07BPEFOPGM@FCT_ANY@  1005410c     flags.obj
 0002:00008114       ??_C@_0L@CDAEILNM@FCT_STREAM@ 10054114     flags.obj
 0002:00008120       ??_C@_0L@IADFDBJB@FCT_COLUMN@ 10054120     flags.obj
 0002:0000812c       ??_C@_0O@KJFMBLFE@LINK_HARDLINK@ 1005412c     flags.obj
 0002:0000813c       ??_C@_0O@OOAFIIDA@LINK_JUNCTION@ 1005413c     flags.obj
 0002:0000814c       ??_C@_0O@FIAPLKLH@LINK_VOLMOUNT@ 1005414c     flags.obj
 0002:0000815c       ??_C@_0BB@JDBEPJDK@LINK_SYMLINKFILE@ 1005415c     flags.obj
 0002:00008170       ??_C@_0BA@GFPIOFMG@LINK_SYMLINKDIR@ 10054170     flags.obj
 0002:00008180       ??_C@_0N@PJENIJFN@LINK_SYMLINK@ 10054180     flags.obj
 0002:00008190       ??_C@_08HNOHKPBK@CPM_FULL@ 10054190     flags.obj
 0002:0000819c       ??_C@_08LAEGFKJE@CPM_REAL@ 1005419c     flags.obj
 0002:000081a8       ??_C@_0L@NPJNPCJM@CPM_NATIVE@ 100541a8     flags.obj
 0002:000081b4       ??_C@_0L@NCFOENCC@VS_RELEASE@ 100541b4     flags.obj
 0002:000081c0       ??_C@_08BDGLHPMJ@VS_ALPHA@ 100541c0     flags.obj
 0002:000081cc       ??_C@_07OKFPMINB@VS_BETA@  100541cc     flags.obj
 0002:000081d4       ??_C@_05MMFLPJEB@VS_RC@    100541d4     flags.obj
 0002:000081dc       ??_C@_0L@IIIJLOAF@VS_SPECIAL@ 100541dc     flags.obj
 0002:000081e8       ??_C@_0L@EAMAICHL@VS_PRIVATE@ 100541e8     flags.obj
 0002:000081f4       ??_C@_0BC@OOKLINPG@OPEN_LEFTDISKMENU@ 100541f4     flags.obj
 0002:00008208       ??_C@_0BB@CEFDHHLF@OPEN_PLUGINSMENU@ 10054208     flags.obj
 0002:0000821c       ??_C@_0O@IEJHJCNB@OPEN_FINDLIST@ 1005421c     flags.obj
 0002:0000822c       ??_C@_0O@OGDCDPNG@OPEN_SHORTCUT@ 1005422c     flags.obj
 0002:0000823c       ??_C@_0BB@JHCCMIPF@OPEN_COMMANDLINE@ 1005423c     flags.obj
 0002:00008250       ??_C@_0M@DMJLHMGM@OPEN_EDITOR@ 10054250     flags.obj
 0002:0000825c       ??_C@_0M@MOBCONI@OPEN_VIEWER@ 1005425c     flags.obj
 0002:00008268       ??_C@_0P@LCDNLGDE@OPEN_FILEPANEL@ 10054268     flags.obj
 0002:00008278       ??_C@_0M@LEBKLGKD@OPEN_DIALOG@ 10054278     flags.obj
 0002:00008284       ??_C@_0N@CBHPGAKB@OPEN_ANALYSE@ 10054284     flags.obj
 0002:00008294       ??_C@_0BD@NFNGGFHI@OPEN_RIGHTDISKMENU@ 10054294     flags.obj
 0002:000082a8       ??_C@_0P@FOKOAMLC@OPEN_FROMMACRO@ 100542a8     flags.obj
 0002:000082b8       ??_C@_0O@NEDDJIHC@OPEN_LUAMACRO@ 100542b8     flags.obj
 0002:000082c8       ??_C@_0P@GBMLNMMI@MCT_MACROPARSE@ 100542c8     flags.obj
 0002:000082d8       ??_C@_0P@GNPFPCF@MCT_LOADMACROS@ 100542d8     flags.obj
 0002:000082e8       ??_C@_0P@HMDDACMI@MCT_ENUMMACROS@ 100542e8     flags.obj
 0002:000082f8       ??_C@_0BA@MOCJHMJK@MCT_WRITEMACROS@ 100542f8     flags.obj
 0002:00008308       ??_C@_0N@IGJGAHKE@MCT_GETMACRO@ 10054308     flags.obj
 0002:00008318       ??_C@_0BC@NFGGBILF@MCT_RECORDEDMACRO@ 10054318     flags.obj
 0002:0000832c       ??_C@_0N@OLCKOJMI@MCT_DELMACRO@ 1005432c     flags.obj
 0002:0000833c       ??_C@_0BC@NALHIHJ@MCT_RUNSTARTMACRO@ 1005433c     flags.obj
 0002:00008350       ??_C@_0P@HOMHAEFB@MCT_EXECSTRING@ 10054350     flags.obj
 0002:00008360       ??_C@_0O@CDBDPKIC@MCT_PANELSORT@ 10054360     flags.obj
 0002:00008370       ??_C@_0BH@PKKJIOHM@MCT_GETCUSTOMSORTMODES@ 10054370     flags.obj
 0002:00008388       ??_C@_0N@FOPIOCHO@MCT_ADDMACRO@ 10054388     flags.obj
 0002:00008398       ??_C@_0N@BHFJFHA@MCT_KEYMACRO@ 10054398     flags.obj
 0002:000083a8       ??_C@_0BB@LPDAOGB@MCT_CANPANELSORT@ 100543a8     flags.obj
 0002:000083bc       ??_C@_0BC@IOECJI@MPRT_NORMALFINISH@ 100543bc     flags.obj
 0002:000083d0       ??_C@_0BB@PMCBIGCA@MPRT_ERRORFINISH@ 100543d0     flags.obj
 0002:000083e4       ??_C@_0BA@BCBAEEOI@MPRT_ERRORPARSE@ 100543e4     flags.obj
 0002:000083f4       ??_C@_09EJDAADCN@MPRT_KEYS@ 100543f4     flags.obj
 0002:00008400       ??_C@_0L@GEHHCKFA@MPRT_PRINT@ 10054400     flags.obj
 0002:0000840c       ??_C@_0BA@OBIDLEIM@MPRT_PLUGINCALL@ 1005440c     flags.obj
 0002:0000841c       ??_C@_0BA@EJFFOAMM@MPRT_PLUGINMENU@ 1005441c     flags.obj
 0002:0000842c       ??_C@_0BC@LEDOPMKI@MPRT_PLUGINCONFIG@ 1005442c     flags.obj
 0002:00008440       ??_C@_0BD@HHINMPPI@MPRT_PLUGINCOMMAND@ 10054440     flags.obj
 0002:00008454       ??_C@_0O@IEMNLPAB@MPRT_USERMENU@ 10054454     flags.obj
 0002:00008464       ??_C@_0BA@GEAFHJNF@MPRT_HASNOMACRO@ 10054464     flags.obj
 0002:00008474       ??_C@_0BC@PNCKAHJO@FE_CHANGEVIEWMODE@ 10054474     flags.obj
 0002:00008488       ??_C@_09DENIDBMJ@FE_REDRAW@ 10054488     flags.obj
 0002:00008494       ??_C@_07CLNPDBLG@FE_IDLE@  10054494     flags.obj
 0002:0000849c       ??_C@_08DENCGKED@FE_CLOSE@ 1005449c     flags.obj
 0002:000084a8       ??_C@_08MOMCCKPB@FE_BREAK@ 100544a8     flags.obj
 0002:000084b4       ??_C@_0L@LELAIPLL@FE_COMMAND@ 100544b4     flags.obj
 0002:000084c0       ??_C@_0M@FIECADDF@FE_GOTFOCUS@ 100544c0     flags.obj
 0002:000084cc       ??_C@_0N@DGHFKMFL@FE_KILLFOCUS@ 100544cc     flags.obj
 0002:000084dc       ??_C@_0BE@PONEECEM@FE_CHANGESORTPARAMS@ 100544dc     flags.obj
 0002:000084f0       ??_C@_0M@HNDHDHHO@FCF_FG_4BIT@ 100544f0     flags.obj
 0002:000084fc       ??_C@_0M@PJHNDJIE@FCF_BG_4BIT@ 100544fc     flags.obj
 0002:00008508       ??_C@_0N@HMKJBHOA@FCF_4BITMASK@ 10054508     flags.obj
 0002:00008518       ??_C@_0BC@HCOAIAEK@FCF_INHERIT_STYLE@ 10054518     flags.obj
 0002:0000852c       ??_C@_0BB@PJFLJJLD@FCF_RAWATTR_MASK@ 1005452c     flags.obj
 0002:00008540       ??_C@_0M@LFMGCKHG@FCF_FG_BOLD@ 10054540     flags.obj
 0002:0000854c       ??_C@_0O@FAPDECBF@FCF_FG_ITALIC@ 1005454c     flags.obj
 0002:0000855c       ??_C@_0BB@NPEFGEGA@FCF_FG_UNDERLINE@ 1005455c     flags.obj
 0002:00008570       ??_C@_0BC@KABNHAEN@FCF_FG_UNDERLINE2@ 10054570     flags.obj
 0002:00008584       ??_C@_0BA@DJMNLMK@FCF_FG_OVERLINE@ 10054584     flags.obj
 0002:00008594       ??_C@_0BB@NJMJIPGP@FCF_FG_STRIKEOUT@ 10054594     flags.obj
 0002:000085a8       ??_C@_0N@HJOMADOA@FCF_FG_FAINT@ 100545a8     flags.obj
 0002:000085b8       ??_C@_0N@NHLHILNJ@FCF_FG_BLINK@ 100545b8     flags.obj
 0002:000085c8       ??_C@_0O@LGBGBIGB@FCF_STYLEMASK@ 100545c8     flags.obj
 0002:000085d8       ??_C@_08BKNBBLHK@FCF_NONE@ 100545d8     flags.obj
 0002:000085e4       ??_C@_08FKIDFHCM@CDF_NONE@ 100545e4     flags.obj
 0002:000085f0       ??_C@_0N@ELMEMNDH@FMSG_WARNING@ 100545f0     flags.obj
 0002:00008600       ??_C@_0P@HHIGLJAP@FMSG_ERRORTYPE@ 10054600     flags.obj
 0002:00008610       ??_C@_0BE@FHOOILPH@FMSG_KEEPBACKGROUND@ 10054610     flags.obj
 0002:00008624       ??_C@_0P@KBEMNNEP@FMSG_LEFTALIGN@ 10054624     flags.obj
 0002:00008634       ??_C@_0O@FOIOKDHJ@FMSG_ALLINONE@ 10054634     flags.obj
 0002:00008644       ??_C@_0L@BGALGPOK@FMSG_MB_OK@ 10054644     flags.obj
 0002:00008650       ??_C@_0BB@JGAPGIEP@FMSG_MB_OKCANCEL@ 10054650     flags.obj
 0002:00008664       ??_C@_0BJ@BKJADAHA@FMSG_MB_ABORTRETRYIGNORE@ 10054664     flags.obj
 0002:00008680       ??_C@_0O@GPCAPHCL@FMSG_MB_YESNO@ 10054680     flags.obj
 0002:00008690       ??_C@_0BE@IBNOLCGP@FMSG_MB_YESNOCANCEL@ 10054690     flags.obj
 0002:000086a4       ??_C@_0BE@OCLAIENB@FMSG_MB_RETRYCANCEL@ 100546a4     flags.obj
 0002:000086b8       ??_C@_09NEGPLEAH@FMSG_NONE@ 100546b8     flags.obj
 0002:000086c4       ??_C@_0N@DHJCDIKM@DIF_BOXCOLOR@ 100546c4     flags.obj
 0002:000086d4       ??_C@_09IAEPIICA@DIF_GROUP@ 100546d4     flags.obj
 0002:000086e0       ??_C@_0N@GCKJNBCM@DIF_LEFTTEXT@ 100546e0     flags.obj
 0002:000086f0       ??_C@_0P@BGPBEDHH@DIF_MOVESELECT@ 100546f0     flags.obj
 0002:00008700       ??_C@_0BC@PDKFKKEI@DIF_SHOWAMPERSAND@ 10054700     flags.obj
 0002:00008714       ??_C@_0BA@BLCOKAAO@DIF_CENTERGROUP@ 10054714     flags.obj
 0002:00008724       ??_C@_0P@MKFBJPOB@DIF_NOBRACKETS@ 10054724     flags.obj
 0002:00008734       ??_C@_0BF@JBCDBJCL@DIF_MANUALADDHISTORY@ 10054734     flags.obj
 0002:0000874c       ??_C@_0O@JKNMBNLA@DIF_SEPARATOR@ 1005474c     flags.obj
 0002:0000875c       ??_C@_0P@CGILDLOA@DIF_SEPARATOR2@ 1005475c     flags.obj
 0002:0000876c       ??_C@_0L@NBPFNGLB@DIF_EDITOR@ 1005476c     flags.obj
 0002:00008778       ??_C@_0BE@PFICAGJF@DIF_LISTNOAMPERSAND@ 10054778     flags.obj
 0002:0000878c       ??_C@_0O@FFJNBMAD@DIF_LISTNOBOX@ 1005478c     flags.obj
 0002:0000879c       ??_C@_0M@IPFBMFDN@DIF_HISTORY@ 1005479c     flags.obj
 0002:000087a8       ??_C@_0P@EGFAEEDC@DIF_BTNNOCLOSE@ 100547a8     flags.obj
 0002:000087b8       ??_C@_0P@KOJCCCGB@DIF_CENTERTEXT@ 100547b8     flags.obj
 0002:000087c8       ??_C@_0BC@ODEMBOPK@DIF_SEPARATORUSER@ 100547c8     flags.obj
 0002:000087dc       ??_C@_0O@IKJBMPOF@DIF_SETSHIELD@ 100547dc     flags.obj
 0002:000087ec       ??_C@_0P@EEJEDBLH@DIF_EDITEXPAND@ 100547ec     flags.obj
 0002:000087fc       ??_C@_0BB@EIMEKEFP@DIF_DROPDOWNLIST@ 100547fc     flags.obj
 0002:00008810       ??_C@_0BD@MNGIOLFF@DIF_USELASTHISTORY@ 10054810     flags.obj
 0002:00008824       ??_C@_0N@MOCGNIKC@DIF_MASKEDIT@ 10054824     flags.obj
 0002:00008834       ??_C@_0BD@LPDHCLJI@DIF_LISTTRACKMOUSE@ 10054834     flags.obj
 0002:00008848       ??_C@_0BK@LEFIBDOA@DIF_LISTTRACKMOUSEINFOCUS@ 10054848     flags.obj
 0002:00008864       ??_C@_0BC@JNLDMGBD@DIF_SELECTONENTRY@ 10054864     flags.obj
 0002:00008878       ??_C@_0L@KKNJDNBK@DIF_3STATE@ 10054878     flags.obj
 0002:00008884       ??_C@_0N@GBGHICKO@DIF_EDITPATH@ 10054884     flags.obj
 0002:00008894       ??_C@_0BB@NPNALIGO@DIF_LISTWRAPMODE@ 10054894     flags.obj
 0002:000088a8       ??_C@_0BD@MFOKKGGF@DIF_NOAUTOCOMPLETE@ 100548a8     flags.obj
 0002:000088bc       ??_C@_0BG@MONEJILE@DIF_LISTAUTOHIGHLIGHT@ 100548bc     flags.obj
 0002:000088d4       ??_C@_0BA@JNOKLHOL@DIF_LISTNOCLOSE@ 100548d4     flags.obj
 0002:000088e4       ??_C@_0BB@GMKDKOOP@DIF_EDITPATHEXEC@ 100548e4     flags.obj
 0002:000088f8       ??_C@_0L@EPNFOPAK@DIF_HIDDEN@ 100548f8     flags.obj
 0002:00008904       ??_C@_0N@KOGKCAKJ@DIF_READONLY@ 10054904     flags.obj
 0002:00008914       ??_C@_0M@NLLDINIM@DIF_NOFOCUS@ 10054914     flags.obj
 0002:00008920       ??_C@_0M@HCFLMDHK@DIF_DISABLE@ 10054920     flags.obj
 0002:0000892c       ??_C@_0BC@CHAAKEJO@DIF_DEFAULTBUTTON@ 1005492c     flags.obj
 0002:00008940       ??_C@_09LCJIOEMN@DIF_FOCUS@ 10054940     flags.obj
 0002:0000894c       ??_C@_0O@KJADCBBN@DIF_RIGHTTEXT@ 1005494c     flags.obj
 0002:0000895c       ??_C@_0N@LAEOODAD@DIF_WORDWRAP@ 1005495c     flags.obj
 0002:0000896c       ??_C@_08KFOHCPDE@DIF_NONE@ 1005496c     flags.obj
 0002:00008978       ??_C@_0N@EDHAFIIL@LIF_SELECTED@ 10054978     flags.obj
 0002:00008988       ??_C@_0M@BMGIEAIL@LIF_CHECKED@ 10054988     flags.obj
 0002:00008994       ??_C@_0O@KJIFADIG@LIF_SEPARATOR@ 10054994     flags.obj
 0002:000089a4       ??_C@_0M@HEFHLFIE@LIF_DISABLE@ 100549a4     flags.obj
 0002:000089b0       ??_C@_0L@PKDDGEEG@LIF_GRAYED@ 100549b0     flags.obj
 0002:000089bc       ??_C@_0L@PFBGAOEP@LIF_HIDDEN@ 100549bc     flags.obj
 0002:000089c8       ??_C@_0BD@HEPCOIEH@LIF_DELETEUSERDATA@ 100549c8     flags.obj
 0002:000089dc       ??_C@_08BODPINCM@LIF_NONE@ 100549dc     flags.obj
 0002:000089e8       ??_C@_0BC@BGAENNBJ@LIFIND_EXACTMATCH@ 100549e8     flags.obj
 0002:000089fc       ??_C@_0M@FPOGKIGO@LIFIND_NONE@ 100549fc     flags.obj
 0002:00008a08       ??_C@_0BA@OOIEKCFB@LINFO_SHOWNOBOX@ 10054a08     flags.obj
 0002:00008a18       ??_C@_0BE@DECCEGNO@LINFO_AUTOHIGHLIGHT@ 10054a18     flags.obj
 0002:00008a2c       ??_C@_0BH@BADLEILJ@LINFO_REVERSEHIGHLIGHT@ 10054a2c     flags.obj
 0002:00008a44       ??_C@_0P@KLBMHNCG@LINFO_WRAPMODE@ 10054a44     flags.obj
 0002:00008a54       ??_C@_0BE@OHJCOKAE@LINFO_SHOWAMPERSAND@ 10054a54     flags.obj
 0002:00008a68       ??_C@_0L@EPACPANF@LINFO_NONE@ 10054a68     flags.obj
 0002:00008a74       ??_C@_0N@OLGDMHKL@FDLG_WARNING@ 10054a74     flags.obj
 0002:00008a84       ??_C@_0BB@DKMEBDJJ@FDLG_SMALLDIALOG@ 10054a84     flags.obj
 0002:00008a98       ??_C@_0BC@ONGLDAJN@FDLG_NODRAWSHADOW@ 10054a98     flags.obj
 0002:00008aac       ??_C@_0BB@NPLEEAKK@FDLG_NODRAWPANEL@ 10054aac     flags.obj
 0002:00008ac0       ??_C@_0BG@GHNOOENB@FDLG_KEEPCONSOLETITLE@ 10054ac0     flags.obj
 0002:00008ad8       ??_C@_0O@MKFABCNE@FDLG_NONMODAL@ 10054ad8     flags.obj
 0002:00008ae8       ??_C@_09NNFHCBNL@FDLG_NONE@ 10054ae8     flags.obj
 0002:00008af4       ??_C@_0N@JOOGIBAO@MIF_SELECTED@ 10054af4     flags.obj
 0002:00008b04       ??_C@_0M@IHMNAMOE@MIF_CHECKED@ 10054b04     flags.obj
 0002:00008b10       ??_C@_0O@DEIKOCPA@MIF_SEPARATOR@ 10054b10     flags.obj
 0002:00008b20       ??_C@_0M@OPPCPJOL@MIF_DISABLE@ 10054b20     flags.obj
 0002:00008b2c       ??_C@_0L@DLLNLLIG@MIF_GRAYED@ 10054b2c     flags.obj
 0002:00008b38       ??_C@_0L@DEJINBIP@MIF_HIDDEN@ 10054b38     flags.obj
 0002:00008b44       ??_C@_08JEEJJGP@MIF_NONE@  10054b44     flags.obj
 0002:00008b50       ??_C@_0BE@FALMPPJK@FMENU_SHOWAMPERSAND@ 10054b50     flags.obj
 0002:00008b64       ??_C@_0P@HICDNKDJ@FMENU_WRAPMODE@ 10054b64     flags.obj
 0002:00008b74       ??_C@_0BE@IDAMFDEA@FMENU_AUTOHIGHLIGHT@ 10054b74     flags.obj
 0002:00008b88       ??_C@_0BL@OKAIKPMN@FMENU_REVERSEAUTOHIGHLIGHT@ 10054b88     flags.obj
 0002:00008ba4       ??_C@_0BJ@FCEONOJC@FMENU_CHANGECONSOLETITLE@ 10054ba4     flags.obj
 0002:00008bc0       ??_C@_0BA@GDFPJAAD@FMENU_SHOWNOBOX@ 10054bc0     flags.obj
 0002:00008bd0       ??_C@_0BD@PMEPMEOJ@FMENU_SHOWSHORTBOX@ 10054bd0     flags.obj
 0002:00008be4       ??_C@_0BE@PDNJFEDO@FMENU_SHOWSINGLEBOX@ 10054be4     flags.obj
 0002:00008bf8       ??_C@_0BD@JBJJGCBE@FMENU_NODRAWSHADOW@ 10054bf8     flags.obj
 0002:00008c0c       ??_C@_0L@DGFIEOMD@FMENU_NONE@ 10054c0c     flags.obj
 0002:00008c18       ??_C@_0O@JEAJLDHC@PPIF_SELECTED@ 10054c18     flags.obj
 0002:00008c28       ??_C@_0BC@LPBDBIOM@PPIF_PROCESSDESCR@ 10054c28     flags.obj
 0002:00008c3c       ??_C@_09OIFMMGNJ@PPIF_NONE@ 10054c3c     flags.obj
 0002:00008c48       ??_C@_0BC@BONLDOOD@PFLAGS_SHOWHIDDEN@ 10054c48     flags.obj
 0002:00008c5c       ??_C@_0BB@BCAJEJEH@PFLAGS_HIGHLIGHT@ 10054c5c     flags.obj
 0002:00008c70       ??_C@_0BI@BFAFODJ@PFLAGS_REVERSESORTORDER@ 10054c70     flags.obj
 0002:00008c88       ??_C@_0BF@KJNCJPKN@PFLAGS_USESORTGROUPS@ 10054c88     flags.obj
 0002:00008ca0       ??_C@_0BF@LBBAIOCD@PFLAGS_SELECTEDFIRST@ 10054ca0     flags.obj
 0002:00008cb8       ??_C@_0BB@KDANIJNM@PFLAGS_REALNAMES@ 10054cb8     flags.obj
 0002:00008ccc       ??_C@_0BB@ILEHDKFJ@PFLAGS_PANELLEFT@ 10054ccc     flags.obj
 0002:00008ce0       ??_C@_0BI@EHHAJLOH@PFLAGS_DIRECTORIESFIRST@ 10054ce0     flags.obj
 0002:00008cf8       ??_C@_0BA@KJEPHDOM@PFLAGS_USECRC32@ 10054cf8     flags.obj
 0002:00008d08       ??_C@_0O@DBPJGING@PFLAGS_PLUGIN@ 10054d08     flags.obj
 0002:00008d18       ??_C@_0P@MLDEBNPK@PFLAGS_VISIBLE@ 10054d18     flags.obj
 0002:00008d28       ??_C@_0N@EOFAELOJ@PFLAGS_FOCUS@ 10054d28     flags.obj
 0002:00008d38       ??_C@_0BI@EOCCAHFA@PFLAGS_ALTERNATIVENAMES@ 10054d38     flags.obj
 0002:00008d50       ??_C@_0BA@GHMDCHHI@PFLAGS_SHORTCUT@ 10054d50     flags.obj
 0002:00008d60       ??_C@_0M@NEMAHHGP@PFLAGS_NONE@ 10054d60     flags.obj
 0002:00008d6c       ??_C@_0M@IDNADAFL@VF_NONMODAL@ 10054d6c     flags.obj
 0002:00008d78       ??_C@_0BB@OCDDPIKL@VF_DELETEONCLOSE@ 10054d78     flags.obj
 0002:00008d8c       ??_C@_0N@LDHALKKM@VF_ENABLE_F6@ 10054d8c     flags.obj
 0002:00008d9c       ??_C@_0BC@DLGKMECC@VF_DISABLEHISTORY@ 10054d9c     flags.obj
 0002:00008db0       ??_C@_0BD@DHJCMLFI@VF_IMMEDIATERETURN@ 10054db0     flags.obj
 0002:00008dc4       ??_C@_0BJ@OGNFHEJG@VF_DELETEONLYFILEONCLOSE@ 10054dc4     flags.obj
 0002:00008de0       ??_C@_07CJJFHP@VF_NONE@    10054de0     flags.obj
 0002:00008de8       ??_C@_0M@PIFGAPFH@EF_NONMODAL@ 10054de8     flags.obj
 0002:00008df4       ??_C@_0N@DBHFPBEO@EF_CREATENEW@ 10054df4     flags.obj
 0002:00008e04       ??_C@_0N@LKLNHALI@EF_ENABLE_F6@ 10054e04     flags.obj
 0002:00008e14       ??_C@_0BC@PPEPEFFI@EF_DISABLEHISTORY@ 10054e14     flags.obj
 0002:00008e28       ??_C@_0BB@KGPIDKFC@EF_DELETEONCLOSE@ 10054e28     flags.obj
 0002:00008e3c       ??_C@_0BD@IHIGHGPL@EF_IMMEDIATERETURN@ 10054e3c     flags.obj
 0002:00008e50       ??_C@_0BJ@ILCPOFKL@EF_DELETEONLYFILEONCLOSE@ 10054e50     flags.obj
 0002:00008e6c       ??_C@_09IJMPFPLB@EF_LOCKED@ 10054e6c     flags.obj
 0002:00008e78       ??_C@_0BC@GFHJGKD@EF_DISABLESAVEPOS@ 10054e78     flags.obj
 0002:00008e8c       ??_C@_0BB@NILAHAFO@EF_OPENMODE_MASK@ 10054e8c     flags.obj
 0002:00008ea0       ??_C@_0BC@GAIDEJIA@EF_OPENMODE_QUERY@ 10054ea0     flags.obj
 0002:00008eb4       ??_C@_0BG@BFKJJBAG@EF_OPENMODE_NEWIFOPEN@ 10054eb4     flags.obj
 0002:00008ecc       ??_C@_0BI@KGOKGPEI@EF_OPENMODE_USEEXISTING@ 10054ecc     flags.obj
 0002:00008ee4       ??_C@_0BI@EJBKKDJ@EF_OPENMODE_BREAKIFOPEN@ 10054ee4     flags.obj
 0002:00008efc       ??_C@_0BJ@MOLGCBMH@EF_OPENMODE_RELOADIFOPEN@ 10054efc     flags.obj
 0002:00008f18       ??_C@_07MBPCONNA@EN_NONE@  10054f18     flags.obj
 0002:00008f20       ??_C@_0BC@HHNGCBAM@FHELP_NOSHOWERROR@ 10054f20     flags.obj
 0002:00008f34       ??_C@_0P@GANNLHEJ@FHELP_SELFHELP@ 10054f34     flags.obj
 0002:00008f44       ??_C@_0O@FLGGLFLC@FHELP_FARHELP@ 10054f44     flags.obj
 0002:00008f54       ??_C@_0BB@KNKDPNI@FHELP_CUSTOMFILE@ 10054f54     flags.obj
 0002:00008f68       ??_C@_0BB@IHFFPJJA@FHELP_CUSTOMPATH@ 10054f68     flags.obj
 0002:00008f7c       ??_C@_0L@OOIMFPBD@FHELP_GUID@ 10054f7c     flags.obj
 0002:00008f88       ??_C@_0BC@PNPOIHMG@FHELP_USECONTENTS@ 10054f88     flags.obj
 0002:00008f9c       ??_C@_0L@MAGMKNFN@FHELP_NONE@ 10054f9c     flags.obj
 0002:00008fa8       ??_C@_0BE@GEGKIINM@KMFLAGS_SILENTCHECK@ 10054fa8     flags.obj
 0002:00008fbc       ??_C@_0BM@BBOPLPKC@KMFLAGS_NOSENDKEYSTOPLUGINS@ 10054fbc     flags.obj
 0002:00008fd8       ??_C@_0BF@PHHPAAOK@KMFLAGS_ENABLEOUTPUT@ 10054fd8     flags.obj
 0002:00008ff0       ??_C@_0BB@NCECNBPK@KMFLAGS_LANGMASK@ 10054ff0     flags.obj
 0002:00009004       ??_C@_0M@HFBACHCP@KMFLAGS_LUA@ 10055004     flags.obj
 0002:00009010       ??_C@_0BD@JHNPMIGP@KMFLAGS_MOONSCRIPT@ 10055010     flags.obj
 0002:00009024       ??_C@_0N@GIJCDFJI@KMFLAGS_NONE@ 10055024     flags.obj
 0002:00009034       ??_C@_0O@GKOLBMFK@AKMFLAGS_NONE@ 10055034     flags.obj
 0002:00009044       ??_C@_0P@LMBMJIMF@FSETCLR_REDRAW@ 10055044     flags.obj
 0002:00009054       ??_C@_0N@LCOHPDHN@FSETCLR_NONE@ 10055054     flags.obj
 0002:00009064       ??_C@_0N@MLMCEKPH@WIF_MODIFIED@ 10055064     flags.obj
 0002:00009074       ??_C@_0M@ICPAPCOF@WIF_CURRENT@ 10055074     flags.obj
 0002:00009080       ??_C@_09FPGEBDGO@WIF_MODAL@ 10055080     flags.obj
 0002:0000908c       ??_C@_08DAKKFBIA@WIF_NONE@ 1005508c     flags.obj
 0002:00009098       ??_C@_0BG@JMJAOELH@VOPT_SAVEFILEPOSITION@ 10055098     flags.obj
 0002:000090b0       ??_C@_0BI@NCAHLEBN@VOPT_AUTODETECTCODEPAGE@ 100550b0     flags.obj
 0002:000090c8       ??_C@_0BC@FGLBHLDI@VOPT_SHOWTITLEBAR@ 100550c8     flags.obj
 0002:000090dc       ??_C@_0BA@GAIDGLME@VOPT_SHOWKEYBAR@ 100550dc     flags.obj
 0002:000090ec       ??_C@_0BD@LEEGOJKA@VOPT_SHOWSCROLLBAR@ 100550ec     flags.obj
 0002:00009100       ??_C@_0P@NEIKPMJJ@VOPT_QUICKVIEW@ 10055100     flags.obj
 0002:00009110       ??_C@_09FIOJMNJ@VOPT_NONE@ 10055110     flags.obj
 0002:0000911c       ??_C@_0N@ILNDJNNO@VSMFL_REDRAW@ 1005511c     flags.obj
 0002:0000912c       ??_C@_0L@DLLCFLOD@VSMFL_NONE@ 1005512c     flags.obj
 0002:00009138       ??_C@_0N@GHEHKHJN@VSP_NOREDRAW@ 10055138     flags.obj
 0002:00009148       ??_C@_0M@LHNGMHFO@VSP_PERCENT@ 10055148     flags.obj
 0002:00009154       ??_C@_0N@JGGGCNIP@VSP_RELATIVE@ 10055154     flags.obj
 0002:00009164       ??_C@_0BA@JKDMJLJG@VSP_NORETNEWPOS@ 10055164     flags.obj
 0002:00009174       ??_C@_08MOKEMBNE@VSP_NONE@ 10055174     flags.obj
 0002:00009180       ??_C@_08FAPBJAKB@VMF_WRAP@ 10055180     flags.obj
 0002:0000918c       ??_C@_0N@GHBDMLON@VMF_WORDWRAP@ 1005518c     flags.obj
 0002:0000919c       ??_C@_08KDJLELDJ@VMF_NONE@ 1005519c     flags.obj
 0002:000091a8       ??_C@_0BB@EDGIEBDF@ECF_TABMARKFIRST@ 100551a8     flags.obj
 0002:000091bc       ??_C@_0BD@DKGCCJNG@ECF_TABMARKCURRENT@ 100551bc     flags.obj
 0002:000091d0       ??_C@_0P@BAFEMBAJ@ECF_AUTODELETE@ 100551d0     flags.obj
 0002:000091e0       ??_C@_08CDFMCHLP@ECF_NONE@ 100551e0     flags.obj
 0002:000091ec       ??_C@_0BA@KNNLMGCA@FIB_ENABLEEMPTY@ 100551ec     flags.obj
 0002:000091fc       ??_C@_0N@DLDJCGJI@FIB_PASSWORD@ 100551fc     flags.obj
 0002:0000920c       ??_C@_0O@DOHEGELC@FIB_EXPANDENV@ 1005520c     flags.obj
 0002:0000921c       ??_C@_0BF@CEMIHIOK@FIB_NOUSELASTHISTORY@ 1005521c     flags.obj
 0002:00009234       ??_C@_0M@KJOJJDIM@FIB_BUTTONS@ 10055234     flags.obj
 0002:00009240       ??_C@_0BA@COBBDHNL@FIB_NOAMPERSAND@ 10055240     flags.obj
 0002:00009250       ??_C@_0N@LBOCEEGH@FIB_EDITPATH@ 10055250     flags.obj
 0002:00009260       ??_C@_0BB@DCODFLEL@FIB_EDITPATHEXEC@ 10055260     flags.obj
 0002:00009274       ??_C@_08HPFOCDKB@FIB_NONE@ 10055274     flags.obj
 0002:00009280       ??_C@_0L@NMBLFMBN@FPF_LOADED@ 10055280     flags.obj
 0002:0000928c       ??_C@_08GKECKCCJ@FPF_ANSI@ 1005528c     flags.obj
 0002:00009298       ??_C@_08OIOFCNLC@FPF_NONE@ 10055298     flags.obj
 0002:000092a4       ??_C@_0L@HODJIPGA@PN_CMPNAME@ 100552a4     flags.obj
 0002:000092b0       ??_C@_0P@KDEENAHJ@PN_CMPNAMELIST@ 100552b0     flags.obj
 0002:000092c0       ??_C@_0BA@BJCCEIOI@PN_GENERATENAME@ 100552c0     flags.obj
 0002:000092d0       ??_C@_0N@FEGPCCPJ@PN_CHECKMASK@ 100552d0     flags.obj
 0002:000092e0       ??_C@_0M@NOOLKEBH@PN_SKIPPATH@ 100552e0     flags.obj
 0002:000092ec       ??_C@_0BE@OPDBOAAE@PN_SHOWERRORMESSAGE@ 100552ec     flags.obj
 0002:00009300       ??_C@_07PFKJNCJP@PN_NONE@  10055300     flags.obj
 0002:00009308       ??_C@_0BG@GOMJDMCK@XLAT_SWITCHKEYBLAYOUT@ 10055308     flags.obj
 0002:00009320       ??_C@_0BE@KOIJDNLA@XLAT_SWITCHKEYBBEEP@ 10055320     flags.obj
 0002:00009334       ??_C@_0BH@KBFAFPNA@XLAT_USEKEYBLAYOUTNAME@ 10055334     flags.obj
 0002:0000934c       ??_C@_0BH@IANKLOAC@XLAT_CONVERTALLCMDLINE@ 1005534c     flags.obj
 0002:00009364       ??_C@_09JCNLKBBK@XLAT_NONE@ 10055364     flags.obj
 0002:00009370       ??_C@_0N@PJEDCNNJ@FRS_RETUPDIR@ 10055370     flags.obj
 0002:00009380       ??_C@_09GHEPLOHO@FRS_RECUR@ 10055380     flags.obj
 0002:0000938c       ??_C@_0BA@JCPHOEAE@FRS_SCANSYMLINK@ 1005538c     flags.obj
 0002:0000939c       ??_C@_08JPCGJJKG@FRS_NONE@ 1005539c     flags.obj
 0002:000093a8       ??_C@_0P@LJPBHEIE@MLF_SHOWERRMSG@ 100553a8     flags.obj
 0002:000093b8       ??_C@_0BF@LMAGFLHF@MLF_DONOTUPDATEPANEL@ 100553b8     flags.obj
 0002:000093d0       ??_C@_0P@EPFBLPAE@MLF_HOLDTARGET@ 100553d0     flags.obj
 0002:000093e0       ??_C@_08EBKEJHAL@MLF_NONE@ 100553e0     flags.obj
 0002:000093ec       ??_C@_0M@JDMKDBDH@FFFS_COMMAS@ 100553ec     flags.obj
 0002:000093f8       ??_C@_0P@JPMLNBKL@FFFS_FLOATSIZE@ 100553f8     flags.obj
 0002:00009408       ??_C@_0BE@NPKCCEJ@FFFS_SHOWBYTESINDEX@ 10055408     flags.obj
 0002:0000941c       ??_C@_0O@FPIOAIMC@FFFS_ECONOMIC@ 1005541c     flags.obj
 0002:0000942c       ??_C@_0O@HFIGPFIH@FFFS_THOUSAND@ 1005542c     flags.obj
 0002:0000943c       ??_C@_0BC@LLLANJJO@FFFS_MINSIZEINDEX@ 1005543c     flags.obj
 0002:00009450       ??_C@_0BH@PEGBPJKE@FFFS_MINSIZEINDEX_MASK@ 10055450     flags.obj
 0002:00009468       ??_C@_09PBPAKNEI@FFFS_NONE@ 10055468     flags.obj
 0002:00009474       ??_C@_0L@NHEJGKCF@PF_PRELOAD@ 10055474     flags.obj
 0002:00009480       ??_C@_0BB@GCINAIGN@PF_DISABLEPANELS@ 10055480     flags.obj
 0002:00009494       ??_C@_09OENCMPGE@PF_EDITOR@ 10055494     flags.obj
 0002:000094a0       ??_C@_09NEKIJNNA@PF_VIEWER@ 100554a0     flags.obj
 0002:000094ac       ??_C@_0P@MBLBBCNK@PF_FULLCMDLINE@ 100554ac     flags.obj
 0002:000094bc       ??_C@_09GMFDAFKL@PF_DIALOG@ 100554bc     flags.obj
 0002:000094c8       ??_C@_07MGEGJMPI@PF_NONE@  100554c8     flags.obj
 0002:000094d0       ??_C@_0BD@EGELEIIG@IPLFLAGS_SEPARATOR@ 100554d0     flags.obj
 0002:000094e4       ??_C@_0O@JBNJFHHK@IPLFLAGS_NONE@ 100554e4     flags.obj
 0002:000094f4       ??_C@_0BD@KGHJOBGM@PMFLAGS_FULLSCREEN@ 100554f4     flags.obj
 0002:00009508       ??_C@_0BH@GDAAKEMH@PMFLAGS_DETAILEDSTATUS@ 10055508     flags.obj
 0002:00009520       ??_C@_0BI@BMHIBDMH@PMFLAGS_ALIGNEXTENSIONS@ 10055520     flags.obj
 0002:00009538       ??_C@_0BH@KOFCBJBO@PMFLAGS_CASECONVERSION@ 10055538     flags.obj
 0002:00009550       ??_C@_0N@DLFMCMOB@PMFLAGS_NONE@ 10055550     flags.obj
 0002:00009560       ??_C@_0BD@PBMGDJEM@OPIF_DISABLEFILTER@ 10055560     flags.obj
 0002:00009574       ??_C@_0BH@FHBKALPD@OPIF_DISABLESORTGROUPS@ 10055574     flags.obj
 0002:0000958c       ??_C@_0BJ@NGLIANCL@OPIF_DISABLEHIGHLIGHTING@ 1005558c     flags.obj
 0002:000095a8       ??_C@_0N@JANKJMLP@OPIF_ADDDOTS@ 100555a8     flags.obj
 0002:000095b8       ??_C@_0BC@HOFHNJIG@OPIF_RAWSELECTION@ 100555b8     flags.obj
 0002:000095cc       ??_C@_0P@OFEDJCO@OPIF_REALNAMES@ 100555cc     flags.obj
 0002:000095dc       ??_C@_0BD@FPGMNAPD@OPIF_SHOWNAMESONLY@ 100555dc     flags.obj
 0002:000095f0       ??_C@_0BJ@NMIFAPJD@OPIF_SHOWRIGHTALIGNNAMES@ 100555f0     flags.obj
 0002:0000960c       ??_C@_0BG@HGPMKHIE@OPIF_SHOWPRESERVECASE@ 1005560c     flags.obj
 0002:00009624       ??_C@_0BE@GJEJHNKJ@OPIF_COMPAREFATTIME@ 10055624     flags.obj
 0002:00009638       ??_C@_0BB@PELHBPAM@OPIF_EXTERNALGET@ 10055638     flags.obj
 0002:0000964c       ??_C@_0BB@CFFPNDFK@OPIF_EXTERNALPUT@ 1005564c     flags.obj
 0002:00009660       ??_C@_0BE@LKEMICNM@OPIF_EXTERNALDELETE@ 10055660     flags.obj
 0002:00009674       ??_C@_0BD@JIMJPFEP@OPIF_EXTERNALMKDIR@ 10055674     flags.obj
 0002:00009688       ??_C@_0BJ@CALDMPLF@OPIF_USEATTRHIGHLIGHTING@ 10055688     flags.obj
 0002:000096a4       ??_C@_0O@JHHHMHIG@OPIF_USECRC32@ 100556a4     flags.obj
 0002:000096b4       ??_C@_0BB@PFDFAFHG@OPIF_USEFREESIZE@ 100556b4     flags.obj
 0002:000096c8       ??_C@_0O@FJPLJDBC@OPIF_SHORTCUT@ 100556c8     flags.obj
 0002:000096d8       ??_C@_09DOPJBMLM@OPIF_NONE@ 100556d8     flags.obj
 0002:000096e4       ??_C@_0L@GEHHKNBL@OPM_SILENT@ 100556e4     flags.obj
 0002:000096f0       ??_C@_08EKEBOKEP@OPM_FIND@ 100556f0     flags.obj
 0002:000096fc       ??_C@_08EHBLNDLO@OPM_VIEW@ 100556fc     flags.obj
 0002:00009708       ??_C@_08LAAGEMJG@OPM_EDIT@ 10055708     flags.obj
 0002:00009714       ??_C@_0N@NDGKAFDM@OPM_TOPLEVEL@ 10055714     flags.obj
 0002:00009724       ??_C@_09EBKAPHPA@OPM_DESCR@ 10055724     flags.obj
 0002:00009730       ??_C@_0O@OPDAGBBE@OPM_QUICKVIEW@ 10055730     flags.obj
 0002:00009740       ??_C@_08LCEGJCAC@OPM_PGDN@ 10055740     flags.obj
 0002:0000974c       ??_C@_0N@HKCLLJDG@OPM_COMMANDS@ 1005574c     flags.obj
 0002:0000975c       ??_C@_08EGEBMPBD@OPM_NONE@ 1005575c     flags.obj
 0002:00009768       ??_C@_0M@MIGJPBPE@FOSF_ACTIVE@ 10055768     flags.obj
 0002:00009774       ??_C@_09FMOOJHDF@FOSF_NONE@ 10055774     flags.obj
 0002:00009780       ??_C@_09HNBBLIGN@PCIF_NONE@ 10055780     flags.obj
 0002:0000978c       ??_C@_0BA@MAEBFMHC@FOREGROUND_BLUE@ 1005578c     flags.obj
 0002:0000979c       ??_C@_0BB@PDFNMAI@FOREGROUND_GREEN@ 1005579c     flags.obj
 0002:000097b0       ??_C@_0P@PBJHCFGA@FOREGROUND_RED@ 100557b0     flags.obj
 0002:000097c0       ??_C@_0BF@OOGEJCC@FOREGROUND_INTENSITY@ 100557c0     flags.obj
 0002:000097d8       ??_C@_0BA@PIFINJCK@BACKGROUND_BLUE@ 100557d8     flags.obj
 0002:000097e8       ??_C@_0BB@GKLNBMEL@BACKGROUND_GREEN@ 100557e8     flags.obj
 0002:000097fc       ??_C@_0P@DANALJMC@BACKGROUND_RED@ 100557fc     flags.obj
 0002:0000980c       ??_C@_0BF@NIGKKPCF@BACKGROUND_INTENSITY@ 1005580c     flags.obj
 0002:00009824       ??_C@_0N@FEFOEFHG@CTRL_C_EVENT@ 10055824     flags.obj
 0002:00009834       ??_C@_0BB@ELEIIFAE@CTRL_BREAK_EVENT@ 10055834     flags.obj
 0002:00009848       ??_C@_0BB@KMPDMOKK@CTRL_CLOSE_EVENT@ 10055848     flags.obj
 0002:0000985c       ??_C@_0BC@MCKCEPAL@CTRL_LOGOFF_EVENT@ 1005585c     flags.obj
 0002:00009870       ??_C@_0BE@BCNEFGKM@CTRL_SHUTDOWN_EVENT@ 10055870     flags.obj
 0002:00009884       ??_C@_0BC@BBOPHMOM@ENABLE_LINE_INPUT@ 10055884     flags.obj
 0002:00009898       ??_C@_0BC@JPFKLHOC@ENABLE_ECHO_INPUT@ 10055898     flags.obj
 0002:000098ac       ??_C@_0BH@EHINFMOF@ENABLE_PROCESSED_INPUT@ 100558ac     flags.obj
 0002:000098c4       ??_C@_0BE@BLAHACNB@ENABLE_WINDOW_INPUT@ 100558c4     flags.obj
 0002:000098d8       ??_C@_0BD@BJECBJPO@ENABLE_MOUSE_INPUT@ 100558d8     flags.obj
 0002:000098ec       ??_C@_0BD@KJBPOMPN@ENABLE_INSERT_MODE@ 100558ec     flags.obj
 0002:00009900       ??_C@_0BH@BJKMFKAO@ENABLE_QUICK_EDIT_MODE@ 10055900     flags.obj
 0002:00009918       ??_C@_0BG@CBCHHIEH@ENABLE_EXTENDED_FLAGS@ 10055918     flags.obj
 0002:00009930       ??_C@_0BF@PEBFEBKN@ENABLE_AUTO_POSITION@ 10055930     flags.obj
 0002:00009948       ??_C@_0BI@MHKNPIFM@ENABLE_PROCESSED_OUTPUT@ 10055948     flags.obj
 0002:00009960       ??_C@_0BK@CDKLKCHJ@ENABLE_WRAP_AT_EOL_OUTPUT@ 10055960     flags.obj
 0002:0000997c       ??_C@_09JBABGNAE@KEY_EVENT@ 1005597c     flags.obj
 0002:00009988       ??_C@_0M@CPILDGOO@MOUSE_EVENT@ 10055988     flags.obj
 0002:00009994       ??_C@_0BJ@OHDOHJKG@WINDOW_BUFFER_SIZE_EVENT@ 10055994     flags.obj
 0002:000099b0       ??_C@_0L@MPODFLFH@MENU_EVENT@ 100559b0     flags.obj
 0002:000099bc       ??_C@_0M@LNGHCCGJ@FOCUS_EVENT@ 100559bc     flags.obj
 0002:000099c8       ??_C@_0M@MKBGBFGO@CAPSLOCK_ON@ 100559c8     flags.obj
 0002:000099d4       ??_C@_0N@EMEOEKDA@ENHANCED_KEY@ 100559d4     flags.obj
 0002:000099e4       ??_C@_0BC@GDHABBAP@RIGHT_ALT_PRESSED@ 100559e4     flags.obj
 0002:000099f8       ??_C@_0BB@MCADLJJO@LEFT_ALT_PRESSED@ 100559f8     flags.obj
 0002:00009a0c       ??_C@_0BD@NEHHNAHO@RIGHT_CTRL_PRESSED@ 10055a0c     flags.obj
 0002:00009a20       ??_C@_0BC@FDNOAAAE@LEFT_CTRL_PRESSED@ 10055a20     flags.obj
 0002:00009a34       ??_C@_0O@OGDFJMBK@SHIFT_PRESSED@ 10055a34     flags.obj
 0002:00009a44       ??_C@_0L@IMGKKBIM@NUMLOCK_ON@ 10055a44     flags.obj
 0002:00009a50       ??_C@_0O@LAHFNPLG@SCROLLLOCK_ON@ 10055a50     flags.obj
 0002:00009a60       ??_C@_0BN@HACKHGAB@FROM_LEFT_1ST_BUTTON_PRESSED@ 10055a60     flags.obj
 0002:00009a80       ??_C@_0BJ@JECFAJNJ@RIGHTMOST_BUTTON_PRESSED@ 10055a80     flags.obj
 0002:00009a9c       ??_C@_0BN@BJCFPKCG@FROM_LEFT_2ND_BUTTON_PRESSED@ 10055a9c     flags.obj
 0002:00009abc       ??_C@_0BN@PMJNFPGM@FROM_LEFT_3RD_BUTTON_PRESSED@ 10055abc     flags.obj
 0002:00009adc       ??_C@_0BN@CNMHAAPD@FROM_LEFT_4TH_BUTTON_PRESSED@ 10055adc     flags.obj
 0002:00009afc       ??_C@_0M@KKBDEELB@MOUSE_MOVED@ 10055afc     flags.obj
 0002:00009b08       ??_C@_0N@EDCKBGJE@DOUBLE_CLICK@ 10055b08     flags.obj
 0002:00009b18       ??_C@_0O@GABDOPO@MOUSE_WHEELED@ 10055b18     flags.obj
 0002:00009b28       ??_C@_0BA@OOKCCMHH@KEY_WOW64_32KEY@ 10055b28     flags.obj
 0002:00009b38       ??_C@_0BA@DBCPEIGE@KEY_WOW64_64KEY@ 10055b38     flags.obj
 0002:00009b50       _Keys                      10055b50     flags.obj
 0002:0000a6b0       _Vals                      100566b0     flags.obj
 0002:0000bd68       ??_C@_06ICDCBJPI@Colors@   10057d68     keysandcolors.obj
 0002:0000bd70       ??_C@_05GALAPKHH@Guids@    10057d70     keysandcolors.obj
 0002:0000e0f4       ??_C@_01EEMJAFIK@?6@       1005a0f4     lflua.obj
 0002:0000e0f8       ??_C@_0BB@BJDGDOHH@cannot?5?$CFs?5?$CFs?3?5?$CFs@ 1005a0f8     lflua.obj
 0002:0000e10c       ??_C@_03PKPBNCAL@?o?$LL?$LP@ 1005a10c     lflua.obj
 0002:0000e110       ??_C@_06CCPPALKB@?$DNstdin@ 1005a110     lflua.obj
 0002:0000e118       ??_C@_01EOFPKCAF@?$EA@     1005a118     lflua.obj
 0002:0000e11c       ??_C@_04PMOCAHAA@open@     1005a11c     lflua.obj
 0002:0000e124       ??_C@_15JJPIMNBO@?$AAr?$AAb@ 1005a124     lflua.obj
 0002:0000e12c       ??_C@_06IEGCHAII@reopen@   1005a12c     lflua.obj
 0002:0000e134       ??_C@_04POLDLDMI@read@     1005a134     lflua.obj
 0002:0000e13c       ??_C@_02LOCGON@?$AA?$AA@   1005a13c     lflua.obj
 0002:0000e140       ??_C@_09KIEPBIJC@far_regex@ 1005a140     lregex.obj
 0002:0000e14c       ??_C@_0BO@PBOFMCLL@attempt?5to?5access?5freed?5regex@ 1005a14c     lregex.obj
 0002:0000e16c       ??_C@_07IHINEPFG@?$CFs?5?$CI?$CFp?$CJ@ 1005a16c     lregex.obj
 0002:0000e174       ??_C@_01KMDKNFGN@?1@       1005a174     lregex.obj
 0002:0000e178       ??_C@_0BE@BBBEAHLK@RECTL_CREATE?5failed@ 1005a178     lregex.obj
 0002:0000e18c       ??_C@_0BL@HEFMPIBG@invalid?5regular?5expression@ 1005a18c     lregex.obj
 0002:0000e1a8       ??_C@_0BK@JCLHPPNA@cannot?5add?5?$CFd?5stack?5slots@ 1005a1a8     lregex.obj
 0002:0000e1c4       ??_C@_0BM@MOHHGMBK@string?5or?5table?5or?5function@ 1005a1c4     lregex.obj
 0002:0000e1e0       ??_C@_0CG@IDFLGMFM@replace?5string?3?5invalid?5capture@ 1005a1e0     lregex.obj
 0002:0000e208       ??_C@_0BJ@IMAIDFKH@invalid?5replacement?5type@ 1005a208     lregex.obj
 0002:0000e224       ??_C@_0BE@KPDOHKBE@invalid?5return?5type@ 1005a224     lregex.obj
 0002:0000e238       ??_C@_04CKFJHKAP@find@     1005a238     lregex.obj
 0002:0000e240       ??_C@_04GOLEAPFD@gsub@     1005a240     lregex.obj
 0002:0000e248       ??_C@_05FNONLPDI@match@    1005a248     lregex.obj
 0002:0000e250       ??_C@_04MGEIEJAD@exec@     1005a250     lregex.obj
 0002:0000e258       ??_C@_05GFGPIPHI@findW@    1005a258     lregex.obj
 0002:0000e260       ??_C@_05HPGHPNC@gsubW@     1005a260     lregex.obj
 0002:0000e268       ??_C@_06NNKFJOLC@matchW@   1005a268     lregex.obj
 0002:0000e270       ??_C@_05GMDFNCGA@execW@    1005a270     lregex.obj
 0002:0000e278       ??_C@_0O@OJAOCNID@bracketscount@ 1005a278     lregex.obj
 0002:0000e288       ??_C@_04BDLIKKMN@__gc@     1005a288     lregex.obj
 0002:0000e290       ??_C@_06DPFCLDIO@gmatch@   1005a290     lregex.obj
 0002:0000e298       ??_C@_07PPMFDHAH@gmatchW@  1005a298     lregex.obj
 0002:0000e2a0       ??_C@_05FGAODPCE@regex@    1005a2a0     lregex.obj
 0002:0000e2a8       _regex_methods             1005a2a8     lregex.obj
 0002:0000e308       _regex_functions           1005a308     lregex.obj
 0002:0000e368       ??_C@_0BC@PMGNICBE@MacroPluginReturn@ 1005a368     luamacro.obj
 0002:0000e37c       ??_C@_02JIEIHMJD@wl@       1005a37c     luamacro.obj
 0002:0000e380       ??_C@_15PMCGDJNJ@?$AAO?$AAK@ 1005a380     luamacro.obj
 0002:0000e388       ??_C@_1BC@GBFPAMBP@?$AAL?$AAu?$AAa?$AAM?$AAa?$AAc?$AAr?$AAo@ 1005a388     luamacro.obj
 0002:0000e3a0       ??_C@_1FA@DAFHIDEP@?$AAt?$AAo?$AAo?$AA?5?$AAm?$AAa?$AAn?$AAy?$AA?5?$AAv?$AAa?$AAl?$AAu?$AAe?$AAs@ 1005a3a0     luamacro.obj
 0002:0000e3f0       ??_C@_0BN@ICDOMFBB@invalid?5argument?5?$CD?$CFd?5to?5?8?$CFs?8@ 1005a3f0     luamacro.obj
 0002:0000e410       ??_C@_0BB@FCMFBGOM@invalid?5argument@ 1005a410     luamacro.obj
 0002:0000e434       ??_C@_0BA@MDNLMOMP@far_usercontrol@ 1005a434     lusercontrol.obj
 0002:0000e444       ??_C@_0BH@DOPNHMGD@bounds?5checking?5failed@ 1005a444     lusercontrol.obj
 0002:0000e45c       ??_C@_09LDLEBFOB@rawhandle@ 1005a45c     lusercontrol.obj
 0002:0000e468       ??_C@_04IMAAEPPE@Char@     1005a468     lusercontrol.obj
 0002:0000e470       ??_C@_0L@PLFFHFAH@Attributes@ 1005a470     lusercontrol.obj
 0002:0000e47c       ??_C@_0BD@BPIMECDH@X?5must?5be?5positive@ 1005a47c     lusercontrol.obj
 0002:0000e490       ??_C@_0BD@MIGOMCGP@Y?5must?5be?5positive@ 1005a490     lusercontrol.obj
 0002:0000e4a4       ??_C@_05MNDELLDN@__len@    1005a4a4     lusercontrol.obj
 0002:0000e4ac       ??_C@_0L@GADKNKH@__newindex@ 1005a4ac     lusercontrol.obj
 0002:0000e4b8       ??_C@_0BC@KFJDHEIC@CreateUserControl@ 1005a4b8     lusercontrol.obj
 0002:0000e4cc       _usercontrol_methods       1005a4cc     lusercontrol.obj
 0002:0000e4f4       _usercontrol_functions     1005a4f4     lusercontrol.obj
 0002:0000e504       ??_C@_07PHPIFDKI@LBUTTON@  1005a504     service.obj
 0002:0000e50c       ??_C@_07JOMJHALB@RBUTTON@  1005a50c     service.obj
 0002:0000e514       ??_C@_06JHILMIHF@CANCEL@   1005a514     service.obj
 0002:0000e51c       ??_C@_07DLFCFDDG@MBUTTON@  1005a51c     service.obj
 0002:0000e524       ??_C@_08OPILMHEG@XBUTTON1@ 1005a524     service.obj
 0002:0000e530       ??_C@_08MEKGJEIF@XBUTTON2@ 1005a530     service.obj
 0002:0000e53c       ??_C@_04FJBHJJME@BACK@     1005a53c     service.obj
 0002:0000e544       ??_C@_03CJMDHCGG@TAB@      1005a544     service.obj
 0002:0000e548       ??_C@_05PONODPI@CLEAR@     1005a548     service.obj
 0002:0000e550       ??_C@_06LJMOENAO@RETURN@   1005a550     service.obj
 0002:0000e558       ??_C@_05OAHIEJBI@SHIFT@    1005a558     service.obj
 0002:0000e560       ??_C@_07DBEDOPMC@CONTROL@  1005a560     service.obj
 0002:0000e568       ??_C@_04IILMDFMO@MENU@     1005a568     service.obj
 0002:0000e570       ??_C@_05DIAHPDGL@PAUSE@    1005a570     service.obj
 0002:0000e578       ??_C@_07OPCFNGJB@CAPITAL@  1005a578     service.obj
 0002:0000e580       ??_C@_04KGDAIAGM@KANA@     1005a580     service.obj
 0002:0000e588       ??_C@_05PPKJGOLB@JUNJA@    1005a588     service.obj
 0002:0000e590       ??_C@_05JEIAEFOF@FINAL@    1005a590     service.obj
 0002:0000e598       ??_C@_05CHABPOPI@HANJA@    1005a598     service.obj
 0002:0000e5a0       ??_C@_06CDPDIIDH@ESCAPE@   1005a5a0     service.obj
 0002:0000e5a8       ??_C@_0L@ODNCKDCK@NONCONVERT@ 1005a5a8     service.obj
 0002:0000e5b4       ??_C@_06INBBKPI@ACCEPT@    1005a5b4     service.obj
 0002:0000e5bc       ??_C@_0L@HEHNEBED@MODECHANGE@ 1005a5bc     service.obj
 0002:0000e5c8       ??_C@_05CAEOFMEP@SPACE@    1005a5c8     service.obj
 0002:0000e5d0       ??_C@_05BFDHCIJM@PRIOR@    1005a5d0     service.obj
 0002:0000e5d8       ??_C@_04MOKMKBJN@NEXT@     1005a5d8     service.obj
 0002:0000e5e0       ??_C@_03JMGAKCCH@END@      1005a5e0     service.obj
 0002:0000e5e4       ??_C@_04GHGFPGNC@HOME@     1005a5e4     service.obj
 0002:0000e5ec       ??_C@_04KCNEHMIH@LEFT@     1005a5ec     service.obj
 0002:0000e5f4       ??_C@_02NAHCJHOC@UP@       1005a5f4     service.obj
 0002:0000e5f8       ??_C@_05PMAFOJDE@RIGHT@    1005a5f8     service.obj
 0002:0000e600       ??_C@_04FANAOELO@DOWN@     1005a600     service.obj
 0002:0000e608       ??_C@_06LCPJPOPK@SELECT@   1005a608     service.obj
 0002:0000e610       ??_C@_05ECKPOFCN@PRINT@    1005a610     service.obj
 0002:0000e618       ??_C@_07LBDEDADF@EXECUTE@  1005a618     service.obj
 0002:0000e620       ??_C@_08EMOKHGD@SNAPSHOT@  1005a620     service.obj
 0002:0000e62c       ??_C@_06OEMEAEKN@INSERT@   1005a62c     service.obj
 0002:0000e634       ??_C@_06FKDAMKFP@DELETE@   1005a634     service.obj
 0002:0000e63c       ??_C@_04DOKPJKJF@HELP@     1005a63c     service.obj
 0002:0000e644       ??_C@_01GBGANLPD@0@        1005a644     service.obj
 0002:0000e648       ??_C@_01HIHLOKLC@1@        1005a648     service.obj
 0002:0000e64c       ??_C@_01FDFGLJHB@2@        1005a64c     service.obj
 0002:0000e650       ??_C@_01EKENIIDA@3@        1005a650     service.obj
 0002:0000e654       ??_C@_01FAMBOPH@4@         1005a654     service.obj
 0002:0000e658       ??_C@_01BMBHCPLG@5@        1005a658     service.obj
 0002:0000e65c       ??_C@_01DHDKHMHF@6@        1005a65c     service.obj
 0002:0000e660       ??_C@_01COCBENDE@7@        1005a660     service.obj
 0002:0000e664       ??_C@_01KJLJFBPL@8@        1005a664     service.obj
 0002:0000e668       ??_C@_01LAKCGALK@9@        1005a668     service.obj
 0002:0000e66c       ??_C@_01FHEEJDEE@A@        1005a66c     service.obj
 0002:0000e670       ??_C@_01HMGJMAIH@B@        1005a670     service.obj
 0002:0000e674       ??_C@_01GFHCPBMG@C@        1005a674     service.obj
 0002:0000e678       ??_C@_01CKDDGHAB@D@        1005a678     service.obj
 0002:0000e67c       ??_C@_01DDCIFGEA@E@        1005a67c     service.obj
 0002:0000e680       ??_C@_01BIAFAFID@F@        1005a680     service.obj
 0002:0000e684       ??_C@_01BBODEMC@G@         1005a684     service.obj
 0002:0000e688       ??_C@_01IGIGCIAN@H@        1005a688     service.obj
 0002:0000e68c       ??_C@_01JPJNBJEM@I@        1005a68c     service.obj
 0002:0000e690       ??_C@_01LELAEKIP@J@        1005a690     service.obj
 0002:0000e694       ??_C@_01KNKLHLMO@K@        1005a694     service.obj
 0002:0000e698       ??_C@_01OCOKONAJ@L@        1005a698     service.obj
 0002:0000e69c       ??_C@_01PLPBNMEI@M@        1005a69c     service.obj
 0002:0000e6a0       ??_C@_01NANMIPIL@N@        1005a6a0     service.obj
 0002:0000e6a4       ??_C@_01MJMHLOMK@O@        1005a6a4     service.obj
 0002:0000e6a8       ??_C@_01EJNLAFE@P@         1005a6a8     service.obj
 0002:0000e6ac       ??_C@_01BNIGIBBF@Q@        1005a6ac     service.obj
 0002:0000e6b0       ??_C@_01DGKLNCNG@R@        1005a6b0     service.obj
 0002:0000e6b4       ??_C@_01CPLAODJH@S@        1005a6b4     service.obj
 0002:0000e6b8       ??_C@_01GAPBHFFA@T@        1005a6b8     service.obj
 0002:0000e6bc       ??_C@_01HJOKEEBB@U@        1005a6bc     service.obj
 0002:0000e6c0       ??_C@_01FCMHBHNC@V@        1005a6c0     service.obj
 0002:0000e6c4       ??_C@_01ELNMCGJD@W@        1005a6c4     service.obj
 0002:0000e6c8       ??_C@_01MMEEDKFM@X@        1005a6c8     service.obj
 0002:0000e6cc       ??_C@_01NFFPALBN@Y@        1005a6cc     service.obj
 0002:0000e6d0       ??_C@_01POHCFINO@Z@        1005a6d0     service.obj
 0002:0000e6d4       ??_C@_04ODLFFOHF@LWIN@     1005a6d4     service.obj
 0002:0000e6dc       ??_C@_04DMGFHHJG@RWIN@     1005a6dc     service.obj
 0002:0000e6e4       ??_C@_04GKGJFGJO@APPS@     1005a6e4     service.obj
 0002:0000e6ec       ??_C@_05DJAECLDN@SLEEP@    1005a6ec     service.obj
 0002:0000e6f4       ??_C@_07NHIPMMJH@NUMPAD0@  1005a6f4     service.obj
 0002:0000e6fc       ??_C@_07MOJEPNNG@NUMPAD1@  1005a6fc     service.obj
 0002:0000e704       ??_C@_07OFLJKOBF@NUMPAD2@  1005a704     service.obj
 0002:0000e70c       ??_C@_07PMKCJPFE@NUMPAD3@  1005a70c     service.obj
 0002:0000e714       ??_C@_07LDODAJJD@NUMPAD4@  1005a714     service.obj
 0002:0000e71c       ??_C@_07KKPIDINC@NUMPAD5@  1005a71c     service.obj
 0002:0000e724       ??_C@_07IBNFGLBB@NUMPAD6@  1005a724     service.obj
 0002:0000e72c       ??_C@_07JIMOFKFA@NUMPAD7@  1005a72c     service.obj
 0002:0000e734       ??_C@_07BPFGEGJP@NUMPAD8@  1005a734     service.obj
 0002:0000e73c       ??_C@_07GENHHNO@NUMPAD9@   1005a73c     service.obj
 0002:0000e744       ??_C@_08LDEOAAGM@MULTIPLY@ 1005a744     service.obj
 0002:0000e750       ??_C@_03BOJFLAKG@ADD@      1005a750     service.obj
 0002:0000e754       ??_C@_09POPINEFK@SEPARATOR@ 1005a754     service.obj
 0002:0000e760       ??_C@_08MGBEENML@SUBTRACT@ 1005a760     service.obj
 0002:0000e76c       ??_C@_07LJPMJDLL@DECIMAL@  1005a76c     service.obj
 0002:0000e774       ??_C@_06FBFCJJMP@DIVIDE@   1005a774     service.obj
 0002:0000e77c       ??_C@_02LCPENACN@F1@       1005a77c     service.obj
 0002:0000e780       ??_C@_02JJNJIDOO@F2@       1005a780     service.obj
 0002:0000e784       ??_C@_02IAMCLCKP@F3@       1005a784     service.obj
 0002:0000e788       ??_C@_02MPIDCEGI@F4@       1005a788     service.obj
 0002:0000e78c       ??_C@_02NGJIBFCJ@F5@       1005a78c     service.obj
 0002:0000e790       ??_C@_02PNLFEGOK@F6@       1005a790     service.obj
 0002:0000e794       ??_C@_02OEKOHHKL@F7@       1005a794     service.obj
 0002:0000e798       ??_C@_02GDDGGLGE@F8@       1005a798     service.obj
 0002:0000e79c       ??_C@_02HKCNFKCF@F9@       1005a79c     service.obj
 0002:0000e7a0       ??_C@_03JKCLJOFG@F10@      1005a7a0     service.obj
 0002:0000e7a4       ??_C@_03IDDAKPBH@F11@      1005a7a4     service.obj
 0002:0000e7a8       ??_C@_03KIBNPMNE@F12@      1005a7a8     service.obj
 0002:0000e7ac       ??_C@_03LBAGMNJF@F13@      1005a7ac     service.obj
 0002:0000e7b0       ??_C@_03POEHFLFC@F14@      1005a7b0     service.obj
 0002:0000e7b4       ??_C@_03OHFMGKBD@F15@      1005a7b4     service.obj
 0002:0000e7b8       ??_C@_03MMHBDJNA@F16@      1005a7b8     service.obj
 0002:0000e7bc       ??_C@_03NFGKAIJB@F17@      1005a7bc     service.obj
 0002:0000e7c0       ??_C@_03FCPCBEFO@F18@      1005a7c0     service.obj
 0002:0000e7c4       ??_C@_03ELOJCFBP@F19@      1005a7c4     service.obj
 0002:0000e7c8       ??_C@_03JIGNCAAP@F20@      1005a7c8     service.obj
 0002:0000e7cc       ??_C@_03IBHGBBEO@F21@      1005a7cc     service.obj
 0002:0000e7d0       ??_C@_03KKFLECIN@F22@      1005a7d0     service.obj
 0002:0000e7d4       ??_C@_03LDEAHDMM@F23@      1005a7d4     service.obj
 0002:0000e7d8       ??_C@_03PMABOFAL@F24@      1005a7d8     service.obj
 0002:0000e7dc       ??_C@_07FLMEHHJP@NUMLOCK@  1005a7dc     service.obj
 0002:0000e7e4       ??_C@_06FNIKALAE@SCROLL@   1005a7e4     service.obj
 0002:0000e7ec       ??_C@_0O@DBBJDALK@OEM_NEC_EQUAL@ 1005a7ec     service.obj
 0002:0000e7fc       ??_C@_0P@JKGCFGCD@OEM_FJ_MASSHOU@ 1005a7fc     service.obj
 0002:0000e80c       ??_C@_0P@NIEOFNLG@OEM_FJ_TOUROKU@ 1005a80c     service.obj
 0002:0000e81c       ??_C@_0M@IBEHGLCM@OEM_FJ_LOYA@ 1005a81c     service.obj
 0002:0000e828       ??_C@_0M@FOJHECMP@OEM_FJ_ROYA@ 1005a828     service.obj
 0002:0000e834       ??_C@_06EPHNCIMI@LSHIFT@   1005a834     service.obj
 0002:0000e83c       ??_C@_06HIJMMPFL@RSHIFT@   1005a83c     service.obj
 0002:0000e844       ??_C@_08IKMONEBG@LCONTROL@ 1005a844     service.obj
 0002:0000e850       ??_C@_08OOMMENPF@RCONTROL@ 1005a850     service.obj
 0002:0000e85c       ??_C@_05IHMGKJGH@LMENU@    1005a85c     service.obj
 0002:0000e864       ??_C@_05LOBKMKIM@RMENU@    1005a864     service.obj
 0002:0000e86c       ??_C@_0N@OAJIELLG@BROWSER_BACK@ 1005a86c     service.obj
 0002:0000e87c       ??_C@_0BA@ENOAJOGH@BROWSER_FORWARD@ 1005a87c     service.obj
 0002:0000e88c       ??_C@_0BA@GDNDIDGJ@BROWSER_REFRESH@ 1005a88c     service.obj
 0002:0000e89c       ??_C@_0N@HKPDGANH@BROWSER_STOP@ 1005a89c     service.obj
 0002:0000e8ac       ??_C@_0P@BEAEBJDD@BROWSER_SEARCH@ 1005a8ac     service.obj
 0002:0000e8bc       ??_C@_0BC@BOMJIH@BROWSER_FAVORITES@ 1005a8bc     service.obj
 0002:0000e8d0       ??_C@_0N@NOOKCEKA@BROWSER_HOME@ 1005a8d0     service.obj
 0002:0000e8e0       ??_C@_0M@ENOHKBMG@VOLUME_MUTE@ 1005a8e0     service.obj
 0002:0000e8ec       ??_C@_0M@JOOBBDNO@VOLUME_DOWN@ 1005a8ec     service.obj
 0002:0000e8f8       ??_C@_09MGPMNMJC@VOLUME_UP@ 1005a8f8     service.obj
 0002:0000e904       ??_C@_0BB@KLAENPA@MEDIA_NEXT_TRACK@ 1005a904     service.obj
 0002:0000e918       ??_C@_0BB@CMOIJKPH@MEDIA_PREV_TRACK@ 1005a918     service.obj
 0002:0000e92c       ??_C@_0L@KBJOCDHK@MEDIA_STOP@ 1005a92c     service.obj
 0002:0000e938       ??_C@_0BB@HAEMIJHO@MEDIA_PLAY_PAUSE@ 1005a938     service.obj
 0002:0000e94c       ??_C@_0M@GCIKMBID@LAUNCH_MAIL@ 1005a94c     service.obj
 0002:0000e958       ??_C@_0BE@FADJJAPM@LAUNCH_MEDIA_SELECT@ 1005a958     service.obj
 0002:0000e96c       ??_C@_0M@MGLJIDDM@LAUNCH_APP1@ 1005a96c     service.obj
 0002:0000e978       ??_C@_0M@ONJENAPP@LAUNCH_APP2@ 1005a978     service.obj
 0002:0000e984       ??_C@_05OIODNPAD@OEM_1@    1005a984     service.obj
 0002:0000e98c       ??_C@_08LDJEIPBH@OEM_PLUS@ 1005a98c     service.obj
 0002:0000e998       ??_C@_09CLPFJEOD@OEM_COMMA@ 1005a998     service.obj
 0002:0000e9a4       ??_C@_09OGMLCNMG@OEM_MINUS@ 1005a9a4     service.obj
 0002:0000e9b0       ??_C@_0L@DNNMNDGM@OEM_PERIOD@ 1005a9b0     service.obj
 0002:0000e9bc       ??_C@_05MDMOIMMA@OEM_2@    1005a9bc     service.obj
 0002:0000e9c4       ??_C@_05NKNFLNIB@OEM_3@    1005a9c4     service.obj
 0002:0000e9cc       ??_C@_05JFJECLEG@OEM_4@    1005a9cc     service.obj
 0002:0000e9d4       ??_C@_05IMIPBKAH@OEM_5@    1005a9d4     service.obj
 0002:0000e9dc       ??_C@_05KHKCEJME@OEM_6@    1005a9dc     service.obj
 0002:0000e9e4       ??_C@_05LOLJHIIF@OEM_7@    1005a9e4     service.obj
 0002:0000e9ec       ??_C@_05DJCBGEEK@OEM_8@    1005a9ec     service.obj
 0002:0000e9f4       ??_C@_07PEFKMFIE@OEM_102@  1005a9f4     service.obj
 0002:0000e9fc       ??_C@_0L@EFLJCPAM@PROCESSKEY@ 1005a9fc     service.obj
 0002:0000ea08       ??_C@_06HOICDKCB@PACKET@   1005aa08     service.obj
 0002:0000ea10       ??_C@_09CAKPMKHM@OEM_RESET@ 1005aa10     service.obj
 0002:0000ea1c       ??_C@_08INMNLJCK@OEM_JUMP@ 1005aa1c     service.obj
 0002:0000ea28       ??_C@_07JNOAEEG@OEM_PA1@   1005aa28     service.obj
 0002:0000ea30       ??_C@_07CCPDFHIF@OEM_PA2@  1005aa30     service.obj
 0002:0000ea38       ??_C@_07DLOIGGME@OEM_PA3@  1005aa38     service.obj
 0002:0000ea40       ??_C@_0L@OCAIHDP@OEM_WSCTRL@ 1005aa40     service.obj
 0002:0000ea4c       ??_C@_04BNGOAFAJ@ATTN@     1005aa4c     service.obj
 0002:0000ea54       ??_C@_05HGAHFFFL@CRSEL@    1005aa54     service.obj
 0002:0000ea5c       ??_C@_05OKOOKOOH@EXSEL@    1005aa5c     service.obj
 0002:0000ea64       ??_C@_05CCFENDFJ@EREOF@    1005aa64     service.obj
 0002:0000ea6c       ??_C@_04MKCNCBEG@PLAY@     1005aa6c     service.obj
 0002:0000ea74       ??_C@_04LGBIGMFG@ZOOM@     1005aa74     service.obj
 0002:0000ea7c       ??_C@_06LJIOOKLP@NONAME@   1005aa7c     service.obj
 0002:0000ea84       ??_C@_03KCLDMPAE@PA1@      1005aa84     service.obj
 0002:0000ea88       ??_C@_09MBBEHOCK@OEM_CLEAR@ 1005aa88     service.obj
 0002:0000ea94       ??_C@_09GJGOMOL@lua51?4dll@ 1005aa94     service.obj
 0002:0000eaa0       ??_C@_0M@PLOBHAKE@luaopen_bit@ 1005aaa0     service.obj
 0002:0000eaac       ??_C@_0M@IALDMMNC@luaopen_ffi@ 1005aaac     service.obj
 0002:0000eab8       ??_C@_0M@DOFFFIEL@luaopen_jit@ 1005aab8     service.obj
 0002:0000eac4       ??_C@_0BK@FFJEICME@integer?5or?5light?5userdata@ 1005aac4     service.obj
 0002:0000eae0       ??_C@_0BD@PNJHLBDA@invalid?5flag?3?5?$CC?$CFs?$CC@ 1005aae0     service.obj
 0002:0000eaf4       ??_C@_0N@JJLBBDOC@invalid?5flag@ 1005aaf4     service.obj
 0002:0000eb04       ??_C@_0BJ@MIKGPOKL@invalid?5flag?5combination@ 1005ab04     service.obj
 0002:0000eb20       ??_C@_08KJKIOMBF@3?40?40?4?$CFd@ 1005ab20     service.obj
 0002:0000eb2c       ??_C@_0P@EANMLDOP@MousePositionX@ 1005ab2c     service.obj
 0002:0000eb3c       ??_C@_0P@FJMHICKO@MousePositionY@ 1005ab3c     service.obj
 0002:0000eb4c       ??_C@_0M@BJAICPIE@ButtonState@ 1005ab4c     service.obj
 0002:0000eb58       ??_C@_0L@EMFBJIPA@EventFlags@ 1005ab58     service.obj
 0002:0000eb64       ??_C@_07EEJLMCNH@CurLine@  1005ab64     service.obj
 0002:0000eb6c       ??_C@_06EDBJMJDC@CurPos@   1005ab6c     service.obj
 0002:0000eb74       ??_C@_09EGONKHKB@CurTabPos@ 1005ab74     service.obj
 0002:0000eb80       ??_C@_0O@OKGGHEJK@TopScreenLine@ 1005ab80     service.obj
 0002:0000eb90       ??_C@_07GDAKJHLE@LeftPos@  1005ab90     service.obj
 0002:0000eb98       ??_C@_08LLJICOLD@Overtype@ 1005ab98     service.obj
 0002:0000eba4       ??_C@_0L@GEIEADPN@ModuleName@ 1005aba4     service.obj
 0002:0000ebb0       ??_C@_09HOIHBHIM@ModuleDir@ 1005abb0     service.obj
 0002:0000ebbc       ??_C@_0L@JLHCLFBG@PluginGuid@ 1005abbc     service.obj
 0002:0000ebc8       ??_C@_08GGMFPBHM@EditorID@ 1005abc8     service.obj
 0002:0000ebd4       ??_C@_0M@CPDBGLHN@WindowSizeX@ 1005abd4     service.obj
 0002:0000ebe0       ??_C@_0M@DGCKFKDM@WindowSizeY@ 1005abe0     service.obj
 0002:0000ebec       ??_C@_0L@PMKENHMA@TotalLines@ 1005abec     service.obj
 0002:0000ebf8       ??_C@_09HKBEFIPN@BlockType@ 1005abf8     service.obj
 0002:0000ec04       ??_C@_0P@GAEEHNHE@BlockStartLine@ 1005ac04     service.obj
 0002:0000ec14       ??_C@_07KHIHFBFN@Options@  1005ac14     service.obj
 0002:0000ec1c       ??_C@_07FLDNELFM@TabSize@  1005ac1c     service.obj
 0002:0000ec24       ??_C@_0O@EBLDFOPH@BookmarkCount@ 1005ac24     service.obj
 0002:0000ec34       ??_C@_0BF@ODFKBFAK@SessionBookmarkCount@ 1005ac34     service.obj
 0002:0000ec4c       ??_C@_08CPAOHJDL@CurState@ 1005ac4c     service.obj
 0002:0000ec58       ??_C@_0N@DAJMJAE@StringLength@ 1005ac58     service.obj
 0002:0000ec68       ??_C@_08JPMALCFA@SelStart@ 1005ac68     service.obj
 0002:0000ec74       ??_C@_06JLEHDHII@SelEnd@   1005ac74     service.obj
 0002:0000ec7c       ??_C@_0L@IFNFGDGN@StringText@ 1005ac7c     service.obj
 0002:0000ec88       ??_C@_09IBGOAAEM@StringEOL@ 1005ac88     service.obj
 0002:0000ec94       ??_C@_06MFLCIING@redraw@   1005ac94     service.obj
 0002:0000ec9c       ??_C@_07HICINA@restore@    1005ac9c     service.obj
 0002:0000eca4       ??_C@_0CG@LAKEGANL@must?5be?5?8redraw?8?0?5?8restore?8?0?5or@ 1005aca4     service.obj
 0002:0000eccc       ??_C@_04LIDDHMOL@Line@     1005accc     service.obj
 0002:0000ecd4       ??_C@_06OIIFPIKD@Cursor@   1005acd4     service.obj
 0002:0000ecdc       ??_C@_0L@GDDEHGKI@ScreenLine@ 1005acdc     service.obj
 0002:0000ece8       ??_C@_0O@CIAFMMMB@BlockStartPos@ 1005ace8     service.obj
 0002:0000ecf8       ??_C@_0L@EKLJJHPF@BlockWidth@ 1005acf8     service.obj
 0002:0000ed04       ??_C@_0M@NKKGBDGK@BlockHeight@ 1005ad04     service.obj
 0002:0000ed10       ??_C@_09JFPCGCOC@StartLine@ 1005ad10     service.obj
 0002:0000ed1c       ??_C@_08JBNOANJG@StartPos@ 1005ad1c     service.obj
 0002:0000ed28       ??_C@_07DCKCOCOC@EndLine@  1005ad28     service.obj
 0002:0000ed30       ??_C@_06KGHIGMHC@EndPos@   1005ad30     service.obj
 0002:0000ed38       ??_C@_0BA@HNIJJEO@ForegroundColor@ 1005ad38     service.obj
 0002:0000ed48       ??_C@_0BA@DPMBBMBG@BackgroundColor@ 1005ad48     service.obj
 0002:0000ed58       ??_C@_0O@NHKEGDJF@GUID?5required@ 1005ad58     service.obj
 0002:0000ed68       ??_C@_0BJ@BMOGHFAN@table?5or?5number?5expected@ 1005ad68     service.obj
 0002:0000ed84       ??_C@_08KGEIBGG@Priority@  1005ad84     service.obj
 0002:0000ed90       ??_C@_05PDOBBJNA@Color@    1005ad90     service.obj
 0002:0000ed98       ??_C@_09KDLBEGCN@EventType@ 1005ad98     service.obj
 0002:0000eda4       ??_C@_07HPHPOAEG@KeyDown@  1005ada4     service.obj
 0002:0000edac       ??_C@_0M@FGGHEADP@RepeatCount@ 1005adac     service.obj
 0002:0000edb8       ??_C@_0BA@KCCLHPM@VirtualScanCode@ 1005adb8     service.obj
 0002:0000edc8       ??_C@_0M@PBJKDIHH@UnicodeChar@ 1005adc8     service.obj
 0002:0000edd4       ??_C@_05GIPJKPFG@SizeX@    1005add4     service.obj
 0002:0000eddc       ??_C@_05HBOCJOBH@SizeY@    1005addc     service.obj
 0002:0000ede4       ??_C@_09GEJJJAHL@CommandId@ 1005ade4     service.obj
 0002:0000edf0       ??_C@_08GPNNBNIL@SetFocus@ 1005adf0     service.obj
 0002:0000edfc       ??_C@_0M@BEDENHPD@invalid?5key@ 1005adfc     service.obj
 0002:0000ee08       ??_C@_19IBCFILMC@?$AAM?$AAe?$AAn?$AAu@ 1005ae08     service.obj
 0002:0000ee14       ??_C@_0BN@JBAMKCCJ@must?5be?5table?0?5string?5or?5nil@ 1005ae14     service.obj
 0002:0000ee34       ??_C@_09FDAFFNEA@MaxHeight@ 1005ae34     service.obj
 0002:0000ee40       ??_C@_06DDHCBBGN@Bottom@   1005ae40     service.obj
 0002:0000ee48       ??_C@_09CFELDMD@HelpTopic@ 1005ae48     service.obj
 0002:0000ee54       ??_C@_0M@GGMLPAIK@SelectIndex@ 1005ae54     service.obj
 0002:0000ee60       ??_C@_02HOGEDOAB@Id@       1005ae60     service.obj
 0002:0000ee64       ??_C@_05LCLENNFI@table@    1005ae64     service.obj
 0002:0000ee6c       ??_C@_06ICGJLFIM@string@   1005ae6c     service.obj
 0002:0000ee74       ??_C@_07FJOBMBFC@checked@  1005ae74     service.obj
 0002:0000ee7c       ??_C@_09MOAJOJKN@separator@ 1005ae7c     service.obj
 0002:0000ee88       ??_C@_07DBNODEFN@disable@  1005ae88     service.obj
 0002:0000ee90       ??_C@_06JHIAOIKD@grayed@   1005ae90     service.obj
 0002:0000ee98       ??_C@_06JIKFICKK@hidden@   1005ae98     service.obj
 0002:0000eea0       ??_C@_08CJLOJPNI@selected@ 1005aea0     service.obj
 0002:0000eeac       ??_C@_08MMCKBNNI@AccelKey@ 1005aeac     service.obj
 0002:0000eeb8       ??_C@_08PNHLLJE@BreakKey@  1005aeb8     service.obj
 0002:0000eec4       ??_C@_15FMBEJGOH@?$AAO?$AAk@ 1005aec4     service.obj
 0002:0000eecc       ??_C@_1BC@IBCAPFAE@?$AAO?$AAk?$AAC?$AAa?$AAn?$AAc?$AAe?$AAl@ 1005aecc     service.obj
 0002:0000eee0       ??_C@_1CC@HODOHOHB@?$AAA?$AAb?$AAo?$AAr?$AAt?$AAR?$AAe?$AAt?$AAr?$AAy?$AAI?$AAg?$AAn?$AAo?$AAr@ 1005aee0     service.obj
 0002:0000ef04       ??_C@_1M@GGPOIMAD@?$AAY?$AAe?$AAs?$AAN?$AAo@ 1005af04     service.obj
 0002:0000ef10       ??_C@_1BI@BNDFIGCI@?$AAY?$AAe?$AAs?$AAN?$AAo?$AAC?$AAa?$AAn?$AAc?$AAe?$AAl@ 1005af10     service.obj
 0002:0000ef28       ??_C@_1BI@KMMIHPHF@?$AAR?$AAe?$AAt?$AAr?$AAy?$AAC?$AAa?$AAn?$AAc?$AAe?$AAl@ 1005af28     service.obj
 0002:0000ef40       ??_C@_1DG@LMKDDADI@?$AA?$DM?$AAn?$AAo?$AAn?$AA?9?$AAs?$AAt?$AAr?$AAi?$AAn?$AAg?$AA?5?$AAe?$AAr?$AAr@ 1005af40     service.obj
 0002:0000ef78       ??_C@_15IEGBJKPD@?$AA?3?$AA?6@ 1005af78     service.obj
 0002:0000ef80       ??_C@_19FFLPMPBO@?$AA?6?$AA?5?$AA?5?$AA?5@ 1005af80     service.obj
 0002:0000ef8c       ??_C@_15JCKODCLA@?$AA?6?$AA?7@ 1005af8c     service.obj
 0002:0000ef94       ??_C@_1M@ILHOPKA@?$AAE?$AAr?$AAr?$AAo?$AAr@ 1005af94     service.obj
 0002:0000efa0       ??_C@_08FNIIFOJC@tostring@ 1005afa0     service.obj
 0002:0000efac       ??_C@_0BJ@JOELOGM@cannot?5convert?5to?5string@ 1005afac     service.obj
 0002:0000efc8       ??_C@_1BA@HHOMBECE@?$AAM?$AAe?$AAs?$AAs?$AAa?$AAg?$AAe@ 1005afc8     service.obj
 0002:0000efd8       ??_C@_17PAGBAIDI@?$AA?$DL?$AAO?$AAK@ 1005afd8     service.obj
 0002:0000efe0       ??_C@_09ENKGJCEC@OwnerGuid@ 1005afe0     service.obj
 0002:0000efec       ??_C@_0N@CCPLCIHE@PluginHandle@ 1005afec     service.obj
 0002:0000effc       ??_C@_0N@HEHBMBNM@PluginObject@ 1005affc     service.obj
 0002:0000f00c       ??_C@_09BKHPOLGD@PanelType@ 1005b00c     service.obj
 0002:0000f018       ??_C@_04GOOOJOPP@left@     1005b018     service.obj
 0002:0000f020       ??_C@_03FGFCOCMD@top@      1005b020     service.obj
 0002:0000f024       ??_C@_05DHJDAOHK@right@    1005b024     service.obj
 0002:0000f02c       ??_C@_06PMMPCIPB@bottom@   1005b02c     service.obj
 0002:0000f034       ??_C@_09MCEJMINN@PanelRect@ 1005b034     service.obj
 0002:0000f040       ??_C@_0M@DDGFKGKJ@ItemsNumber@ 1005b040     service.obj
 0002:0000f04c       ??_C@_0BE@EOBAHHNK@SelectedItemsNumber@ 1005b04c     service.obj
 0002:0000f060       ??_C@_0M@JMILNLLF@CurrentItem@ 1005b060     service.obj
 0002:0000f06c       ??_C@_0N@CDHIFJIH@TopPanelItem@ 1005b06c     service.obj
 0002:0000f07c       ??_C@_08IMMBLBLF@ViewMode@ 1005b07c     service.obj
 0002:0000f088       ??_C@_08CENECNJD@SortMode@ 1005b088     service.obj
 0002:0000f094       ??_C@_04FABLJDN@Name@      1005b094     service.obj
 0002:0000f09c       ??_C@_05LOJBNELM@Param@    1005b09c     service.obj
 0002:0000f0a4       ??_C@_04PBAHLACE@File@     1005b0a4     service.obj
 0002:0000f0ac       ??_C@_08HGEAFCFN@PluginId@ 1005b0ac     service.obj
 0002:0000f0b8       ??_C@_0BA@MLHECKCE@table?5or?5string@ 1005b0b8     service.obj
 0002:0000f0c8       ??_C@_0BD@CKJHMJBG@non?9positive?5index@ 1005b0c8     service.obj
 0002:0000f0dc       ??_C@_0BA@GNKNKKDM@number?5or?5table@ 1005b0dc     service.obj
 0002:0000f0ec       ??_C@_0CI@DDAJHJKO@?$CFs?5?9?5unsupported?5type?5in?5dialog@ 1005b0ec     service.obj
 0002:0000f114       ??_C@_0CD@JIANOKII@unsupported?5flag?5in?5dialog?5item@ 1005b114     service.obj
 0002:0000f138       ??_C@_0CB@EOGFCCCC@value?5at?5index?5?$CFd?5is?5not?5a?5tabl@ 1005b138     service.obj
 0002:0000f15c       ??_C@_0O@FEBHKEHB@closed?5dialog@ 1005b15c     service.obj
 0002:0000f16c       ??_C@_0BK@NEMPGLFN@operation?5not?5implemented@ 1005b16c     service.obj
 0002:0000f188       ??_C@_04KPCPLBPL@Left@     1005b188     service.obj
 0002:0000f190       ??_C@_03PGGAENPN@Top@      1005b190     service.obj
 0002:0000f194       ??_C@_05DADPALEM@Right@    1005b194     service.obj
 0002:0000f19c       ??_C@_0CK@JHNDGJBB@element?5?$CD?$CFd?5in?5argument?5?$CD4?5is?5n@ 1005b19c     service.obj
 0002:0000f1c8       ??_C@_0L@CECHCPAP@StartIndex@ 1005b1c8     service.obj
 0002:0000f1d4       ??_C@_05IJGIMMHE@Count@    1005b1d4     service.obj
 0002:0000f1dc       ??_C@_07NOCIGAPP@Pattern@  1005b1dc     service.obj
 0002:0000f1e4       ??_C@_09IMOCKOO@SelectPos@ 1005b1e4     service.obj
 0002:0000f1f0       ??_C@_06DJONBJOP@TopPos@   1005b1f0     service.obj
 0002:0000f1f8       ??_C@_09OGCBKCAK@MaxLength@ 1005b1f8     service.obj
 0002:0000f204       ??_C@_05FNNGFGLF@Index@    1005b204     service.obj
 0002:0000f20c       ??_C@_07GHGHLGFI@GetType@  1005b20c     service.obj
 0002:0000f214       ??_C@_07MMLMCDAI@ValType@  1005b214     service.obj
 0002:0000f21c       ??_C@_05LPIJGKJ@Value@     1005b21c     service.obj
 0002:0000f224       ??_C@_0L@LPFMIAHH@helpstring@ 1005b224     service.obj
 0002:0000f230       ??_C@_0P@NABDHFON@getvaluestring@ 1005b230     service.obj
 0002:0000f240       ??_C@_0BJ@IINAPFDG@Items?$FL?$CFd?$FN?5is?5not?5a?5table@ 1005b240     service.obj
 0002:0000f25c       ??_C@_0CC@GBOJFNBI@error?5occured?5in?5dialog?5procedu@ 1005b25c     service.obj
 0002:0000f280       ??_C@_0M@EHMONPJO@?$CFs?5?$CIclosed?$CJ@ 1005b280     service.obj
 0002:0000f28c       ??_C@_08GDAJJKGC@ViewerID@ 1005b28c     service.obj
 0002:0000f298       ??_C@_07MJHBHMFM@FilePos@  1005b298     service.obj
 0002:0000f2a0       ??_C@_07FBAHDBGN@CurMode@  1005b2a0     service.obj
 0002:0000f2a8       ??_C@_06IMBBKDFH@iParam@   1005b2a8     service.obj
 0002:0000f2b0       ??_C@_1BE@CGKCNEEP@?$AAI?$AAn?$AAp?$AAu?$AAt?$AA?5?$AAB?$AAo?$AAx@ 1005b2b0     service.obj
 0002:0000f2c4       ??_C@_1CA@PCDNIBFH@?$AAE?$AAn?$AAt?$AAe?$AAr?$AA?5?$AAt?$AAh?$AAe?$AA?5?$AAt?$AAe?$AAx?$AAt?$AA?3@ 1005b2c4     service.obj
 0002:0000f2e4       ??_C@_15GALJLHBD@?$AA?$DO?$AA?$DO@ 1005b2e4     service.obj
 0002:0000f2ec       ??_C@_0BG@GAFLOAPP@command?5not?5supported@ 1005b2ec     service.obj
 0002:0000f304       ??_C@_09MIJAKHKB@Completed@ 1005b304     service.obj
 0002:0000f310       ??_C@_05KGEAEGFG@Total@    1005b310     service.obj
 0002:0000f318       ??_C@_0P@DJOANNIK@?$CFd?4?$CFd?4?$CFd?4?$CFd?4?$CFd@ 1005b318     service.obj
 0002:0000f328       ??_C@_03FCCPIJGJ@Pos@      1005b328     service.obj
 0002:0000f32c       ??_C@_08NNKIOIN@TypeName@  1005b32c     service.obj
 0002:0000f338       ??_C@_07ONPPLIAF@ErrCode@  1005b338     service.obj
 0002:0000f340       ??_C@_07LJDOKIBM@ErrPosX@  1005b340     service.obj
 0002:0000f348       ??_C@_07KACFJJFN@ErrPosY@  1005b348     service.obj
 0002:0000f350       ??_C@_06HBEFEBCM@ErrSrc@   1005b350     service.obj
 0002:0000f358       ??_C@_06LDIMCHFC@?$CF?$CKs?$CFs?5@ 1005b358     service.obj
 0002:0000f360       ??_C@_09HNJDNMKK@?$CF?$CF?$CFdd?$CF?$CFs?5@ 1005b360     service.obj
 0002:0000f36c       ??_C@_0CC@JIGPFMKG@global?5?$GAtostring?8?5is?5not?5functi@ 1005b36c     service.obj
 0002:0000f390       ??_C@_0CH@OINAPBOJ@tostring?$CI?$CJ?5returned?5a?5non?9strin@ 1005b390     service.obj
 0002:0000f3b8       ??_C@_04CIMGMMMG@text@     1005b3b8     service.obj
 0002:0000f3c0       ??_C@_03CAOIPBNL@arg@      1005b3c0     service.obj
 0002:0000f3c8       ??_C@_0ME@JDKAEDFJ@local?5items?0n?$DN?4?4?4?6local?5bottom?$DN@ 1005b3c8     service.obj
 0002:0000f48c       ??_C@_0CG@FGNNCNLL@attempt?5to?5access?5invalid?5file?5@ 1005b48c     service.obj
 0002:0000f4b4       ??_C@_07BJOIOONN@Strings@  1005b4b4     service.obj
 0002:0000f4bc       ??_C@_08FGAFMHLF@DiskMenu@ 1005b4bc     service.obj
 0002:0000f4c8       ??_C@_0L@NHENMPLN@PluginMenu@ 1005b4c8     service.obj
 0002:0000f4d4       ??_C@_0N@IEACHFBM@PluginConfig@ 1005b4d4     service.obj
 0002:0000f4e4       ??_C@_05GCJGCMFJ@PInfo@    1005b4e4     service.obj
 0002:0000f4ec       ??_C@_05HMEFBOHK@GInfo@    1005b4ec     service.obj
 0002:0000f4f4       ??_C@_0N@GAMEMCEE@invalid?5GUID@ 1005b4f4     service.obj
 0002:0000f504       ??_C@_0BP@NJEEOHDB@attempt?5to?5access?5closed?5timer@ 1005b504     service.obj
 0002:0000f524       ??_C@_05LGELBCGM@Close@    1005b524     service.obj
 0002:0000f52c       ??_C@_07DOAOMMKG@Enabled@  1005b52c     service.obj
 0002:0000f534       ??_C@_08KDKDEPAG@Interval@ 1005b534     service.obj
 0002:0000f540       ??_C@_07CIINKFND@OnTimer@  1005b540     service.obj
 0002:0000f548       ??_C@_06EFCDMIMC@Closed@   1005b548     service.obj
 0002:0000f550       ??_C@_0CE@LHJCBGGH@attempt?5to?5call?5non?9existent?5me@ 1005b550     service.obj
 0002:0000f574       ??_C@_0BO@PNFLEJKN@attempt?5to?5access?5a?5closed?5?$CFs@ 1005b574     service.obj
 0002:0000f594       ??_C@_04OKOFBOPB@Time@     1005b594     service.obj
 0002:0000f59c       ??_C@_04LADJNOK@Lock@      1005b59c     service.obj
 0002:0000f5a4       ??_C@_09KFKKEOOH@GetFilesW@ 1005b5a4     service.obj
 0002:0000f5b0       ??_C@_0BE@OGGJBMCE@insufficient?5memory@ 1005b5b0     service.obj
 0002:0000f5c4       ??_C@_09MMBIJGAH@PutFilesW@ 1005b5c4     service.obj
 0002:0000f5d0       ??_C@_0N@HPKKMFEI@GetFindDataW@ 1005b5d0     service.obj
 0002:0000f5e0       ??_C@_0O@GNDAADHN@FreeFindDataW@ 1005b5e0     service.obj
 0002:0000f5f0       ??_C@_0O@BCOALCIL@SetDirectoryW@ 1005b5f0     service.obj
 0002:0000f600       ??_C@_0P@LKPINHLK@FreeFileFilter@ 1005b600     service.obj
 0002:0000f610       ??_C@_0BA@JGEOEAE@OpenFiltersMenu@ 1005b610     service.obj
 0002:0000f620       ??_C@_0BB@OPPOFOAK@StartingToFilter@ 1005b620     service.obj
 0002:0000f634       ??_C@_0P@JDMCHDIM@IsFileInFilter@ 1005b634     service.obj
 0002:0000f644       ??_C@_04MIIPNNEF@send@     1005b644     service.obj
 0002:0000f64c       ??_C@_06JBKGCNBB@Delete@   1005b64c     service.obj
 0002:0000f654       ??_C@_04PAFOOALK@Enum@     1005b654     service.obj
 0002:0000f65c       ??_C@_04HJMOFLDF@Free@     1005b65c     service.obj
 0002:0000f664       ??_C@_03NNDHPFFO@Get@      1005b664     service.obj
 0002:0000f668       ??_C@_03CEMDFJG@Set@       1005b668     service.obj
 0002:0000f66c       ??_C@_0N@OELJMCEC@CreateSubkey@ 1005b66c     service.obj
 0002:0000f67c       ??_C@_0L@CPCKAMD@OpenSubkey@ 1005b67c     service.obj
 0002:0000f688       ??_C@_08EGJLHNCO@AddColor@ 1005b688     service.obj
 0002:0000f694       ??_C@_0BD@DOFEEDDC@AddSessionBookmark@ 1005b694     service.obj
 0002:0000f6a8       ??_C@_0BG@IGFHDIIN@ClearSessionBookmarks@ 1005b6a8     service.obj
 0002:0000f6c0       ??_C@_08PDEJHGJI@DelColor@ 1005b6c0     service.obj
 0002:0000f6cc       ??_C@_0M@LPIECDD@DeleteBlock@ 1005b6cc     service.obj
 0002:0000f6d8       ??_C@_0L@BCLIBKOC@DeleteChar@ 1005b6d8     service.obj
 0002:0000f6e4       ??_C@_0BG@KOELEFCN@DeleteSessionBookmark@ 1005b6e4     service.obj
 0002:0000f6fc       ??_C@_0N@EKENACAE@DeleteString@ 1005b6fc     service.obj
 0002:0000f70c       ??_C@_06MJDIICIN@Editor@   1005b70c     service.obj
 0002:0000f714       ??_C@_0L@HDLPOLMA@ExpandTabs@ 1005b714     service.obj
 0002:0000f720       ??_C@_0N@MGAOADJN@GetBookmarks@ 1005b720     service.obj
 0002:0000f730       ??_C@_08JOPFJIPE@GetColor@ 1005b730     service.obj
 0002:0000f73c       ??_C@_0M@FECPLAMN@GetFileName@ 1005b73c     service.obj
 0002:0000f748       ??_C@_07NAJNLNAF@GetInfo@  1005b748     service.obj
 0002:0000f750       ??_C@_0N@KIILHCLH@GetSelection@ 1005b750     service.obj
 0002:0000f760       ??_C@_0BE@LBJJGOGD@GetSessionBookmarks@ 1005b760     service.obj
 0002:0000f774       ??_C@_09HBLKHMEA@GetString@ 1005b774     service.obj
 0002:0000f780       ??_C@_0L@IDFHDAHP@GetStringW@ 1005b780     service.obj
 0002:0000f78c       ??_C@_0N@ICPGLOEG@InsertString@ 1005b78c     service.obj
 0002:0000f79c       ??_C@_0L@JMOIGJIA@InsertText@ 1005b79c     service.obj
 0002:0000f7a8       ??_C@_0M@BINOKANK@InsertTextW@ 1005b7a8     service.obj
 0002:0000f7b4       ??_C@_0BE@CNGODNDI@NextSessionBookmark@ 1005b7b4     service.obj
 0002:0000f7c8       ??_C@_0BE@IEBIGOAP@PrevSessionBookmark@ 1005b7c8     service.obj
 0002:0000f7dc       ??_C@_0N@FNCEPAJJ@ProcessInput@ 1005b7dc     service.obj
 0002:0000f7ec       ??_C@_04GMBKPCGK@Quit@     1005b7ec     service.obj
 0002:0000f7f4       ??_C@_09KINLOJJJ@ReadInput@ 1005b7f4     service.obj
 0002:0000f800       ??_C@_09DBPLBJBJ@RealToTab@ 1005b800     service.obj
 0002:0000f80c       ??_C@_06KAPLBEK@Redraw@    1005b80c     service.obj
 0002:0000f814       ??_C@_08FBDDPFPJ@SaveFile@ 1005b814     service.obj
 0002:0000f820       ??_C@_06HJGPBJLE@Select@   1005b820     service.obj
 0002:0000f828       ??_C@_09PPEOOGEC@SetKeyBar@ 1005b828     service.obj
 0002:0000f834       ??_C@_08CCKJEGOF@SetParam@ 1005b834     service.obj
 0002:0000f840       ??_C@_0M@GKIFPNAD@SetPosition@ 1005b840     service.obj
 0002:0000f84c       ??_C@_09FPPPFNNC@SetString@ 1005b84c     service.obj
 0002:0000f858       ??_C@_0L@JNHIIHDG@SetStringW@ 1005b858     service.obj
 0002:0000f864       ??_C@_08GMCCAJLF@SetTitle@ 1005b864     service.obj
 0002:0000f870       ??_C@_08JNAOBKMI@GetTitle@ 1005b870     service.obj
 0002:0000f87c       ??_C@_0BF@LIMPGNED@SubscribeChangeEvent@ 1005b87c     service.obj
 0002:0000f894       ??_C@_09JFBCONJH@TabToReal@ 1005b894     service.obj
 0002:0000f8a0       ??_C@_08IBJJAHJG@UndoRedo@ 1005b8a0     service.obj
 0002:0000f8ac       ??_C@_07JMDLHPJF@SetMode@  1005b8ac     service.obj
 0002:0000f8b4       ??_C@_06PJECNADJ@Viewer@   1005b8b4     service.obj
 0002:0000f8bc       ??_C@_0P@OAACIGEB@BeginSelection@ 1005b8bc     service.obj
 0002:0000f8cc       ??_C@_0BB@PJGDGIKA@CheckPanelsExist@ 1005b8cc     service.obj
 0002:0000f8e0       ??_C@_0P@DFBDDHFA@ClearSelection@ 1005b8e0     service.obj
 0002:0000f8f0       ??_C@_0N@BHLDKHDJ@EndSelection@ 1005b8f0     service.obj
 0002:0000f900       ??_C@_0L@KOHCMOPM@GetCmdLine@ 1005b900     service.obj
 0002:0000f90c       ??_C@_0O@NLDIMJEA@GetCmdLinePos@ 1005b90c     service.obj
 0002:0000f91c       ??_C@_0BE@CBPLLCEH@GetCmdLineSelection@ 1005b91c     service.obj
 0002:0000f930       ??_C@_0P@CMFANDFM@GetColumnTypes@ 1005b930     service.obj
 0002:0000f940       ??_C@_0BA@DJGLDCBG@GetColumnWidths@ 1005b940     service.obj
 0002:0000f950       ??_C@_0BE@JPAIJBCI@GetCurrentPanelItem@ 1005b950     service.obj
 0002:0000f964       ??_C@_0BC@NGKPIKGL@GetPanelDirectory@ 1005b964     service.obj
 0002:0000f978       ??_C@_0P@GODLFFFJ@GetPanelFormat@ 1005b978     service.obj
 0002:0000f988       ??_C@_0BB@LCMBHPNI@GetPanelHostFile@ 1005b988     service.obj
 0002:0000f99c       ??_C@_0N@HPIPGDFA@GetPanelInfo@ 1005b99c     service.obj
 0002:0000f9ac       ??_C@_0N@HAFLAIHA@GetPanelItem@ 1005b9ac     service.obj
 0002:0000f9bc       ??_C@_0P@HCBKDPMP@GetPanelPrefix@ 1005b9bc     service.obj
 0002:0000f9cc       ??_C@_0BF@MEMFMMGB@GetSelectedPanelItem@ 1005b9cc     service.obj
 0002:0000f9e4       ??_C@_0O@HEGDGAJG@GetUserScreen@ 1005b9e4     service.obj
 0002:0000f9f4       ??_C@_0O@EHOCCHAL@InsertCmdLine@ 1005b9f4     service.obj
 0002:0000fa04       ??_C@_0O@OMMHIHHH@IsActivePanel@ 1005ba04     service.obj
 0002:0000fa14       ??_C@_0M@LCEPDNPK@RedrawPanel@ 1005ba14     service.obj
 0002:0000fa20       ??_C@_0P@OPKJJMLB@SetActivePanel@ 1005ba20     service.obj
 0002:0000fa30       ??_C@_0L@LAFNHJLF@SetCmdLine@ 1005ba30     service.obj
 0002:0000fa3c       ??_C@_0O@KECGHKDH@SetCmdLinePos@ 1005ba3c     service.obj
 0002:0000fa4c       ??_C@_0BE@IPNAPCDL@SetCmdLineSelection@ 1005ba4c     service.obj
 0002:0000fa60       ??_C@_0BE@PAPEKLCP@SetDirectoriesFirst@ 1005ba60     service.obj
 0002:0000fa74       ??_C@_0BC@PDKEABHF@SetPanelDirectory@ 1005ba74     service.obj
 0002:0000fa88       ??_C@_0N@NMDFLOPL@SetSelection@ 1005ba88     service.obj
 0002:0000fa98       ??_C@_0M@CMMMGIDG@SetSortMode@ 1005ba98     service.obj
 0002:0000faa4       ??_C@_0N@HCHLALN@SetSortOrder@ 1005baa4     service.obj
 0002:0000fab4       ??_C@_0O@LHNNDOB@SetUserScreen@ 1005bab4     service.obj
 0002:0000fac4       ??_C@_0M@IENJPEBA@SetViewMode@ 1005bac4     service.obj
 0002:0000fad0       ??_C@_0M@EICBHAOA@UpdatePanel@ 1005bad0     service.obj
 0002:0000fadc       ??_C@_0BC@BIIKJLKB@PluginStartupInfo@ 1005badc     service.obj
 0002:0000faf0       ??_C@_0L@PJAHNOGM@DialogInit@ 1005baf0     service.obj
 0002:0000fafc       ??_C@_09DBEDLMHB@DialogRun@ 1005bafc     service.obj
 0002:0000fb08       ??_C@_0L@DLFLHLOO@DialogFree@ 1005bb08     service.obj
 0002:0000fb14       ??_C@_0P@HLOFPDFP@SendDlgMessage@ 1005bb14     service.obj
 0002:0000fb24       ??_C@_0L@CKELNLCE@GetDlgItem@ 1005bb24     service.obj
 0002:0000fb30       ??_C@_0L@DEGEGMGN@SetDlgItem@ 1005bb30     service.obj
 0002:0000fb3c       ??_C@_0BK@EBIPEKDH@SubscribeDialogDrawEvents@ 1005bb3c     service.obj
 0002:0000fb58       ??_C@_0L@MCFABBED@GetDirList@ 1005bb58     service.obj
 0002:0000fb64       ??_C@_06KCCBBIBJ@GetMsg@   1005bb64     service.obj
 0002:0000fb6c       ??_C@_0BB@HIDBFOJJ@GetPluginDirList@ 1005bb6c     service.obj
 0002:0000fb80       ??_C@_04IFEHPILC@Menu@     1005bb80     service.obj
 0002:0000fb88       ??_C@_07BEIHKDLJ@Message@  1005bb88     service.obj
 0002:0000fb90       ??_C@_0O@CGLFPNOD@RestoreScreen@ 1005bb90     service.obj
 0002:0000fba0       ??_C@_0L@PGGGPLFK@SaveScreen@ 1005bba0     service.obj
 0002:0000fbac       ??_C@_0L@HABDNHIM@FreeScreen@ 1005bbac     service.obj
 0002:0000fbb8       ??_C@_08DAHHHDJC@ShowHelp@ 1005bbb8     service.obj
 0002:0000fbc4       ??_C@_08IAADAJIH@InputBox@ 1005bbc4     service.obj
 0002:0000fbd0       ??_C@_0L@HHLOIHOP@AdvControl@ 1005bbd0     service.obj
 0002:0000fbdc       ??_C@_0N@GHGEMEN@MacroLoadAll@ 1005bbdc     service.obj
 0002:0000fbec       ??_C@_0N@NAGBAPAE@MacroSaveAll@ 1005bbec     service.obj
 0002:0000fbfc       ??_C@_0O@KGHDMPAJ@MacroGetState@ 1005bbfc     service.obj
 0002:0000fc0c       ??_C@_0N@PNLHCOIE@MacroGetArea@ 1005bc0c     service.obj
 0002:0000fc1c       ??_C@_09KGKKBHMO@MacroPost@ 1005bc1c     service.obj
 0002:0000fc28       ??_C@_0L@KBAKOGFP@MacroCheck@ 1005bc28     service.obj
 0002:0000fc34       ??_C@_08KAFLEHAN@MacroAdd@ 1005bc34     service.obj
 0002:0000fc40       ??_C@_0M@KFMHCNNB@MacroDelete@ 1005bc40     service.obj
 0002:0000fc4c       ??_C@_0BC@MJDKBAPF@MacroGetLastError@ 1005bc4c     service.obj
 0002:0000fc60       ??_C@_0N@COEPENFH@MacroExecute@ 1005bc60     service.obj
 0002:0000fc70       ??_C@_0BB@BICELPOF@CreateFileFilter@ 1005bc70     service.obj
 0002:0000fc84       ??_C@_0L@CHJBHF@LoadPlugin@ 1005bc84     service.obj
 0002:0000fc90       ??_C@_0N@DHIONCLI@UnloadPlugin@ 1005bc90     service.obj
 0002:0000fca0       ??_C@_0BB@IJHIBGJA@ForcedLoadPlugin@ 1005bca0     service.obj
 0002:0000fcb4       ??_C@_0L@DACPHGGH@FindPlugin@ 1005bcb4     service.obj
 0002:0000fcc0       ??_C@_0BF@KLOGLFMF@GetPluginInformation@ 1005bcc0     service.obj
 0002:0000fcd8       ??_C@_0L@JIDCIJHM@GetPlugins@ 1005bcd8     service.obj
 0002:0000fce4       ??_C@_0P@IKAEEPOB@IsPluginLoaded@ 1005bce4     service.obj
 0002:0000fcf4       ??_C@_0P@HMKEDHIE@CreateSettings@ 1005bcf4     service.obj
 0002:0000fd04       ??_C@_0N@GOMOBHDB@FreeSettings@ 1005bd04     service.obj
 0002:0000fd14       ??_C@_0M@IFKFGKML@ColorDialog@ 1005bd14     service.obj
 0002:0000fd20       ??_C@_0BA@EOCNNPOG@CopyToClipboard@ 1005bd20     service.obj
 0002:0000fd30       ??_C@_0BD@PLIHDKFC@PasteFromClipboard@ 1005bd30     service.obj
 0002:0000fd44       ??_C@_0BC@FJDIKOMH@InputRecordToName@ 1005bd44     service.obj
 0002:0000fd58       ??_C@_0BC@FFNOIDFI@NameToInputRecord@ 1005bd58     service.obj
 0002:0000fd6c       ??_C@_08HGLFNLMB@LStricmp@ 1005bd6c     service.obj
 0002:0000fd78       ??_C@_09GALOFBAC@LStrnicmp@ 1005bd78     service.obj
 0002:0000fd84       ??_C@_0M@KPPMMAOL@ProcessName@ 1005bd84     service.obj
 0002:0000fd90       ??_C@_0M@KFCNKLDK@GetPathRoot@ 1005bd90     service.obj
 0002:0000fd9c       ??_C@_0BE@EPGHGPJC@GetReparsePointInfo@ 1005bd9c     service.obj
 0002:0000fdb0       ??_C@_08DNJCLFF@LIsAlpha@  1005bdb0     service.obj
 0002:0000fdbc       ??_C@_0M@LKJIEECA@LIsAlphanum@ 1005bdbc     service.obj
 0002:0000fdc8       ??_C@_08MAHKICD@LIsLower@  1005bdc8     service.obj
 0002:0000fdd4       ??_C@_08FHLJMDJK@LIsUpper@ 1005bdd4     service.obj
 0002:0000fde0       ??_C@_09LPKAHGM@LLowerBuf@ 1005bde0     service.obj
 0002:0000fdec       ??_C@_09GLKFOOEP@LUpperBuf@ 1005bdec     service.obj
 0002:0000fdf8       ??_C@_06ILCHIEBO@MkTemp@   1005bdf8     service.obj
 0002:0000fe00       ??_C@_06DKBBJCCG@MkLink@   1005be00     service.obj
 0002:0000fe08       ??_C@_0N@CCDDAJK@TruncPathStr@ 1005be08     service.obj
 0002:0000fe18       ??_C@_08BNEIIKEJ@TruncStr@ 1005be18     service.obj
 0002:0000fe24       ??_C@_0BA@CLEHBIPM@RecursiveSearch@ 1005be24     service.obj
 0002:0000fe34       ??_C@_0M@HKHGOOHG@ConvertPath@ 1005be34     service.obj
 0002:0000fe40       ??_C@_04OCDKHGII@XLat@     1005be40     service.obj
 0002:0000fe48       ??_C@_0P@BGLLKGOI@FormatFileSize@ 1005be48     service.obj
 0002:0000fe58       ??_C@_08KJBLDCDF@FarClock@ 1005be58     service.obj
 0002:0000fe64       ??_C@_0BD@ELMHPHAC@CPluginStartupInfo@ 1005be64     service.obj
 0002:0000fe78       ??_C@_0BE@DJLJEKBK@GetCurrentDirectory@ 1005be78     service.obj
 0002:0000fe8c       ??_C@_0N@MOMBJEKA@GetFileOwner@ 1005be8c     service.obj
 0002:0000fe9c       ??_C@_0BB@JBNBALEM@GetNumberOfLinks@ 1005be9c     service.obj
 0002:0000feb0       ??_C@_0BB@OPAJHEIC@GetLuafarVersion@ 1005beb0     service.obj
 0002:0000fec4       ??_C@_0O@BJEAJNBH@MakeMenuItems@ 1005bec4     service.obj
 0002:0000fed4       ??_C@_0BB@HLFLDCHO@RunDefaultScript@ 1005bed4     service.obj
 0002:0000fee8       ??_C@_04JLAJABDJ@Show@     1005bee8     service.obj
 0002:0000fef0       ??_C@_05NHFJDMOA@Timer@    1005bef0     service.obj
 0002:0000fef8       ??_C@_0BD@KCMHFGFP@FileTimeResolution@ 1005bef8     service.obj
 0002:0000ff0c       ??_C@_04CPPPJGME@Host@     1005bf0c     service.obj
 0002:0000ff14       ??_C@_0N@ECMJOJJG@MacroCallFar@ 1005bf14     service.obj
 0002:0000ff24       ??_C@_0BC@JJHHFNMP@FarMacroCallToLua@ 1005bf24     service.obj
 0002:0000ff38       ??_C@_06GIFLLBB@editor@    1005bf38     service.obj
 0002:0000ff40       ??_C@_06DGPPOJKF@viewer@   1005bf40     service.obj
 0002:0000ff48       ??_C@_01DICPFPGM@k@        1005bf48     service.obj
 0002:0000ff4c       ??_C@_06BPGFKLEK@__mode@   1005bf4c     service.obj
 0002:0000ff54       ??_C@_1CC@OPOAGCKN@?$AA?2?$AAl?$AAu?$AAa?$AAf?$AAa?$AAr?$AA_?$AAi?$AAn?$AAi?$AAt?$AA?4?$AAl?$AAu@ 1005bf54     service.obj
 0002:0000ff78       ??_C@_1BG@BDOBMIBP@?$AAF?$AAA?$AAR?$AAP?$AAR?$AAO?$AAF?$AAI?$AAL?$AAE@ 1005bf78     service.obj
 0002:0000ff90       ??_C@_02KFNNKBCK@io@       1005bf90     service.obj
 0002:0000ff94       ??_C@_02EHCHIAMF@os@       1005bf94     service.obj
 0002:0000ff98       ??_C@_04CFDJAKFL@math@     1005bf98     service.obj
 0002:0000ffa0       ??_C@_07GAJMMAJO@unicode@  1005bfa0     service.obj
 0002:0000ffa8       ??_C@_04LHHHFLPP@utf8@     1005bfa8     service.obj
 0002:0000ffb0       ??_C@_03JECLAOEA@win@      1005bfb0     service.obj
 0002:0000ffb4       ??_C@_05NDNJFBEF@cfind@    1005bfb4     service.obj
 0002:0000ffbc       ??_C@_03EDMBFDDG@bit@      1005bfbc     service.obj
 0002:0000ffc0       ??_C@_03IGHFHLNJ@jit@      1005bfc0     service.obj
 0002:0000ffc4       ??_C@_08LBNNGFKE@_PRELOAD@ 1005bfc4     service.obj
 0002:0000ffd0       ??_C@_03DIJDOPEA@ffi@      1005bfd0     service.obj
 0002:0000ffd4       ??_C@_06ONNDGCDK@dofile@   1005bfd4     service.obj
 0002:0000ffdc       ??_C@_08BNNFLGCJ@loadfile@ 1005bfdc     service.obj
 0002:0000ffe8       ??_C@_06JLGJNGCD@luafar@   1005bfe8     service.obj
 0002:0000fff0       ??_C@_03OFAPEBGM@?$CFs?6@  1005bff0     service.obj
 0002:0000fff4       _filefilter_methods        1005bff4     service.obj
 0002:0001002c       _SettingsType              1005c02c     service.obj
 0002:00010040       _VirtualKeyStrings         1005c040     service.obj
 0002:00010440       _FAR_FLAGSTABLE            1005c440     service.obj
 0002:0001044c       _SettingsHandles           1005c44c     service.obj
 0002:00010468       _FAKE_PLUGIN_DATA_KEY      1005c468     service.obj
 0002:00010478       _SavedScreenType           1005c478     service.obj
 0002:00010488       _editor_funcs              1005c488     service.obj
 0002:000105d0       _panel_funcs               1005c5d0     service.obj
 0002:000106e8       _far_Dialog                1005c6e8     service.obj
 0002:00010918       _FarTimerType              1005c918     service.obj
 0002:00010924       _FarTimerQueueKey          1005c924     service.obj
 0002:00010950       _api_functions             1005c950     service.obj
 0002:000109bc       _far_host_funcs            1005c9bc     service.obj
 0002:000109f0       _far_funcs                 1005c9f0     service.obj
 0002:00010c78       _FAR_DN_STORAGE            1005cc78     service.obj
 0002:00010cf8       _timer_methods             1005ccf8     service.obj
 0002:00010d20       _dialog_methods            1005cd20     service.obj
 0002:00010d48       _FarFileFilterType         1005cd48     service.obj
 0002:00010d58       _viewer_funcs              1005cd58     service.obj
 0002:00010da8       _Settings_methods          1005cda8     service.obj
 0002:00010df8       _FAR_VIRTUALKEYS           1005cdf8     service.obj
 0002:00010e10       _FarDialogType             1005ce10     service.obj
 0002:00010e1c       _AddMacroDataType          1005ce1c     service.obj
 0002:00010e34       _PluginHandleType          1005ce34     service.obj
 0002:00010e44       ??_C@_0BO@BNLBHKJN@unable?5to?5dump?5given?5function@ 1005ce44     slnunico.obj
 0002:00010e64       ??_C@_02HIBBOKEN@?2r@      1005ce64     slnunico.obj
 0002:00010e68       ??_C@_04MPDIABOK@?2000@    1005ce68     slnunico.obj
 0002:00010e70       ??_C@_05GGBDHNF@?9?$CL?5?$CD0@ 1005ce70     slnunico.obj
 0002:00010e78       ??_C@_0CA@COOMGCAO@invalid?5format?5?$CIrepeated?5flags?$CJ@ 1005ce78     slnunico.obj
 0002:00010e98       ??_C@_0CN@KALFEKPN@invalid?5format?5?$CIwidth?5or?5precis@ 1005ce98     slnunico.obj
 0002:00010ec8       ??_C@_0CC@KIPBEOBI@invalid?5option?5?8?$CF?$CF?$CFc?8?5to?5?8forma@ 1005cec8     slnunico.obj
 0002:00010eec       ??_C@_04GGLOKIEE@dump@     1005ceec     slnunico.obj
 0002:00010ef4       ??_C@_06DLEPGFEF@format@   1005cef4     slnunico.obj
 0002:00010efc       ??_C@_03HOKODIMJ@rep@      1005cefc     slnunico.obj
 0002:00010f00       ??_C@_09GCBMKPBD@utf8valid@ 1005cf00     slnunico.obj
 0002:00010f34       ??_C@_0BE@LDJANOJE@?$CFs?5expected?0?5got?5?$CFs@ 1005cf34     lutf8lib.obj
 0002:00010f48       ??_C@_0BD@MJACNLBA@invalid?5UTF?98?5code@ 1005cf48     lutf8lib.obj
 0002:00010f5c       ??_C@_0BP@MEEJFMAG@initial?5position?5out?5of?5string@ 1005cf5c     lutf8lib.obj
 0002:00010f7c       ??_C@_0BN@IINPNO@final?5position?5out?5of?5string@ 1005cf7c     lutf8lib.obj
 0002:00010f9c       ??_C@_0N@FCPHIMMG@out?5of?5range@ 1005cf9c     lutf8lib.obj
 0002:00010fac       ??_C@_0BG@DFAIEAEC@string?5slice?5too?5long@ 1005cfac     lutf8lib.obj
 0002:00010fc4       ??_C@_0BD@JFBPAFFP@value?5out?5of?5range@ 1005cfc4     lutf8lib.obj
 0002:00010fd8       ??_C@_0O@FJKLBAIJ@number?1string@ 1005cfd8     lutf8lib.obj
 0002:00010fe8       ??_C@_0BE@MHMGJPCL@invalid?5escape?5?8?$CFc?8@ 1005cfe8     lutf8lib.obj
 0002:00010ffc       ??_C@_0O@BGLHAEFA@invalid?5index@ 1005cffc     lutf8lib.obj
 0002:0001100c       ??_C@_0BG@OBAFCJJL@position?5out?5of?5range@ 1005d00c     lutf8lib.obj
 0002:00011024       ??_C@_0CI@HDBIKOFJ@initial?5position?5is?5a?5continuat@ 1005d024     lutf8lib.obj
 0002:0001104c       ??_C@_0BL@JNACDPC@invalid?5capture?5index?5?$CF?$CF?$CFd@ 1005d04c     lutf8lib.obj
 0002:00011068       ??_C@_0BI@ECNPHIBF@invalid?5pattern?5capture@ 1005d068     lutf8lib.obj
 0002:00011080       ??_C@_0CD@PLJBIEHA@malformed?5pattern?5?$CIends?5with?5?8?$CF@ 1005d080     lutf8lib.obj
 0002:000110a4       ??_C@_0CA@CFGACOGB@malformed?5pattern?5?$CImissing?5?8?$FN?8?$CJ@ 1005d0a4     lutf8lib.obj
 0002:000110c4       ??_C@_0CP@FCNHBCLO@malformed?5pattern?5?$CImissing?5argu@ 1005d0c4     lutf8lib.obj
 0002:000110f4       ??_C@_0BC@IMEAEJPD@too?5many?5captures@ 1005d0f4     lutf8lib.obj
 0002:00011108       ??_C@_0BE@LPFFPFJG@pattern?5too?5complex@ 1005d108     lutf8lib.obj
 0002:0001111c       ??_C@_0CD@LOJJMDBH@missing?5?8?$FL?8?5after?5?8?$CF?$CFf?8?5in?5patt@ 1005d11c     lutf8lib.obj
 0002:00011140       ??_C@_0BG@LEHNKOGD@invalid?5capture?5index@ 1005d140     lutf8lib.obj
 0002:00011158       ??_C@_0BD@BFKNEALP@unfinished?5capture@ 1005d158     lutf8lib.obj
 0002:0001116c       ??_C@_0L@NLFJOONJ@?$FO$?$CK?$CL?$DP?4?$CI?$FL?$CF?9@ 1005d16c     lutf8lib.obj
 0002:00011178       ??_C@_0CK@KLCOLAN@invalid?5use?5of?5?8?$CFc?8?5in?5replacem@ 1005d178     lutf8lib.obj
 0002:000111a4       ??_C@_0CB@LPDIHGGA@invalid?5replacement?5value?5?$CIa?5?$CFs@ 1005d1a4     lutf8lib.obj
 0002:000111c8       ??_C@_0BP@PPPOBACA@string?1function?1table?5expected@ 1005d1c8     lutf8lib.obj
 0002:000111e8       ??_C@_06KLHHMIGM@offset@   1005d1e8     lutf8lib.obj
 0002:000111f0       ??_C@_05CFHFIAJO@codes@    1005d1f0     lutf8lib.obj
 0002:000111f8       ??_C@_09HHCEKEIA@codepoint@ 1005d1f8     lutf8lib.obj
 0002:00011204       ??_C@_03BKCJCHLK@len@      1005d204     lutf8lib.obj
 0002:00011208       ??_C@_07KOIEOCCE@reverse@  1005d208     lutf8lib.obj
 0002:00011210       ??_C@_05IPJEPLHL@lower@    1005d210     lutf8lib.obj
 0002:00011218       ??_C@_05NECKJAMC@upper@    1005d218     lutf8lib.obj
 0002:00011220       ??_C@_05PHLGJONK@title@    1005d220     lutf8lib.obj
 0002:00011228       ??_C@_04MLGPBLN@fold@      1005d228     lutf8lib.obj
 0002:00011230       ??_C@_04IHGKJMLH@byte@     1005d230     lutf8lib.obj
 0002:00011238       ??_C@_04ENMBGAPA@char@     1005d238     lutf8lib.obj
 0002:00011240       ??_C@_06CHNIFGOF@escape@   1005d240     lutf8lib.obj
 0002:00011248       ??_C@_06OAOPNKHP@insert@   1005d248     lutf8lib.obj
 0002:00011250       ??_C@_06LEMKAMD@remove@    1005d250     lutf8lib.obj
 0002:00011258       ??_C@_07BAPMOMKI@charpos@  1005d258     lutf8lib.obj
 0002:00011260       ??_C@_04CJGEDOF@next@      1005d260     lutf8lib.obj
 0002:00011268       ??_C@_05IGKADHGO@width@    1005d268     lutf8lib.obj
 0002:00011270       ??_C@_0L@OLBIGGEG@widthindex@ 1005d270     lutf8lib.obj
 0002:0001127c       ??_C@_08GEDFKPFE@ncasecmp@ 1005d27c     lutf8lib.obj
 0002:00011288       ??_C@_0M@GMACFGDH@charpattern@ 1005d288     lutf8lib.obj
 0002:000112c0       ??_C@_05DFJCHPDH@input@    1005d2c0     uliolib51.obj
 0002:000112c8       ??_C@_06DKIGHACF@output@   1005d2c8     uliolib51.obj
 0002:000112d0       ??_C@_06DJHOIPC@?$CFs?3?5?$CFs@ 1005d2d0     uliolib51.obj
 0002:000112d8       ??_C@_02DKCKIIND@?$CFs@    1005d2d8     uliolib51.obj
 0002:000112dc       ??_C@_05KCHOJJD@FILE?$CK@  1005d2dc     uliolib51.obj
 0002:000112e4       ??_C@_0M@IBKPHHKH@closed?5file@ 1005d2e4     uliolib51.obj
 0002:000112f0       ??_C@_04DAMGJPCA@file@     1005d2f0     uliolib51.obj
 0002:000112f8       ??_C@_0BN@LPOOHAOM@attempt?5to?5use?5a?5closed?5file@ 1005d2f8     uliolib51.obj
 0002:00011318       ??_C@_0BL@PEFGCPAG@cannot?5close?5standard?5file@ 1005d318     uliolib51.obj
 0002:00011334       ??_C@_07DMJMBBKE@__close@  1005d334     uliolib51.obj
 0002:0001133c       ??_C@_0O@PLFAPHPG@file?5?$CIclosed?$CJ@ 1005d33c     uliolib51.obj
 0002:0001134c       ??_C@_09BPMAMLLD@file?5?$CI?$CFp?$CJ@ 1005d34c     uliolib51.obj
 0002:00011358       ??_C@_17OBBFBLGE@?$AAr?$AAw?$AAa@ 1005d358     uliolib51.obj
 0002:00011360       ??_C@_0CP@DHGANCPP@invalid?5mode?5?8?$CFs?8?5?$CIshould?5match@ 1005d360     uliolib51.obj
 0002:00011390       ??_C@_0BL@JMNLNGCA@standard?5?$CFs?5file?5is?5closed@ 1005d390     uliolib51.obj
 0002:000113ac       ??_C@_13CIFDLIMG@?$AAw@    1005d3ac     uliolib51.obj
 0002:000113b0       ??_C@_03DLDNIBIK@?$CFlf@   1005d3b0     uliolib51.obj
 0002:000113b4       ??_C@_0BD@IOJAAODF@too?5many?5arguments@ 1005d3b4     uliolib51.obj
 0002:000113c8       ??_C@_0P@PJFAGLMH@invalid?5option@ 1005d3c8     uliolib51.obj
 0002:000113d8       ??_C@_0P@CENJCLHM@invalid?5format@ 1005d3d8     uliolib51.obj
 0002:000113e8       ??_C@_0BH@PBGIDLEF@file?5is?5already?5closed@ 1005d3e8     uliolib51.obj
 0002:00011400       ??_C@_05CGOEHEFE@?$CF?414g@ 1005d400     uliolib51.obj
 0002:00011408       ??_C@_03KCHOJKKI@set@      1005d408     uliolib51.obj
 0002:0001140c       ??_C@_03LIBLMJMB@cur@      1005d40c     uliolib51.obj
 0002:00011410       ??_C@_03JBJLGPFL@end@      1005d410     uliolib51.obj
 0002:00011414       ??_C@_0BP@MGCOJADF@not?5an?5integer?5in?5proper?5range@ 1005d414     uliolib51.obj
 0002:00011434       ??_C@_02KAJCLHKP@no@       1005d434     uliolib51.obj
 0002:00011438       ??_C@_04PLMLMMEO@full@     1005d438     uliolib51.obj
 0002:00011440       ??_C@_04HJPCFDOP@line@     1005d440     uliolib51.obj
 0002:00011448       ??_C@_0DB@KKADAMFH@rawhandle?5is?5only?5available?5in?5@ 1005d448     uliolib51.obj
 0002:0001147c       ??_C@_05LBOHBHFK@close@    1005d47c     uliolib51.obj
 0002:00011484       ??_C@_05GLCAEPFP@flush@    1005d484     uliolib51.obj
 0002:0001148c       ??_C@_05DENOCHIP@lines@    1005d48c     uliolib51.obj
 0002:00011494       ??_C@_05IACAFMHP@popen@    1005d494     uliolib51.obj
 0002:0001149c       ??_C@_07FKJPAINK@tmpfile@  1005d49c     uliolib51.obj
 0002:000114a4       ??_C@_05NGFEDHGN@write@    1005d4a4     uliolib51.obj
 0002:000114ac       ??_C@_04EDECCOGL@seek@     1005d4ac     uliolib51.obj
 0002:000114b4       ??_C@_07HHBPNGAN@setvbuf@  1005d4b4     uliolib51.obj
 0002:000114bc       ??_C@_05MHOFLBOO@stdin@    1005d4bc     uliolib51.obj
 0002:000114c4       ??_C@_06DJDOIFHB@stdout@   1005d4c4     uliolib51.obj
 0002:000114cc       ??_C@_06FJGNEBG@stderr@    1005d4cc     uliolib51.obj
 0002:000115c8       ??_C@_0BN@GMPFCLAN@unable?5to?5get?5ModuleFileName@ 1005d5c8     uloadlib51.obj
 0002:000115e8       ??_C@_13MGDFOILI@?$AA?$CB@ 1005d5e8     uloadlib51.obj
 0002:000115ec       ??_C@_09GMLHALBF@LOADLIB?3?5@ 1005d5ec     uloadlib51.obj
 0002:000115f8       ??_C@_04HDOCAJNK@?$CFs?$CFs@ 1005d5f8     uloadlib51.obj
 0002:00011600       ??_C@_08HNNNOMMJ@_LOADLIB@ 1005d600     uloadlib51.obj
 0002:0001160c       ??_C@_04HKFDNBLD@init@     1005d60c     uloadlib51.obj
 0002:00011614       ??_C@_13FPGAJAPJ@?$AA?2@   1005d614     uloadlib51.obj
 0002:00011618       ??_C@_13JOFGPIOO@?$AA?4@   1005d618     uloadlib51.obj
 0002:0001161c       ??_C@_0BO@COFCKCAL@?8package?4?$CFs?8?5must?5be?5a?5string@ 1005d61c     uloadlib51.obj
 0002:0001163c       ??_C@_0CE@EPEHLLIH@?8package?4?$CFs?8?5contains?5invalid?5U@ 1005d63c     uloadlib51.obj
 0002:00011660       ??_C@_13HGPDMIBE@?$AA?$DP@ 1005d660     uloadlib51.obj
 0002:00011664       ??_C@_0P@NEBKIMDC@?6?7no?5file?5?8?$CFs?8@ 1005d664     uloadlib51.obj
 0002:00011674       ??_C@_0CO@KHMIPLKM@error?5loading?5module?5?8?$CFs?8?5from?5@ 1005d674     uloadlib51.obj
 0002:000116a4       ??_C@_04LNEJFJGI@path@     1005d6a4     uloadlib51.obj
 0002:000116ac       ??_C@_01IDAFKMJL@_@        1005d6ac     uloadlib51.obj
 0002:000116b0       ??_C@_01LFCBOECM@?4@       1005d6b0     uloadlib51.obj
 0002:000116b4       ??_C@_0L@KHKMBFOE@luaopen_?$CFs@ 1005d6b4     uloadlib51.obj
 0002:000116c0       ??_C@_05EEMJHCCC@cpath@    1005d6c0     uloadlib51.obj
 0002:000116c8       ??_C@_0BO@KOILFIGK@?6?7no?5module?5?8?$CFs?8?5in?5file?5?8?$CFs?8@ 1005d6c8     uloadlib51.obj
 0002:000116e8       ??_C@_0CC@CCJHFBLH@?8package?4preload?8?5must?5be?5a?5tab@ 1005d6e8     uloadlib51.obj
 0002:0001170c       ??_C@_0CB@NPNABMBF@?6?7no?5field?5package?4preload?$FL?8?$CFs?8@ 1005d70c     uloadlib51.obj
 0002:00011730       ??_C@_07PINPBNPB@_LOADED@  1005d730     uloadlib51.obj
 0002:00011738       ??_C@_0CL@DIEJCPFH@loop?5or?5previous?5error?5loading?5@ 1005d738     uloadlib51.obj
 0002:00011764       ??_C@_07JAOCDFCG@loaders@  1005d764     uloadlib51.obj
 0002:0001176c       ??_C@_0CC@IGEJMOFI@?8package?4loaders?8?5must?5be?5a?5tab@ 1005d76c     uloadlib51.obj
 0002:00011790       ??_C@_0BJ@HFHHABH@module?5?8?$CFs?8?5not?5found?3?$CFs@ 1005d790     uloadlib51.obj
 0002:000117ac       ??_C@_01INIBCBCB@f@        1005d7ac     uloadlib51.obj
 0002:000117b0       ??_C@_0CI@GKOMOAFD@?8module?8?5not?5called?5from?5a?5Lua?5@ 1005d7b0     uloadlib51.obj
 0002:000117d8       ??_C@_02CCIJHOCI@_M@       1005d7d8     uloadlib51.obj
 0002:000117dc       ??_C@_05ICMCJINN@_NAME@    1005d7dc     uloadlib51.obj
 0002:000117e4       ??_C@_08HONLOGDK@_PACKAGE@ 1005d7e4     uloadlib51.obj
 0002:000117f0       ??_C@_0BO@CBJIAGLF@name?5conflict?5for?5module?5?8?$CFs?8@ 1005d7f0     uloadlib51.obj
 0002:00011810       ??_C@_17KOAMMDLI@?$AA?$DL?$AA?$AB?$AA?$DL@ 1005d810     uloadlib51.obj
 0002:00011818       ??_C@_15HKKNGJC@?$AA?$DL?$AA?$DL@ 1005d818     uloadlib51.obj
 0002:00011820       ??_C@_13GGAHEHIG@?$AA?$AB@ 1005d820     uloadlib51.obj
 0002:00011824       ??_C@_07KOEABFCN@loadlib@  1005d824     uloadlib51.obj
 0002:0001182c       ??_C@_06LNOHAKGK@seeall@   1005d82c     uloadlib51.obj
 0002:00011834       ??_C@_06BIEEJMKO@module@   1005d834     uloadlib51.obj
 0002:0001183c       ??_C@_07FFLLPPLH@require@  1005d83c     uloadlib51.obj
 0002:00011848       ??_C@_1HE@JLDBNBHO@?$AA?4?$AA?2?$AA?$DP?$AA?4?$AAl?$AAu?$AAa?$AA?$DL?$AA?$CB?$AA?2?$AAl?$AAu?$AAa?$AA?2?$AA?$DP@ 1005d848     uloadlib51.obj
 0002:000118bc       ??_C@_1BC@ILFFIBFI@?$AAL?$AAU?$AAA?$AA_?$AAP?$AAA?$AAT?$AAH@ 1005d8bc     uloadlib51.obj
 0002:000118d0       ??_C@_1DM@FGPGEDD@?$AA?4?$AA?2?$AA?$DP?$AA?4?$AAd?$AAl?$AAl?$AA?$DL?$AA?$CB?$AA?2?$AA?$DP?$AA?4?$AAd?$AAl?$AAl@ 1005d8d0     uloadlib51.obj
 0002:0001190c       ??_C@_1BE@EFNILHBI@?$AAL?$AAU?$AAA?$AA_?$AAC?$AAP?$AAA?$AAT?$AAH@ 1005d90c     uloadlib51.obj
 0002:00011920       ??_C@_1BE@CKNDCMBB@?$AA?2?$AA?6?$AA?$DL?$AA?6?$AA?$DP?$AA?6?$AA?$CB?$AA?6?$AA?9@ 1005d920     uloadlib51.obj
 0002:00011934       ??_C@_06HEJKKHEK@config@   1005d934     uloadlib51.obj
 0002:0001193c       ??_C@_06IILMCCFO@loaded@   1005d93c     uloadlib51.obj
 0002:00011994       ??_C@_0BB@BLJKPILH@system?5error?5?$CFd?6@ 1005d994     ustring.obj
 0002:000119a8       ??_C@_0BJ@MEAJDMDL@invalid?5multibyte?5string@ 1005d9a8     ustring.obj
 0002:000119c4       ??_C@_0BG@ELIKBHAO@invalid?5UTF?916?5string@ 1005d9c4     ustring.obj
 0002:000119dc       ??_C@_0M@KJGJBDLL@MaxCharSize@ 1005d9dc     ustring.obj
 0002:000119e8       ??_C@_0M@IMOFNPBB@DefaultChar@ 1005d9e8     ustring.obj
 0002:000119f4       ??_C@_08HIIJAENB@LeadByte@ 1005d9f4     ustring.obj
 0002:00011a00       ??_C@_0BD@CBNPFFPH@UnicodeDefaultChar@ 1005da00     ustring.obj
 0002:00011a14       ??_C@_0N@DJCOCBOB@CodePageName@ 1005da14     ustring.obj
 0002:00011a24       ??_C@_0N@IFJMFGJK@unknown?5type@ 1005da24     ustring.obj
 0002:00011a34       ??_C@_0BC@GPFCFLGN@no?5root?5directory@ 1005da34     ustring.obj
 0002:00011a48       ??_C@_09HPGMKNKO@removable@ 1005da48     ustring.obj
 0002:00011a54       ??_C@_05OFLEIIDM@fixed@    1005da54     ustring.obj
 0002:00011a5c       ??_C@_06IMIHEKN@remote@    1005da5c     ustring.obj
 0002:00011a64       ??_C@_05POABADMF@cdrom@    1005da64     ustring.obj
 0002:00011a6c       ??_C@_07BHCBOAMP@ramdisk@  1005da6c     ustring.obj
 0002:00011a74       ??_C@_0L@PLJFMBIJ@MemoryLoad@ 1005da74     ustring.obj
 0002:00011a80       ??_C@_09MMAOIBBJ@TotalPhys@ 1005da80     ustring.obj
 0002:00011a8c       ??_C@_09KFOEOLH@AvailPhys@ 1005da8c     ustring.obj
 0002:00011a98       ??_C@_0O@PEEMGPEP@TotalPageFile@ 1005da98     ustring.obj
 0002:00011aa8       ??_C@_0O@LLHOKNF@AvailPageFile@ 1005daa8     ustring.obj
 0002:00011ab8       ??_C@_0N@LCJEOHMM@TotalVirtual@ 1005dab8     ustring.obj
 0002:00011ac8       ??_C@_0N@EGHLANBF@AvailVirtual@ 1005dac8     ustring.obj
 0002:00011ad8       ??_C@_0BF@KKNLCGDE@AvailExtendedVirtual@ 1005dad8     ustring.obj
 0002:00011af0       ??_C@_0P@KJDDGAFH@FileAttributes@ 1005daf0     ustring.obj
 0002:00011b00       ??_C@_0BE@DEHGONAH@EnumSystemCodePages@ 1005db00     ustring.obj
 0002:00011b14       ??_C@_06FMJLOCAF@GetACP@   1005db14     ustring.obj
 0002:00011b1c       ??_C@_09HLFMNDA@GetCPInfo@ 1005db1c     ustring.obj
 0002:00011b28       ??_C@_0O@PIBBCLJF@GetCurrentDir@ 1005db28     ustring.obj
 0002:00011b38       ??_C@_0N@IIBOJKJ@GetDriveType@ 1005db38     ustring.obj
 0002:00011b48       ??_C@_0M@KHMMJMNI@GetFileAttr@ 1005db48     ustring.obj
 0002:00011b54       ??_C@_0M@ONGMCNNE@GetKeyState@ 1005db54     ustring.obj
 0002:00011b60       ??_C@_0BH@KKAFOIJJ@GetLogicalDriveStrings@ 1005db60     ustring.obj
 0002:00011b78       ??_C@_08OMCNFONF@GetOEMCP@ 1005db78     ustring.obj
 0002:00011b84       ??_C@_0N@EBDGNADB@GetConsoleCP@ 1005db84     ustring.obj
 0002:00011b94       ??_C@_0N@DFIIBMHN@SetConsoleCP@ 1005db94     ustring.obj
 0002:00011ba4       ??_C@_0BD@LLGELLLN@GetConsoleOutputCP@ 1005dba4     ustring.obj
 0002:00011bb8       ??_C@_0BD@EBEOINFF@SetConsoleOutputCP@ 1005dbb8     ustring.obj
 0002:00011bcc       ??_C@_0BD@IHIHPGDL@GlobalMemoryStatus@ 1005dbcc     ustring.obj
 0002:00011be0       ??_C@_0BE@HCIKGJGE@MultiByteToWideChar@ 1005dbe0     ustring.obj
 0002:00011bf4       ??_C@_09EPINLGBH@OemToUtf8@ 1005dbf4     ustring.obj
 0002:00011c00       ??_C@_0BC@NFCPMJFM@OutputDebugString@ 1005dc00     ustring.obj
 0002:00011c14       ??_C@_0BA@MNJFBAJH@SHGetFolderPath@ 1005dc14     ustring.obj
 0002:00011c24       ??_C@_0L@PMCLJMMJ@SearchPath@ 1005dc24     ustring.obj
 0002:00011c30       ??_C@_0O@IHAPJIOC@SetCurrentDir@ 1005dc30     ustring.obj
 0002:00011c40       ??_C@_0M@KINCEKFL@SetFileAttr@ 1005dc40     ustring.obj
 0002:00011c4c       ??_C@_05PFDOMJEF@Sleep@    1005dc4c     ustring.obj
 0002:00011c54       ??_C@_0M@KJELMDJD@Utf16ToUtf8@ 1005dc54     ustring.obj
 0002:00011c60       ??_C@_09LCEKPEGC@Utf8ToOem@ 1005dc60     ustring.obj
 0002:00011c6c       ??_C@_0M@GJGCILHG@Utf8ToUtf16@ 1005dc6c     ustring.obj
 0002:00011c78       ??_C@_04NDFIEGPL@Uuid@     1005dc78     ustring.obj
 0002:00011c80       ??_C@_0BE@LJADKLBD@WideCharToMultiByte@ 1005dc80     ustring.obj
 0002:00011c94       ??_C@_04GFOHBGIO@subW@     1005dc94     ustring.obj
 0002:00011c9c       ??_C@_06FHFOAHML@system@   1005dc9c     ustring.obj
 0002:00011ca4       ??_C@_04NOFELICG@lenW@     1005dca4     ustring.obj
 0002:00011cac       ??_C@_07JOJHCKGP@ustring@  1005dcac     ustring.obj
 0002:00011cb8       _ustring_funcs             1005dcb8     ustring.obj
 0002:00011db0       ??_C@_0DJ@KKHMCMAP@bad?5field?5?$FL?$CFd?$FN?5in?5table?5stackpo@ 1005ddb0     util.obj
 0002:00011dec       ??_C@_0DJ@PFHHGAMM@bad?5field?5?8?$CFs?8?5in?5table?5stackpo@ 1005ddec     util.obj
 0002:00011e28       ??_C@_06EBGNBFIA@number@   1005de28     util.obj
 0002:00011e30       ??_C@_04CBBMIBLK@HKLM@     1005de30     win.obj
 0002:00011e38       ??_C@_04LEMDOLAJ@HKCC@     1005de38     win.obj
 0002:00011e40       ??_C@_04OHBKMIBJ@HKCR@     1005de40     win.obj
 0002:00011e48       ??_C@_04KIFLFONO@HKCU@     1005de48     win.obj
 0002:00011e50       ??_C@_03DLBIJLAB@HKU@      1005de50     win.obj
 0002:00011e54       ??_C@_0DA@DKALLFDI@must?5be?5?8HKLM?8?0?5?8HKCC?8?0?5?8HKCR?8?0@ 1005de54     win.obj
 0002:00011e84       ??_C@_05KDALNKAH@dword@    1005de84     win.obj
 0002:00011e8c       ??_C@_06FNFBAEBE@binary@   1005de8c     win.obj
 0002:00011e94       ??_C@_0N@CBOMHLPN@expandstring@ 1005de94     win.obj
 0002:00011ea4       ??_C@_0M@PEGIPCHN@multistring@ 1005dea4     win.obj
 0002:00011eb0       ??_C@_0BH@NOJOGNJM@unsupported?5value?5type@ 1005deb0     win.obj
 0002:00011ec8       ??_C@_0BD@MJODDCFG@OpenRegKey?5failed?4@ 1005dec8     win.obj
 0002:00011edc       ??_C@_0BI@COLHBIIE@RegQueryValueEx?5failed?4@ 1005dedc     win.obj
 0002:00011ef4       ??_C@_1BK@BIGILECK@?$AAA?$AAd?$AAv?$AAa?$AAp?$AAi?$AA3?$AA2?$AA?4?$AAd?$AAl?$AAl@ 1005def4     win.obj
 0002:00011f10       ??_C@_0BA@LILAPHGE@RegDeleteKeyExW@ 1005df10     win.obj
 0002:00011f20       ??_C@_0BG@HHFHBIKG@RegOpenKeyExW?5failed?4@ 1005df20     win.obj
 0002:00011f38       ??_C@_05DFPNHDMN@wYear@    1005df38     win.obj
 0002:00011f40       ??_C@_06MGNNJGBJ@wMonth@   1005df40     win.obj
 0002:00011f48       ??_C@_0L@OAHPHHP@wDayOfWeek@ 1005df48     win.obj
 0002:00011f54       ??_C@_04NBLBJIPP@wDay@     1005df54     win.obj
 0002:00011f5c       ??_C@_05BMOPCGDH@wHour@    1005df5c     win.obj
 0002:00011f64       ??_C@_07HPODENI@wMinute@   1005df64     win.obj
 0002:00011f6c       ??_C@_07IIEDHHJN@wSecond@  1005df6c     win.obj
 0002:00011f74       ??_C@_0O@HBAPEOKP@wMilliseconds@ 1005df74     win.obj
 0002:00011f84       ??_C@_01LKDEMHDF@s@        1005df84     win.obj
 0002:00011f88       ??_C@_0BA@IAFODGNM@CursorPositionX@ 1005df88     win.obj
 0002:00011f98       ??_C@_0BA@JJEFAHJN@CursorPositionY@ 1005df98     win.obj
 0002:00011fa8       ??_C@_0L@NFCEOFBF@WindowLeft@ 1005dfa8     win.obj
 0002:00011fb4       ??_C@_09JHGOALHG@WindowTop@ 1005dfb4     win.obj
 0002:00011fc0       ??_C@_0M@HHPHMPGH@WindowRight@ 1005dfc0     win.obj
 0002:00011fcc       ??_C@_0N@JPIJCAOJ@WindowBottom@ 1005dfcc     win.obj
 0002:00011fdc       ??_C@_0BD@DOLDEII@MaximumWindowSizeX@ 1005dfdc     win.obj
 0002:00011ff0       ??_C@_0BD@BKPAAFMJ@MaximumWindowSizeY@ 1005dff0     win.obj
 0002:00012004       ??_C@_01PFHFFBPC@t@        1005e004     win.obj
 0002:00012008       ??_C@_0BJ@LPJMBJJL@directory?5already?5exists@ 1005e008     win.obj
 0002:00012024       ??_C@_02NIKKAELB@XP@       1005e024     win.obj
 0002:00012028       ??_C@_05OFKKJCED@XPSP1@    1005e028     win.obj
 0002:00012030       ??_C@_05MOIHMBIA@XPSP2@    1005e030     win.obj
 0002:00012038       ??_C@_05NHJMPAMB@XPSP3@    1005e038     win.obj
 0002:00012040       ??_C@_05FGFMDFJC@Vista@    1005e040     win.obj
 0002:00012048       ??_C@_08ENCCDKOP@VistaSP1@ 1005e048     win.obj
 0002:00012054       ??_C@_08GGAPGJCM@VistaSP2@ 1005e054     win.obj
 0002:00012060       ??_C@_02PJEKLOOM@W7@       1005e060     win.obj
 0002:00012064       ??_C@_05DPOOILML@W7SP1@    1005e064     win.obj
 0002:0001206c       ??_C@_02HONCKCCD@W8@       1005e06c     win.obj
 0002:00012070       ??_C@_04HCPPKHCP@W8?41@    1005e070     win.obj
 0002:00012078       ??_C@_03HCIOKOKM@W10@      1005e078     win.obj
 0002:0001207c       ??_C@_06LGMEBDBC@Server@   1005e07c     win.obj
 0002:00012084       ??_C@_0BH@CNFJKJGO@invalid?5argument?5value@ 1005e084     win.obj
 0002:0001209c       ??_C@_0BK@LNHOAEDA@must?5be?5string?5or?5integer@ 1005e09c     win.obj
 0002:000120b8       ??_C@_0BK@JGAEKFII@invalid?5value?5at?5key?5?8?$CFs?8@ 1005e0b8     win.obj
 0002:000120d4       ??_C@_0O@CFPMOCDP@CompareString@ 1005e0d4     win.obj
 0002:000120e4       ??_C@_08PPLNFCGA@CopyFile@ 1005e0e4     win.obj
 0002:000120f0       ??_C@_09INHPLKKM@CreateDir@ 1005e0f0     win.obj
 0002:000120fc       ??_C@_0L@GPLPOFDC@DeleteFile@ 1005e0fc     win.obj
 0002:00012108       ??_C@_0N@FOJPHHPH@DeleteRegKey@ 1005e108     win.obj
 0002:00012118       ??_C@_0P@PCCDOIAL@DeleteRegValue@ 1005e118     win.obj
 0002:00012128       ??_C@_0L@DGAGCFOP@EnumRegKey@ 1005e128     win.obj
 0002:00012134       ??_C@_0N@PFFNCIBD@EnumRegValue@ 1005e134     win.obj
 0002:00012144       ??_C@_0L@MGMEFCAE@ExtractKey@ 1005e144     win.obj
 0002:00012150       ??_C@_0N@HALOIPMN@ExtractKeyEx@ 1005e150     win.obj
 0002:00012160       ??_C@_0N@DNBFBBHK@IsWinVersion@ 1005e160     win.obj
 0002:00012170       ??_C@_0BI@EKFDIGHI@FileTimeToLocalFileTime@ 1005e170     win.obj
 0002:00012188       ??_C@_0BF@KPJNHALE@FileTimeToSystemTime@ 1005e188     win.obj
 0002:000121a0       ??_C@_0BL@NAIJNMLL@GetConsoleScreenBufferInfo@ 1005e1a0     win.obj
 0002:000121bc       ??_C@_06CALCCDMF@GetEnv@   1005e1bc     win.obj
 0002:000121c4       ??_C@_0M@EINGHLOA@GetFileInfo@ 1005e1c4     win.obj
 0002:000121d0       ??_C@_0N@HDKONBLE@GetFileTimes@ 1005e1d0     win.obj
 0002:000121e0       ??_C@_09GFGIAJLD@GetRegKey@ 1005e1e0     win.obj
 0002:000121ec       ??_C@_0BI@ENMDHCMK@GetSystemTimeAsFileTime@ 1005e1ec     win.obj
 0002:00012204       ??_C@_0P@GGGHOPAD@GetVirtualKeys@ 1005e204     win.obj
 0002:00012214       ??_C@_0P@MIPPOCAO@IsProcess64bit@ 1005e214     win.obj
 0002:00012224       ??_C@_08CALLHOCI@MoveFile@ 1005e224     win.obj
 0002:00012230       ??_C@_09EDKALOCB@RemoveDir@ 1005e230     win.obj
 0002:0001223c       ??_C@_0L@HBAGBENL@RenameFile@ 1005e23c     win.obj
 0002:00012248       ??_C@_06LDCDJLBI@SetEnv@   1005e248     win.obj
 0002:00012250       ??_C@_0N@HBABNPI@SetFileTimes@ 1005e250     win.obj
 0002:00012260       ??_C@_09ELCNCICB@SetRegKey@ 1005e260     win.obj
 0002:0001226c       ??_C@_0N@BFFIJKHB@ShellExecute@ 1005e26c     win.obj
 0002:0001227c       ??_C@_0BF@HBHGIPOG@SystemTimeToFileTime@ 1005e27c     win.obj
 0002:00012294       ??_C@_06DNONFAKH@wcscmp@   1005e294     win.obj
 0002:0001229c       ??_C@_0N@OCKOJJEP@WriteConsole@ 1005e29c     win.obj
 0002:000122b0       _win_funcs                 1005e2b0     win.obj
 0002:000123b0       ??_C@_0O@NLDKAIKN@EncodePointer@ 1005e3b0     vc_crt_fix_impl.obj
 0002:000123c0       ??_C@_0O@KBPMFGHI@DecodePointer@ 1005e3c0     vc_crt_fix_impl.obj
 0002:000123d0       ??_C@_0BD@GIGEJCNH@GetModuleHandleExW@ 1005e3d0     vc_crt_fix_impl.obj
 0002:000123e4       ??_C@_0BE@NBEJPEJA@InitializeSListHead@ 1005e3e4     vc_crt_fix_impl.obj
 0002:000123f8       ??_C@_0BG@PLLPFLHB@InterlockedFlushSList@ 1005e3f8     vc_crt_fix_impl.obj
 0002:00012410       ??_C@_0BJ@PNEEKDOK@InterlockedPopEntrySList@ 1005e410     vc_crt_fix_impl.obj
 0002:0001242c       ??_C@_0BK@JFGGAIOA@InterlockedPushEntrySList@ 1005e42c     vc_crt_fix_impl.obj
 0002:00012448       ??_C@_0BL@FOECAEGO@InterlockedPushListSListEx@ 1005e448     vc_crt_fix_impl.obj
 0002:00012464       ??_C@_0BD@FHMMIGCI@RtlFirstEntrySList@ 1005e464     vc_crt_fix_impl.obj
 0002:00012478       ??_C@_0BA@FGPHPMJB@QueryDepthSList@ 1005e478     vc_crt_fix_impl.obj
 0002:00012488       ??_C@_0BJ@NLNFLAMA@GetNumaHighestNodeNumber@ 1005e488     vc_crt_fix_impl.obj
 0002:000124a4       ??_C@_0BP@KHGALBC@GetLogicalProcessorInformation@ 1005e4a4     vc_crt_fix_impl.obj
 0002:000124c4       ??_C@_0BI@BKLFFAPO@SetThreadStackGuarantee@ 1005e4c4     vc_crt_fix_impl.obj
 0002:000124dc       ??_C@_0BM@HCFOFFN@InitializeCriticalSectionEx@ 1005e4dc     vc_crt_fix_impl.obj
 0002:000124f8       ??_C@_0BA@IHGNDAEB@CompareStringEx@ 1005e4f8     vc_crt_fix_impl.obj
 0002:00012528       __real@3ff0000000000000    1005e528     service.obj
 0002:00012530       __real@4059000000000000    1005e530     service.obj
 0002:00012538       __real@41e0000000000000    1005e538     service.obj
 0002:00012540       __real@41f0000000000000    1005e540     service.obj
 0002:00012548       __real@43e0000000000000    1005e548     util.obj
 0002:00012550       __real@bff0000000000000    1005e550     exported.obj
 0002:000125b8       __load_config_used         1005e5b8     LIBCMT:loadcfg.obj
 0002:0001265c       ??_R4exception@std@@6B@    1005e65c     libvcruntime:frame.obj
 0002:00012670       ??_R3exception@std@@8      1005e670     libvcruntime:frame.obj
 0002:00012680       ??_R2exception@std@@8      1005e680     libvcruntime:frame.obj
 0002:00012688       ??_R1A@?0A@EA@exception@std@@8 1005e688     libvcruntime:frame.obj
 0002:000126a4       ??_R4bad_exception@std@@6B@ 1005e6a4     libvcruntime:frame.obj
 0002:000126b8       ??_R3bad_exception@std@@8  1005e6b8     libvcruntime:frame.obj
 0002:000126c8       ??_R2bad_exception@std@@8  1005e6c8     libvcruntime:frame.obj
 0002:000126d4       ??_R1A@?0A@EA@bad_exception@std@@8 1005e6d4     libvcruntime:frame.obj
 0002:000126f0       ??_R4type_info@@6B@        1005e6f0     LIBCMT:std_type_info_static.obj
 0002:00012704       ??_R3type_info@@8          1005e704     LIBCMT:std_type_info_static.obj
 0002:00012714       ??_R2type_info@@8          1005e714     LIBCMT:std_type_info_static.obj
 0002:0001271c       ??_R1A@?0A@EA@type_info@@8 1005e71c     LIBCMT:std_type_info_static.obj
 0002:00012740       ___safe_se_handler_table   1005e740     <linker-defined>
 0002:00012a58       ___rtc_iaa                 1005ea58     LIBCMT:initsect.obj
 0002:00012a5c       ___rtc_izz                 1005ea5c     LIBCMT:initsect.obj
 0002:00012a60       ___rtc_taa                 1005ea60     LIBCMT:initsect.obj
 0002:00012a64       ___rtc_tzz                 1005ea64     LIBCMT:initsect.obj
 0002:00012c24       __TI2?AVbad_exception@std@@ 1005ec24     libvcruntime:frame.obj
 0002:00012c34       __CTA2?AVbad_exception@std@@ 1005ec34     libvcruntime:frame.obj
 0002:00012c40       __CT??_R0?AVbad_exception@std@@@8??0bad_exception@std@@QAE@ABV01@@Z12 1005ec40     libvcruntime:frame.obj
 0002:00012c5c       __CT??_R0?AVexception@std@@@8??0exception@std@@QAE@ABV01@@Z12 1005ec5c     libvcruntime:frame.obj
 0002:0001388c       __IMPORT_DESCRIPTOR_KERNEL32 1005f88c     kernel32:KERNEL32.dll
 0002:000138a0       __IMPORT_DESCRIPTOR_ADVAPI32 1005f8a0     advapi32:ADVAPI32.dll
 0002:000138b4       __IMPORT_DESCRIPTOR_USER32 1005f8b4     user32:USER32.dll
 0002:000138c8       __IMPORT_DESCRIPTOR_SHELL32 1005f8c8     shell32:SHELL32.dll
 0002:000138dc       __IMPORT_DESCRIPTOR_RPCRT4 1005f8dc     rpcrt4:RPCRT4.dll
 0002:000138f0       __IMPORT_DESCRIPTOR_lua51  1005f8f0     lua51:lua51.dll
 0002:00013904       __NULL_IMPORT_DESCRIPTOR   1005f904     kernel32:KERNEL32.dll
 0003:00000000       ___scrt_native_dllmain_reason 10061000     LIBCMT:utility.obj
 0003:00000004       ___security_cookie_complement 10061004     LIBCMT:gs_cookie.obj
 0003:00000008       ___security_cookie         10061008     LIBCMT:gs_cookie.obj
 0003:0000000c       ___isa_enabled             1006100c     LIBCMT:cpu_disp.obj
 0003:00000020       __NLG_Destination          10061020     libvcruntime:exsup.obj
 0003:00000030       __iob                      10061030     libucrt:_file.obj
 0003:000000e0       ___abort_behavior          100610e0     libucrt:abort.obj
 0003:000000e8       ___acrt_initial_locale_data 100610e8     libucrt:nlsdata.obj
 0003:000001a0       ___acrt_initial_locale_pointers 100611a0     libucrt:nlsdata.obj
 0003:000001a8       ___acrt_wide_c_locale_string 100611a8     libucrt:nlsdata.obj
 0003:000001b0       ___badioinfo               100611b0     libucrt:ioinit.obj
 0003:000001f0       __lookuptrailbytes         100611f0     libucrt:read.obj
 0003:000002f0       __pwctype                  100612f0     libucrt:ctype.obj
 0003:000002f8       ___acrt_initial_multibyte_data 100612f8     libucrt:mbctype.obj
 0003:00000818       ___globallocalestatus      10061818     libucrt:glstatus.obj
 0003:00000820       ___acrt_lconv_c            10061820     libucrt:localeconv.obj
 0003:00000870       ___acrt_lconv_static_decimal 10061870     libucrt:localeconv.obj
 0003:00000874       ___acrt_lconv_static_W_decimal 10061874     libucrt:localeconv.obj
 0003:00000890       __fltused                  10061890     LIBCMT:fltused.obj
 0003:000008a0       _GetPluginData             100618a0     service.obj
 0003:0000b9f0       ??_R0?AVbad_exception@std@@@8 1006c9f0     libvcruntime:frame.obj
 0003:0000ba10       ??_R0?AVexception@std@@@8  1006ca10     libvcruntime:frame.obj
 0003:0000ba2c       ??_R0?AVtype_info@@@8      1006ca2c     LIBCMT:std_type_info_static.obj
 0003:0000bd6c       ___scrt_current_native_startup_state 1006cd6c     LIBCMT:utility.obj
 0003:0000bd70       ___scrt_native_startup_lock 1006cd70     LIBCMT:utility.obj
 0003:0000bd94       ___isa_available           1006cd94     LIBCMT:cpu_disp.obj
 0003:0000bd98       ___favor                   1006cd98     LIBCMT:cpu_disp.obj
 0003:0000bd9c       ___scrt_debugger_hook_flag 1006cd9c     LIBCMT:utility_desktop.obj
 0003:0000bda0       ?__type_info_root_node@@3U__type_info_node@@A 1006cda0     LIBCMT:tncleanup.obj
 0003:0000bda8       ?__WinRTOutOfMemoryExceptionCallback@@3P6GPAXXZA 1006cda8     libvcruntime:ehhelpers.obj
 0003:0000bdf0       ?pArgList@UnDecorator@@0PAVReplicator@@A 1006cdf0     libvcruntime:undname.obj
 0003:0000bdf4       ?pZNameList@UnDecorator@@0PAVReplicator@@A 1006cdf4     libvcruntime:undname.obj
 0003:0000bdf8       ?pTemplateArgList@UnDecorator@@0PAVReplicator@@A 1006cdf8     libvcruntime:undname.obj
 0003:0000bdfc       ?gName@UnDecorator@@0PBDB  1006cdfc     libvcruntime:undname.obj
 0003:0000be00       ?name@UnDecorator@@0PBDB   1006ce00     libvcruntime:undname.obj
 0003:0000be04       ?disableFlags@UnDecorator@@0KA 1006ce04     libvcruntime:undname.obj
 0003:0000be08       ?fExplicitTemplateParams@UnDecorator@@0_NA 1006ce08     libvcruntime:undname.obj
 0003:0000be09       ?fGetTemplateArgumentList@UnDecorator@@0_NA 1006ce09     libvcruntime:undname.obj
 0003:0000be0c       ?m_pGetParameter@UnDecorator@@0P6APADJ@ZA 1006ce0c     libvcruntime:undname.obj
 0003:0000be10       ?m_CHPENameOffset@UnDecorator@@0KA 1006ce10     libvcruntime:undname.obj
 0003:0000be14       ?m_recursionLevel@UnDecorator@@0KA 1006ce14     libvcruntime:undname.obj
 0003:0000be4c       ___pPurecall               1006ce4c     libvcruntime:purevirt_data.obj
 0003:0000be50       __nstream                  1006ce50     libucrt:_file.obj
 0003:0000be54       ___piob                    1006ce54     libucrt:_file.obj
 0003:0000be58       __cflush                   1006ce58     libucrt:_file.obj
 0003:0000be84       ?c_exit_complete@?1???R<lambda_6e4b09c48022b2350581041d5f6b0c4c>@@QBE@XZ@4_NA 1006ce84     libucrt:exit.obj
 0003:0000bf90       __environ_table            1006cf90     libucrt:environment_initialization.obj
 0003:0000bf94       __wenviron_table           1006cf94     libucrt:environment_initialization.obj
 0003:0000bf98       ___dcrt_initial_wide_environment 1006cf98     libucrt:environment_initialization.obj
 0003:0000bf9c       ___dcrt_initial_narrow_environment 1006cf9c     libucrt:environment_initialization.obj
 0003:0000bfa0       ___acrt_atexit_table       1006cfa0     libucrt:onexit.obj
 0003:0000bfac       ___acrt_at_quick_exit_table 1006cfac     libucrt:onexit.obj
 0003:0000bfc8       ___acrt_stdout_buffer      1006cfc8     libucrt:_sftbuf.obj
 0003:0000bfcc       ___acrt_stderr_buffer      1006cfcc     libucrt:_sftbuf.obj
 0003:0000bfd0       ___acrt_locale_changed_data 1006cfd0     libucrt:wsetlocale.obj
 0003:0000bfd4       ___acrt_current_locale_data 1006cfd4     libucrt:nlsdata.obj
 0003:0000bfd8       ___pioinfo                 1006cfd8     libucrt:ioinit.obj
 0003:0000c1d8       __nhandle                  1006d1d8     libucrt:ioinit.obj
 0003:0000c41c       __commode                  1006d41c     libucrt:ncommode.obj
 0003:0000c420       __mbctype                  1006d420     libucrt:mbctype.obj
 0003:0000c424       __mbcasemap                1006d424     libucrt:mbctype.obj
 0003:0000c428       ___acrt_current_multibyte_data 1006d428     libucrt:mbctype.obj
 0003:0000c434       __pgmptr                   1006d434     libucrt:argv_data.obj
 0003:0000c438       ___argc                    1006d438     libucrt:argv_data.obj
 0003:0000c43c       ___argv                    1006d43c     libucrt:argv_data.obj
 0003:0000c440       ___wargv                   1006d440     libucrt:argv_data.obj
 0003:0000c444       __acmdln                   1006d444     libucrt:argv_data.obj
 0003:0000c448       __wcmdln                   1006d448     libucrt:argv_data.obj
 0003:0000c44c       ___acrt_heap               1006d44c     libucrt:heap_handle.obj
 0003:0000c45c       ___acrt_lconv_static_null  1006d45c     libucrt:localeconv.obj
 0003:0000c460       ___acrt_lconv_static_W_null 1006d460     libucrt:localeconv.obj
 0003:0000c464       __umaskval                 1006d464     libucrt:umask.obj
 0003:0000c474       __fmode                    1006d474     libucrt:txtmode.obj
 0003:0000c478       ___fastflag                1006d478     libucrt:fp_flags.obj
 0003:0000c538       ?Ptr@?1???R<lambda_1>@?1??XorPointer@@YAPAXPAX@Z@QBE@XZ@4PAXA 1006d538     vc_crt_fix_impl.obj
 0003:0000c540       ___dyn_tls_init_callback   1006d540     <common>
 0003:0000c544       ___scrt_ucrt_dll_is_in_use 1006d544     <common>
 0003:0000c548       __pmatherr                 1006d548     <common>
 0003:0000c54c       ___use_sse2_mathfcns       1006d54c     <common>
 0003:0000c550       _EnumCP                    1006d550     <common>
 0003:0000c558       ?_OptionsStorage@?1??__local_stdio_printf_options@@9@9 1006d558     <common>
 0003:0000c560       ?_OptionsStorage@?1??__local_stdio_scanf_options@@9@9 1006d560     <common>

 entry point at        0001:0002c34b

 Static symbols

 0000:fff8b000       .debug$S                   10000000     luafar3.exp
 0000:fff8b000       .debug$S                   10000000     advapi32:ADVAPI32.dll
 0000:fff8b000       .debug$S                   10000000     advapi32:ADVAPI32.dll
 0000:fff8b000       .debug$S                   10000000     advapi32:ADVAPI32.dll
 0000:fff8b000       .debug$S                   10000000     advapi32:ADVAPI32.dll
 0000:fff8b000       .debug$S                   10000000     advapi32:ADVAPI32.dll
 0000:fff8b000       .debug$S                   10000000     advapi32:ADVAPI32.dll
 0000:fff8b000       .debug$S                   10000000     advapi32:ADVAPI32.dll
 0000:fff8b000       .debug$S                   10000000     advapi32:ADVAPI32.dll
 0000:fff8b000       .debug$S                   10000000     advapi32:ADVAPI32.dll
 0000:fff8b000       .debug$S                   10000000     kernel32:KERNEL32.dll
 0000:fff8b000       .debug$S                   10000000     kernel32:KERNEL32.dll
 0000:fff8b000       .debug$S                   10000000     kernel32:KERNEL32.dll
 0000:fff8b000       .debug$S                   10000000     kernel32:KERNEL32.dll
 0000:fff8b000       .debug$S                   10000000     kernel32:KERNEL32.dll
 0000:fff8b000       .debug$S                   10000000     kernel32:KERNEL32.dll
 0000:fff8b000       .debug$S                   10000000     kernel32:KERNEL32.dll
 0000:fff8b000       .debug$S                   10000000     kernel32:KERNEL32.dll
 0000:fff8b000       .debug$S                   10000000     kernel32:KERNEL32.dll
 0000:fff8b000       .debug$S                   10000000     kernel32:KERNEL32.dll
 0000:fff8b000       .debug$S                   10000000     kernel32:KERNEL32.dll
 0000:fff8b000       .debug$S                   10000000     kernel32:KERNEL32.dll
 0000:fff8b000       .debug$S                   10000000     kernel32:KERNEL32.dll
 0000:fff8b000       .debug$S                   10000000     kernel32:KERNEL32.dll
 0000:fff8b000       .debug$S                   10000000     kernel32:KERNEL32.dll
 0000:fff8b000       .debug$S                   10000000     kernel32:KERNEL32.dll
 0000:fff8b000       .debug$S                   10000000     kernel32:KERNEL32.dll
 0000:fff8b000       .debug$S                   10000000     kernel32:KERNEL32.dll
 0000:fff8b000       .debug$S                   10000000     kernel32:KERNEL32.dll
 0000:fff8b000       .debug$S                   10000000     kernel32:KERNEL32.dll
 0000:fff8b000       .debug$S                   10000000     kernel32:KERNEL32.dll
 0000:fff8b000       .debug$S                   10000000     kernel32:KERNEL32.dll
 0000:fff8b000       .debug$S                   10000000     kernel32:KERNEL32.dll
 0000:fff8b000       .debug$S                   10000000     kernel32:KERNEL32.dll
 0000:fff8b000       .debug$S                   10000000     kernel32:KERNEL32.dll
 0000:fff8b000       .debug$S                   10000000     kernel32:KERNEL32.dll
 0000:fff8b000       .debug$S                   10000000     kernel32:KERNEL32.dll
 0000:fff8b000       .debug$S                   10000000     kernel32:KERNEL32.dll
 0000:fff8b000       .debug$S                   10000000     kernel32:KERNEL32.dll
 0000:fff8b000       .debug$S                   10000000     kernel32:KERNEL32.dll
 0000:fff8b000       .debug$S                   10000000     kernel32:KERNEL32.dll
 0000:fff8b000       .debug$S                   10000000     kernel32:KERNEL32.dll
 0000:fff8b000       .debug$S                   10000000     kernel32:KERNEL32.dll
 0000:fff8b000       .debug$S                   10000000     kernel32:KERNEL32.dll
 0000:fff8b000       .debug$S                   10000000     kernel32:KERNEL32.dll
 0000:fff8b000       .debug$S                   10000000     kernel32:KERNEL32.dll
 0000:fff8b000       .debug$S                   10000000     kernel32:KERNEL32.dll
 0000:fff8b000       .debug$S                   10000000     kernel32:KERNEL32.dll
 0000:fff8b000       .debug$S                   10000000     kernel32:KERNEL32.dll
 0000:fff8b000       .debug$S                   10000000     kernel32:KERNEL32.dll
 0000:fff8b000       .debug$S                   10000000     kernel32:KERNEL32.dll
 0000:fff8b000       .debug$S                   10000000     kernel32:KERNEL32.dll
 0000:fff8b000       .debug$S                   10000000     kernel32:KERNEL32.dll
 0000:fff8b000       .debug$S                   10000000     kernel32:KERNEL32.dll
 0000:fff8b000       .debug$S                   10000000     kernel32:KERNEL32.dll
 0000:fff8b000       .debug$S                   10000000     kernel32:KERNEL32.dll
 0000:fff8b000       .debug$S                   10000000     kernel32:KERNEL32.dll
 0000:fff8b000       .debug$S                   10000000     kernel32:KERNEL32.dll
 0000:fff8b000       .debug$S                   10000000     kernel32:KERNEL32.dll
 0000:fff8b000       .debug$S                   10000000     kernel32:KERNEL32.dll
 0000:fff8b000       .debug$S                   10000000     kernel32:KERNEL32.dll
 0000:fff8b000       .debug$S                   10000000     kernel32:KERNEL32.dll
 0000:fff8b000       .debug$S                   10000000     kernel32:KERNEL32.dll
 0000:fff8b000       .debug$S                   10000000     kernel32:KERNEL32.dll
 0000:fff8b000       .debug$S                   10000000     kernel32:KERNEL32.dll
 0000:fff8b000       .debug$S                   10000000     kernel32:KERNEL32.dll
 0000:fff8b000       .debug$S                   10000000     kernel32:KERNEL32.dll
 0000:fff8b000       .debug$S                   10000000     kernel32:KERNEL32.dll
 0000:fff8b000       .debug$S                   10000000     kernel32:KERNEL32.dll
 0000:fff8b000       .debug$S                   10000000     kernel32:KERNEL32.dll
 0000:fff8b000       .debug$S                   10000000     kernel32:KERNEL32.dll
 0000:fff8b000       .debug$S                   10000000     kernel32:KERNEL32.dll
 0000:fff8b000       .debug$S                   10000000     kernel32:KERNEL32.dll
 0000:fff8b000       .debug$S                   10000000     kernel32:KERNEL32.dll
 0000:fff8b000       .debug$S                   10000000     kernel32:KERNEL32.dll
 0000:fff8b000       .debug$S                   10000000     kernel32:KERNEL32.dll
 0000:fff8b000       .debug$S                   10000000     kernel32:KERNEL32.dll
 0000:fff8b000       .debug$S                   10000000     kernel32:KERNEL32.dll
 0000:fff8b000       .debug$S                   10000000     kernel32:KERNEL32.dll
 0000:fff8b000       .debug$S                   10000000     kernel32:KERNEL32.dll
 0000:fff8b000       .debug$S                   10000000     kernel32:KERNEL32.dll
 0000:fff8b000       .debug$S                   10000000     kernel32:KERNEL32.dll
 0000:fff8b000       .debug$S                   10000000     kernel32:KERNEL32.dll
 0000:fff8b000       .debug$S                   10000000     kernel32:KERNEL32.dll
 0000:fff8b000       .debug$S                   10000000     kernel32:KERNEL32.dll
 0000:fff8b000       .debug$S                   10000000     kernel32:KERNEL32.dll
 0000:fff8b000       .debug$S                   10000000     kernel32:KERNEL32.dll
 0000:fff8b000       .debug$S                   10000000     kernel32:KERNEL32.dll
 0000:fff8b000       .debug$S                   10000000     kernel32:KERNEL32.dll
 0000:fff8b000       .debug$S                   10000000     kernel32:KERNEL32.dll
 0000:fff8b000       .debug$S                   10000000     kernel32:KERNEL32.dll
 0000:fff8b000       .debug$S                   10000000     kernel32:KERNEL32.dll
 0000:fff8b000       .debug$S                   10000000     kernel32:KERNEL32.dll
 0000:fff8b000       .debug$S                   10000000     kernel32:KERNEL32.dll
 0000:fff8b000       .debug$S                   10000000     kernel32:KERNEL32.dll
 0000:fff8b000       .debug$S                   10000000     kernel32:KERNEL32.dll
 0000:fff8b000       .debug$S                   10000000     kernel32:KERNEL32.dll
 0000:fff8b000       .debug$S                   10000000     kernel32:KERNEL32.dll
 0000:fff8b000       .debug$S                   10000000     kernel32:KERNEL32.dll
 0000:fff8b000       .debug$S                   10000000     kernel32:KERNEL32.dll
 0000:fff8b000       .debug$S                   10000000     kernel32:KERNEL32.dll
 0000:fff8b000       .debug$S                   10000000     kernel32:KERNEL32.dll
 0000:fff8b000       .debug$S                   10000000     kernel32:KERNEL32.dll
 0000:fff8b000       .debug$S                   10000000     kernel32:KERNEL32.dll
 0000:fff8b000       .debug$S                   10000000     kernel32:KERNEL32.dll
 0000:fff8b000       .debug$S                   10000000     kernel32:KERNEL32.dll
 0000:fff8b000       .debug$S                   10000000     kernel32:KERNEL32.dll
 0000:fff8b000       .debug$S                   10000000     kernel32:KERNEL32.dll
 0000:fff8b000       .debug$S                   10000000     kernel32:KERNEL32.dll
 0000:fff8b000       .debug$S                   10000000     kernel32:KERNEL32.dll
 0000:fff8b000       .debug$S                   10000000     kernel32:KERNEL32.dll
 0000:fff8b000       .debug$S                   10000000     kernel32:KERNEL32.dll
 0000:fff8b000       .debug$S                   10000000     kernel32:KERNEL32.dll
 0000:fff8b000       .debug$S                   10000000     kernel32:KERNEL32.dll
 0000:fff8b000       .debug$S                   10000000     kernel32:KERNEL32.dll
 0000:fff8b000       .debug$S                   10000000     kernel32:KERNEL32.dll
 0000:fff8b000       .debug$S                   10000000     kernel32:KERNEL32.dll
 0000:fff8b000       .debug$S                   10000000     kernel32:KERNEL32.dll
 0000:fff8b000       .debug$S                   10000000     kernel32:KERNEL32.dll
 0000:fff8b000       .debug$S                   10000000     kernel32:KERNEL32.dll
 0000:fff8b000       .debug$S                   10000000     kernel32:KERNEL32.dll
 0000:fff8b000       .debug$S                   10000000     kernel32:KERNEL32.dll
 0000:fff8b000       .debug$S                   10000000     kernel32:KERNEL32.dll
 0000:fff8b000       .debug$S                   10000000     kernel32:KERNEL32.dll
 0000:fff8b000       .debug$S                   10000000     kernel32:KERNEL32.dll
 0000:fff8b000       .debug$S                   10000000     kernel32:KERNEL32.dll
 0000:fff8b000       .debug$S                   10000000     kernel32:KERNEL32.dll
 0000:fff8b000       .debug$S                   10000000     kernel32:KERNEL32.dll
 0000:fff8b000       .debug$S                   10000000     kernel32:KERNEL32.dll
 0000:fff8b000       .debug$S                   10000000     kernel32:KERNEL32.dll
 0000:fff8b000       .debug$S                   10000000     kernel32:KERNEL32.dll
 0000:fff8b000       .debug$S                   10000000     kernel32:KERNEL32.dll
 0000:fff8b000       .debug$S                   10000000     kernel32:KERNEL32.dll
 0000:fff8b000       .debug$S                   10000000     kernel32:KERNEL32.dll
 0000:fff8b000       .debug$S                   10000000     rpcrt4:RPCRT4.dll
 0000:fff8b000       .debug$S                   10000000     rpcrt4:RPCRT4.dll
 0000:fff8b000       .debug$S                   10000000     rpcrt4:RPCRT4.dll
 0000:fff8b000       .debug$S                   10000000     rpcrt4:RPCRT4.dll
 0000:fff8b000       .debug$S                   10000000     shell32:SHELL32.dll
 0000:fff8b000       .debug$S                   10000000     shell32:SHELL32.dll
 0000:fff8b000       .debug$S                   10000000     user32:USER32.dll
 0000:fff8b000       .debug$S                   10000000     lua51:lua51.dll
 0000:fff8b000       .debug$S                   10000000     lua51:lua51.dll
 0000:fff8b000       .debug$S                   10000000     lua51:lua51.dll
 0000:fff8b000       .debug$S                   10000000     lua51:lua51.dll
 0000:fff8b000       .debug$S                   10000000     lua51:lua51.dll
 0000:fff8b000       .debug$S                   10000000     lua51:lua51.dll
 0000:fff8b000       .debug$S                   10000000     lua51:lua51.dll
 0000:fff8b000       .debug$S                   10000000     lua51:lua51.dll
 0000:fff8b000       .debug$S                   10000000     lua51:lua51.dll
 0000:fff8b000       .debug$S                   10000000     lua51:lua51.dll
 0000:fff8b000       .debug$S                   10000000     lua51:lua51.dll
 0000:fff8b000       .debug$S                   10000000     lua51:lua51.dll
 0000:fff8b000       .debug$S                   10000000     lua51:lua51.dll
 0000:fff8b000       .debug$S                   10000000     lua51:lua51.dll
 0000:fff8b000       .debug$S                   10000000     lua51:lua51.dll
 0000:fff8b000       .debug$S                   10000000     lua51:lua51.dll
 0000:fff8b000       .debug$S                   10000000     lua51:lua51.dll
 0000:fff8b000       .debug$S                   10000000     lua51:lua51.dll
 0000:fff8b000       .debug$S                   10000000     lua51:lua51.dll
 0000:fff8b000       .debug$S                   10000000     lua51:lua51.dll
 0000:fff8b000       .debug$S                   10000000     lua51:lua51.dll
 0000:fff8b000       .debug$S                   10000000     lua51:lua51.dll
 0000:fff8b000       .debug$S                   10000000     lua51:lua51.dll
 0000:fff8b000       .debug$S                   10000000     lua51:lua51.dll
 0000:fff8b000       .debug$S                   10000000     lua51:lua51.dll
 0000:fff8b000       .debug$S                   10000000     lua51:lua51.dll
 0000:fff8b000       .debug$S                   10000000     lua51:lua51.dll
 0000:fff8b000       .debug$S                   10000000     lua51:lua51.dll
 0000:fff8b000       .debug$S                   10000000     lua51:lua51.dll
 0000:fff8b000       .debug$S                   10000000     lua51:lua51.dll
 0000:fff8b000       .debug$S                   10000000     lua51:lua51.dll
 0000:fff8b000       .debug$S                   10000000     lua51:lua51.dll
 0000:fff8b000       .debug$S                   10000000     lua51:lua51.dll
 0000:fff8b000       .debug$S                   10000000     lua51:lua51.dll
 0000:fff8b000       .debug$S                   10000000     lua51:lua51.dll
 0000:fff8b000       .debug$S                   10000000     lua51:lua51.dll
 0000:fff8b000       .debug$S                   10000000     lua51:lua51.dll
 0000:fff8b000       .debug$S                   10000000     lua51:lua51.dll
 0000:fff8b000       .debug$S                   10000000     lua51:lua51.dll
 0000:fff8b000       .debug$S                   10000000     lua51:lua51.dll
 0000:fff8b000       .debug$S                   10000000     lua51:lua51.dll
 0000:fff8b000       .debug$S                   10000000     lua51:lua51.dll
 0000:fff8b000       .debug$S                   10000000     lua51:lua51.dll
 0000:fff8b000       .debug$S                   10000000     lua51:lua51.dll
 0000:fff8b000       .debug$S                   10000000     lua51:lua51.dll
 0000:fff8b000       .debug$S                   10000000     lua51:lua51.dll
 0000:fff8b000       .debug$S                   10000000     lua51:lua51.dll
 0000:fff8b000       .debug$S                   10000000     lua51:lua51.dll
 0000:fff8b000       .debug$S                   10000000     lua51:lua51.dll
 0000:fff8b000       .debug$S                   10000000     lua51:lua51.dll
 0000:fff8b000       .debug$S                   10000000     lua51:lua51.dll
 0000:fff8b000       .debug$S                   10000000     lua51:lua51.dll
 0000:fff8b000       .debug$S                   10000000     lua51:lua51.dll
 0000:fff8b000       .debug$S                   10000000     lua51:lua51.dll
 0000:fff8b000       .debug$S                   10000000     lua51:lua51.dll
 0000:fff8b000       .debug$S                   10000000     lua51:lua51.dll
 0000:fff8b000       .debug$S                   10000000     lua51:lua51.dll
 0000:fff8b000       .debug$S                   10000000     lua51:lua51.dll
 0000:fff8b000       .debug$S                   10000000     lua51:lua51.dll
 0000:fff8b000       .debug$S                   10000000     lua51:lua51.dll
 0000:fff8b000       .debug$S                   10000000     lua51:lua51.dll
 0000:fff8b000       .debug$S                   10000000     lua51:lua51.dll
 0000:fff8b000       .debug$S                   10000000     lua51:lua51.dll
 0000:fff8b000       .debug$S                   10000000     lua51:lua51.dll
 0000:fff8b000       .debug$S                   10000000     lua51:lua51.dll
 0000:fff8b000       .debug$S                   10000000     lua51:lua51.dll
 0000:fff8b000       .debug$S                   10000000     lua51:lua51.dll
 0000:fff8b000       .debug$S                   10000000     lua51:lua51.dll
 0000:fff8b000       .debug$S                   10000000     lua51:lua51.dll
 0000:fff8b000       .debug$S                   10000000     lua51:lua51.dll
 0000:fff8b000       .debug$S                   10000000     lua51:lua51.dll
 0000:fff8b000       .debug$S                   10000000     lua51:lua51.dll
 0000:fff8b000       .debug$S                   10000000     lua51:lua51.dll
 0000:fff8b000       .debug$S                   10000000     lua51:lua51.dll
 0000:fff8b000       .debug$S                   10000000     lua51:lua51.dll
 0000:fff8b000       .debug$S                   10000000     lua51:lua51.dll
 0000:fff8b000       .debug$S                   10000000     lua51:lua51.dll
 0000:fff8b000       .debug$S                   10000000     lua51:lua51.dll
 0000:fff8b000       .debug$S                   10000000     lua51:lua51.dll
 0000:fff8b000       .debug$S                   10000000     lua51:lua51.dll
 0000:fff8b000       .debug$S                   10000000     lua51:lua51.dll
 0000:fff8b000       .debug$S                   10000000     lua51:lua51.dll
 0000:fff8b000       .debug$S                   10000000     lua51:lua51.dll
 0000:fff8b000       .debug$S                   10000000     lua51:lua51.dll
 0000:fff8b000       .debug$S                   10000000     lua51:lua51.dll
 0000:fff8b000       .debug$S                   10000000     lua51:lua51.dll
 0000:fff8b000       .debug$S                   10000000     lua51:lua51.dll
 0000:fff8b000       .debug$S                   10000000     lua51:lua51.dll
 0000:fff8b000       .debug$S                   10000000     lua51:lua51.dll
 0001:00000320       _band                      10001320 f   bit64.obj
 0001:00000390       _bor                       10001390 f   bit64.obj
 0001:00000400       _bxor                      10001400 f   bit64.obj
 0001:00000470       _bnot                      10001470 f   bit64.obj
 0001:000004a0       _lshift                    100014a0 f   bit64.obj
 0001:00000510       _rshift                    10001510 f   bit64.obj
 0001:00000580       _arshift                   10001580 f   bit64.obj
 0001:000005f0       _f_new                     100015f0 f   bit64.obj
 0001:00000870       _f_tostring                10001870 f   bit64.obj
 0001:000008d0       _f_type                    100018d0 f   bit64.obj
 0001:00000950       _f_add                     10001950 f   bit64.obj
 0001:000009c0       _f_sub                     100019c0 f   bit64.obj
 0001:00000a10       _f_mul                     10001a10 f   bit64.obj
 0001:00000ab0       _f_div                     10001ab0 f   bit64.obj
 0001:00000bd0       _f_mod                     10001bd0 f   bit64.obj
 0001:00000c30       _f_unm                     10001c30 f   bit64.obj
 0001:00000c60       _f_eq                      10001c60 f   bit64.obj
 0001:00000cc0       _f_lt                      10001cc0 f   bit64.obj
 0001:00000d20       _f_le                      10001d20 f   bit64.obj
 0001:00000d80       _f_tonumber                10001d80 f   bit64.obj
 0001:000026a0       _RegisterObject            100036a0 f   exported.obj
 0001:00002710       _PushAnalyseInfo           10003710 f   exported.obj
 0001:00003384       $LN20                      10004384     exported.obj
 0001:00003420       _FillFarMacroCall_Callback@12 10004420 f   exported.obj
 0001:00003470       _FillFarMacroCall          10004470 f   exported.obj
 0001:00004e64       $LN37                      10005e64     exported.obj
 0001:00004e70       $LN36                      10005e70     exported.obj
 0001:00005980       _getF                      10006980 f   lflua.obj
 0001:000059e0       _errfile                   100069e0 f   lflua.obj
 0001:000077d0       _FL_PushParams             100087d0 f   luamacro.obj
 0001:000079b0       $LN31                      100089b0     luamacro.obj
 0001:000079e0       _InitMPR                   100089e0 f   luamacro.obj
 0001:00007f20       _MacroCallFarCallback@12   10008f20 f   luamacro.obj
 0001:00008200       _uc_tostring               10009200 f   lusercontrol.obj
 0001:00008270       _uc_index                  10009270 f   lusercontrol.obj
 0001:000083d0       _uc_newindex               100093d0 f   lusercontrol.obj
 0001:00008540       _uc_New                    10009540 f   lusercontrol.obj
 0001:00008700       _OptHandle                 10009700 f   service.obj
 0001:00008760       $LN11                      10009760     service.obj
 0001:00008780       _get_env_flag              10009780 f   service.obj
 0001:000088f8       $LN20                      100098f8     service.obj
 0001:00008910       _check_env_flag            10009910 f   service.obj
 0001:00008c54       $LN38                      10009c54     service.obj
 0001:00008cf0       _CheckFlagsFromTable       10009cf0 f   service.obj
 0001:00008db0       _GetRealPluginData         10009db0 f   service.obj
 0001:00008dd0       _GetFakePluginData         10009dd0 f   service.obj
 0001:00008e10       _PluginHandle_rawhandle    10009e10 f   service.obj
 0001:00008f90       _far_GetFileOwner          10009f90 f   service.obj
 0001:000091f0       _far_GetNumberOfLinks      1000a1f0 f   service.obj
 0001:000092c0       _far_GetLuafarVersion      1000a2c0 f   service.obj
 0001:000093e0       _FillEditorSetPosition     1000a3e0 f   service.obj
 0001:00009bd0       _far_PluginStartupInfo     1000abd0 f   service.obj
 0001:00009da0       _far_GetCurrentDirectory   1000ada0 f   service.obj
 0001:00009e80       _push_ev_filename          1000ae80 f   service.obj
 0001:00009fd0       _editor_GetFileName        1000afd0 f   service.obj
 0001:0000a010       _editor_GetInfo            1000b010 f   service.obj
 0001:0000a390       _FastGetString             1000b390 f   service.obj
 0001:0000a430       __EditorGetString          1000b430 f   service.obj
 0001:0000a810       _editor_GetString          1000b810 f   service.obj
 0001:0000a820       _editor_GetStringW         1000b820 f   service.obj
 0001:0000a840       __EditorSetString          1000b840 f   service.obj
 0001:0000aa60       _editor_SetString          1000ba60 f   service.obj
 0001:0000aa70       _editor_SetStringW         1000ba70 f   service.obj
 0001:0000aa90       _editor_InsertString       1000ba90 f   service.obj
 0001:0000aaf0       _editor_DeleteString       1000baf0 f   service.obj
 0001:0000ab40       __EditorInsertText         1000bb40 f   service.obj
 0001:0000acb0       _editor_InsertText         1000bcb0 f   service.obj
 0001:0000acc0       _editor_InsertTextW        1000bcc0 f   service.obj
 0001:0000ace0       _editor_DeleteChar         1000bce0 f   service.obj
 0001:0000ad30       _editor_DeleteBlock        1000bd30 f   service.obj
 0001:0000ad80       _editor_UndoRedo           1000bd80 f   service.obj
 0001:0000adf0       _FillKeyBarTitles          1000bdf0 f   service.obj
 0001:0000afe0       _SetKeyBar                 1000bfe0 f   service.obj
 0001:0000b140       _editor_SetKeyBar          1000c140 f   service.obj
 0001:0000b160       _viewer_SetKeyBar          1000c160 f   service.obj
 0001:0000b170       _editor_SetParam           1000c170 f   service.obj
 0001:0000b3f0       _editor_SetPosition        1000c3f0 f   service.obj
 0001:0000b4d0       _editor_Redraw             1000c4d0 f   service.obj
 0001:0000b520       _editor_ExpandTabs         1000c520 f   service.obj
 0001:0000b580       _PushBookmarks             1000c580 f   service.obj
 0001:0000b750       _editor_GetBookmarks       1000c750 f   service.obj
 0001:0000b770       _editor_GetSessionBookmarks 1000c770 f   service.obj
 0001:0000b790       _editor_AddSessionBookmark 1000c790 f   service.obj
 0001:0000b7e0       _editor_ClearSessionBookmarks 1000c7e0 f   service.obj
 0001:0000b830       _editor_DeleteSessionBookmark 1000c830 f   service.obj
 0001:0000b890       _editor_NextSessionBookmark 1000c890 f   service.obj
 0001:0000b8e0       _editor_PrevSessionBookmark 1000c8e0 f   service.obj
 0001:0000b930       _editor_SetTitle           1000c930 f   service.obj
 0001:0000ba20       _editor_GetTitle           1000ca20 f   service.obj
 0001:0000bb30       _editor_Quit               1000cb30 f   service.obj
 0001:0000bb80       _FillEditorSelect          1000cb80 f   service.obj
 0001:0000bd00       _editor_Select             1000cd00 f   service.obj
 0001:0000be00       _editor_GetSelection       1000ce00 f   service.obj
 0001:0000c1d0       __EditorTabConvert         1000d1d0 f   service.obj
 0001:0000c270       _editor_TabToReal          1000d270 f   service.obj
 0001:0000c290       _editor_RealToTab          1000d290 f   service.obj
 0001:0000c530       _GetOptGuid                1000d530 f   service.obj
 0001:0000c5d0       _editor_AddColor           1000d5d0 f   service.obj
 0001:0000c7e0       _editor_DelColor           1000d7e0 f   service.obj
 0001:0000c890       _editor_GetColor           1000d890 f   service.obj
 0001:0000caa0       _editor_SaveFile           1000daa0 f   service.obj
 0001:0000cff8       $LN54                      1000dff8     service.obj
 0001:0000d010       $LN53                      1000e010     service.obj
 0001:0000d020       _editor_ReadInput          1000e020 f   service.obj
 0001:0000d428       $LN46                      1000e428     service.obj
 0001:0000d440       $LN45                      1000e440     service.obj
 0001:0000d450       _OptInputRecord            1000e450 f   service.obj
 0001:0000d4f0       _editor_ProcessInput       1000e4f0 f   service.obj
 0001:0000d570       _editor_SubscribeChangeEvent 1000e570 f   service.obj
 0001:0000d610       _far_Menu                  1000e610 f   service.obj
 0001:0000e9d0       _far_Message               1000f9d0 f   service.obj
 0001:0000ee00       _panel_CheckPanelsExist    1000fe00 f   service.obj
 0001:0000ee40       _panel_ClosePanel          1000fe40 f   service.obj
 0001:0000ef40       _panel_GetPanelInfo        1000ff40 f   service.obj
 0001:0000f250       _get_panel_item            10010250 f   service.obj
 0001:0000f350       _panel_GetPanelItem        10010350 f   service.obj
 0001:0000f370       _panel_GetSelectedPanelItem 10010370 f   service.obj
 0001:0000f390       _panel_GetCurrentPanelItem 10010390 f   service.obj
 0001:0000f3b0       _get_string_info           100103b0 f   service.obj
 0001:0000f4f0       _panel_GetPanelFormat      100104f0 f   service.obj
 0001:0000f510       _panel_GetPanelHostFile    10010510 f   service.obj
 0001:0000f530       _panel_GetColumnTypes      10010530 f   service.obj
 0001:0000f550       _panel_GetColumnWidths     10010550 f   service.obj
 0001:0000f570       _panel_GetPanelPrefix      10010570 f   service.obj
 0001:0000f590       _panel_RedrawPanel         10010590 f   service.obj
 0001:0000f690       _SetPanelBooleanProperty   10010690 f   service.obj
 0001:0000f720       _SetPanelIntegerProperty   10010720 f   service.obj
 0001:0000f7b0       _panel_SetSortOrder        100107b0 f   service.obj
 0001:0000f7d0       _panel_SetDirectoriesFirst 100107d0 f   service.obj
 0001:0000f7f0       _panel_UpdatePanel         100107f0 f   service.obj
 0001:0000f810       _panel_SetSortMode         10010810 f   service.obj
 0001:0000f830       _panel_SetViewMode         10010830 f   service.obj
 0001:0000f850       _panel_GetPanelDirectory   10010850 f   service.obj
 0001:0000fb20       _panel_SetPanelDirectory   10010b20 f   service.obj
 0001:0000ff90       _panel_GetCmdLine          10010f90 f   service.obj
 0001:00010080       _panel_SetCmdLine          10011080 f   service.obj
 0001:00010160       _panel_GetCmdLinePos       10011160 f   service.obj
 0001:000101c0       _panel_SetCmdLinePos       100111c0 f   service.obj
 0001:00010210       _panel_InsertCmdLine       10011210 f   service.obj
 0001:000102f0       _panel_GetCmdLineSelection 100112f0 f   service.obj
 0001:000103a0       _panel_SetCmdLineSelection 100113a0 f   service.obj
 0001:00010440       _ChangePanelSelection      10011440 f   service.obj
 0001:00010660       _panel_SetSelection        10011660 f   service.obj
 0001:00010680       _panel_ClearSelection      10011680 f   service.obj
 0001:00010690       _panel_BeginSelection      10011690 f   service.obj
 0001:00010710       _panel_EndSelection        10011710 f   service.obj
 0001:00010790       _panel_SetUserScreen       10011790 f   service.obj
 0001:000107e0       _panel_GetUserScreen       100117e0 f   service.obj
 0001:00010830       _panel_IsActivePanel       10011830 f   service.obj
 0001:00010880       _panel_SetActivePanel      10011880 f   service.obj
 0001:00010900       _far_GetDirList            10011900 f   service.obj
 0001:00010a40       _far_GetPluginDirList      10011a40 f   service.obj
 0001:00010ba0       _far_RestoreScreen         10011ba0 f   service.obj
 0001:00010c10       _far_FreeScreen            10011c10 f   service.obj
 0001:00010c60       _far_SaveScreen            10011c60 f   service.obj
 0001:00010f40       _SetFarDialogItem          10011f40 f   service.obj
 0001:000114d0       _PushDlgItem               100124d0 f   service.obj
 0001:00011a90       _PushDlgItemNum            10012a90 f   service.obj
 0001:00011b40       _SetDlgItem                10012b40 f   service.obj
 0001:00011cc0       _far_SendDlgMessage        10012cc0 f   service.obj
 0001:00012f18       $LN180                     10013f18     service.obj
 0001:00012f24       $LN179                     10013f24     service.obj
 0001:00012f68       $LN182                     10013f68     service.obj
 0001:00012ff0       $LN181                     10013ff0     service.obj
 0001:00013254       $LN31                      10014254     service.obj
 0001:00013264       $LN30                      10014264     service.obj
 0001:0001327c       $LN33                      1001427c     service.obj
 0001:000132a0       $LN32                      100142a0     service.obj
 0001:00013534       $LN30                      10014534     service.obj
 0001:0001354c       $LN29                      1001454c     service.obj
 0001:00013730       _far_DialogInit            10014730 f   service.obj
 0001:00013b80       _far_DialogRun             10014b80 f   service.obj
 0001:00013c40       _far_DialogFree            10014c40 f   service.obj
 0001:00013cb0       _dialog_tostring           10014cb0 f   service.obj
 0001:00013d10       _dialog_rawhandle          10014d10 f   service.obj
 0001:00013d60       _far_GetDlgItem            10014d60 f   service.obj
 0001:00013dd0       _far_SetDlgItem            10014dd0 f   service.obj
 0001:00013e40       _far_SubscribeDialogDrawEvents 10014e40 f   service.obj
 0001:00013e60       _editor_Editor             10014e60 f   service.obj
 0001:000140f0       _viewer_Viewer             100150f0 f   service.obj
 0001:00014350       _viewer_GetFileName        10015350 f   service.obj
 0001:00014390       _viewer_GetInfo            10015390 f   service.obj
 0001:00014620       _viewer_Quit               10015620 f   service.obj
 0001:00014660       _viewer_Redraw             10015660 f   service.obj
 0001:000146a0       _viewer_Select             100156a0 f   service.obj
 0001:00014740       _viewer_SetPosition        10015740 f   service.obj
 0001:00014910       _viewer_SetMode            10015910 f   service.obj
 0001:00014a20       _far_ShowHelp              10015a20 f   service.obj
 0001:00014c50       _far_InputBox              10015c50 f   service.obj
 0001:000151c0       _far_GetMsg                100161c0 f   service.obj
 0001:000152d0       _far_Text                  100162d0 f   service.obj
 0001:00015420       _far_CopyToClipboard       10016420 f   service.obj
 0001:00015530       _far_PasteFromClipboard    10016530 f   service.obj
 0001:00015620       _far_InputRecordToName     10016620 f   service.obj
 0001:000158d0       _far_NameToInputRecord     100168d0 f   service.obj
 0001:000159c0       _far_LStricmp              100169c0 f   service.obj
 0001:00015b20       _far_LStrnicmp             10016b20 f   service.obj
 0001:00015c90       _far_ProcessName           10016c90 f   service.obj
 0001:00016030       _far_GetReparsePointInfo   10017030 f   service.obj
 0001:000161b0       _far_LIsAlpha              100171b0 f   service.obj
 0001:00016280       _far_LIsAlphanum           10017280 f   service.obj
 0001:00016350       _far_LIsLower              10017350 f   service.obj
 0001:00016420       _far_LIsUpper              10017420 f   service.obj
 0001:000164f0       _convert_buf               100174f0 f   service.obj
 0001:000165c0       _far_LLowerBuf             100175c0 f   service.obj
 0001:000165e0       _far_LUpperBuf             100175e0 f   service.obj
 0001:00016600       _far_MkTemp                10017600 f   service.obj
 0001:00016790       _far_MkLink                10017790 f   service.obj
 0001:000169d0       _far_GetPathRoot           100179d0 f   service.obj
 0001:00016b30       _truncstring               10017b30 f   service.obj
 0001:00016cf0       _far_TruncPathStr          10017cf0 f   service.obj
 0001:00016d10       _far_TruncStr              10017d10 f   service.obj
 0001:00016d30       _FrsUserFunc@12            10017d30 f   service.obj
 0001:00016ea0       _far_RecursiveSearch       10017ea0 f   service.obj
 0001:000171e0       _far_ConvertPath           100181e0 f   service.obj
 0001:00017380       _far_AdvControl            10018380 f   service.obj
 0001:00017af4       $LN56                      10018af4     service.obj
 0001:00017b38       $LN55                      10018b38     service.obj
 0001:00017b60       _far_MacroLoadAll          10018b60 f   service.obj
 0001:00017cf0       _far_MacroSaveAll          10018cf0 f   service.obj
 0001:00017d30       _far_MacroGetState         10018d30 f   service.obj
 0001:00017d70       _far_MacroGetArea          10018d70 f   service.obj
 0001:00017db0       _MacroSendString           10018db0 f   service.obj
 0001:00017f80       _far_MacroPost             10018f80 f   service.obj
 0001:00017f90       _far_MacroCheck            10018f90 f   service.obj
 0001:00017fb0       _far_MacroGetLastError     10018fb0 f   service.obj
 0001:00018220       _far_MacroAdd              10019220 f   service.obj
 0001:000185f0       _far_MacroDelete           100195f0 f   service.obj
 0001:00018680       _AddMacroData_gc           10019680 f   service.obj
 0001:00018710       _far_MacroExecute          10019710 f   service.obj
 0001:00018910       _far_CPluginStartupInfo    10019910 f   service.obj
 0001:000189d0       _far_MakeMenuItems         100199d0 f   service.obj
 0001:00018cf0       _far_Show                  10019cf0 f   service.obj
 0001:00018e20       _far_CreateFileFilter      10019e20 f   service.obj
 0001:00018ec0       _filefilter_Free           10019ec0 f   service.obj
 0001:00018f30       _filefilter_gc             10019f30 f   service.obj
 0001:00018fa0       _filefilter_tostring       10019fa0 f   service.obj
 0001:00019000       _filefilter_OpenMenu       1001a000 f   service.obj
 0001:00019070       _filefilter_Starting       1001a070 f   service.obj
 0001:000190e0       _filefilter_IsFileInFilter 1001a0e0 f   service.obj
 0001:00019190       _plugin_load               1001a190 f   service.obj
 0001:000192b0       _far_LoadPlugin            1001a2b0 f   service.obj
 0001:000192c0       _far_ForcedLoadPlugin      1001a2c0 f   service.obj
 0001:000192e0       _far_UnloadPlugin          1001a2e0 f   service.obj
 0001:00019330       _far_FindPlugin            1001a330 f   service.obj
 0001:00019470       _PutPluginMenuItemToTable  1001a470 f   service.obj
 0001:00019620       _PutVersionInfoToTable     1001a620 f   service.obj
 0001:00019770       _far_GetPluginInformation  1001a770 f   service.obj
 0001:00019cd0       _far_GetPlugins            1001acd0 f   service.obj
 0001:00019da0       _far_IsPluginLoaded        1001ada0 f   service.obj
 0001:00019eb0       _far_XLat                  1001aeb0 f   service.obj
 0001:0001a0f0       _far_FormatFileSize        1001b0f0 f   service.obj
 0001:0001a2b0       _far_FarClock              1001b2b0 f   service.obj
 0001:0001a370       _far_Timer                 1001b370 f   service.obj
 0001:0001a500       _timer_Close               1001b500 f   service.obj
 0001:0001a5a0       _timer_gc                  1001b5a0 f   service.obj
 0001:0001a610       _timer_tostring            1001b610 f   service.obj
 0001:0001a670       _timer_index               1001b670 f   service.obj
 0001:0001a830       _timer_newindex            1001b830 f   service.obj
 0001:0001a9e0       _far_CreateSettings        1001b9e0 f   service.obj
 0001:0001abe0       _Settings_set              1001bbe0 f   service.obj
 0001:0001ae30       _Settings_get              1001be30 f   service.obj
 0001:0001b060       _Settings_delete           1001c060 f   service.obj
 0001:0001b1a0       _Settings_createsubkey     1001c1a0 f   service.obj
 0001:0001b3e0       _Settings_opensubkey       1001c3e0 f   service.obj
 0001:0001b520       _Settings_enum             1001c520 f   service.obj
 0001:0001ba30       _Settings_free             1001ca30 f   service.obj
 0001:0001bab0       _far_FreeSettings          1001cab0 f   service.obj
 0001:0001bb40       _Settings_tostring         1001cb40 f   service.obj
 0001:0001bba0       _far_ColorDialog           1001cba0 f   service.obj
 0001:0001bcf0       _far_RunDefaultScript      1001ccf0 f   service.obj
 0001:0001bd20       _far_FileTimeResolution    1001cd20 f   service.obj
 0001:0001bd80       _GetPluginModuleHandle     1001cd80 f   service.obj
 0001:0001be00       _far_host_GetFiles         1001ce00 f   service.obj
 0001:0001c0a0       _far_host_PutFiles         1001d0a0 f   service.obj
 0001:0001c340       _far_host_GetFindData      1001d340 f   service.obj
 0001:0001c4a0       _far_host_FreeUserData     1001d4a0 f   service.obj
 0001:0001c590       _far_host_SetDirectory     1001d590 f   service.obj
 0001:0001c780       _luaopen_far               1001d780 f   service.obj
 0001:0001ce20       _CustomAllocator           1001de20 f   service.obj
 0001:0001d230       _str_rep                   1001e230 f   slnunico.obj
 0001:0001d2c0       _writer                    1001e2c0 f   slnunico.obj
 0001:0001d2e0       _str_dump                  1001e2e0 f   slnunico.obj
 0001:0001d370       _str_format                1001e370 f   slnunico.obj
 0001:0001d9b0       $LN84                      1001e9b0     slnunico.obj
 0001:0001d9cc       $LN83                      1001e9cc     slnunico.obj
 0001:0001da00       $LN89                      1001ea00     slnunico.obj
 0001:0001da10       $LN88                      1001ea10     slnunico.obj
 0001:0001da70       _utf8_valid                1001ea70 f   slnunico.obj
 0001:0001db70       _utf8_decode               1001eb70 f   lutf8lib.obj
 0001:0001dc10       _utf8_next                 1001ec10 f   lutf8lib.obj
 0001:0001dc40       _utf8_length               1001ec40 f   lutf8lib.obj
 0001:0001dc80       _utf8_offset               1001ec80 f   lutf8lib.obj
 0001:0001dd20       _utf8_range                1001ed20 f   lutf8lib.obj
 0001:0001de00       _find_in_range             1001ee00 f   lutf8lib.obj
 0001:0001de60       _utf8_isdigit              1001ee60 f   lutf8lib.obj
 0001:0001dec0       _utf8_islower              1001eec0 f   lutf8lib.obj
 0001:0001df20       _utf8_iscompose            1001ef20 f   lutf8lib.obj
 0001:0001df80       _utf8_tolower              1001ef80 f   lutf8lib.obj
 0001:0001dfe0       _utf8_toupper              1001efe0 f   lutf8lib.obj
 0001:0001e040       _utf8_totitle              1001f040 f   lutf8lib.obj
 0001:0001e0a0       _utf8_tofold               1001f0a0 f   lutf8lib.obj
 0001:0001e100       _utf8_width                1001f100 f   lutf8lib.obj
 0001:0001e220       _utf8_safe_decode          1001f220 f   lutf8lib.obj
 0001:0001e2c0       _Lutf8_len                 1001f2c0 f   lutf8lib.obj
 0001:0001e420       _Lutf8_sub                 1001f420 f   lutf8lib.obj
 0001:0001e4a0       _Lutf8_reverse             1001f4a0 f   lutf8lib.obj
 0001:0001e620       _Lutf8_byte                1001f620 f   lutf8lib.obj
 0001:0001e6d0       _Lutf8_codepoint           1001f6d0 f   lutf8lib.obj
 0001:0001e820       _Lutf8_char                1001f820 f   lutf8lib.obj
 0001:0001e930       _Lutf8_lower               1001f930 f   lutf8lib.obj
 0001:0001ead0       _Lutf8_upper               1001fad0 f   lutf8lib.obj
 0001:0001ec70       _Lutf8_title               1001fc70 f   lutf8lib.obj
 0001:0001ee10       _Lutf8_fold                1001fe10 f   lutf8lib.obj
 0001:0001efb0       _Lutf8_escape              1001ffb0 f   lutf8lib.obj
 0001:0001f1c4       $LN55                      100201c4     lutf8lib.obj
 0001:0001f1d4       $LN54                      100201d4     lutf8lib.obj
 0001:0001f220       _Lutf8_insert              10020220 f   lutf8lib.obj
 0001:0001f350       _Lutf8_remove              10020350 f   lutf8lib.obj
 0001:0001f440       _push_offset               10020440 f   lutf8lib.obj
 0001:0001f4e0       _Lutf8_charpos             100204e0 f   lutf8lib.obj
 0001:0001f5b0       _Lutf8_offset              100205b0 f   lutf8lib.obj
 0001:0001f700       _Lutf8_next                10020700 f   lutf8lib.obj
 0001:0001f780       _iter_aux                  10020780 f   lutf8lib.obj
 0001:0001f860       _iter_auxstrict            10020860 f   lutf8lib.obj
 0001:0001f880       _iter_auxlax               10020880 f   lutf8lib.obj
 0001:0001f890       _Lutf8_codes               10020890 f   lutf8lib.obj
 0001:0001f8f0       _Lutf8_width               100208f0 f   lutf8lib.obj
 0001:0001fa00       _Lutf8_widthindex          10020a00 f   lutf8lib.obj
 0001:0001fae0       _Lutf8_ncasecmp            10020ae0 f   lutf8lib.obj
 0001:0001fbc0       _classend                  10020bc0 f   lutf8lib.obj
 0001:0001fc80       _match_class               10020c80 f   lutf8lib.obj
 0001:00020074       $LN163                     10021074     lutf8lib.obj
 0001:000200a8       $LN162                     100210a8     lutf8lib.obj
 0001:000200d0       _matchbracketclass         100210d0 f   lutf8lib.obj
 0001:000201c0       _singlematch               100211c0 f   lutf8lib.obj
 0001:00020270       _matchbalance              10021270 f   lutf8lib.obj
 0001:000203c0       _start_capture             100213c0 f   lutf8lib.obj
 0001:00020410       _match                     10021410 f   lutf8lib.obj
 0001:000209dc       $LN207                     100219dc     lutf8lib.obj
 0001:000209f4       $LN209                     100219f4     lutf8lib.obj
 0001:00020a04       $LN208                     10021a04     lutf8lib.obj
 0001:00020a3c       $LN215                     10021a3c     lutf8lib.obj
 0001:00020a50       $LN214                     10021a50     lutf8lib.obj
 0001:00020a70       _get_index                 10021a70 f   lutf8lib.obj
 0001:00020ac0       _push_captures             10021ac0 f   lutf8lib.obj
 0001:00020ba0       _find_aux                  10021ba0 f   lutf8lib.obj
 0001:00020f80       _Lutf8_find                10021f80 f   lutf8lib.obj
 0001:00020fa0       _Lutf8_match               10021fa0 f   lutf8lib.obj
 0001:00020fb0       _gmatch_aux                10021fb0 f   lutf8lib.obj
 0001:000210e0       _Lutf8_gmatch              100220e0 f   lutf8lib.obj
 0001:00021130       _add_s                     10022130 f   lutf8lib.obj
 0001:00021350       _Lutf8_gsub                10022350 f   lutf8lib.obj
 0001:00021900       _pushresult                10022900 f   uliolib51.obj
 0001:00021a10       _fileerror                 10022a10 f   uliolib51.obj
 0001:00021ae0       _io_type                   10022ae0 f   uliolib51.obj
 0001:00021b90       _io_noclose                10022b90 f   uliolib51.obj
 0001:00021bc0       _io_pclose                 10022bc0 f   uliolib51.obj
 0001:00021c40       _io_fclose                 10022c40 f   uliolib51.obj
 0001:00021cc0       _io_close                  10022cc0 f   uliolib51.obj
 0001:00021d40       _io_gc                     10022d40 f   uliolib51.obj
 0001:00021d90       _io_tostring               10022d90 f   uliolib51.obj
 0001:00021de0       _io_open                   10022de0 f   uliolib51.obj
 0001:00022050       _io_popen                  10023050 f   uliolib51.obj
 0001:00022200       _io_tmpfile                10023200 f   uliolib51.obj
 0001:00022280       _g_iofile                  10023280 f   uliolib51.obj
 0001:00022400       _io_input                  10023400 f   uliolib51.obj
 0001:00022420       _io_output                 10023420 f   uliolib51.obj
 0001:00022440       _f_lines                   10023440 f   uliolib51.obj
 0001:000224a0       _io_lines                  100234a0 f   uliolib51.obj
 0001:00022630       _read_line                 10023630 f   uliolib51.obj
 0001:00022730       _read_chars                10023730 f   uliolib51.obj
 0001:000227f0       _g_read                    100237f0 f   uliolib51.obj
 0001:00022b40       $LN68                      10023b40     uliolib51.obj
 0001:00022b54       $LN67                      10023b54     uliolib51.obj
 0001:00022b70       _io_read                   10023b70 f   uliolib51.obj
 0001:00022bc0       _f_read                    10023bc0 f   uliolib51.obj
 0001:00022c10       _io_readline               10023c10 f   uliolib51.obj
 0001:00022cf0       _g_write                   10023cf0 f   uliolib51.obj
 0001:00022df0       _io_write                  10023df0 f   uliolib51.obj
 0001:00022e40       _f_write                   10023e40 f   uliolib51.obj
 0001:00022e90       _f_seek                    10023e90 f   uliolib51.obj
 0001:00022fd0       _f_setvbuf                 10023fd0 f   uliolib51.obj
 0001:00023090       _io_flush                  10024090 f   uliolib51.obj
 0001:00023130       _f_flush                   10024130 f   uliolib51.obj
 0001:000231c0       _f_rawhandle               100241c0 f   uliolib51.obj
 0001:00023440       _gctm                      10024440 f   uloadlib51.obj
 0001:00023470       _ll_loadfunc               10024470 f   uloadlib51.obj
 0001:00023620       _ll_loadlib                10024620 f   uloadlib51.obj
 0001:00023720       _findfile                  10024720 f   uloadlib51.obj
 0001:00023a80       _loaderror                 10024a80 f   uloadlib51.obj
 0001:00023b50       _loader_Lua                10024b50 f   uloadlib51.obj
 0001:00023ba0       _mkfuncname                10024ba0 f   uloadlib51.obj
 0001:00023bf0       _loader_C                  10024bf0 f   uloadlib51.obj
 0001:00023c80       _loader_Croot              10024c80 f   uloadlib51.obj
 0001:00023d20       _loader_preload            10024d20 f   uloadlib51.obj
 0001:00023da0       _ll_require                10024da0 f   uloadlib51.obj
 0001:00023f80       _ll_module                 10024f80 f   uloadlib51.obj
 0001:00024180       _ll_seeall                 10025180 f   uloadlib51.obj
 0001:000241f0       _setpath                   100251f0 f   uloadlib51.obj
 0001:00025998       $LN26                      10026998     ustring.obj
 0001:000269f0       _ustring_OutputDebugString 100279f0 f   ustring.obj
 0001:00026b30       _ustring_system            10027b30 f   ustring.obj
 0001:00027210       _win_GetEnv                10028210 f   win.obj
 0001:00027450       _win_SetEnv                10028450 f   win.obj
 0001:000275b0       _CheckHKey                 100285b0 f   win.obj
 0001:00027710       _win_SetRegKey             10028710 f   win.obj
 0001:00027c70       _win_GetRegKey             10028c70 f   win.obj
 0001:00027fac       $LN48                      10028fac     win.obj
 0001:00027fd0       _win_DeleteRegKey          10028fd0 f   win.obj
 0001:00028130       _win_DeleteRegValue        10029130 f   win.obj
 0001:00028360       _win_EnumRegKey            10029360 f   win.obj
 0001:000285d0       _win_EnumRegValue          100295d0 f   win.obj
 0001:00028840       _win_ExtractKey            10029840 f   win.obj
 0001:000288e0       _win_ExtractKeyEx          100298e0 f   win.obj
 0001:00028960       _PushWinFindData           10029960 f   win.obj
 0001:00028b90       _win_GetFileInfo           10029b90 f   win.obj
 0001:00028ca0       _win_GetSystemTimeAsFileTime 10029ca0 f   win.obj
 0001:00028cd0       _win_FileTimeToSystemTime  10029cd0 f   win.obj
 0001:00028ee0       _win_SystemTimeToFileTime  10029ee0 f   win.obj
 0001:00029190       _win_FileTimeToLocalFileTime 1002a190 f   win.obj
 0001:00029220       _win_CompareString         1002a220 f   win.obj
 0001:000294b0       _win_wcscmp                1002a4b0 f   win.obj
 0001:00029610       _win_GetVirtualKeys        1002a610 f   win.obj
 0001:00029630       _win_GetConsoleScreenBufferInfo 1002a630 f   win.obj
 0001:00029890       _win_CopyFile              1002a890 f   win.obj
 0001:00029a20       _win_MoveFile              1002aa20 f   win.obj
 0001:00029c00       _win_DeleteFile            1002ac00 f   win.obj
 0001:00029cd0       _mkdir                     1002acd0 f   win.obj
 0001:00029e80       _win_CreateDir             1002ae80 f   win.obj
 0001:0002a040       _win_RemoveDir             1002b040 f   win.obj
 0001:0002a110       _win_ShellExecute          1002b110 f   win.obj
 0001:0002a400       _win_IsProcess64bit        1002b400 f   win.obj
 0001:0002ade0       _PutFileTimeToTableEx      1002bde0 f   win.obj
 0001:0002ae30       _win_GetFileTimes          1002be30 f   win.obj
 0001:0002afa0       _ExtractFileTime           1002bfa0 f   win.obj
 0001:0002b040       _win_SetFileTimes          1002c040 f   win.obj
 0001:0002b2c0       ?DecodePointer@implementation@?1??DecodePointerWrapper@@YGPAXPAX@Z@SGPAX0@Z 1002c2c0 f   vc_crt_fix_impl.obj
 0001:0002b2c0       ?EncodePointer@implementation@?1??EncodePointerWrapper@@YGPAXPAX@Z@SGPAX0@Z 1002c2c0 f   vc_crt_fix_impl.obj
 0001:0002b3d0       ?GetModuleHandleExW@implementation@?1??GetModuleHandleExWWrapper@@YGHKPB_WPAPAUHINSTANCE__@@@Z@SGHK01@Z 1002c3d0 f   vc_crt_fix_impl.obj
 0001:0002b4a0       ?InitializeSListHead@implementation@slist@@YGXPAT_SLIST_HEADER@@@Z 1002c4a0 f   vc_crt_fix_impl.obj
 0001:0002b560       ?InterlockedFlushSList@implementation@slist@@YGPAU_SINGLE_LIST_ENTRY@@PAT_SLIST_HEADER@@@Z 1002c560 f   vc_crt_fix_impl.obj
 0001:0002b590       ?InterlockedPopEntrySList@implementation@slist@@YGPAU_SINGLE_LIST_ENTRY@@PAT_SLIST_HEADER@@@Z 1002c590 f   vc_crt_fix_impl.obj
 0001:0002b5e0       ?InterlockedPushEntrySList@implementation@slist@@YGPAU_SINGLE_LIST_ENTRY@@PAT_SLIST_HEADER@@PAU3@@Z 1002c5e0 f   vc_crt_fix_impl.obj
 0001:0002b620       ?InterlockedPushListSListEx@implementation@slist@@YGPAU_SINGLE_LIST_ENTRY@@PAT_SLIST_HEADER@@PAU3@1K@Z 1002c620 f   vc_crt_fix_impl.obj
 0001:0002b660       ?RtlFirstEntrySList@implementation@slist@@YGPAU_SINGLE_LIST_ENTRY@@PAT_SLIST_HEADER@@@Z 1002c660 f   vc_crt_fix_impl.obj
 0001:0002b690       ?QueryDepthSList@implementation@slist@@YGGPAT_SLIST_HEADER@@@Z 1002c690 f   vc_crt_fix_impl.obj
 0001:0002b940       ?GetNumaHighestNodeNumber@implementation@?1??GetNumaHighestNodeNumberWrapper@@YGHPAK@Z@SGH0@Z 1002c940 f   vc_crt_fix_impl.obj
 0001:0002b9b0       ?GetLogicalProcessorInformation@implementation@?1??GetLogicalProcessorInformationWrapper@@YGHPAU_SYSTEM_LOGICAL_PROCESSOR_INFORMATION@@PAK@Z@SGH01@Z 1002c9b0 f   vc_crt_fix_impl.obj
 0001:0002ba10       ?SetThreadStackGuarantee@implementation@?1??SetThreadStackGuaranteeWrapper@@YGHPAK@Z@SGH0@Z 1002ca10 f   vc_crt_fix_impl.obj
 0001:0002ba70       ?InitializeCriticalSectionEx@implementation@?1??InitializeCriticalSectionExWrapper@@YGHPAU_RTL_CRITICAL_SECTION@@KK@Z@SGH0KK@Z 1002ca70 f   vc_crt_fix_impl.obj
 0001:0002baf0       ?CompareStringEx@implementation@?1??CompareStringExWrapper@@YGHPB_WK0H0HPAU_nlsversioninfo@@PAXJ@Z@SGH0K0H0H12J@Z 1002caf0 f   vc_crt_fix_impl.obj
 0001:0002bb70       ?CompareStringEx@implementation@?1??LCMapStringExWrapper@@YGHPB_WK0HPA_WHPAU_nlsversioninfo@@PAXJ@Z@SGH0K0H1H23J@Z 1002cb70 f   vc_crt_fix_impl.obj
 0001:0002bcf6       ?find_pe_section@@YAPAU_IMAGE_SECTION_HEADER@@QAEI@Z 1002ccf6 f   LIBCMT:utility.obj
 0001:0002c010       ?dllmain_crt_dispatch@@YGHQAUHINSTANCE__@@KQAX@Z 1002d010 f   LIBCMT:dll_dllmain.obj
 0001:0002c063       ?dllmain_crt_process_attach@@YAHQAUHINSTANCE__@@QAX@Z 1002d063 f   LIBCMT:dll_dllmain.obj
 0001:0002c16a       ?dllmain_crt_process_detach@@YAH_N@Z 1002d16a f   LIBCMT:dll_dllmain.obj
 0001:0002c21a       ?dllmain_dispatch@@YAHQAUHINSTANCE__@@KQAX@Z 1002d21a f   LIBCMT:dll_dllmain.obj
 0001:0002c320       ?dllmain_raw@@YGHQAUHINSTANCE__@@KQAX@Z 1002d320 f   LIBCMT:dll_dllmain.obj
 0001:0002c670       $$000000                   1002d670     LIBCMT:sehprolg4.obj
 0001:0002c6cb       ___get_entropy             1002d6cb f   LIBCMT:gs_support.obj
 0001:0002cbe0       $$000000                   1002dbe0     libvcruntime:strchr.obj
 0001:0002cd10       $$000000                   1002dd10     libvcruntime:strrchr.obj
 0001:0002d29c       ?_FilterSetCurrentException@@YAKPAU_EXCEPTION_POINTERS@@E@Z 1002e29c f   libvcruntime:ehhelpers.obj
 0001:0002d3f0       _ValidateLocalCookies      1002e3f0 f   libvcruntime:chandler4.obj
 0001:0002d590       $$000000                   1002e590     libvcruntime:memset.obj
 0001:0002d889       ??$BuildCatchObjectHelperInternal@V__FrameHandler3@@@@YAHPAUEHExceptionRecord@@PAXPBU_s_HandlerType@@PBU_s_CatchableType@@@Z 1002e889 f   libvcruntime:frame.obj
 0001:0002d9c7       ??$BuildCatchObjectInternal@V__FrameHandler3@@@@YAXPAUEHExceptionRecord@@PAXPBU_s_HandlerType@@PBU_s_CatchableType@@@Z 1002e9c7 f   libvcruntime:frame.obj
 0001:0002da60       ??$CatchIt@V__FrameHandler3@@@@YAXPAUEHExceptionRecord@@PAUEHRegistrationNode@@PAU_CONTEXT@@PAXPBU_s_FuncInfo@@PBU_s_HandlerType@@PBU_s_CatchableType@@PBU_s_TryBlockMapEntry@@H1EE@Z 1002ea60 f   libvcruntime:frame.obj
 0001:0002dae0       ??$FindHandler@V__FrameHandler3@@@@YAXPAUEHExceptionRecord@@PAUEHRegistrationNode@@PAU_CONTEXT@@PAXPBU_s_FuncInfo@@EH1@Z 1002eae0 f   libvcruntime:frame.obj
 0001:0002de96       ??$FindHandlerForForeignException@V__FrameHandler3@@@@YAXPAUEHExceptionRecord@@PAUEHRegistrationNode@@PAU_CONTEXT@@PAXPBU_s_FuncInfo@@HH1@Z 1002ee96 f   libvcruntime:frame.obj
 0001:0002e218       ?CallCatchBlock@@YAPAXPAUEHExceptionRecord@@PAUEHRegistrationNode@@PAU_CONTEXT@@PBU_s_FuncInfo@@PAXHK@Z 1002f218 f   libvcruntime:frame.obj
 0001:0002e3dc       ?CallUnexpected@@YAXPBU_s_ESTypeList@@@Z 1002f3dc f   libvcruntime:frame.obj
 0001:0002e3fc       __catch$?CallUnexpected@@YAXPBU_s_ESTypeList@@@Z$0 1002f3fc f   libvcruntime:frame.obj
 0001:0002e416       ?ExFilterRethrow@@YAHPAU_EXCEPTION_POINTERS@@@Z 1002f416 f   libvcruntime:frame.obj
 0001:0002e560       ?IsInExceptionSpec@@YAEPAUEHExceptionRecord@@PBU_s_ESTypeList@@@Z 1002f560 f   libvcruntime:frame.obj
 0001:0002e640       $$000000                   1002f640     libvcruntime:lowhelpr.obj
 0001:0002e760       $$000000                   1002f760     libvcruntime:exsup4.obj
 0001:0002e7f0       __unwind_handler4          1002f7f0 f   libvcruntime:exsup4.obj
 0001:0002e8c7       ?try_get_first_available_module@@YAPAUHINSTANCE__@@QBW4module_id@?A0x1172487b@@0@Z 1002f8c7 f   libvcruntime:winapi_downlevel.obj
 0001:0002e973       ?try_get_function@@YAPAXW4function_id@?A0x1172487b@@QBDQBW4module_id@2@2@Z 1002f973 f   libvcruntime:winapi_downlevel.obj
 0001:0002ec30       $$000000                   1002fc30     libvcruntime:memmove.obj
 0001:0002ee94       TrailingUpVec              1002fe94     libvcruntime:memmove.obj
 0001:0002ef40       TrailingDownVec            1002ff40     libvcruntime:memmove.obj
 0001:0002f1b0       $$000000                   100301b0     libvcruntime:exsup.obj
 0001:0002f1d1       __unwind_handler           100301d1 f   libvcruntime:exsup.obj
 0001:0002f2f0       $$000000                   100302f0     libvcruntime:memcpy.obj
 0001:0002f554       TrailingUpVec              10030554     libvcruntime:memcpy.obj
 0001:0002f600       TrailingDownVec            10030600     libvcruntime:memcpy.obj
 0001:0002f864       ??$?RV<lambda_c29ee0499b841886b80d843682cc403a>@@AAV<lambda_0be4ab1c2a6918fda4e39227d83ea893>@@V<lambda_5a3ed3da325c8ea037a470278c0f2d16>@@@?$__crt_seh_guarded_call@H@@QAEH$$QAV<lambda_c29ee0499b841886b80d843682cc403a>@@AAV<lambda_0be4ab1c2a6918fda4e39227d83ea893>@@$$QAV<lambda_5a3ed3da325c8ea037a470278c0f2d16>@@@Z 10030864 f   libucrt:output.obj
 0001:0002f8bf       ??$common_vsprintf@Vstandard_base@__crt_stdio_output@@D@@YAH_KQADIQBDQAU__crt_locale_pointers@@1@Z 100308bf f   libucrt:output.obj
 0001:0002fa3d       ??$common_vsprintf@Vstandard_base@__crt_stdio_output@@_W@@YAH_KQA_WIQB_WQAU__crt_locale_pointers@@QAD@Z 10030a3d f   libucrt:output.obj
 0001:00030217       ??R<lambda_0be4ab1c2a6918fda4e39227d83ea893>@@QBEHXZ 10031217 f   libucrt:output.obj
 0001:000305ec       $LN53                      100315ec     libucrt:output.obj
 0001:00030700       $LN53                      10031700     libucrt:output.obj
 0001:0003081c       $LN53                      1003181c     libucrt:output.obj
 0001:00031618       $LN20                      10032618     libucrt:output.obj
 0001:0003162c       $LN17                      1003262c     libucrt:output.obj
 0001:000326c3       ___hw_cw_sse2              100336c3 f   libucrt:ieee87.obj
 0001:00032b49       __hw_cw                    10033b49 f   libucrt:ieee87.obj
 0001:00032be7       ??$common_fsopen@_W@@YAPAU_iobuf@@QB_W0H@Z 10033be7 f   libucrt:fopen.obj
 0001:00032fd8       ??$common_freopen@_W@@YAHQAPAU_iobuf@@QB_W1V__crt_stdio_stream@@H@Z 10033fd8 f   libucrt:freopen.obj
 0001:0003366d       _memcpy_s                  1003466d f   libucrt:cfout.obj
 0001:0003366d       _memcpy_s                  1003466d f   libucrt:mbctype.obj
 0001:0003366d       _memcpy_s                  1003466d f   libucrt:fread.obj
 0001:0003366d       _memcpy_s                  1003466d f   libucrt:input.obj
 0001:000336ee       ??$common_strerror@D@@YAPADH@Z 100346ee f   libucrt:strerror.obj
 0001:000339c0       $$000000                   100349c0     libucrt:strncmp.obj
 0001:00033b60       $$000000                   10034b60     libucrt:strncpy.obj
 0001:00033c90       $$000000                   10034c90     libucrt:strpbrk.obj
 0001:00033cd0       ??$common_popen@_W@@YAPAU_iobuf@@QB_W0@Z 10034cd0 f   libucrt:popen.obj
 0001:00033dfa       ??$common_popen_nolock@_W@@YAPAU_iobuf@@QB_W0HAAY01H@Z 10034dfa f   libucrt:popen.obj
 0001:00034069       ??$convert_popen_type_to_fdopen_mode@_W@@YA?AU?$fdopen_mode@_W@?A0xe43b7539@@QB_W@Z 10035069 f   libucrt:popen.obj
 0001:000340ee       ??$get_executable_path@_W@@YAPB_WQB_W@Z 100350ee f   libucrt:popen.obj
 0001:00034261       ?idtab@@YAPAUprocess_handle_pair@?A0xe43b7539@@QAU_iobuf@@@Z 10035261 f   libucrt:popen.obj
 0001:000343b4       ??$?RV<lambda_2866be3712abc81a800a822484c830d8>@@AAV<lambda_39ca0ed439415581b5b15c265174cece>@@V<lambda_2b24c74d71094a6cd0cb82e44167d71b>@@@?$__crt_seh_guarded_call@X@@QAEX$$QAV<lambda_2866be3712abc81a800a822484c830d8>@@AAV<lambda_39ca0ed439415581b5b15c265174cece>@@$$QAV<lambda_2b24c74d71094a6cd0cb82e44167d71b>@@@Z 100353b4 f   libucrt:fflush.obj
 0001:00034440       ??$?RV<lambda_2cc53f568c5a2bb6f192f930a45d44ea>@@AAV<lambda_ab61a845afdef5b7c387490eaf3616ee>@@V<lambda_c2ffc0b7726aa6be21d5f0026187e748>@@@?$__crt_seh_guarded_call@X@@QAEX$$QAV<lambda_2cc53f568c5a2bb6f192f930a45d44ea>@@AAV<lambda_ab61a845afdef5b7c387490eaf3616ee>@@$$QAV<lambda_c2ffc0b7726aa6be21d5f0026187e748>@@@Z 10035440 f   libucrt:fflush.obj
 0001:000344ec       ??$?RV<lambda_6d20deecaf4856105ebacbad442d1079>@@AAV<lambda_9a32fed5bf61b6b509b2d3f6003082a1>@@V<lambda_63ea2239ed67c638ddbae41947fdf875>@@@?$__crt_seh_guarded_call@H@@QAEH$$QAV<lambda_6d20deecaf4856105ebacbad442d1079>@@AAV<lambda_9a32fed5bf61b6b509b2d3f6003082a1>@@$$QAV<lambda_63ea2239ed67c638ddbae41947fdf875>@@@Z 100354ec f   libucrt:fflush.obj
 0001:0003454c       ?common_flush_all@@YAH_N@Z 1003554c f   libucrt:fflush.obj
 0001:00034599       ?common_flush_all_should_try_to_flush_stream@@YA_NV__crt_stdio_stream@@QAH@Z 10035599 f   libucrt:fflush.obj
 0001:000345cc       ?is_stream_flushable_or_commitable@@YA_NJ@Z 100355cc f   libucrt:fflush.obj
 0001:000347ac       ??$common_fgets@D@@YAPADQADHV__crt_stdio_stream@@@Z 100357ac f   libucrt:fgets.obj
 0001:00034879       ??$generate_tmpfile_file_name@D@@YA_NQADI@Z 10035879 f   libucrt:tmpfile.obj
 0001:000348ed       ??$get_tmpfile_buffer_nolock@D@@YAPADW4buffer_id@?A0x5b9a7937@@@Z 100358ed f   libucrt:tmpfile.obj
 0001:00034928       ??$initialize_tmpfile_buffer_nolock@D@@YA_NW4buffer_id@?A0x5b9a7937@@@Z 10035928 f   libucrt:tmpfile.obj
 0001:000349de       ?common_tmpfile@@YAHQAPAU_iobuf@@H@Z 100359de f   libucrt:tmpfile.obj
 0001:00034a5a       ?common_tmpfile_nolock@@YAHQAPAU_iobuf@@H@Z 10035a5a f   libucrt:tmpfile.obj
 0001:00034c25       ??$?RV<lambda_4ac01c32aa5b53846f05d0620572872e>@@AAV<lambda_5856287d7ecd2be6c9197bb4007c3f6e>@@V<lambda_e7a9868ed898c75c0f0637692d94351a>@@@?$__crt_seh_guarded_call@I@@QAEI$$QAV<lambda_4ac01c32aa5b53846f05d0620572872e>@@AAV<lambda_5856287d7ecd2be6c9197bb4007c3f6e>@@$$QAV<lambda_e7a9868ed898c75c0f0637692d94351a>@@@Z 10035c25 f   libucrt:fwrite.obj
 0001:00034c80       ??R<lambda_5856287d7ecd2be6c9197bb4007c3f6e>@@QBEIXZ 10035c80 f   libucrt:fwrite.obj
 0001:00034ea7       ??$?RV<lambda_70c0770dcc4f6ec6272bb01dc82d3c91>@@AAV<lambda_ca71763b3c0644891230e4f79ea54fa6>@@V<lambda_ca266f0f09348b8765c113e3a39a2bc1>@@@?$__crt_seh_guarded_call@H@@QAEH$$QAV<lambda_70c0770dcc4f6ec6272bb01dc82d3c91>@@AAV<lambda_ca71763b3c0644891230e4f79ea54fa6>@@$$QAV<lambda_ca266f0f09348b8765c113e3a39a2bc1>@@@Z 10035ea7 f   libucrt:setvbuf.obj
 0001:00034f02       ??R<lambda_ca71763b3c0644891230e4f79ea54fa6>@@QBEHXZ 10035f02 f   libucrt:setvbuf.obj
 0001:00034f9c       ?set_buffer@@YAHV__crt_stdio_stream@@QADIH@Z 10035f9c f   libucrt:setvbuf.obj
 0001:00035051       ??$?RV<lambda_274ecf0a8038e561263518ab346655e8>@@AAV<lambda_21448eb78dd3c4a522ed7c65a98d88e6>@@V<lambda_0ca1de2171e49cefb1e8dc85c06db622>@@@?$__crt_seh_guarded_call@H@@QAEH$$QAV<lambda_274ecf0a8038e561263518ab346655e8>@@AAV<lambda_21448eb78dd3c4a522ed7c65a98d88e6>@@$$QAV<lambda_0ca1de2171e49cefb1e8dc85c06db622>@@@Z 10036051 f   libucrt:input.obj
 0001:00035b03       $LN38                      10036b03     libucrt:input.obj
 0001:00035c27       $LN37                      10036c27     libucrt:input.obj
 0001:0003642e       ??R<lambda_0b87716a0b73cdfba1cd37fcaaa20711>@@QBE_NXZ 1003742e f   libucrt:input.obj
 0001:0003642e       ??R<lambda_c7c3f778895f47e7f4eff38a8fef279a>@@QBE_NXZ 1003742e f   libucrt:input.obj
 0001:0003642e       ??R<lambda_e41f1170c8800e4a6fed1afad60fab6f>@@QBE_NXZ 1003742e f   libucrt:input.obj
 0001:00036458       ??R<lambda_21448eb78dd3c4a522ed7c65a98d88e6>@@QBEHXZ 10037458 f   libucrt:input.obj
 0001:00039018       $LN22                      1003a018     libucrt:input.obj
 0001:00039766       $LN19                      1003a766     libucrt:input.obj
 0001:0003977a       $LN16                      1003a77a     libucrt:input.obj
 0001:0003998e       ??$common_ftell@_J@@YA_JV__crt_stdio_stream@@@Z 1003a98e f   libucrt:ftell.obj
 0001:00039a0e       ??$common_ftell_nolock@_J@@YA_JV__crt_stdio_stream@@@Z 1003aa0e f   libucrt:ftell.obj
 0001:00039b92       ?common_ftell_read_mode_nolock@@YA_JV__crt_stdio_stream@@_J1@Z 1003ab92 f   libucrt:ftell.obj
 0001:00039d51       ?common_ftell_translated_utf8_nolock@@YA_JV__crt_stdio_stream@@_J@Z 1003ad51 f   libucrt:ftell.obj
 0001:00039eea       ?count_newline_bytes@@YA_JQBD0W4__crt_lowio_text_mode@@@Z 1003aeea f   libucrt:ftell.obj
 0001:00039ff8       ?common_fseek@@YAHV__crt_stdio_stream@@_JH@Z 1003aff8 f   libucrt:fseek.obj
 0001:0003a083       ?common_fseek_binary_mode_read_only_fast_track_nolock@@YA_NV__crt_stdio_stream@@_JH@Z 1003b083 f   libucrt:fseek.obj
 0001:0003a15c       ?common_fseek_nolock@@YAHV__crt_stdio_stream@@_JH@Z 1003b15c f   libucrt:fseek.obj
 0001:0003a255       ??$common_dupenv_s@_W@@YAHQAPA_WQAIQB_WHQBDH@Z 1003b255 f   libucrt:getenv.obj
 0001:0003a2ba       ??$common_dupenv_s_nolock@_W@@YAHQAPA_WQAIQB_WHQBDH@Z 1003b2ba f   libucrt:getenv.obj
 0001:0003a366       ??$common_getenv@_W@@YAPA_WQB_W@Z 1003b366 f   libucrt:getenv.obj
 0001:0003a3e5       ??$common_getenv_nolock@_W@@YAPA_WQB_W@Z 1003b3e5 f   libucrt:getenv.obj
 0001:0003a492       ??$common_system@_W@@YAHQB_W@Z 1003b492 f   libucrt:system.obj
 0001:0003a753       ??$?RV<lambda_03b1d95aef87969028cfba75ccab2455>@@AAV<lambda_6e4b09c48022b2350581041d5f6b0c4c>@@V<lambda_22bdf7517842c4b3e53723af5aa32b9e>@@@?$__crt_seh_guarded_call@X@@QAEX$$QAV<lambda_03b1d95aef87969028cfba75ccab2455>@@AAV<lambda_6e4b09c48022b2350581041d5f6b0c4c>@@$$QAV<lambda_22bdf7517842c4b3e53723af5aa32b9e>@@@Z 1003b753 f   libucrt:exit.obj
 0001:0003a7a0       ??R<lambda_6e4b09c48022b2350581041d5f6b0c4c>@@QBE@XZ 1003b7a0 f   libucrt:exit.obj
 0001:0003a87a       ?atexit_exception_filter@@YAHK@Z 1003b87a f   libucrt:exit.obj
 0001:0003a88d       ?common_exit@@YAXHW4_crt_exit_cleanup_mode@@W4_crt_exit_return_mode@@@Z 1003b88d f   libucrt:exit.obj
 0001:0003a8f1       ?exit_or_terminate_process@@YAXI@Z 1003b8f1 f   libucrt:exit.obj
 0001:0003a933       ?is_managed_app@@YA_NXZ    1003b933 f   libucrt:exit.obj
 0001:0003a976       ?try_cor_exit_process@@YAXI@Z 1003b976 f   libucrt:exit.obj
 0001:0003aa04       ??$common_configure_argv@D@@YAHW4_crt_argv_mode@@@Z 1003ba04 f   libucrt:argv_parsing.obj
 0001:0003ab3a       ??$parse_command_line@D@@YAXPADPAPAD0PAI2@Z 1003bb3a f   libucrt:argv_parsing.obj
 0001:0003ad0b       ??$common_get_or_create_environment_nolock@_W@@YAPAPA_WXZ 1003bd0b f   libucrt:environment_initialization.obj
 0001:0003ad37       ??$common_initialize_environment_nolock@D@@YAHXZ 1003bd37 f   libucrt:environment_initialization.obj
 0001:0003ad8a       ??$common_initialize_environment_nolock@_W@@YAHXZ 1003bd8a f   libucrt:environment_initialization.obj
 0001:0003add8       ??$create_environment@D@@YAQAPADQAD@Z 1003bdd8 f   libucrt:environment_initialization.obj
 0001:0003aea8       ??$create_environment@_W@@YAQAPA_WQA_W@Z 1003bea8 f   libucrt:environment_initialization.obj
 0001:0003afb5       ??$free_environment@D@@YAXQAPAD@Z 1003bfb5 f   libucrt:environment_initialization.obj
 0001:0003afb5       ??$free_environment@_W@@YAXQAPA_W@Z 1003bfb5 f   libucrt:environment_initialization.obj
 0001:0003afe4       ??$initialize_environment_by_cloning_nolock@_W@@YAHXZ 1003bfe4 f   libucrt:environment_initialization.obj
 0001:0003b08a       ??$uninitialize_environment_internal@D@@YAXAAPAPAD@Z 1003c08a f   libucrt:environment_initialization.obj
 0001:0003b0a5       ??$uninitialize_environment_internal@_W@@YAXAAPAPA_W@Z 1003c0a5 f   libucrt:environment_initialization.obj
 0001:0003b101       ??$?RV<lambda_69a2805e680e0e292e8ba93315fe43a8>@@AAV<lambda_f03950bc5685219e0bcd2087efbe011e>@@V<lambda_03fcd07e894ec930e3f35da366ca99d6>@@@?$__crt_seh_guarded_call@H@@QAEH$$QAV<lambda_69a2805e680e0e292e8ba93315fe43a8>@@AAV<lambda_f03950bc5685219e0bcd2087efbe011e>@@$$QAV<lambda_03fcd07e894ec930e3f35da366ca99d6>@@@Z 1003c101 f   libucrt:onexit.obj
 0001:0003b15c       ??$?RV<lambda_8e746cf0007f6ed984d6f78af1fec997>@@AAV<lambda_22ebabd17bc4fa466a2aca6d8deb888d>@@V<lambda_18ed0c0b38a6dc0daf1e7ac6d6adf05e>@@@?$__crt_seh_guarded_call@H@@QAEH$$QAV<lambda_8e746cf0007f6ed984d6f78af1fec997>@@AAV<lambda_22ebabd17bc4fa466a2aca6d8deb888d>@@$$QAV<lambda_18ed0c0b38a6dc0daf1e7ac6d6adf05e>@@@Z 1003c15c f   libucrt:onexit.obj
 0001:0003b1d6       ??R<lambda_22ebabd17bc4fa466a2aca6d8deb888d>@@QBEHXZ 1003c1d6 f   libucrt:onexit.obj
 0001:0003b2ff       ??R<lambda_f03950bc5685219e0bcd2087efbe011e>@@QBEHXZ 1003c2ff f   libucrt:onexit.obj
 0001:0003b478       _initialize_environment    1003c478 f   libucrt:initialization.obj
 0001:0003b478       _initialize_global_state_isolation 1003c478 f   libucrt:initialization.obj
 0001:0003b478       _report_memory_leaks       1003c478 f   libucrt:initialization.obj
 0001:0003b478       _uninitialize_c            1003c478 f   libucrt:initialization.obj
 0001:0003b478       _uninitialize_global_state_isolation 1003c478 f   libucrt:initialization.obj
 0001:0003b47b       _initialize_global_variables 1003c47b f   libucrt:initialization.obj
 0001:0003b488       _initialize_c              1003c488 f   libucrt:initialization.obj
 0001:0003b4a2       _uninitialize_environment  1003c4a2 f   libucrt:initialization.obj
 0001:0003b4aa       _initialize_pointers       1003c4aa f   libucrt:initialization.obj
 0001:0003b4d8       _uninitialize_vcruntime    1003c4d8 f   libucrt:initialization.obj
 0001:0003b4e1       _uninitialize_allocated_memory 1003c4e1 f   libucrt:initialization.obj
 0001:0003b4f8       _uninitialize_allocated_io_buffers 1003c4f8 f   libucrt:initialization.obj
 0001:0003b548       ??R<lambda_af42a3ee9806e9a7305d451646e05244>@@QBEXAAPAU__crt_multibyte_data@@@Z 1003c548 f   libucrt:initialization.obj
 0001:0003b68c       ?_strupr_s_l_stat@@YAHQADIQAU__crt_locale_pointers@@@Z 1003c68c f   libucrt:strupr.obj
 0001:0003ceb0       ??$?RV<lambda_15ade71b0218206bbe3333a0c9b79046>@@AAV<lambda_da44e0f8b0f19ba52fefafb335991732>@@V<lambda_207f2d024fc103971653565357d6cd41>@@@?$__crt_seh_guarded_call@X@@QAEX$$QAV<lambda_15ade71b0218206bbe3333a0c9b79046>@@AAV<lambda_da44e0f8b0f19ba52fefafb335991732>@@$$QAV<lambda_207f2d024fc103971653565357d6cd41>@@@Z 1003deb0 f   libucrt:per_thread_data.obj
 0001:0003cf02       ??$?RV<lambda_38edbb1296d33220d7e4dd0ed76b244a>@@AAV<lambda_5ce1d447e08cb34b2473517608e21441>@@V<lambda_fb385d3da700c9147fc39e65dd577a8c>@@@?$__crt_seh_guarded_call@X@@QAEX$$QAV<lambda_38edbb1296d33220d7e4dd0ed76b244a>@@AAV<lambda_5ce1d447e08cb34b2473517608e21441>@@$$QAV<lambda_fb385d3da700c9147fc39e65dd577a8c>@@@Z 1003df02 f   libucrt:per_thread_data.obj
 0001:0003cf6d       ??$?RV<lambda_6affb1475c98b40b75cdec977db92e3c>@@AAV<lambda_b8d4b9c228a6ecc3f80208dbb4b4a104>@@V<lambda_608742c3c92a14382c1684fc64f96c88>@@@?$__crt_seh_guarded_call@X@@QAEX$$QAV<lambda_6affb1475c98b40b75cdec977db92e3c>@@AAV<lambda_b8d4b9c228a6ecc3f80208dbb4b4a104>@@$$QAV<lambda_608742c3c92a14382c1684fc64f96c88>@@@Z 1003df6d f   libucrt:per_thread_data.obj
 0001:0003cfc2       ??$?RV<lambda_a7e850c220f1c8d1e6efeecdedd162c6>@@AAV<lambda_46720907175c18b6c9d2717bc0d2d362>@@V<lambda_9048902d66e8d99359bc9897bbb930a8>@@@?$__crt_seh_guarded_call@X@@QAEX$$QAV<lambda_a7e850c220f1c8d1e6efeecdedd162c6>@@AAV<lambda_46720907175c18b6c9d2717bc0d2d362>@@$$QAV<lambda_9048902d66e8d99359bc9897bbb930a8>@@@Z 1003dfc2 f   libucrt:per_thread_data.obj
 0001:0003d01c       ?construct_ptd@@YAXQAU__acrt_ptd@@QAPAU__crt_locale_data@@@Z 1003e01c f   libucrt:per_thread_data.obj
 0001:0003d0b5       ?destroy_fls@@YGXPAX@Z     1003e0b5 f   libucrt:per_thread_data.obj
 0001:0003d0d6       ?destroy_ptd@@YAXQAU__acrt_ptd@@@Z 1003e0d6 f   libucrt:per_thread_data.obj
 0001:0003d1a3       ?replace_current_thread_locale_nolock@@YAXQAU__acrt_ptd@@QAU__crt_locale_data@@@Z 1003e1a3 f   libucrt:per_thread_data.obj
 0001:0003d528       ?fp_format_a@@YAHQBNPADIQADIH_NIQAU__crt_locale_pointers@@@Z 1003e528 f   libucrt:cvt.obj
 0001:0003d841       ?fp_format_e@@YAHQBNQADI1IH_NIQAU__crt_locale_pointers@@@Z 1003e841 f   libucrt:cvt.obj
 0001:0003d8e3       ?fp_format_e_internal@@YAHQADIH_NIQAU_strflt@@1QAU__crt_locale_pointers@@@Z 1003e8e3 f   libucrt:cvt.obj
 0001:0003da2b       ?fp_format_f@@YAHQBNQADI1IHQAU__crt_locale_pointers@@@Z 1003ea2b f   libucrt:cvt.obj
 0001:0003dab6       ?fp_format_f_internal@@YAHQADIHQAU_strflt@@_NQAU__crt_locale_pointers@@@Z 1003eab6 f   libucrt:cvt.obj
 0001:0003db87       ?fp_format_g@@YAHQBNQADI1IH_NIQAU__crt_locale_pointers@@@Z 1003eb87 f   libucrt:cvt.obj
 0001:0003dc48       ?fp_format_nan_or_infinity@@YAHW4__acrt_fp_class@@_NPADI1@Z 1003ec48 f   libucrt:cvt.obj
 0001:0003dcdd       ?shift_bytes@@YAXQADI0H@Z  1003ecdd f   libucrt:cvt.obj
 0001:0003df9e       ??$?RV<lambda_e5124f882df8998aaf41531e079ba474>@@AAV<lambda_3e16ef9562a7dcce91392c22ab16ea36>@@V<lambda_e25ca0880e6ef98be67edffd8c599615>@@@?$__crt_seh_guarded_call@X@@QAEX$$QAV<lambda_e5124f882df8998aaf41531e079ba474>@@AAV<lambda_3e16ef9562a7dcce91392c22ab16ea36>@@$$QAV<lambda_e25ca0880e6ef98be67edffd8c599615>@@@Z 1003ef9e f   libucrt:wsetlocale.obj
 0001:0003e03e       ?initialize_inherited_file_handles_nolock@@YAXXZ 1003f03e f   libucrt:ioinit.obj
 0001:0003e0f4       ?initialize_stdio_handles_nolock@@YAXXZ 1003f0f4 f   libucrt:ioinit.obj
 0001:0003e234       ??$?RV<lambda_218ce3db14220d0be481dae8ef3383b6>@@AAV<lambda_628dfdc04ba53c8bfc02c9951375f3f5>@@V<lambda_57dc472bd5c9d5f3b2cbca59b8a843ae>@@@?$__crt_seh_guarded_call@H@@QAEH$$QAV<lambda_218ce3db14220d0be481dae8ef3383b6>@@AAV<lambda_628dfdc04ba53c8bfc02c9951375f3f5>@@$$QAV<lambda_57dc472bd5c9d5f3b2cbca59b8a843ae>@@@Z 1003f234 f   libucrt:close.obj
 0001:0003e48d       ?find_or_allocate_unused_stream_nolock@@YA?AV__crt_stdio_stream@@XZ 1003f48d f   libucrt:stream.obj
 0001:0003e5f3       ??$?RV<lambda_cbab9ec6f41b0180b23cc171c22676b0>@@AAV<lambda_44731a7d0e6d81c3e6aa82d741081786>@@V<lambda_4b292cb8dd18144e164572427af410ab>@@@?$__crt_seh_guarded_call@P6AXH@Z@@QAEP6AXH@Z$$QAV<lambda_cbab9ec6f41b0180b23cc171c22676b0>@@AAV<lambda_44731a7d0e6d81c3e6aa82d741081786>@@$$QAV<lambda_4b292cb8dd18144e164572427af410ab>@@@Z 1003f5f3 f   libucrt:signal.obj
 0001:0003e657       ?get_global_action_nolock@@YAPAP6AXH@ZH@Z 1003f657 f   libucrt:signal.obj
 0001:0003e699       ?siglookup@@YAPAU__crt_signal_action_t@@HQAU1@@Z 1003f699 f   libucrt:signal.obj
 0001:0003ec99       ??$common_openfile@_W@@YAPAU_iobuf@@QB_W0HV__crt_stdio_stream@@@Z 1003fc99 f   libucrt:openfile.obj
 0001:0003ee98       ?try_get_AreFileApisANSI@@YAP6GHXZXZ 1003fe98 f   libucrt:winapi_thunks.obj
 0001:0003eeb2       ?try_get_CompareStringEx@@YAP6GHPB_WK0H0HPAU_nlsversioninfo@@PAXJ@ZXZ 1003feb2 f   libucrt:winapi_thunks.obj
 0001:0003eecc       ?try_get_LCMapStringEx@@YAP6GHPB_WK0HPA_WHPAU_nlsversioninfo@@PAXJ@ZXZ 1003fecc f   libucrt:winapi_thunks.obj
 0001:0003eee6       ?try_get_LocaleNameToLCID@@YAP6GKPB_WK@ZXZ 1003fee6 f   libucrt:winapi_thunks.obj
 0001:0003ef00       ?try_get_first_available_module@@YAPAUHINSTANCE__@@QBW4module_id@?A0x391cf84c@@0@Z 1003ff00 f   libucrt:winapi_thunks.obj
 0001:0003efc7       ?try_get_function@@YAPAXW4function_id@?A0x391cf84c@@QBDQBW4module_id@2@2@Z 1003ffc7 f   libucrt:winapi_thunks.obj
 0001:0003f3ea       ??$common_refill_and_read_nolock@D@@YAHV__crt_stdio_stream@@@Z 100403ea f   libucrt:_filbuf.obj
 0001:0003f57f       ??$common_lseek@J@@YAJHJH@Z 1004057f f   libucrt:lseek.obj
 0001:0003f671       ??$common_lseek@_J@@YA_JH_JH@Z 10040671 f   libucrt:lseek.obj
 0001:0003f77d       ??$common_lseek_nolock@J@@YAJHJH@Z 1004077d f   libucrt:lseek.obj
 0001:0003f7d4       ??$common_lseek_nolock@_J@@YA_JH_JH@Z 100407d4 f   libucrt:lseek.obj
 0001:0003f850       ?common_lseek_do_seek_nolock@@YAJQAXJH@Z 10040850 f   libucrt:lseek.obj
 0001:0003f96c       ??$translate_text_mode_nolock@D@@YAHHQADI@Z 1004096c f   libucrt:read.obj
 0001:0003facd       ??$translate_text_mode_nolock@_W@@YAHHQA_WI@Z 10040acd f   libucrt:read.obj
 0001:0003fc9e       ?translate_ansi_or_utf8_nolock@@YAHHQADIQA_WI@Z 10040c9e f   libucrt:read.obj
 0001:0003fdf5       ?translate_utf16_from_console_nolock@@YAHHQA_WI@Z 10040df5 f   libucrt:read.obj
 0001:00040340       ??$common_tcsncpy_s@D@@YAHQADIQBDI@Z 10041340 f   libucrt:strncpy_s.obj
 0001:00040726       ??$common_getpath@_W@@YAPA_WQB_WQA_WI@Z 10041726 f   libucrt:getpath.obj
 0001:00040856       ??$__acrt_convert_wcs_mbs_cp@D_WV<lambda_62f6974d9771e494a5ea317cc32e971c>@@U__crt_win32_buffer_internal_dynamic_resizing@@@@YAHQBDAAV?$__crt_win32_buffer@_WU__crt_win32_buffer_internal_dynamic_resizing@@@@ABV<lambda_62f6974d9771e494a5ea317cc32e971c>@@I@Z 10041856 f   libucrt:createprocessa.obj
 0001:00040dbd       ??$common_fdopen@_W@@YAPAU_iobuf@@HQB_W@Z 10041dbd f   libucrt:fdopen.obj
 0001:00040ec1       ??$?RV<lambda_9e9de3de5fa147e2223d7db92bc10aa6>@@AAV<lambda_38ce7e780aa69e748d6df282ebc68efe>@@V<lambda_8ca6da459f0f6780f1cff60fdc3d00e5>@@@?$__crt_seh_guarded_call@H@@QAEH$$QAV<lambda_9e9de3de5fa147e2223d7db92bc10aa6>@@AAV<lambda_38ce7e780aa69e748d6df282ebc68efe>@@$$QAV<lambda_8ca6da459f0f6780f1cff60fdc3d00e5>@@@Z 10041ec1 f   libucrt:commit.obj
 0001:00040fe0       ?write_double_translated_ansi_nolock@@YA?AUwrite_result@?A0x17268360@@HQBDI@Z 10041fe0 f   libucrt:write.obj
 0001:0004138a       ?write_double_translated_unicode_nolock@@YA?AUwrite_result@?A0x17268360@@QBDI@Z 1004238a f   libucrt:write.obj
 0001:000413f2       ?write_requires_double_translation_nolock@@YA_NH@Z 100423f2 f   libucrt:write.obj
 0001:00041463       ?write_text_ansi_nolock@@YA?AUwrite_result@?A0x17268360@@HQBDI@Z 10042463 f   libucrt:write.obj
 0001:0004153e       ?write_text_utf16le_nolock@@YA?AUwrite_result@?A0x17268360@@HQBDI@Z 1004253e f   libucrt:write.obj
 0001:00041627       ?write_text_utf8_nolock@@YA?AUwrite_result@?A0x17268360@@HQBDI@Z 10042627 f   libucrt:write.obj
 0001:00041a2d       ??$common_xtox@_KD@@YAH_KQADII_N@Z 10042a2d f   libucrt:xtoa.obj
 0001:00041af4       ??$common_xtox_s@_KD@@YAH_KQADII_N@Z 10042af4 f   libucrt:xtoa.obj
 0001:00041c5c       ??$common_sopen_dispatch@D@@YAHQBDHHHQAHH@Z 10042c5c f   libucrt:open.obj
 0001:00041d1d       ??$common_sopen_dispatch@_W@@YAHQB_WHHHQAHH@Z 10042d1d f   libucrt:open.obj
 0001:00041dde       ?configure_text_mode@@YAHHUfile_options@?A0xa9d50aae@@HAAW4__crt_lowio_text_mode@@@Z 10042dde f   libucrt:open.obj
 0001:00042031       ?create_file@@YAPAXQB_WQAU_SECURITY_ATTRIBUTES@@Ufile_options@?A0xa9d50aae@@@Z 10043031 f   libucrt:open.obj
 0001:00042056       ?decode_open_create_flags@@YAKH@Z 10043056 f   libucrt:open.obj
 0001:000420c6       ?decode_options@@YA?AUfile_options@?A0xa9d50aae@@HHH@Z 100430c6 f   libucrt:open.obj
 0001:00042240       ?truncate_ctrl_z_if_present@@YAHH@Z 10043240 f   libucrt:open.obj
 0001:0004276e       ??$common_flush_and_write_nolock@D@@YAHHV__crt_stdio_stream@@@Z 1004376e f   libucrt:_flsbuf.obj
 0001:00042883       ??$write_buffer_nolock@D@@YA_NDV__crt_stdio_stream@@@Z 10043883 f   libucrt:_flsbuf.obj
 0001:0004294f       ?stream_is_at_end_of_file_nolock@@YA_NV__crt_stdio_stream@@@Z 1004394f f   libucrt:_flsbuf.obj
 0001:00042b19       ??$?RV<lambda_1f7e3ac85ca3635646511ad93ac0febe>@@AAV<lambda_555255fdfb9471e5fa7bfca50021c162>@@V<lambda_24f51f8b0c33fe186c624e6675644b7a>@@@?$__crt_seh_guarded_call@_N@@QAE_N$$QAV<lambda_1f7e3ac85ca3635646511ad93ac0febe>@@AAV<lambda_555255fdfb9471e5fa7bfca50021c162>@@$$QAV<lambda_24f51f8b0c33fe186c624e6675644b7a>@@@Z 10043b19 f   libucrt:spawnv.obj
 0001:00042b74       ??$common_spawnv@_W@@YAHHQB_WQBQB_W1@Z 10043b74 f   libucrt:spawnv.obj
 0001:00042d7d       ??$execute_command@_W@@YAHHQB_WQBQB_W1@Z 10043d7d f   libucrt:spawnv.obj
 0001:00042f90       ??R<lambda_555255fdfb9471e5fa7bfca50021c162>@@QBE_NXZ 10043f90 f   libucrt:spawnv.obj
 0001:000430ce       ?accumulate_inheritable_handles@@YA_NQAPAEQAI_N@Z 100440ce f   libucrt:spawnv.obj
 0001:00043112       ??$common_spawnvp@_W@@YAHHQB_WQBQB_W1@Z 10044112 f   libucrt:spawnvp.obj
 0001:0004344b       ?<lambda_invoker_cdecl>@<lambda_838c7f62c73c983481e27c09e84b0b5d>@@CAHPBX0@Z 1004444b f   libucrt:argv_wildcards.obj
 0001:00043463       ??$__acrt_convert_wcs_mbs_cp@_WDV<lambda_28bda7af82a03b66c1cb3803a755f95d>@@U__crt_win32_buffer_internal_dynamic_resizing@@@@YAHQB_WAAV?$__crt_win32_buffer@DU__crt_win32_buffer_internal_dynamic_resizing@@@@ABV<lambda_28bda7af82a03b66c1cb3803a755f95d>@@I@Z 10044463 f   libucrt:argv_wildcards.obj
 0001:00043532       ??$common_expand_argv_wildcards@D@@YAHQAPADQAPAPAD@Z 10044532 f   libucrt:argv_wildcards.obj
 0001:00043721       ??$copy_and_add_argument_to_buffer@D@@YAHQBD0IAAV?$argument_list@D@?A0x5f5c8891@@@Z 10044721 f   libucrt:argv_wildcards.obj
 0001:000437d2       ??$expand_argument_wildcards@D@@YAHQAD0AAV?$argument_list@D@?A0x5f5c8891@@@Z 100447d2 f   libucrt:argv_wildcards.obj
 0001:00043a65       ?expand_if_necessary@?$argument_list@D@?A0x5f5c8891@@AAEHXZ 10044a65 f   libucrt:argv_wildcards.obj
 0001:00043af7       ??$__acrt_convert_wcs_mbs_cp@_WDV<lambda_0fec1a7b3f42a53036604e18c2d5e07e>@@U__crt_win32_buffer_no_resizing@@@@YAHQB_WAAV?$__crt_win32_buffer@DU__crt_win32_buffer_no_resizing@@@@ABV<lambda_0fec1a7b3f42a53036604e18c2d5e07e>@@I@Z 10044af7 f   libucrt:getmodulefilenamea.obj
 0001:00043c9a       ??$?RV<lambda_ceb1ee4838e85a9d631eb091e2fbe199>@@AAV<lambda_ae742caa10f662c28703da3d2ea5e57e>@@V<lambda_cd08b5d6af4937fe54fc07d0c9bf6b37>@@@?$__crt_seh_guarded_call@X@@QAEX$$QAV<lambda_ceb1ee4838e85a9d631eb091e2fbe199>@@AAV<lambda_ae742caa10f662c28703da3d2ea5e57e>@@$$QAV<lambda_cd08b5d6af4937fe54fc07d0c9bf6b37>@@@Z 10044c9a f   libucrt:mbctype.obj
 0001:00043ce7       ??R<lambda_ae742caa10f662c28703da3d2ea5e57e>@@QBEXXZ 10044ce7 f   libucrt:mbctype.obj
 0001:00043d6a       ?CPtoLocaleName@@YAPB_WH@Z 10044d6a f   libucrt:mbctype.obj
 0001:00043da8       ?getSystemCP@@YAHH@Z       10044da8 f   libucrt:mbctype.obj
 0001:00043e19       ?setSBCS@@YAXPAU__crt_multibyte_data@@@Z 10044e19 f   libucrt:mbctype.obj
 0001:00043e7e       ?setSBUpLow@@YAXPAU__crt_multibyte_data@@@Z 10044e7e f   libucrt:mbctype.obj
 0001:00043fff       ?setmbcp_internal@@YAHH_NQAU__acrt_ptd@@QAPAU__crt_multibyte_data@@@Z 10044fff f   libucrt:mbctype.obj
 0001:00044118       ?update_thread_multibyte_data_internal@@YAPAU__crt_multibyte_data@@QAU__acrt_ptd@@QAPAU1@@Z 10045118 f   libucrt:mbctype.obj
 0001:00044406       ?x_ismbbtype_l@@YAHPAU__crt_locale_pointers@@IHH@Z 10045406 f   libucrt:ismbbyte.obj
 0001:000445b7       ?find_end_of_double_null_terminated_sequence@@YAPB_WQB_W@Z 100455b7 f   libucrt:get_environment_from_os.obj
 0001:000446c2       ??$common_set_variable_in_environment_nolock@_W@@YAHQA_WH@Z 100456c2 f   libucrt:setenv.obj
 0001:00044915       ??$copy_environment@_W@@YAPAPA_WQAPA_W@Z 10045915 f   libucrt:setenv.obj
 0001:000449d3       ??$ensure_current_environment_is_not_initial_environment_nolock@_W@@YAXXZ 100459d3 f   libucrt:setenv.obj
 0001:000449ed       ??$find_in_environment_nolock@_W@@YAHQB_WI@Z 100459ed f   libucrt:setenv.obj
 0001:00044bf5       ?__acrt_LCMapStringA_stat@@YAHPAU__crt_locale_pointers@@PB_WKPBDHPADHHH@Z 10045bf5 f   libucrt:lcmapstringa.obj
 0001:00044e69       ??R<lambda_3d301b9e52f5099be73030e1f0bf487e>@@QBEIPBD@Z 10045e69 f   libucrt:mbrtowc.obj
 0001:000469fb       ?free_crt_array_internal@@YAXQAPBXI@Z 100479fb f   libucrt:inittime.obj
 0001:000471bc       ?GetTableIndexFromLocaleName@@YAHPB_W@Z 100481bc f   libucrt:lcidtoname_downlevel.obj
 0001:000475fd       ?to_abstract_control@@YA?AW4__acrt_fenv_abstract_control@@W4__acrt_fenv_machine_sse_control@@@Z 100485fd f   libucrt:_fenvutils.obj
 0001:000476b9       ?to_abstract_control@@YA?AW4__acrt_fenv_abstract_control@@W4__acrt_fenv_machine_x87_control@@@Z 100486b9 f   libucrt:_fenvutils.obj
 0001:00047772       ?to_machine_sse_control@@YA?AW4__acrt_fenv_machine_sse_control@@W4__acrt_fenv_abstract_control@@@Z 10048772 f   libucrt:_fenvutils.obj
 0001:0004783f       ?to_machine_x87_control@@YA?AW4__acrt_fenv_machine_x87_control@@W4__acrt_fenv_abstract_control@@@Z 1004883f f   libucrt:_fenvutils.obj
 0001:00047c28       ??$construct_command_line@_W@@YAHQBQB_WQAPA_W@Z 10048c28 f   libucrt:cenvarg.obj
 0001:00047d16       ??$construct_environment_block@_W@@YAHQBQB_WQAPA_W@Z 10048d16 f   libucrt:cenvarg.obj
 0001:00048004       ??R<lambda_31d3e4c6a34e5ddcb7af9cf02b7cd71c>@@QBEPA_WXZ 10049004 f   libucrt:cenvarg.obj
 0001:000480d0       ?swap@@YAXPAD0I@Z          100490d0 f   libucrt:qsort.obj
 0001:000485f8       ?initialize_multibyte@@YAHXZ 100495f8 f   libucrt:multibyte_initializer.obj
 0001:00048880       $$000000                   10049880     libucrt:log10_impl.obj
 0001:00048990       $$000000                   10049990     libucrt:ceil_pentium4.obj
 0001:00048ac0       $$000000                   10049ac0     libucrt:_strnicm.obj
 0001:00048b21       ?__dcrt_lowio_initialize_console_output@@YAXXZ 10049b21 f   libucrt:initcon.obj
 0001:00048be0       $$000000                   10049be0     libucrt:log10_pentium4.obj
 0001:00048e70       $$000000                   10049e70     libucrt:87tran.obj
 0001:00049080       $$000000                   1004a080     libucrt:87disp.obj
 0001:000492e0       $$000000                   1004a2e0     libucrt:common.obj
 0001:00049470       $$000000                   1004a470     libucrt:genexcep.obj
 0001:0004a4b0       $$000000                   1004b4b0     LIBCMT:ulldvrm.obj
 0001:0004a550       $$000000                   1004b550     LIBCMT:sehprolg4gs.obj
 0001:0004a5b0       $$000000                   1004b5b0     LIBCMT:llmul.obj
 0001:0004a5f0       $$000000                   1004b5f0     LIBCMT:llshl.obj
 0001:0004a610       $$000000                   1004b610     LIBCMT:ullshr.obj
 0001:0004a630       $$000000                   1004b630     LIBCMT:lldiv.obj
 0001:0004a6e0       $$000000                   1004b6e0     LIBCMT:chkstk.obj
 0001:0004a710       $$000000                   1004b710     LIBCMT:alloca16.obj
 0001:0004a740       $$000000                   1004b740     LIBCMT:lldvrm.obj
 0001:0004a820       $$000000                   1004b820     LIBCMT:ftol2.obj
 0001:0004ab40       $$000000                   1004bb40     LIBCMT:llrem.obj
 0001:0004ac00       $$000000                   1004bc00     LIBCMT:llshr.obj
 0001:0004ac30       $$000000                   1004bc30     libvcruntime:memchr.obj
 0001:0004ace0       __ehhandler$??__FDeleter@?1??InitializeSListHead@implementation@slist@@YGXPAT_SLIST_HEADER@@@Z@YAXXZ 1004bce0 f   vc_crt_fix_impl.obj
 0001:0004acfb       __ehhandler$?CallUnexpected@@YAXPBU_s_ESTypeList@@@Z 1004bcfb f   libvcruntime:frame.obj
 0001:0004ad20       ??__FDeleter@?1??InitializeSListHead@implementation@slist@@YGXPAT_SLIST_HEADER@@@Z@YAXXZ 1004bd20 f   vc_crt_fix_impl.obj
 0002:00000410       _GS_ExceptionPointers      1004c410     LIBCMT:gs_report.obj
 0002:00000460       ?tokenTable@@3QBUStringLiteral@@B 1004c460     libvcruntime:undname.obj
 0002:000004e0       ?nameTable@@3QBUStringLiteral@@B 1004c4e0     libvcruntime:undname.obj
 0002:00000778       ?rttiTable@@3QBUStringLiteral@@B 1004c778     libvcruntime:undname.obj
 0002:000007a0       ?IndirectionName@@3QBUStringLiteral@@B 1004c7a0     libvcruntime:undname.obj
 0002:000007d0       ?PrefixName@@3QBUStringLiteral@@B 1004c7d0     libvcruntime:undname.obj
 0002:00000dfc       ?module_names@?A0x1172487b@@3QBQB_WB 1004cdfc     libvcruntime:winapi_downlevel.obj
 0002:00000ea4       ?candidate_modules@?1??try_get_FlsAlloc@@YAP6GKP6GXPAX@Z@ZXZ@4QBW4module_id@?A0x1172487b@@B 1004cea4     libvcruntime:winapi_downlevel.obj
 0002:00000eb8       ?candidate_modules@?1??try_get_FlsFree@@YAP6GHK@ZXZ@4QBW4module_id@?A0x1172487b@@B 1004ceb8     libvcruntime:winapi_downlevel.obj
 0002:00000ec8       ?candidate_modules@?1??try_get_FlsGetValue@@YAP6GPAXK@ZXZ@4QBW4module_id@?A0x1172487b@@B 1004cec8     libvcruntime:winapi_downlevel.obj
 0002:00000edc       ?candidate_modules@?1??try_get_FlsSetValue@@YAP6GHKPAX@ZXZ@4QBW4module_id@?A0x1172487b@@B 1004cedc     libvcruntime:winapi_downlevel.obj
 0002:00000ef0       ?candidate_modules@?1??try_get_InitializeCriticalSectionEx@@YAP6GHPAU_RTL_CRITICAL_SECTION@@KK@ZXZ@4QBW4module_id@?A0x1172487b@@B 1004cef0     libvcruntime:winapi_downlevel.obj
 0002:00000f70       ?errtable@@3QBUerrentry@?A0x31fdb9ec@@B 1004cf70     libucrt:errno.obj
 0002:00001118       ?default_cmd_exe@?1???$common_popen_nolock@_W@@YAPAU_iobuf@@QB_W0HAAY01H@Z@4QB_WB 1004d118     libucrt:popen.obj
 0002:00001128       ?slash_c@?1???$common_popen_nolock@_W@@YAPAU_iobuf@@QB_W0HAAY01H@Z@4QB_WB 1004d128     libucrt:popen.obj
 0002:00001134       ?comspec_name@?1???$get_comspec@_W@@YAPB_WXZ@4QB_WB 1004d134     libucrt:popen.obj
 0002:00001144       ?backslash@?L@???$get_executable_path@_W@@YAPB_WQB_W@Z@4QB_WB 1004d144     libucrt:popen.obj
 0002:00001148       ?path_name@?1???$get_path@_W@@YAPB_WXZ@4QB_WB 1004d148     libucrt:popen.obj
 0002:00001a60       ?large_power_indices@?1??multiply_by_power_of_ten@__crt_strtox@@YA_NAAUbig_integer@2@I@Z@4QBUunpack_index@?1??12@YA_N0I@Z@B 1004da60     libucrt:input.obj
 0002:00001d28       ?comspec_name@?1???$common_system@_W@@YAHQB_W@Z@4QB_WB 1004dd28     libucrt:system.obj
 0002:00001d38       ?cmd_exe@?1???$common_system@_W@@YAHQB_W@Z@4QB_WB 1004dd38     libucrt:system.obj
 0002:00001d48       ?slash_c@?1???$common_system@_W@@YAHQB_W@Z@4QB_WB 1004dd48     libucrt:system.obj
 0002:00001e18       ___acrt_initializers       1004de18     libucrt:initialization.obj
 0002:00001e98       ?strings@?1??fp_format_nan_or_infinity@@YAHW4__acrt_fp_class@@_NPADI1@Z@4QAY03QBDA 1004de98     libucrt:cvt.obj
 0002:000023e0       _over                      1004e3e0     libucrt:fpctrl.obj
 0002:000023ec       _under                     1004e3ec     libucrt:fpctrl.obj
 0002:00002430       ?module_names@?A0x391cf84c@@3QBQB_WB 1004e430     libucrt:winapi_thunks.obj
 0002:000028a8       ?candidate_modules@?1??try_get_AreFileApisANSI@@YAP6GHXZXZ@4QBW4module_id@?A0x391cf84c@@B 1004e8a8     libucrt:winapi_thunks.obj
 0002:000028bc       ?candidate_modules@?1??try_get_CompareStringEx@@YAP6GHPB_WK0H0HPAU_nlsversioninfo@@PAXJ@ZXZ@4QBW4module_id@?A0x391cf84c@@B 1004e8bc     libucrt:winapi_thunks.obj
 0002:000028c4       ?candidate_modules@?1??try_get_FlsAlloc@@YAP6GKP6GXPAX@Z@ZXZ@4QBW4module_id@?A0x391cf84c@@B 1004e8c4     libucrt:winapi_thunks.obj
 0002:000028cc       ?candidate_modules@?1??try_get_FlsFree@@YAP6GHK@ZXZ@4QBW4module_id@?A0x391cf84c@@B 1004e8cc     libucrt:winapi_thunks.obj
 0002:000028d4       ?candidate_modules@?1??try_get_FlsGetValue@@YAP6GPAXK@ZXZ@4QBW4module_id@?A0x391cf84c@@B 1004e8d4     libucrt:winapi_thunks.obj
 0002:000028dc       ?candidate_modules@?1??try_get_FlsSetValue@@YAP6GHKPAX@ZXZ@4QBW4module_id@?A0x391cf84c@@B 1004e8dc     libucrt:winapi_thunks.obj
 0002:000028e4       ?candidate_modules@?1??try_get_InitializeCriticalSectionEx@@YAP6GHPAU_RTL_CRITICAL_SECTION@@KK@ZXZ@4QBW4module_id@?A0x391cf84c@@B 1004e8e4     libucrt:winapi_thunks.obj
 0002:000028ec       ?candidate_modules@?1??try_get_LCMapStringEx@@YAP6GHPB_WK0HPA_WHPAU_nlsversioninfo@@PAXJ@ZXZ@4QBW4module_id@?A0x391cf84c@@B 1004e8ec     libucrt:winapi_thunks.obj
 0002:00002904       ?candidate_modules@?1??try_get_LocaleNameToLCID@@YAP6GKPB_WK@ZXZ@4QBW4module_id@?A0x391cf84c@@B 1004e904     libucrt:winapi_thunks.obj
 0002:00002920       ?candidate_modules@?1??try_get_AppPolicyGetProcessTerminationMethod@@YAP6GJPAXPAW4AppPolicyProcessTerminationMethod@@@ZXZ@4QBW4module_id@?A0x391cf84c@@B 1004e920     libucrt:winapi_thunks.obj
 0002:00003544       ?dot_slash@?CB@???$common_spawnv@_W@@YAHHQB_WQBQB_W1@Z@4QB_WB 1004f544     libucrt:spawnv.obj
 0002:0000354c       ?extensions@?CP@???$common_spawnv@_W@@YAHHQB_WQBQB_W1@Z@4QAY04$$CB_WA 1004f54c     libucrt:spawnv.obj
 0002:00003574       ?_mb_locale_names@@3QBQB_WB 1004f574     libucrt:mbctype.obj
 0002:000035b8       ?large_power_indices@?1??multiply_by_power_of_ten@__crt_strtox@@YA_NAAUbig_integer@2@I@Z@4QBUunpack_index@?1??12@YA_N0I@Z@B 1004f5b8     libucrt:cfout.obj
 0002:00003678       ?LcidToLocaleNameTable@?A0x881e4c05@@3QBULcidToLocaleName@1@B 1004f678     libucrt:lcidtoname_downlevel.obj
 0002:00004798       ?LocaleNameToIndexTable@?A0x881e4c05@@3QBULocaleNameIndex@1@B 10050798     libucrt:lcidtoname_downlevel.obj
 0002:000056e8       ?equal_sign@?BD@???$construct_environment_block@_W@@YAHQBQB_WQAPA_W@Z@4QB_WB 100516e8     libucrt:cenvarg.obj
 0002:000056f0       LOG_name                   100516f0     libucrt:log10_impl.obj
 0002:00005700       _One                       10051700     libucrt:ceil_pentium4.obj
 0002:00005710       _Bns                       10051710     libucrt:ceil_pentium4.obj
 0002:00005720       _Zero                      10051720     libucrt:ceil_pentium4.obj
 0002:00005730       _S                         10051730     libucrt:ceil_pentium4.obj
 0002:00005740       _NegZero                   10051740     libucrt:ceil_pentium4.obj
 0002:00005760       emask                      10051760     libucrt:log10_pentium4.obj
 0002:00005770       CC                         10051770     libucrt:log10_pentium4.obj
 0002:00005780       Magic                      10051780     libucrt:log10_pentium4.obj
 0002:00005790       hi_mask                    10051790     libucrt:log10_pentium4.obj
 0002:000057a0       LOG10_2                    100517a0     libucrt:log10_pentium4.obj
 0002:000057b0       place_L                    100517b0     libucrt:log10_pentium4.obj
 0002:000057d0       One                        100517d0     libucrt:log10_pentium4.obj
 0002:000057e0       Zero                       100517e0     libucrt:log10_pentium4.obj
 0002:000057f0       Two52                      100517f0     libucrt:log10_pentium4.obj
 0002:00005800       Infs                       10051800     libucrt:log10_pentium4.obj
 0002:00005810       NaN                        10051810     libucrt:log10_pentium4.obj
 0002:00005820       coeff                      10051820     libucrt:log10_pentium4.obj
 0002:0000587e       _log2max                   1005187e     libucrt:87tran.obj
 0002:00005888       _smallarg                  10051888     libucrt:87tran.obj
 0002:00005892       _half                      10051892     libucrt:87tran.obj
 0002:000058de       One                        100518de     libucrt:87disp.obj
 0002:000058e6       Three                      100518e6     libucrt:87disp.obj
 0002:000058ee       XAMtoTagTab                100518ee     libucrt:87disp.obj
 0002:00005900       One                        10051900     libucrt:common.obj
 0002:00005914       DblMax                     10051914     libucrt:common.obj
 0002:0000591c       DblMin                     1005191c     libucrt:common.obj
 0002:00005924       IeeeAdjO                   10051924     libucrt:common.obj
 0002:0000592c       IeeeAdjU                   1005192c     libucrt:common.obj
 0002:00005934       _infinity                  10051934     libucrt:common.obj
 0002:0000593c       _zero                      1005193c     libucrt:common.obj
 0002:00006198       ?_names@?1??_get_fname@@9@9 10052198     libucrt:fpexcept.obj
 0002:00006340       two32                      10052340     LIBCMT:ftol2.obj
 0002:00006344       two63                      10052344     LIBCMT:ftol2.obj
 0002:00006348       _NaN                       10052348     LIBCMT:ftol2.obj
 0002:00006440       _metamethods               10052440     bit64.obj
 0002:000064a0       _funcs                     100524a0     bit64.obj
 0002:0000bd78       _colors                    10057d78     keysandcolors.obj
 0002:0000ccd8       _guids                     10058cd8     keysandcolors.obj
 0002:0000e424       _LuamacroGuid              1005a424     luamacro.obj
 0002:00010460       ?key@?3??far_Menu@@9@9     1005c460     service.obj
 0002:00010934       ?C@?3??far_InputRecordToName@@9@9 1005c934     service.obj
 0002:0001093c       ?FarGuid@?1??far_CreateSettings@@9@9 1005c93c     service.obj
 0002:00010c50       _lualibs_extra             1005cc50     service.obj
 0002:00010c90       _lualibs                   1005cc90     service.obj
 0002:00010e08       ?A@?3??far_InputRecordToName@@9@9 1005ce08     service.obj
 0002:00010e2c       ?S@?3??far_InputRecordToName@@9@9 1005ce2c     service.obj
 0002:00010f0c       _uniclib                   1005cf0c     slnunico.obj
 0002:00011294       ?limits@?1??utf8_decode@@9@9 1005d294     lutf8lib.obj
 0002:000112ac       _UTF8PATT                  1005d2ac     lutf8lib.obj
 0002:000114d8       _flib                      1005d4d8     uliolib51.obj
 0002:00011530       _iolib                     1005d530     uliolib51.obj
 0002:00011590       ?mode@?1??f_seek@@9@9      1005d590     uliolib51.obj
 0002:0001159c       ?modenames@?1??f_seek@@9@9 1005d59c     uliolib51.obj
 0002:000115ac       ?modenames@?1??f_setvbuf@@9@9 1005d5ac     uliolib51.obj
 0002:000115bc       ?mode@?1??f_setvbuf@@9@9   1005d5bc     uliolib51.obj
 0002:00011944       _pk_funcs                  1005d944     uloadlib51.obj
 0002:0001195c       _sentinel_                 1005d95c     uloadlib51.obj
 0002:00011960       _ll_funcs                  1005d960     uloadlib51.obj
 0002:00011980       _loaders                   1005d980     uloadlib51.obj
 0002:00012508       ?ntdll@modules@@3QB_WB     1005e508     vc_crt_fix_impl.obj
 0002:00012514       ?kernel32@modules@@3QB_WB  1005e514     vc_crt_fix_impl.obj
 0002:00012a68       __unwindtable$??__FDeleter@?1??InitializeSListHead@implementation@slist@@YGXPAT_SLIST_HEADER@@@Z@YAXXZ 1005ea68     vc_crt_fix_impl.obj
 0002:00012a70       __ehfuncinfo$??__FDeleter@?1??InitializeSListHead@implementation@slist@@YGXPAT_SLIST_HEADER@@@Z@YAXXZ 1005ea70     vc_crt_fix_impl.obj
 0002:00012a98       __sehtable$___scrt_is_nonwritable_in_current_image 1005ea98     LIBCMT:utility.obj
 0002:00012ab8       __sehtable$?dllmain_crt_process_attach@@YAHQAUHINSTANCE__@@QAX@Z 1005eab8     LIBCMT:dll_dllmain.obj
 0002:00012ad8       __sehtable$?dllmain_crt_process_detach@@YAH_N@Z 1005ead8     LIBCMT:dll_dllmain.obj
 0002:00012b00       __sehtable$?dllmain_dispatch@@YAHQAUHINSTANCE__@@KQAX@Z 1005eb00     LIBCMT:dll_dllmain.obj
 0002:00012b20       __sehtable$___DestructExceptionObject 1005eb20     libvcruntime:ehhelpers.obj
 0002:00012b40       __sehtable$?FrameUnwindToState@__FrameHandler3@@SAXPAUEHRegistrationNode@@PAXPBU_s_FuncInfo@@H@Z 1005eb40     libvcruntime:frame.obj
 0002:00012b68       __sehtable$?CallCatchBlock@@YAPAXPAUEHExceptionRecord@@PAUEHRegistrationNode@@PAU_CONTEXT@@PBU_s_FuncInfo@@PAXHK@Z 1005eb68     libvcruntime:frame.obj
 0002:00012b90       __catchsym$?CallUnexpected@@YAXPBU_s_ESTypeList@@@Z$2 1005eb90     libvcruntime:frame.obj
 0002:00012ba0       __unwindtable$?CallUnexpected@@YAXPBU_s_ESTypeList@@@Z 1005eba0     libvcruntime:frame.obj
 0002:00012bb0       __tryblocktable$?CallUnexpected@@YAXPBU_s_ESTypeList@@@Z 1005ebb0     libvcruntime:frame.obj
 0002:00012bc4       __ehfuncinfo$?CallUnexpected@@YAXPBU_s_ESTypeList@@@Z 1005ebc4     libvcruntime:frame.obj
 0002:00012be8       __sehtable$??$BuildCatchObjectHelperInternal@V__FrameHandler3@@@@YAHPAUEHExceptionRecord@@PAXPBU_s_HandlerType@@PBU_s_CatchableType@@@Z 1005ebe8     libvcruntime:frame.obj
 0002:00012c08       __sehtable$??$BuildCatchObjectInternal@V__FrameHandler3@@@@YAXPAUEHExceptionRecord@@PAXPBU_s_HandlerType@@PBU_s_CatchableType@@@Z 1005ec08     libvcruntime:frame.obj
 0002:00012c78       __sehtable$??$?RV<lambda_c29ee0499b841886b80d843682cc403a>@@AAV<lambda_0be4ab1c2a6918fda4e39227d83ea893>@@V<lambda_5a3ed3da325c8ea037a470278c0f2d16>@@@?$__crt_seh_guarded_call@H@@QAEH$$QAV<lambda_c29ee0499b841886b80d843682cc403a>@@AAV<lambda_0be4ab1c2a6918fda4e39227d83ea893>@@$$QAV<lambda_5a3ed3da325c8ea037a470278c0f2d16>@@@Z 1005ec78     libucrt:output.obj
 0002:00012c98       __sehtable$_fclose         1005ec98     libucrt:fclose.obj
 0002:00012cb8       __sehtable$??$common_fsopen@_W@@YAPAU_iobuf@@QB_W0H@Z 1005ecb8     libucrt:fopen.obj
 0002:00012cd8       __sehtable$_fgetc          1005ecd8     libucrt:fgetc.obj
 0002:00012cf8       __sehtable$??$common_freopen@_W@@YAHQAPAU_iobuf@@QB_W1V__crt_stdio_stream@@H@Z 1005ecf8     libucrt:freopen.obj
 0002:00012d18       __sehtable$_rewind         1005ed18     libucrt:rewind.obj
 0002:00012d38       __sehtable$_ungetc         1005ed38     libucrt:ungetc.obj
 0002:00012d58       __sehtable$_fread_s        1005ed58     libucrt:fread.obj
 0002:00012d78       __sehtable$__pclose        1005ed78     libucrt:popen.obj
 0002:00012d98       __sehtable$??$common_popen@_W@@YAPAU_iobuf@@QB_W0@Z 1005ed98     libucrt:popen.obj
 0002:00012db8       __sehtable$??$?RV<lambda_2866be3712abc81a800a822484c830d8>@@AAV<lambda_39ca0ed439415581b5b15c265174cece>@@V<lambda_2b24c74d71094a6cd0cb82e44167d71b>@@@?$__crt_seh_guarded_call@X@@QAEX$$QAV<lambda_2866be3712abc81a800a822484c830d8>@@AAV<lambda_39ca0ed439415581b5b15c265174cece>@@$$QAV<lambda_2b24c74d71094a6cd0cb82e44167d71b>@@@Z 1005edb8     libucrt:fflush.obj
 0002:00012dd8       __sehtable$??$?RV<lambda_2cc53f568c5a2bb6f192f930a45d44ea>@@AAV<lambda_ab61a845afdef5b7c387490eaf3616ee>@@V<lambda_c2ffc0b7726aa6be21d5f0026187e748>@@@?$__crt_seh_guarded_call@X@@QAEX$$QAV<lambda_2cc53f568c5a2bb6f192f930a45d44ea>@@AAV<lambda_ab61a845afdef5b7c387490eaf3616ee>@@$$QAV<lambda_c2ffc0b7726aa6be21d5f0026187e748>@@@Z 1005edd8     libucrt:fflush.obj
 0002:00012df8       __sehtable$??$?RV<lambda_6d20deecaf4856105ebacbad442d1079>@@AAV<lambda_9a32fed5bf61b6b509b2d3f6003082a1>@@V<lambda_63ea2239ed67c638ddbae41947fdf875>@@@?$__crt_seh_guarded_call@H@@QAEH$$QAV<lambda_6d20deecaf4856105ebacbad442d1079>@@AAV<lambda_9a32fed5bf61b6b509b2d3f6003082a1>@@$$QAV<lambda_63ea2239ed67c638ddbae41947fdf875>@@@Z 1005edf8     libucrt:fflush.obj
 0002:00012e18       __sehtable$_clearerr_s     1005ee18     libucrt:clearerr.obj
 0002:00012e38       __sehtable$??$common_fgets@D@@YAPADQADHV__crt_stdio_stream@@@Z 1005ee38     libucrt:fgets.obj
 0002:00012e58       __sehtable$?common_tmpfile_nolock@@YAHQAPAU_iobuf@@H@Z 1005ee58     libucrt:tmpfile.obj
 0002:00012e78       __sehtable$?common_tmpfile@@YAHQAPAU_iobuf@@H@Z 1005ee78     libucrt:tmpfile.obj
 0002:00012e98       __sehtable$??$?RV<lambda_4ac01c32aa5b53846f05d0620572872e>@@AAV<lambda_5856287d7ecd2be6c9197bb4007c3f6e>@@V<lambda_e7a9868ed898c75c0f0637692d94351a>@@@?$__crt_seh_guarded_call@I@@QAEI$$QAV<lambda_4ac01c32aa5b53846f05d0620572872e>@@AAV<lambda_5856287d7ecd2be6c9197bb4007c3f6e>@@$$QAV<lambda_e7a9868ed898c75c0f0637692d94351a>@@@Z 1005ee98     libucrt:fwrite.obj
 0002:00012eb8       __sehtable$??$?RV<lambda_70c0770dcc4f6ec6272bb01dc82d3c91>@@AAV<lambda_ca71763b3c0644891230e4f79ea54fa6>@@V<lambda_ca266f0f09348b8765c113e3a39a2bc1>@@@?$__crt_seh_guarded_call@H@@QAEH$$QAV<lambda_70c0770dcc4f6ec6272bb01dc82d3c91>@@AAV<lambda_ca71763b3c0644891230e4f79ea54fa6>@@$$QAV<lambda_ca266f0f09348b8765c113e3a39a2bc1>@@@Z 1005eeb8     libucrt:setvbuf.obj
 0002:00012ed8       __sehtable$??$?RV<lambda_274ecf0a8038e561263518ab346655e8>@@AAV<lambda_21448eb78dd3c4a522ed7c65a98d88e6>@@V<lambda_0ca1de2171e49cefb1e8dc85c06db622>@@@?$__crt_seh_guarded_call@H@@QAEH$$QAV<lambda_274ecf0a8038e561263518ab346655e8>@@AAV<lambda_21448eb78dd3c4a522ed7c65a98d88e6>@@$$QAV<lambda_0ca1de2171e49cefb1e8dc85c06db622>@@@Z 1005eed8     libucrt:input.obj
 0002:00012ef8       __sehtable$??$common_ftell@_J@@YA_JV__crt_stdio_stream@@@Z 1005eef8     libucrt:ftell.obj
 0002:00012f18       __sehtable$?common_fseek@@YAHV__crt_stdio_stream@@_JH@Z 1005ef18     libucrt:fseek.obj
 0002:00012f38       __sehtable$??$common_getenv@_W@@YAPA_WQB_W@Z 1005ef38     libucrt:getenv.obj
 0002:00012f58       __sehtable$??$common_dupenv_s@_W@@YAHQAPA_WQAIQB_WHQBDH@Z 1005ef58     libucrt:getenv.obj
 0002:00012f78       __sehtable$??R<lambda_6e4b09c48022b2350581041d5f6b0c4c>@@QBE@XZ 1005ef78     libucrt:exit.obj
 0002:00012f98       __sehtable$??$?RV<lambda_03b1d95aef87969028cfba75ccab2455>@@AAV<lambda_6e4b09c48022b2350581041d5f6b0c4c>@@V<lambda_22bdf7517842c4b3e53723af5aa32b9e>@@@?$__crt_seh_guarded_call@X@@QAEX$$QAV<lambda_03b1d95aef87969028cfba75ccab2455>@@AAV<lambda_6e4b09c48022b2350581041d5f6b0c4c>@@$$QAV<lambda_22bdf7517842c4b3e53723af5aa32b9e>@@@Z 1005ef98     libucrt:exit.obj
 0002:00012fb8       __sehtable$??$?RV<lambda_8e746cf0007f6ed984d6f78af1fec997>@@AAV<lambda_22ebabd17bc4fa466a2aca6d8deb888d>@@V<lambda_18ed0c0b38a6dc0daf1e7ac6d6adf05e>@@@?$__crt_seh_guarded_call@H@@QAEH$$QAV<lambda_8e746cf0007f6ed984d6f78af1fec997>@@AAV<lambda_22ebabd17bc4fa466a2aca6d8deb888d>@@$$QAV<lambda_18ed0c0b38a6dc0daf1e7ac6d6adf05e>@@@Z 1005efb8     libucrt:onexit.obj
 0002:00012fd8       __sehtable$??$?RV<lambda_69a2805e680e0e292e8ba93315fe43a8>@@AAV<lambda_f03950bc5685219e0bcd2087efbe011e>@@V<lambda_03fcd07e894ec930e3f35da366ca99d6>@@@?$__crt_seh_guarded_call@H@@QAEH$$QAV<lambda_69a2805e680e0e292e8ba93315fe43a8>@@AAV<lambda_f03950bc5685219e0bcd2087efbe011e>@@$$QAV<lambda_03fcd07e894ec930e3f35da366ca99d6>@@@Z 1005efd8     libucrt:onexit.obj
 0002:00012ff8       __sehtable$_terminate      1005eff8     libucrt:terminate.obj
 0002:00013018       __sehtable$??$?RV<lambda_15ade71b0218206bbe3333a0c9b79046>@@AAV<lambda_da44e0f8b0f19ba52fefafb335991732>@@V<lambda_207f2d024fc103971653565357d6cd41>@@@?$__crt_seh_guarded_call@X@@QAEX$$QAV<lambda_15ade71b0218206bbe3333a0c9b79046>@@AAV<lambda_da44e0f8b0f19ba52fefafb335991732>@@$$QAV<lambda_207f2d024fc103971653565357d6cd41>@@@Z 1005f018     libucrt:per_thread_data.obj
 0002:00013038       __sehtable$??$?RV<lambda_a7e850c220f1c8d1e6efeecdedd162c6>@@AAV<lambda_46720907175c18b6c9d2717bc0d2d362>@@V<lambda_9048902d66e8d99359bc9897bbb930a8>@@@?$__crt_seh_guarded_call@X@@QAEX$$QAV<lambda_a7e850c220f1c8d1e6efeecdedd162c6>@@AAV<lambda_46720907175c18b6c9d2717bc0d2d362>@@$$QAV<lambda_9048902d66e8d99359bc9897bbb930a8>@@@Z 1005f038     libucrt:per_thread_data.obj
 0002:00013058       __sehtable$??$?RV<lambda_38edbb1296d33220d7e4dd0ed76b244a>@@AAV<lambda_5ce1d447e08cb34b2473517608e21441>@@V<lambda_fb385d3da700c9147fc39e65dd577a8c>@@@?$__crt_seh_guarded_call@X@@QAEX$$QAV<lambda_38edbb1296d33220d7e4dd0ed76b244a>@@AAV<lambda_5ce1d447e08cb34b2473517608e21441>@@$$QAV<lambda_fb385d3da700c9147fc39e65dd577a8c>@@@Z 1005f058     libucrt:per_thread_data.obj
 0002:00013078       __sehtable$??$?RV<lambda_6affb1475c98b40b75cdec977db92e3c>@@AAV<lambda_b8d4b9c228a6ecc3f80208dbb4b4a104>@@V<lambda_608742c3c92a14382c1684fc64f96c88>@@@?$__crt_seh_guarded_call@X@@QAEX$$QAV<lambda_6affb1475c98b40b75cdec977db92e3c>@@AAV<lambda_b8d4b9c228a6ecc3f80208dbb4b4a104>@@$$QAV<lambda_608742c3c92a14382c1684fc64f96c88>@@@Z 1005f078     libucrt:per_thread_data.obj
 0002:00013098       __sehtable$??$?RV<lambda_e5124f882df8998aaf41531e079ba474>@@AAV<lambda_3e16ef9562a7dcce91392c22ab16ea36>@@V<lambda_e25ca0880e6ef98be67edffd8c599615>@@@?$__crt_seh_guarded_call@X@@QAEX$$QAV<lambda_e5124f882df8998aaf41531e079ba474>@@AAV<lambda_3e16ef9562a7dcce91392c22ab16ea36>@@$$QAV<lambda_e25ca0880e6ef98be67edffd8c599615>@@@Z 1005f098     libucrt:wsetlocale.obj
 0002:000130b8       __sehtable$___acrt_initialize_lowio 1005f0b8     libucrt:ioinit.obj
 0002:000130d8       __sehtable$??$?RV<lambda_218ce3db14220d0be481dae8ef3383b6>@@AAV<lambda_628dfdc04ba53c8bfc02c9951375f3f5>@@V<lambda_57dc472bd5c9d5f3b2cbca59b8a843ae>@@@?$__crt_seh_guarded_call@H@@QAEH$$QAV<lambda_218ce3db14220d0be481dae8ef3383b6>@@AAV<lambda_628dfdc04ba53c8bfc02c9951375f3f5>@@$$QAV<lambda_57dc472bd5c9d5f3b2cbca59b8a843ae>@@@Z 1005f0d8     libucrt:close.obj
 0002:000130f8       __sehtable$?__acrt_stdio_allocate_stream@@YA?AV__crt_stdio_stream@@XZ 1005f0f8     libucrt:stream.obj
 0002:00013118       __sehtable$_raise          1005f118     libucrt:signal.obj
 0002:00013138       __sehtable$??$?RV<lambda_cbab9ec6f41b0180b23cc171c22676b0>@@AAV<lambda_44731a7d0e6d81c3e6aa82d741081786>@@V<lambda_4b292cb8dd18144e164572427af410ab>@@@?$__crt_seh_guarded_call@P6AXH@Z@@QAEP6AXH@Z$$QAV<lambda_cbab9ec6f41b0180b23cc171c22676b0>@@AAV<lambda_44731a7d0e6d81c3e6aa82d741081786>@@$$QAV<lambda_4b292cb8dd18144e164572427af410ab>@@@Z 1005f138     libucrt:signal.obj
 0002:00013158       __sehtable$___set_fpsr_sse2 1005f158     libucrt:fpctrl.obj
 0002:00013178       __sehtable$__fcloseall     1005f178     libucrt:closeall.obj
 0002:00013198       __sehtable$??$common_lseek@J@@YAJHJH@Z 1005f198     libucrt:lseek.obj
 0002:000131b8       __sehtable$??$common_lseek@_J@@YA_JH_JH@Z 1005f1b8     libucrt:lseek.obj
 0002:000131d8       __sehtable$__read          1005f1d8     libucrt:read.obj
 0002:000131f8       __sehtable$__pipe          1005f1f8     libucrt:pipe.obj
 0002:00013220       __sehtable$??$common_fdopen@_W@@YAPAU_iobuf@@HQB_W@Z 1005f220     libucrt:fdopen.obj
 0002:00013240       __sehtable$??$?RV<lambda_9e9de3de5fa147e2223d7db92bc10aa6>@@AAV<lambda_38ce7e780aa69e748d6df282ebc68efe>@@V<lambda_8ca6da459f0f6780f1cff60fdc3d00e5>@@@?$__crt_seh_guarded_call@H@@QAEH$$QAV<lambda_9e9de3de5fa147e2223d7db92bc10aa6>@@AAV<lambda_38ce7e780aa69e748d6df282ebc68efe>@@$$QAV<lambda_8ca6da459f0f6780f1cff60fdc3d00e5>@@@Z 1005f240     libucrt:commit.obj
 0002:00013260       __sehtable$__write         1005f260     libucrt:write.obj
 0002:00013280       __sehtable$??$common_sopen_dispatch@D@@YAHQBDHHHQAHH@Z 1005f280     libucrt:open.obj
 0002:000132a0       __sehtable$??$common_sopen_dispatch@_W@@YAHQB_WHHHQAHH@Z 1005f2a0     libucrt:open.obj
 0002:000132c0       __sehtable$__rmtmp         1005f2c0     libucrt:rmtmp.obj
 0002:000132e8       __sehtable$??$?RV<lambda_1f7e3ac85ca3635646511ad93ac0febe>@@AAV<lambda_555255fdfb9471e5fa7bfca50021c162>@@V<lambda_24f51f8b0c33fe186c624e6675644b7a>@@@?$__crt_seh_guarded_call@_N@@QAE_N$$QAV<lambda_1f7e3ac85ca3635646511ad93ac0febe>@@AAV<lambda_555255fdfb9471e5fa7bfca50021c162>@@$$QAV<lambda_24f51f8b0c33fe186c624e6675644b7a>@@@Z 1005f2e8     libucrt:spawnv.obj
 0002:00013308       __sehtable$?update_thread_multibyte_data_internal@@YAPAU__crt_multibyte_data@@QAU__acrt_ptd@@QAPAU1@@Z 1005f308     libucrt:mbctype.obj
 0002:00013328       __sehtable$??$?RV<lambda_ceb1ee4838e85a9d631eb091e2fbe199>@@AAV<lambda_ae742caa10f662c28703da3d2ea5e57e>@@V<lambda_cd08b5d6af4937fe54fc07d0c9bf6b37>@@@?$__crt_seh_guarded_call@X@@QAEX$$QAV<lambda_ceb1ee4838e85a9d631eb091e2fbe199>@@AAV<lambda_ae742caa10f662c28703da3d2ea5e57e>@@$$QAV<lambda_cd08b5d6af4937fe54fc07d0c9bf6b37>@@@Z 1005f328     libucrt:mbctype.obj
 0002:00013348       __sehtable$__query_new_handler 1005f348     libucrt:new_handler.obj
 0002:00013368       __sehtable$___acrt_update_thread_locale_data 1005f368     libucrt:locale_refcounting.obj
 0002:00013388       __sehtable$__alloc_osfhnd  1005f388     libucrt:osfinfo.obj
 0002:000133a8       __sehtable$___acrt_lowio_ensure_fh_exists 1005f3a8     libucrt:osfinfo.obj
 0002:000133c8       __sehtable$__IsNonwritableInCurrentImage 1005f3c8     LIBCMT:pesect.obj
 0002:000133f0       .edata                     1005f3f0     luafar3.exp
 0002:00013418       rgpv                       1005f418     luafar3.exp
 0002:000134c4       rgszName                   1005f4c4     luafar3.exp
 0002:00013570       rgwOrd                     1005f570     luafar3.exp
 0002:000135c6       szName                     1005f5c6     luafar3.exp
 0002:000135d2       $N00001                    1005f5d2     luafar3.exp
 0002:000135dd       $N00002                    1005f5dd     luafar3.exp
 0002:000135ed       $N00003                    1005f5ed     luafar3.exp
 0002:000135fb       $N00004                    1005f5fb     luafar3.exp
 0002:00013606       $N00005                    1005f606     luafar3.exp
 0002:00013613       $N00006                    1005f613     luafar3.exp
 0002:00013622       $N00007                    1005f622     luafar3.exp
 0002:0001362d       $N00008                    1005f62d     luafar3.exp
 0002:00013637       $N00009                    1005f637     luafar3.exp
 0002:00013642       $N00010                    1005f642     luafar3.exp
 0002:00013655       $N00011                    1005f655     luafar3.exp
 0002:00013665       $N00012                    1005f665     luafar3.exp
 0002:00013677       $N00013                    1005f677     luafar3.exp
 0002:0001368b       $N00014                    1005f68b     luafar3.exp
 0002:00013697       $N00015                    1005f697     luafar3.exp
 0002:000136a6       $N00016                    1005f6a6     luafar3.exp
 0002:000136b7       $N00017                    1005f6b7     luafar3.exp
 0002:000136c7       $N00018                    1005f6c7     luafar3.exp
 0002:000136db       $N00019                    1005f6db     luafar3.exp
 0002:000136ec       $N00020                    1005f6ec     luafar3.exp
 0002:000136f4       $N00021                    1005f6f4     luafar3.exp
 0002:00013705       $N00022                    1005f705     luafar3.exp
 0002:00013716       $N00023                    1005f716     luafar3.exp
 0002:00013722       $N00024                    1005f722     luafar3.exp
 0002:00013733       $N00025                    1005f733     luafar3.exp
 0002:00013744       $N00026                    1005f744     luafar3.exp
 0002:0001374f       $N00027                    1005f74f     luafar3.exp
 0002:00013757       $N00028                    1005f757     luafar3.exp
 0002:0001376e       $N00029                    1005f76e     luafar3.exp
 0002:00013784       $N00030                    1005f784     luafar3.exp
 0002:0001379a       $N00031                    1005f79a     luafar3.exp
 0002:000137b0       $N00032                    1005f7b0     luafar3.exp
 0002:000137c2       $N00033                    1005f7c2     luafar3.exp
 0002:000137d5       $N00034                    1005f7d5     luafar3.exp
 0002:000137ea       $N00035                    1005f7ea     luafar3.exp
 0002:000137ff       $N00036                    1005f7ff     luafar3.exp
 0002:00013816       $N00037                    1005f816     luafar3.exp
 0002:0001382c       $N00038                    1005f82c     luafar3.exp
 0002:00013838       $N00039                    1005f838     luafar3.exp
 0002:0001384c       $N00040                    1005f84c     luafar3.exp
 0002:0001385d       $N00041                    1005f85d     luafar3.exp
 0002:0001386d       $N00042                    1005f86d     luafar3.exp
 0002:0001387c       $N00043                    1005f87c     luafar3.exp
 0002:000141c6       .idata$6                   100601c6     kernel32:KERNEL32.dll
 0002:0001426c       .idata$6                   1006026c     advapi32:ADVAPI32.dll
 0002:00014288       .idata$6                   10060288     user32:USER32.dll
 0002:000142b8       .idata$6                   100602b8     shell32:SHELL32.dll
 0002:00014306       .idata$6                   10060306     rpcrt4:RPCRT4.dll
 0002:000148ae       .idata$6                   100608ae     lua51:lua51.dll
 0003:00000010       ?__vcrt_flsindex@@3KA      10061010     libvcruntime:per_thread_data.obj
 0003:000000d8       ?errno_no_memory@@3HA      100610d8     libucrt:errno.obj
 0003:000000dc       ?doserrno_no_memory@@3KA   100610dc     libucrt:errno.obj
 0003:000000e4       ?__acrt_flsindex@@3KA      100610e4     libucrt:per_thread_data.obj
 0003:000001e8       ?__DAZ_ENABLED@?1??__set_fpsr_sse2@@9@9 100611e8     libucrt:fpctrl.obj
 0003:00000518       __mbctypes                 10061518     libucrt:mbctype.obj
 0003:00000620       __mbcasemaps               10061620     libucrt:mbctype.obj
 0003:00000720       ?__rgctypeflag@@3PADA      10061720     libucrt:mbctype.obj
 0003:00000728       ?__rgcode_page_info@@3PAUcode_page_info@@A 10061728     libucrt:mbctype.obj
 0003:00000880       ?__dcrt_lowio_console_output_handle@@3PAXA 10061880     libucrt:initcon.obj
 0003:000008b0       _unprintable_table         100618b0     lutf8lib.obj
 0003:00000970       _tolower_table             10061970     lutf8lib.obj
 0003:00001450       _alpha_table               10062450     lutf8lib.obj
 0003:00003370       _doublewidth_table         10064370     lutf8lib.obj
 0003:00003860       _toupper_table             10064860     lutf8lib.obj
 0003:00004420       _xdigit_table              10065420     lutf8lib.obj
 0003:00004470       _upper_table               10065470     lutf8lib.obj
 0003:00004b80       _digit_table               10065b80     lutf8lib.obj
 0003:00004e60       _cntrl_table               10065e60     lutf8lib.obj
 0003:00004f90       _compose_table             10065f90     lutf8lib.obj
 0003:00005dd0       _totitle_table             10066dd0     lutf8lib.obj
 0003:000069b0       _alnum_extend_table        100679b0     lutf8lib.obj
 0003:00006fe0       _graph_table               10067fe0     lutf8lib.obj
 0003:00009560       _lower_table               1006a560     lutf8lib.obj
 0003:00009d10       _tofold_table              1006ad10     lutf8lib.obj
 0003:0000a930       _punct_table               1006b930     lutf8lib.obj
 0003:0000b2f0       _space_table               1006c2f0     lutf8lib.obj
 0003:0000b350       _ambiwidth_table           1006c350     lutf8lib.obj
 0003:0000ba50       _GS_ExceptionRecord        1006ca50     LIBCMT:gs_report.obj
 0003:0000baa0       _GS_ContextRecord          1006caa0     LIBCMT:gs_report.obj
 0003:0000bd74       ?is_initialized_as_dll@@3_NA 1006cd74     LIBCMT:utility.obj
 0003:0000bd75       ?module_local_atexit_table_initialized@@3_NA 1006cd75     LIBCMT:utility.obj
 0003:0000bd78       ?module_local_atexit_table@@3U_onexit_table_t@@A 1006cd78     LIBCMT:utility.obj
 0003:0000bd84       ?module_local_at_quick_exit_table@@3U_onexit_table_t@@A 1006cd84     LIBCMT:utility.obj
 0003:0000bd90       ?__proc_attached@@3HA      1006cd90     LIBCMT:dll_dllmain.obj
 0003:0000bdac       ?__vcrt_startup_thread_ptd@@3U__vcrt_ptd@@A 1006cdac     libvcruntime:per_thread_data.obj
 0003:0000bdd4       ___vcrt_lock_table         1006cdd4     libvcruntime:locks.obj
 0003:0000bdec       ___vcrt_locks_initialized  1006cdec     libvcruntime:locks.obj
 0003:0000be18       ?heap@@3V_HeapManager@@A   1006ce18     libvcruntime:undname.obj
 0003:0000be2c       ?module_handles@@3PAPAUHINSTANCE__@@A 1006ce2c     libvcruntime:winapi_downlevel.obj
 0003:0000be38       ?function_pointers@@3PAPAXA 1006ce38     libvcruntime:winapi_downlevel.obj
 0003:0000be5c       ?__idtabsiz@@3IA           1006ce5c     libucrt:popen.obj
 0003:0000be60       ?__idpairs@@3PAUprocess_handle_pair@?A0xe43b7539@@A 1006ce60     libucrt:popen.obj
 0003:0000be64       ?narrow_tmpfile_buffer_pointers@@3PAPADA 1006ce64     libucrt:tmpfile.obj
 0003:0000be70       ?wide_tmpfile_buffer_pointers@@3PAPA_WA 1006ce70     libucrt:tmpfile.obj
 0003:0000be7c       ?c_termination_complete@@3JA 1006ce7c     libucrt:exit.obj
 0003:0000be80       ?thread_local_exit_callback_func@@3P6GXPAXK0@ZA 1006ce80     libucrt:exit.obj
 0003:0000be88       ?program_name@?1???$common_configure_argv@D@@YAHW4_crt_argv_mode@@@Z@4PADA 1006ce88     libucrt:argv_parsing.obj
 0003:0000bfb8       ?__acrt_invalid_parameter_handler@@3V?$dual_state_global@P6AXPB_W00II@Z@__crt_state_management@@A 1006cfb8     libucrt:invalid_parameter.obj
 0003:0000bfbc       ?internal_state@?1??_mbtowc_l@@9@4U_Mbstatet@@A 1006cfbc     libucrt:mbtowc.obj
 0003:0000bfc4       ?enable_percent_n@@3IA     1006cfc4     libucrt:printf_count_output.obj
 0003:0000c1dc       ?ctrlc_action@@3V?$dual_state_global@P6AXH@Z@__crt_state_management@@A 1006d1dc     libucrt:signal.obj
 0003:0000c1e0       ?ctrlbreak_action@@3V?$dual_state_global@P6AXH@Z@__crt_state_management@@A 1006d1e0     libucrt:signal.obj
 0003:0000c1e4       ?abort_action@@3V?$dual_state_global@P6AXH@Z@__crt_state_management@@A 1006d1e4     libucrt:signal.obj
 0003:0000c1e8       ?term_action@@3V?$dual_state_global@P6AXH@Z@__crt_state_management@@A 1006d1e8     libucrt:signal.obj
 0003:0000c1f0       ?module_handles@@3PAPAUHINSTANCE__@@A 1006d1f0     libucrt:winapi_thunks.obj
 0003:0000c240       ?encoded_function_pointers@@3PAPAXA 1006d240     libucrt:winapi_thunks.obj
 0003:0000c2c8       ?__acrt_lock_table@@3PAU_RTL_CRITICAL_SECTION@@A 1006d2c8     libucrt:locks.obj
 0003:0000c418       ?__acrt_locks_initialized@@3IA 1006d418     libucrt:locks.obj
 0003:0000c42c       ?fSystemSet@@3HA           1006d42c     libucrt:mbctype.obj
 0003:0000c430       ?initialized@?1??__acrt_initialize_multibyte@@9@4_NA 1006d430     libucrt:mbctype.obj
 0003:0000c450       ?__acrt_new_handler@@3V?$dual_state_global@P6AHI@Z@__crt_state_management@@A 1006d450     libucrt:new_handler.obj
 0003:0000c454       ?user_matherr@@3V?$dual_state_global@P6AHPAU_exception@@@Z@__crt_state_management@@A 1006d454     libucrt:matherr.obj
 0003:0000c458       ?__acrt_global_new_mode@@3V?$dual_state_global@J@__crt_state_management@@A 1006d458     libucrt:new_mode.obj
 0003:0000c468       ?internal_pst@?1??__mbrtoc32_utf8@__crt_mbstring@@YAIPA_UPBDIPAU_Mbstatet@@@Z@4U3@A 1006d468     libucrt:mbrtoc32.obj
 0003:0000c470       ?__acrt_app_type@@3W4_crt_app_type@@A 1006d470     libucrt:report_runtime_error.obj
 0003:0000c47c       __pmatherr_set             1006d47c     libucrt:libm_error.obj
 0003:0000c480       _luaopen_bit               1006d480     service.obj
 0003:0000c484       _luaopen_ffi               1006d484     service.obj
 0003:0000c488       _luaopen_jit               1006d488     service.obj
 0003:0000c48c       ?Function@?1??RtlFirstEntrySListWrapper@@9@4@4Q6GPAU_SINGLE_LIST_ENTRY@@PAT_SLIST_HEADER@@@ZA 1006d48c     vc_crt_fix_impl.obj
 0003:0000c490       ?$S17@?1??CompareStringExWrapper@@9@36@4IA 1006d490     vc_crt_fix_impl.obj
 0003:0000c494       ?Cookie@?1??XorPointer@@YAPAXPAX@Z@4IB 1006d494     vc_crt_fix_impl.obj
 0003:0000c498       ?$S1@?1??XorPointer@@YAPAXPAX@Z@4IA 1006d498     vc_crt_fix_impl.obj
 0003:0000c49c       ?Function@?1??CompareStringExWrapper@@9@36@4Q6GHPB_WK0H0HPAU_nlsversioninfo@@PAXJ@ZA 1006d49c     vc_crt_fix_impl.obj
 0003:0000c4a0       ?Function@?1??InterlockedPushEntrySListWrapper@@9@8@4Q6GPAU_SINGLE_LIST_ENTRY@@PAT_SLIST_HEADER@@PAU2@@ZA 1006d4a0     vc_crt_fix_impl.obj
 0003:0000c4a4       ?Function@?1??EncodePointerWrapper@@9@4@4Q6GPAXPAX@ZA 1006d4a4     vc_crt_fix_impl.obj
 0003:0000c4a8       ?Function@?1??DecodePointerWrapper@@9@4@4Q6GPAXPAX@ZA 1006d4a8     vc_crt_fix_impl.obj
 0003:0000c4ac       ?Function@?1??QueryDepthSListWrapper@@9@4@4Q6GGPAT_SLIST_HEADER@@@ZA 1006d4ac     vc_crt_fix_impl.obj
 0003:0000c4b0       ?$S9@?1??InterlockedPushEntrySListWrapper@@9@8@4IA 1006d4b0     vc_crt_fix_impl.obj
 0003:0000c4b4       ?$S11@?1??RtlFirstEntrySListWrapper@@9@4@4IA 1006d4b4     vc_crt_fix_impl.obj
 0003:0000c4b8       ?$S12@?1??QueryDepthSListWrapper@@9@4@4IA 1006d4b8     vc_crt_fix_impl.obj
 0003:0000c4c0       ?Deleter@?1??InitializeSListHead@implementation@slist@@YGXPAT_SLIST_HEADER@@@Z@4Vservice_deleter@23@A 1006d4c0     vc_crt_fix_impl.obj
 0003:0000c4e0       ?$S15@?1??SetThreadStackGuaranteeWrapper@@9@4@4IA 1006d4e0     vc_crt_fix_impl.obj
 0003:0000c4e4       ?Function@?1??SetThreadStackGuaranteeWrapper@@9@4@4Q6GHPAK@ZA 1006d4e4     vc_crt_fix_impl.obj
 0003:0000c4e8       ?Function@?1??LCMapStringExWrapper@@9@36@4Q6GHPB_WK0HPA_WHPAU_nlsversioninfo@@PAXJ@ZA 1006d4e8     vc_crt_fix_impl.obj
 0003:0000c4ec       ?$S3@?1??DecodePointerWrapper@@9@4@4IA 1006d4ec     vc_crt_fix_impl.obj
 0003:0000c4f0       ?Function@?1??InterlockedPushListSListExWrapper@@9@16@4Q6GPAU_SINGLE_LIST_ENTRY@@PAT_SLIST_HEADER@@PAU2@1K@ZA 1006d4f0     vc_crt_fix_impl.obj
 0003:0000c4f4       ?Function@?1??GetModuleHandleExWWrapper@@9@12@4Q6GHKPB_WPAPAUHINSTANCE__@@@ZA 1006d4f4     vc_crt_fix_impl.obj
 0003:0000c4f8       ?$S2@?1??EncodePointerWrapper@@9@4@4IA 1006d4f8     vc_crt_fix_impl.obj
 0003:0000c4fc       ?Function@?1??GetLogicalProcessorInformationWrapper@@9@8@4Q6GHPAU_SYSTEM_LOGICAL_PROCESSOR_INFORMATION@@PAK@ZA 1006d4fc     vc_crt_fix_impl.obj
 0003:0000c500       ?$S18@?1??LCMapStringExWrapper@@9@36@4IA 1006d500     vc_crt_fix_impl.obj
 0003:0000c504       ?$S6@?1??InitializeSListHeadWrapper@@9@4@4IA 1006d504     vc_crt_fix_impl.obj
 0003:0000c508       ?Function@?1??InitializeCriticalSectionExWrapper@@9@12@4Q6GHPAU_RTL_CRITICAL_SECTION@@KK@ZA 1006d508     vc_crt_fix_impl.obj
 0003:0000c50c       ?Function@?1??InterlockedFlushSListWrapper@@9@4@4Q6GPAU_SINGLE_LIST_ENTRY@@PAT_SLIST_HEADER@@@ZA 1006d50c     vc_crt_fix_impl.obj
 0003:0000c510       ?$S14@?1??GetLogicalProcessorInformationWrapper@@9@8@4IA 1006d510     vc_crt_fix_impl.obj
 0003:0000c514       ?$S13@?1??GetNumaHighestNodeNumberWrapper@@9@4@4IA 1006d514     vc_crt_fix_impl.obj
 0003:0000c518       ?Function@?1??InterlockedPopEntrySListWrapper@@9@4@4Q6GPAU_SINGLE_LIST_ENTRY@@PAT_SLIST_HEADER@@@ZA 1006d518     vc_crt_fix_impl.obj
 0003:0000c51c       ?Function@?1??InitializeSListHeadWrapper@@9@4@4Q6GXPAT_SLIST_HEADER@@@ZA 1006d51c     vc_crt_fix_impl.obj
 0003:0000c520       ?$S8@?1??InterlockedPopEntrySListWrapper@@9@4@4IA 1006d520     vc_crt_fix_impl.obj
 0003:0000c524       ?$S5@?1??InitializeSListHead@implementation@slist@@YGXPAT_SLIST_HEADER@@@Z@4IA 1006d524     vc_crt_fix_impl.obj
 0003:0000c528       ?$S7@?1??InterlockedFlushSListWrapper@@9@4@4IA 1006d528     vc_crt_fix_impl.obj
 0003:0000c52c       ?$S10@?1??InterlockedPushListSListExWrapper@@9@16@4IA 1006d52c     vc_crt_fix_impl.obj
 0003:0000c530       ?$S16@?1??InitializeCriticalSectionExWrapper@@9@12@4IA 1006d530     vc_crt_fix_impl.obj
 0003:0000c534       ?$S4@?1??GetModuleHandleExWWrapper@@9@12@4IA 1006d534     vc_crt_fix_impl.obj
 0003:0000c53c       ?Function@?1??GetNumaHighestNodeNumberWrapper@@9@4@4Q6GHPAK@ZA 1006d53c     vc_crt_fix_impl.obj
 0004:00000060       $R000000                   1006e060     luafar3.res
